 TmpPanel

 Timestamp is 5ce5f3d4 (Thu May 23 04:13:56 2019)

 Preferred load address is 0000000180000000

 Start         Length     Name                   Class
 0001:00000000 00000008H .CRT$XCA                CODE
 0001:00000008 00000008H .CRT$XCZ                CODE
 0001:00000010 00000008H .CRT$XIA                CODE
 0001:00000018 00000018H .CRT$XIC                CODE
 0001:00000030 00000008H .CRT$XIZ                CODE
 0001:00000038 00000008H .CRT$XPA                CODE
 0001:00000040 00000010H .CRT$XPX                CODE
 0001:00000050 00000008H .CRT$XPXA               CODE
 0001:00000058 00000008H .CRT$XPZ                CODE
 0001:00000060 00000008H .CRT$XTA                CODE
 0001:00000068 00000008H .CRT$XTZ                CODE
 0001:00000070 00000000H .gfids$y                CODE
 0001:00000070 00007960H .rdata                  CODE
 0001:000079d0 000001f4H .rdata$r                CODE
 0001:00007bc4 000002b4H .rdata$zzzdbg           CODE
 0001:00007e78 00000008H .rtc$IAA                CODE
 0001:00007e80 00000008H .rtc$IZZ                CODE
 0001:00007e88 00000008H .rtc$TAA                CODE
 0001:00007e90 00000010H .rtc$TZZ                CODE
 0001:00007ea0 00012a40H .text$mn                CODE
 0001:0001a8e0 00000020H .text$mn$00             CODE
 0001:0001a900 00000250H .text$x                 CODE
 0001:0001ab50 00001290H .xdata                  CODE
 0001:0001bde0 000000f0H .xdata$x                CODE
 0001:0001bed0 00000192H .edata                  CODE
 0002:00000000 00000a08H .data                   DATA
 0002:00000a08 000000a8H .data$r                 DATA
 0002:00000ab0 00001eb0H .bss                    DATA
 0003:00000000 000014b8H .pdata                  DATA
 0004:00000000 000002e0H .idata$5                DATA
 0004:000002e0 00000010H .00cfg                  DATA
 0004:000002f0 0000003cH .idata$2                DATA
 0004:0000032c 00000014H .idata$3                DATA
 0004:00000340 000002e0H .idata$4                DATA
 0004:00000620 0000067cH .idata$6                DATA
 0005:00000000 00000060H .rsrc$01                DATA
 0005:00000060 00000378H .rsrc$02                DATA

  Address         Publics by Value              Rva+Base               Lib:Object

 0000:00000000       __hybrid_code_map_count    0000000000000000     <absolute>
 0000:00000000       __hybrid_code_map          0000000000000000     <absolute>
 0000:00000000       __guard_iat_count          0000000000000000     <absolute>
 0000:00000000       __guard_longjmp_count      0000000000000000     <absolute>
 0000:00000000       __volatile_metadata        0000000000000000     <absolute>
 0000:00000000       __guard_longjmp_table      0000000000000000     <absolute>
 0000:00000000       __guard_iat_table          0000000000000000     <absolute>
 0000:00000000       __guard_fids_count         0000000000000000     <absolute>
 0000:00000000       ___safe_se_handler_count   0000000000000000     <absolute>
 0000:00000000       __enclave_config           0000000000000000     <absolute>
 0000:00000000       ___safe_se_handler_table   0000000000000000     <absolute>
 0000:00000000       __guard_fids_table         0000000000000000     <absolute>
 0000:00000000       __hybrid_auxiliary_iat     0000000000000000     <absolute>
 0000:00000000       __dynamic_value_reloc_table 0000000000000000     <absolute>
 0000:00000100       __guard_flags              0000000000000100     <absolute>
 0000:00000000       __ImageBase                0000000180000000     <linker-defined>
 0001:00000000       __xc_a                     0000000180001000     LIBCMT:initializers.obj
 0001:00000008       __xc_z                     0000000180001008     LIBCMT:initializers.obj
 0001:00000010       __xi_a                     0000000180001010     LIBCMT:initializers.obj
 0001:00000018       __acrt_multibyte_initializer 0000000180001018     libucrt:multibyte_initializer.obj
 0001:00000020       __acrt_stdio_initializer   0000000180001020     libucrt:stdio_initializer.obj
 0001:00000028       __acrt_tran_fma3_initializer 0000000180001028     libucrt:fma3_initializer.obj
 0001:00000030       __xi_z                     0000000180001030     LIBCMT:initializers.obj
 0001:00000038       __xp_a                     0000000180001038     LIBCMT:initializers.obj
 0001:00000040       __acrt_locale_terminator   0000000180001040     libucrt:locale_initializer.obj
 0001:00000048       __dcrt_console_output_terminator 0000000180001048     libucrt:console_output_initializer.obj
 0001:00000050       __acrt_stdio_terminator    0000000180001050     libucrt:stdio_initializer.obj
 0001:00000058       __xp_z                     0000000180001058     LIBCMT:initializers.obj
 0001:00000060       __xt_a                     0000000180001060     LIBCMT:initializers.obj
 0001:00000068       __xt_z                     0000000180001068     LIBCMT:initializers.obj
 0001:00000070       MainGuid                   0000000180001070     TmpPanel.obj
 0001:00000080       MenuGuid                   0000000180001080     TmpPanel.obj
 0001:00000090       ConfigDialogGuid           0000000180001090     TmpPanel.obj
 0001:000000a0       ??_C@_11LOCGONAA@@         00000001800010a0     TmpPanel.obj
 0001:000000a8       ??_C@_1O@CILPHMLJ@?$AAF?$AAA?$AAR?$AAT?$AAM?$AAP@ 00000001800010a8     TmpPanel.obj
 0001:000000b8       ??_C@_1BM@MDBPDFDA@?$AA?$CF?$AAC?$AAO?$AAM?$AAS?$AAP?$AAE?$AAC?$AA?$CF?$AA?5?$AA?1?$AAc?$AA?5@ 00000001800010b8     TmpPanel.obj
 0001:000000d4       ??_C@_13IMODFHAA@?$AA?9@   00000001800010d4     TmpPanel.obj
 0001:000000d8       ??_C@_15KIOHKAAB@?$AA?$CK?$AA?4@ 00000001800010d8     TmpPanel.obj
 0001:000000e0       ??_C@_1BC@ENICKDH@?$AAC?$AAo?$AAn?$AAt?$AAe?$AAn?$AAt?$AAs@ 00000001800010e0     TmpPanel.obj
 0001:000000f8       ??_C@_19BDAJEHDN@?$AAo?$AAp?$AAe?$AAn@ 00000001800010f8     TmpPanel.obj
 0001:00000108       ??_C@_1BC@DDPAOGMO@?$AAT?$AAm?$AAp?$AAP?$AAa?$AAn?$AAe?$AAl@ 0000000180001108     TmpPanel.obj
 0001:00000120       ??_C@_1EA@PHBPOOLI@?$AAT?$AAe?$AAm?$AAp?$AAo?$AAr?$AAa?$AAr?$AAy?$AA?5?$AAP?$AAa?$AAn?$AAe?$AAl@ 0000000180001120     TmpPanel.obj
 0001:00000160       ??_C@_1DE@BGKMIKPD@?$AAE?$AAu?$AAg?$AAe?$AAn?$AAe?$AA?5?$AAR?$AAo?$AAs?$AAh?$AAa?$AAl?$AA?5?$AA?$CG@ 0000000180001160     TmpPanel.obj
 0001:000001f0       ??_7?$DialogItemBinding@UFarDialogItem@@@@6B@ 00000001800011f0     TmpCfg.obj
 0001:00000200       ??_7PluginCheckBoxBinding@@6B@ 0000000180001200     TmpCfg.obj
 0001:00000210       ??_7PluginRadioButtonBinding@@6B@ 0000000180001210     TmpCfg.obj
 0001:00000220       ??_7PluginEditFieldBinding@@6B@ 0000000180001220     TmpCfg.obj
 0001:00000230       ??_7PluginIntEditFieldBinding@@6B@ 0000000180001230     TmpCfg.obj
 0001:00000240       ??_C@_15EFLNJKHH@?$AA?$CF?$AAu@ 0000000180001240     TmpCfg.obj
 0001:00000248       ??_7PluginUIntEditFieldBinding@@6B@ 0000000180001248     TmpCfg.obj
 0001:00000258       ??_7?$DialogBuilderBase@UFarDialogItem@@@@6B@ 0000000180001258     TmpCfg.obj
 0001:000002a0       ??_7PluginDialogBuilder@@6B@ 00000001800012a0     TmpCfg.obj
 0001:000002e8       ??_C@_1BO@NGDOFANC@?$AAA?$AAd?$AAd?$AAT?$AAo?$AAD?$AAi?$AAs?$AAk?$AAs?$AAM?$AAe?$AAn?$AAu@ 00000001800012e8     TmpCfg.obj
 0001:00000308       ??_C@_1CC@PNNAOHJC@?$AAA?$AAd?$AAd?$AAT?$AAo?$AAP?$AAl?$AAu?$AAg?$AAi?$AAn?$AAs?$AAM?$AAe?$AAn@ 0000000180001308     TmpCfg.obj
 0001:00000330       ??_C@_1BI@CPJJFPIA@?$AAC?$AAo?$AAm?$AAm?$AAo?$AAn?$AAP?$AAa?$AAn?$AAe?$AAl@ 0000000180001330     TmpCfg.obj
 0001:00000348       ??_C@_1BM@FPOJMDKB@?$AAS?$AAa?$AAf?$AAe?$AAM?$AAo?$AAd?$AAe?$AAP?$AAa?$AAn?$AAe?$AAl@ 0000000180001348     TmpCfg.obj
 0001:00000368       ??_C@_1BG@NHJCENND@?$AAA?$AAn?$AAy?$AAI?$AAn?$AAP?$AAa?$AAn?$AAe?$AAl@ 0000000180001368     TmpCfg.obj
 0001:00000380       ??_C@_1BK@BNOFJDBM@?$AAC?$AAo?$AAp?$AAy?$AAC?$AAo?$AAn?$AAt?$AAe?$AAn?$AAt?$AAs@ 0000000180001380     TmpCfg.obj
 0001:000003a0       ??_C@_19OBGHODPD@?$AAM?$AAo?$AAd?$AAe@ 00000001800013a0     TmpCfg.obj
 0001:000003b0       ??_C@_1CA@JNAJBENN@?$AAM?$AAe?$AAn?$AAu?$AAF?$AAo?$AAr?$AAF?$AAi?$AAl?$AAe?$AAl?$AAi?$AAs?$AAt@ 00000001800013b0     TmpCfg.obj
 0001:000003d0       ??_C@_1DC@BNKDLIA@?$AAN?$AAe?$AAw?$AAP?$AAa?$AAn?$AAe?$AAl?$AAF?$AAo?$AAr?$AAS?$AAe?$AAa?$AAr@ 00000001800013d0     TmpCfg.obj
 0001:00000408       ??_C@_1CA@GMFGCAGE@?$AAF?$AAu?$AAl?$AAl?$AAS?$AAc?$AAr?$AAe?$AAe?$AAn?$AAP?$AAa?$AAn?$AAe?$AAl@ 0000000180001408     TmpCfg.obj
 0001:00000428       ??_C@_1BC@JCHBPJL@?$AAL?$AAi?$AAs?$AAt?$AAU?$AAT?$AAF?$AA8@ 0000000180001428     TmpCfg.obj
 0001:00000440       ??_C@_17PBMJFEI@?$AAN?$AA?0?$AAS@ 0000000180001440     TmpCfg.obj
 0001:00000448       ??_C@_1BI@KCJICNAC@?$AAC?$AAo?$AAl?$AAu?$AAm?$AAn?$AAT?$AAy?$AAp?$AAe?$AAs@ 0000000180001448     TmpCfg.obj
 0001:00000460       ??_C@_17FKOBGGOI@?$AA0?$AA?0?$AA8@ 0000000180001460     TmpCfg.obj
 0001:00000468       ??_C@_1BK@IJFPLJEF@?$AAC?$AAo?$AAl?$AAu?$AAm?$AAn?$AAW?$AAi?$AAd?$AAt?$AAh?$AAs@ 0000000180001468     TmpCfg.obj
 0001:00000488       ??_C@_1BE@CNONJJPK@?$AAN?$AAR?$AA?0?$AAS?$AAC?$AA?0?$AAD?$AA?0?$AAT@ 0000000180001488     TmpCfg.obj
 0001:000004a0       ??_C@_1CE@CFCOMBOO@?$AAS?$AAt?$AAa?$AAt?$AAu?$AAs?$AAC?$AAo?$AAl?$AAu?$AAm?$AAn?$AAT?$AAy?$AAp@ 00000001800014a0     TmpCfg.obj
 0001:000004c8       ??_C@_1BA@HANPCFLL@?$AA0?$AA?0?$AA8?$AA?0?$AA0?$AA?0?$AA5@ 00000001800014c8     TmpCfg.obj
 0001:000004d8       ??_C@_1CG@NCCICMEA@?$AAS?$AAt?$AAa?$AAt?$AAu?$AAs?$AAC?$AAo?$AAl?$AAu?$AAm?$AAn?$AAW?$AAi?$AAd@ 00000001800014d8     TmpCfg.obj
 0001:00000500       ??_C@_1O@HIOLBLLI@?$AA?$CK?$AA?4?$AAt?$AAe?$AAm?$AAp@ 0000000180001500     TmpCfg.obj
 0001:00000510       ??_C@_19KOBLENB@?$AAM?$AAa?$AAs?$AAk@ 0000000180001510     TmpCfg.obj
 0001:00000520       ??_C@_17GNJCADOE@?$AAt?$AAm?$AAp@ 0000000180001520     TmpCfg.obj
 0001:00000528       ??_C@_1O@GBAEOCCH@?$AAP?$AAr?$AAe?$AAf?$AAi?$AAx@ 0000000180001528     TmpCfg.obj
 0001:00000538       ??_C@_1O@BJPKKLLM@?$AAC?$AAo?$AAn?$AAf?$AAi?$AAg@ 0000000180001538     TmpCfg.obj
 0001:00000548       ??_C@_1CM@OOGBEAGB@?$AAT?$AAe?$AAm?$AAp?$AAP?$AAa?$AAn?$AAe?$AAl?$AA?4?$AAC?$AAo?$AAl?$AAu?$AAm@ 0000000180001548     TmpCfg.obj
 0001:00000578       ??_C@_1CO@PEIMNADN@?$AAT?$AAe?$AAm?$AAp?$AAP?$AAa?$AAn?$AAe?$AAl?$AA?4?$AAC?$AAo?$AAl?$AAu?$AAm@ 0000000180001578     TmpCfg.obj
 0001:000005a8       ??_C@_1DI@DFFNPDGJ@?$AAT?$AAe?$AAm?$AAp?$AAP?$AAa?$AAn?$AAe?$AAl?$AA?4?$AAS?$AAt?$AAa?$AAt?$AAu@ 00000001800015a8     TmpCfg.obj
 0001:000005e0       ??_C@_1DK@GODNGDDP@?$AAT?$AAe?$AAm?$AAp?$AAP?$AAa?$AAn?$AAe?$AAl?$AA?4?$AAS?$AAt?$AAa?$AAt?$AAu@ 00000001800015e0     TmpCfg.obj
 0001:00000620       ??_C@_1BO@JLKBMGBC@?$AAT?$AAe?$AAm?$AAp?$AAP?$AAa?$AAn?$AAe?$AAl?$AA?4?$AAM?$AAa?$AAs?$AAk@ 0000000180001620     TmpCfg.obj
 0001:00000640       ??_C@_1CC@CFPIPDCG@?$AAT?$AAe?$AAm?$AAp?$AAP?$AAa?$AAn?$AAe?$AAl?$AA?4?$AAP?$AAr?$AAe?$AAf?$AAi@ 0000000180001640     TmpCfg.obj
 0001:00000670       __xmm@ffffffffffffffff0000000000000002 0000000180001670     TmpCfg.obj
 0001:00000680       __xmm@ffffffffffffffffffffffffffffffff 0000000180001680     TmpCfg.obj
 0001:00000690       ??_C@_19NHGNNLNG@?$AA?$CI?$AAR?$AA?$CJ?$AA?5@ 0000000180001690     TmpClass.obj
 0001:000006a0       ??_C@_1O@OCNONAPA@?$AA?5?$AA?$CF?$AAs?$AA?$CF?$AAs?$AA?5@ 00000001800016a0     TmpClass.obj
 0001:000006b0       ??_C@_13FPGAJAPJ@?$AA?2@   00000001800016b0     TmpClass.obj
 0001:000006b4       ??_C@_13BBDEGPLJ@?$AA?$CK@ 00000001800016b4     TmpClass.obj
 0001:000006b8       ??_C@_15DDHGOCBH@?$AA?4?$AA?4@ 00000001800016b8     TmpClass.obj
 0001:000006c0       ??_C@_13JOFGPIOO@?$AA?4@   00000001800016c0     TmpClass.obj
 0001:000006c8       ??_C@_1M@HCONLDPB@?$AAp?$AAa?$AAn?$AAe?$AAl@ 00000001800016c8     TmpClass.obj
 0001:000006d8       ??_C@_1CE@FHMHDLFC@?$AAT?$AAm?$AAp?$AAP?$AAa?$AAn?$AAe?$AAl?$AA?4?$AAS?$AAa?$AAv?$AAe?$AAL?$AAi@ 00000001800016d8     TmpClass.obj
 0001:00000704       ??_C@_15JNBOKNOG@?$AA?$AN?$AA?6@ 0000000180001704     TmpClass.obj
 0001:0000070c       ??_C@_02PCIJFNDE@?$AN?6@   000000018000170c     TmpClass.obj
 0001:00000728       ??_C@_1BC@JIEGIPND@?$AA?5?$AA?5?$AA?5?$AA?$CF?$AAs?$AA?5?$AA?$CF?$AAd@ 0000000180001728     TmpClass.obj
 0001:00000740       ??_C@_19BKJMDJK@?$AA?2?$AA?2?$AA?4?$AA?2@ 0000000180001740     TmpClass.obj
 0001:00000750       ??_C@_1CE@JKDBMIKG@?$AA?2?$AA?2?$AA?4?$AA?2?$AAP?$AAh?$AAy?$AAs?$AAi?$AAc?$AAa?$AAl?$AAD?$AAr?$AAi@ 0000000180001750     TmpClass.obj
 0001:00000778       ??_C@_1BE@BNONMOPA@?$AA?2?$AA?2?$AA?4?$AA?2?$AAc?$AAd?$AAr?$AAo?$AAm@ 0000000180001778     TmpClass.obj
 0001:00000790       __xmm@00000000000000010000000000000001 0000000180001790     TmpClass.obj
 0001:000007a0       ??_C@_1BC@NAEGMMKI@?$AA?2?$AA?2?$AA?$DP?$AA?2?$AAU?$AAN?$AAC?$AA?2@ 00000001800017a0     TmpMix.obj
 0001:000007b8       ??_C@_19MJCDBCKE@?$AA?2?$AA?2?$AA?$DP?$AA?2@ 00000001800017b8     TmpMix.obj
 0001:000007c8       ??_C@_1CC@OPFFOEHP@?$AA?$CF?$AAF?$AAA?$AAR?$AAH?$AAO?$AAM?$AAE?$AA?$CF?$AA?$DL?$AA?$CF?$AAP?$AAA?$AAT?$AAH@ 00000001800017c8     TmpMix.obj
 0001:000007f0       _pDefaultRawDllMain        00000001800017f0     LIBCMT:dll_dllmain.obj
 0001:000007f0       _pRawDllMain               00000001800017f0     LIBCMT:dll_dllmain.obj
 0001:00000800       ??_7exception@std@@6B@     0000000180001800     LIBCMT:throw_bad_alloc.obj
 0001:00000810       ??_C@_0BC@EOODALEL@Unknown?5exception@ 0000000180001810     LIBCMT:throw_bad_alloc.obj
 0001:00000830       ??_7bad_alloc@std@@6B@     0000000180001830     LIBCMT:throw_bad_alloc.obj
 0001:00000840       ??_C@_0P@GHFPNOJB@bad?5allocation@ 0000000180001840     LIBCMT:throw_bad_alloc.obj
 0001:00000858       ??_7bad_array_new_length@std@@6B@ 0000000180001858     LIBCMT:throw_bad_alloc.obj
 0001:00000868       ??_C@_0BF@KINCDENJ@bad?5array?5new?5length@ 0000000180001868     LIBCMT:throw_bad_alloc.obj
 0001:00000888       ??_7type_info@@6B@         0000000180001888     LIBCMT:std_type_info_static.obj
 0001:000008d0       _pDestructExceptionObject  00000001800018d0     libvcruntime:ehhelpers.obj
 0001:00000c18       ??_C@_08EHJDFFNH@__based?$CI@ 0000000180001c18     libvcruntime:undname.obj
 0001:00000c28       ??_C@_07KOLFKCDI@__cdecl@  0000000180001c28     libvcruntime:undname.obj
 0001:00000c30       ??_C@_08GHMPAG@__pascal@   0000000180001c30     libvcruntime:undname.obj
 0001:00000c40       ??_C@_09IFJBGAPI@__stdcall@ 0000000180001c40     libvcruntime:undname.obj
 0001:00000c50       ??_C@_0L@NPHFGOKO@__thiscall@ 0000000180001c50     libvcruntime:undname.obj
 0001:00000c60       ??_C@_0L@JMKHOMEK@__fastcall@ 0000000180001c60     libvcruntime:undname.obj
 0001:00000c70       ??_C@_0N@BCKKPABJ@__vectorcall@ 0000000180001c70     libvcruntime:undname.obj
 0001:00000c80       ??_C@_09HIJEGCPM@__clrcall@ 0000000180001c80     libvcruntime:undname.obj
 0001:00000c8c       ??_C@_06GHPCKEAG@__eabi@   0000000180001c8c     libvcruntime:undname.obj
 0001:00000c98       ??_C@_09IOPIDJLG@__swift_1@ 0000000180001c98     libvcruntime:undname.obj
 0001:00000ca8       ??_C@_09KFNFGKHF@__swift_2@ 0000000180001ca8     libvcruntime:undname.obj
 0001:00000cb8       ??_C@_07JOMMBBKO@__ptr64@  0000000180001cb8     libvcruntime:undname.obj
 0001:00000cc0       ??_C@_0L@PILCLIHE@__restrict@ 0000000180001cc0     libvcruntime:undname.obj
 0001:00000cd0       ??_C@_0M@GFIIJFMG@__unaligned@ 0000000180001cd0     libvcruntime:undname.obj
 0001:00000ce0       ??_C@_09DHDLOLLB@restrict?$CI@ 0000000180001ce0     libvcruntime:undname.obj
 0001:00000cea       ??_C@_00CNPNBAHC@@         0000000180001cea     libvcruntime:undname.obj
 0001:00000cec       ??_C@_04NIHEBCM@?5new@     0000000180001cec     libvcruntime:undname.obj
 0001:00000cf8       ??_C@_07FPCDHGMM@?5delete@ 0000000180001cf8     libvcruntime:undname.obj
 0001:00000d00       ??_C@_01NEMOKFLO@?$DN@     0000000180001d00     libvcruntime:undname.obj
 0001:00000d04       ??_C@_02GPIOPFAK@?$DO?$DO@ 0000000180001d04     libvcruntime:undname.obj
 0001:00000d08       ??_C@_02FODMEDOG@?$DM?$DM@ 0000000180001d08     libvcruntime:undname.obj
 0001:00000d0c       ??_C@_01DCLJPIOD@?$CB@     0000000180001d0c     libvcruntime:undname.obj
 0001:00000d10       ??_C@_02EGOFBIJA@?$DN?$DN@ 0000000180001d10     libvcruntime:undname.obj
 0001:00000d14       ??_C@_02FDNJECIE@?$CB?$DN@ 0000000180001d14     libvcruntime:undname.obj
 0001:00000d18       ??_C@_02GPECMEKF@?$FL?$FN@ 0000000180001d18     libvcruntime:undname.obj
 0001:00000d20       ??_C@_08LHJFAFGD@operator@ 0000000180001d20     libvcruntime:undname.obj
 0001:00000d2c       ??_C@_02HBOOOICD@?9?$DO@   0000000180001d2c     libvcruntime:undname.obj
 0001:00000d30       ??_C@_01NBENCBCI@?$CK@     0000000180001d30     libvcruntime:undname.obj
 0001:00000d34       ??_C@_02ECNGHCIF@?$CL?$CL@ 0000000180001d34     libvcruntime:undname.obj
 0001:00000d38       ??_C@_02BAABKJLB@?9?9@     0000000180001d38     libvcruntime:undname.obj
 0001:00000d3c       ??_C@_01JOAMLHOP@?9@       0000000180001d3c     libvcruntime:undname.obj
 0001:00000d40       ??_C@_01MIFGBAGJ@?$CL@     0000000180001d40     libvcruntime:undname.obj
 0001:00000d44       ??_C@_01HNPIGOCE@?$CG@     0000000180001d44     libvcruntime:undname.obj
 0001:00000d48       ??_C@_03MNHNFDLC@?9?$DO?$CK@ 0000000180001d48     libvcruntime:undname.obj
 0001:00000d4c       ??_C@_01KMDKNFGN@?1@       0000000180001d4c     libvcruntime:undname.obj
 0001:00000d50       ??_C@_01FGNFDNOH@?$CF@     0000000180001d50     libvcruntime:undname.obj
 0001:00000d54       ??_C@_01MNNFJEPP@?$DM@     0000000180001d54     libvcruntime:undname.obj
 0001:00000d58       ??_C@_02EHCHHCKH@?$DM?$DN@ 0000000180001d58     libvcruntime:undname.obj
 0001:00000d5c       ??_C@_01PPODPGHN@?$DO@     0000000180001d5c     libvcruntime:undname.obj
 0001:00000d60       ??_C@_02EEKDKGMJ@?$DO?$DN@ 0000000180001d60     libvcruntime:undname.obj
 0001:00000d64       ??_C@_01IHBHIGKO@?0@       0000000180001d64     libvcruntime:undname.obj
 0001:00000d68       ??_C@_02HCKGKOFO@?$CI?$CJ@ 0000000180001d68     libvcruntime:undname.obj
 0001:00000d6c       ??_C@_01PJKLJHI@?$HO@      0000000180001d6c     libvcruntime:undname.obj
 0001:00000d70       ??_C@_01JKBOJNNK@?$FO@     0000000180001d70     libvcruntime:undname.obj
 0001:00000d74       ??_C@_01DNKMNLPK@?$HM@     0000000180001d74     libvcruntime:undname.obj
 0001:00000d78       ??_C@_02PPKAJPJL@?$CG?$CG@ 0000000180001d78     libvcruntime:undname.obj
 0001:00000d7c       ??_C@_02NONPIBCD@?$HM?$HM@ 0000000180001d7c     libvcruntime:undname.obj
 0001:00000d80       ??_C@_02FPIMKNGF@?$CK?$DN@ 0000000180001d80     libvcruntime:undname.obj
 0001:00000d84       ??_C@_02FOEOMHFC@?$CL?$DN@ 0000000180001d84     libvcruntime:undname.obj
 0001:00000d88       ??_C@_02FKMDLLOA@?9?$DN@   0000000180001d88     libvcruntime:undname.obj
 0001:00000d8c       ??_C@_02FJEHGPIO@?1?$DN@   0000000180001d8c     libvcruntime:undname.obj
 0001:00000d90       ??_C@_02FENAOKFI@?$CF?$DN@ 0000000180001d90     libvcruntime:undname.obj
 0001:00000d94       ??_C@_03IKFCCPFF@?$DO?$DO?$DN@ 0000000180001d94     libvcruntime:undname.obj
 0001:00000d98       ??_C@_03CDNPDDLA@?$DM?$DM?$DN@ 0000000180001d98     libvcruntime:undname.obj
 0001:00000d9c       ??_C@_02FGJGFEAB@?$CG?$DN@ 0000000180001d9c     libvcruntime:undname.obj
 0001:00000da0       ??_C@_02DHLNPPGH@?$HM?$DN@ 0000000180001da0     libvcruntime:undname.obj
 0001:00000da4       ??_C@_02MHEGNOJ@?$FO?$DN@  0000000180001da4     libvcruntime:undname.obj
 0001:00000da8       ??_C@_09IFPLHPGF@?$GAvftable?8@ 0000000180001da8     libvcruntime:undname.obj
 0001:00000db8       ??_C@_09BLBHBJP@?$GAvbtable?8@ 0000000180001db8     libvcruntime:undname.obj
 0001:00000dc8       ??_C@_07FEEIOKP@?$GAvcall?8@ 0000000180001dc8     libvcruntime:undname.obj
 0001:00000dd0       ??_C@_08LLFFHHDJ@?$GAtypeof?8@ 0000000180001dd0     libvcruntime:undname.obj
 0001:00000de0       ??_C@_0BF@KDPPACIK@?$GAlocal?5static?5guard?8@ 0000000180001de0     libvcruntime:undname.obj
 0001:00000df8       ??_C@_08OBABFOLI@?$GAstring?8@ 0000000180001df8     libvcruntime:undname.obj
 0001:00000e08       ??_C@_0BD@JDLKDPAB@?$GAvbase?5destructor?8@ 0000000180001e08     libvcruntime:undname.obj
 0001:00000e20       ??_C@_0BN@DEGPLNFK@?$GAvector?5deleting?5destructor?8@ 0000000180001e20     libvcruntime:undname.obj
 0001:00000e40       ??_C@_0BO@OBMKPJIG@?$GAdefault?5constructor?5closure?8@ 0000000180001e40     libvcruntime:undname.obj
 0001:00000e60       ??_C@_0BN@IMDCHIKM@?$GAscalar?5deleting?5destructor?8@ 0000000180001e60     libvcruntime:undname.obj
 0001:00000e80       ??_C@_0BO@PFGOCPJJ@?$GAvector?5constructor?5iterator?8@ 0000000180001e80     libvcruntime:undname.obj
 0001:00000ea0       ??_C@_0BN@LFPFMEDL@?$GAvector?5destructor?5iterator?8@ 0000000180001ea0     libvcruntime:undname.obj
 0001:00000ec0       ??_C@_0CE@IKBNEHA@?$GAvector?5vbase?5constructor?5itera@ 0000000180001ec0     libvcruntime:undname.obj
 0001:00000ee8       ??_C@_0BL@NILFHHPC@?$GAvirtual?5displacement?5map?8@ 0000000180001ee8     libvcruntime:undname.obj
 0001:00000f08       ??_C@_0CB@JONCMFFK@?$GAeh?5vector?5constructor?5iterator@ 0000000180001f08     libvcruntime:undname.obj
 0001:00000f30       ??_C@_0CA@GCEOPDGL@?$GAeh?5vector?5destructor?5iterator?8@ 0000000180001f30     libvcruntime:undname.obj
 0001:00000f50       ??_C@_0CH@OOJPLCPH@?$GAeh?5vector?5vbase?5constructor?5it@ 0000000180001f50     libvcruntime:undname.obj
 0001:00000f78       ??_C@_0BL@LLKPOHJI@?$GAcopy?5constructor?5closure?8@ 0000000180001f78     libvcruntime:undname.obj
 0001:00000f98       ??_C@_0BA@KBCDOMBN@?$GAudt?5returning?8@ 0000000180001f98     libvcruntime:undname.obj
 0001:00000fa8       ??_C@_03KLGMFNMG@?$GAEH@   0000000180001fa8     libvcruntime:undname.obj
 0001:00000fac       ??_C@_05KHLCHHI@?$GARTTI@  0000000180001fac     libvcruntime:undname.obj
 0001:00000fb8       ??_C@_0BA@KKLDJDLB@?$GAlocal?5vftable?8@ 0000000180001fb8     libvcruntime:undname.obj
 0001:00000fc8       ??_C@_0CE@IIHCMGGL@?$GAlocal?5vftable?5constructor?5clos@ 0000000180001fc8     libvcruntime:undname.obj
 0001:00000fec       ??_C@_06FHBGPFGH@?5new?$FL?$FN@ 0000000180001fec     libvcruntime:undname.obj
 0001:00000ff8       ??_C@_09LBNFPBCA@?5delete?$FL?$FN@ 0000000180001ff8     libvcruntime:undname.obj
 0001:00001008       ??_C@_0P@HJKNJFNN@?$GAomni?5callsig?8@ 0000000180002008     libvcruntime:undname.obj
 0001:00001018       ??_C@_0BL@CNOONJFP@?$GAplacement?5delete?5closure?8@ 0000000180002018     libvcruntime:undname.obj
 0001:00001038       ??_C@_0BN@CKNJLHMB@?$GAplacement?5delete?$FL?$FN?5closure?8@ 0000000180002038     libvcruntime:undname.obj
 0001:00001058       ??_C@_0CG@CFDHKGGD@?$GAmanaged?5vector?5constructor?5ite@ 0000000180002058     libvcruntime:undname.obj
 0001:00001080       ??_C@_0CF@IMGKMJNO@?$GAmanaged?5vector?5destructor?5iter@ 0000000180002080     libvcruntime:undname.obj
 0001:000010a8       ??_C@_0CG@HLDDJMAG@?$GAeh?5vector?5copy?5constructor?5ite@ 00000001800020a8     libvcruntime:undname.obj
 0001:000010d0       ??_C@_0CM@FCBBDIGB@?$GAeh?5vector?5vbase?5copy?5construct@ 00000001800020d0     libvcruntime:undname.obj
 0001:00001100       ??_C@_0BL@CLIPGLGB@?$GAdynamic?5initializer?5for?5?8@ 0000000180002100     libvcruntime:undname.obj
 0001:00001120       ??_C@_0CB@PDBIFEP@?$GAdynamic?5atexit?5destructor?5for?5@ 0000000180002120     libvcruntime:undname.obj
 0001:00001148       ??_C@_0CD@CGAJBKEJ@?$GAvector?5copy?5constructor?5iterat@ 0000000180002148     libvcruntime:undname.obj
 0001:00001170       ??_C@_0CJ@GJELGAMM@?$GAvector?5vbase?5copy?5constructor?5@ 0000000180002170     libvcruntime:undname.obj
 0001:000011a0       ??_C@_0CL@FGIJHLCE@?$GAmanaged?5vector?5copy?5constructo@ 00000001800021a0     libvcruntime:undname.obj
 0001:000011d0       ??_C@_0BM@PMGGMLDN@?$GAlocal?5static?5thread?5guard?8@ 00000001800021d0     libvcruntime:undname.obj
 0001:000011f0       ??_C@_0N@BDNMDMOL@operator?5?$CC?$CC?5@ 00000001800021f0     libvcruntime:undname.obj
 0001:00001200       ??_C@_0BC@GGEBGALA@operator?5co_await@ 0000000180002200     libvcruntime:undname.obj
 0001:00001218       ??_C@_0BC@DAFEJGAK@?5Type?5Descriptor?8@ 0000000180002218     libvcruntime:undname.obj
 0001:00001230       ??_C@_0BM@LDKODKLH@?5Base?5Class?5Descriptor?5at?5?$CI@ 0000000180002230     libvcruntime:undname.obj
 0001:00001250       ??_C@_0BD@LGICGFMM@?5Base?5Class?5Array?8@ 0000000180002250     libvcruntime:undname.obj
 0001:00001268       ??_C@_0BN@MECKDCOJ@?5Class?5Hierarchy?5Descriptor?8@ 0000000180002268     libvcruntime:undname.obj
 0001:00001288       ??_C@_0BK@CFCOFLF@?5Complete?5Object?5Locator?8@ 0000000180002288     libvcruntime:undname.obj
 0001:000012c0       ??_C@_1DM@KHCHBNEB@?$AAa?$AAp?$AAi?$AA?9?$AAm?$AAs?$AA?9?$AAw?$AAi?$AAn?$AA?9?$AAc?$AAo?$AAr?$AAe@ 00000001800022c0     libvcruntime:winapi_downlevel.obj
 0001:00001300       ??_C@_1DK@LPPGFMPP@?$AAa?$AAp?$AAi?$AA?9?$AAm?$AAs?$AA?9?$AAw?$AAi?$AAn?$AA?9?$AAc?$AAo?$AAr?$AAe@ 0000000180002300     libvcruntime:winapi_downlevel.obj
 0001:00001340       ??_C@_1BC@GDMECMAK@?$AAk?$AAe?$AAr?$AAn?$AAe?$AAl?$AA3?$AA2@ 0000000180002340     libvcruntime:winapi_downlevel.obj
 0001:00001358       ??_C@_1BA@PFFKHIOG@?$AAa?$AAp?$AAi?$AA?9?$AAm?$AAs?$AA?9@ 0000000180002358     libvcruntime:winapi_downlevel.obj
 0001:00001368       ??_C@_1BA@IAIFMGEF@?$AAe?$AAx?$AAt?$AA?9?$AAm?$AAs?$AA?9@ 0000000180002368     libvcruntime:winapi_downlevel.obj
 0001:00001380       ??_C@_08KNHFBNJ@FlsAlloc@  0000000180002380     libvcruntime:winapi_downlevel.obj
 0001:00001398       ??_C@_07PEJMOBNF@FlsFree@  0000000180002398     libvcruntime:winapi_downlevel.obj
 0001:000013a8       ??_C@_0M@GDNOONDI@FlsGetValue@ 00000001800023a8     libvcruntime:winapi_downlevel.obj
 0001:000013c0       ??_C@_0M@JCPCPOEF@FlsSetValue@ 00000001800023c0     libvcruntime:winapi_downlevel.obj
 0001:000013d8       ??_C@_0BM@HCFOFFN@InitializeCriticalSectionEx@ 00000001800023d8     libvcruntime:winapi_downlevel.obj
 0001:00001400       __acrt_exception_action_table 0000000180002400     libucrt:exception_filter.obj
 0001:000014c0       __acrt_signal_action_table_count 00000001800024c0     libucrt:exception_filter.obj
 0001:000014c8       __acrt_signal_action_first_fpe_index 00000001800024c8     libucrt:exception_filter.obj
 0001:000014d0       __acrt_signal_action_fpe_count 00000001800024d0     libucrt:exception_filter.obj
 0001:000014d8       ??_C@_1BI@BGOHAHKC@?$AAm?$AAs?$AAc?$AAo?$AAr?$AAe?$AAe?$AA?4?$AAd?$AAl?$AAl?$AA?$AA@ 00000001800024d8     libucrt:exit.obj
 0001:000014f0       ??_C@_0P@MIGLKIOC@CorExitProcess?$AA@ 00000001800024f0     libucrt:exit.obj
 0001:00001788       ??_C@_1M@HPNHIDJI@?$AAj?$AAa?$AA?9?$AAJ?$AAP?$AA?$AA@ 0000000180002788     libucrt:mbctype.obj
 0001:00001798       ??_C@_1M@BIBDDEMK@?$AAz?$AAh?$AA?9?$AAC?$AAN?$AA?$AA@ 0000000180002798     libucrt:mbctype.obj
 0001:000017a8       ??_C@_1M@JLOOOEGK@?$AAk?$AAo?$AA?9?$AAK?$AAR?$AA?$AA@ 00000001800027a8     libucrt:mbctype.obj
 0001:000017b8       ??_C@_1M@CLNBBOPM@?$AAz?$AAh?$AA?9?$AAT?$AAW?$AA?$AA@ 00000001800027b8     libucrt:mbctype.obj
 0001:00001870       ??_C@_1EA@JGEFHKEI@?$AAa?$AAp?$AAi?$AA?9?$AAm?$AAs?$AA?9?$AAw?$AAi?$AAn?$AA?9?$AAc?$AAo?$AAr?$AAe?$AA?9?$AAd?$AAa?$AAt?$AAe?$AAt?$AAi?$AAm?$AAe?$AA?9?$AAl?$AA1?$AA?9?$AA1?$AA?9?$AA1?$AA?$AA@ 0000000180002870     libucrt:winapi_thunks.obj
 0001:000018b0       ??_C@_1DM@KHCHBNEB@?$AAa?$AAp?$AAi?$AA?9?$AAm?$AAs?$AA?9?$AAw?$AAi?$AAn?$AA?9?$AAc?$AAo?$AAr?$AAe?$AA?9?$AAf?$AAi?$AAb?$AAe?$AAr?$AAs?$AA?9?$AAl?$AA1?$AA?9?$AA1?$AA?9?$AA1?$AA?$AA@ 00000001800028b0     libucrt:winapi_thunks.obj
 0001:000018f0       ??_C@_1DI@IJCEHOCB@?$AAa?$AAp?$AAi?$AA?9?$AAm?$AAs?$AA?9?$AAw?$AAi?$AAn?$AA?9?$AAc?$AAo?$AAr?$AAe?$AA?9?$AAf?$AAi?$AAl?$AAe?$AA?9?$AAl?$AA1?$AA?9?$AA2?$AA?9?$AA2?$AA?$AA@ 00000001800028f0     libucrt:winapi_thunks.obj
 0001:00001930       ??_C@_1EI@MPIAOHOC@?$AAa?$AAp?$AAi?$AA?9?$AAm?$AAs?$AA?9?$AAw?$AAi?$AAn?$AA?9?$AAc?$AAo?$AAr?$AAe?$AA?9?$AAl?$AAo?$AAc?$AAa?$AAl?$AAi?$AAz?$AAa?$AAt?$AAi?$AAo?$AAn?$AA?9?$AAl?$AA1?$AA?9@ 0000000180002930     libucrt:winapi_thunks.obj
 0001:00001980       ??_C@_1FK@FPHCKFIE@?$AAa?$AAp?$AAi?$AA?9?$AAm?$AAs?$AA?9?$AAw?$AAi?$AAn?$AA?9?$AAc?$AAo?$AAr?$AAe?$AA?9?$AAl?$AAo?$AAc?$AAa?$AAl?$AAi?$AAz?$AAa?$AAt?$AAi?$AAo?$AAn?$AA?9?$AAo?$AAb?$AAs@ 0000000180002980     libucrt:winapi_thunks.obj
 0001:000019e0       ??_C@_1EM@DILCGIIO@?$AAa?$AAp?$AAi?$AA?9?$AAm?$AAs?$AA?9?$AAw?$AAi?$AAn?$AA?9?$AAc?$AAo?$AAr?$AAe?$AA?9?$AAp?$AAr?$AAo?$AAc?$AAe?$AAs?$AAs?$AAt?$AAh?$AAr?$AAe?$AAa?$AAd?$AAs?$AA?9?$AAl@ 00000001800029e0     libucrt:winapi_thunks.obj
 0001:00001a30       ??_C@_1DM@LNCGDDPN@?$AAa?$AAp?$AAi?$AA?9?$AAm?$AAs?$AA?9?$AAw?$AAi?$AAn?$AA?9?$AAc?$AAo?$AAr?$AAe?$AA?9?$AAs?$AAt?$AAr?$AAi?$AAn?$AAg?$AA?9?$AAl?$AA1?$AA?9?$AA1?$AA?9?$AA0?$AA?$AA@ 0000000180002a30     libucrt:winapi_thunks.obj
 0001:00001a70       ??_C@_1DK@LPPGFMPP@?$AAa?$AAp?$AAi?$AA?9?$AAm?$AAs?$AA?9?$AAw?$AAi?$AAn?$AA?9?$AAc?$AAo?$AAr?$AAe?$AA?9?$AAs?$AAy?$AAn?$AAc?$AAh?$AA?9?$AAl?$AA1?$AA?9?$AA2?$AA?9?$AA0?$AA?$AA@ 0000000180002a70     libucrt:winapi_thunks.obj
 0001:00001ab0       ??_C@_1DO@FPAPJEMD@?$AAa?$AAp?$AAi?$AA?9?$AAm?$AAs?$AA?9?$AAw?$AAi?$AAn?$AA?9?$AAc?$AAo?$AAr?$AAe?$AA?9?$AAs?$AAy?$AAs?$AAi?$AAn?$AAf?$AAo?$AA?9?$AAl?$AA1?$AA?9?$AA2?$AA?9?$AA1?$AA?$AA@ 0000000180002ab0     libucrt:winapi_thunks.obj
 0001:00001af0       ??_C@_1DK@NDHNAHIO@?$AAa?$AAp?$AAi?$AA?9?$AAm?$AAs?$AA?9?$AAw?$AAi?$AAn?$AA?9?$AAc?$AAo?$AAr?$AAe?$AA?9?$AAw?$AAi?$AAn?$AAr?$AAt?$AA?9?$AAl?$AA1?$AA?9?$AA1?$AA?9?$AA0?$AA?$AA@ 0000000180002af0     libucrt:winapi_thunks.obj
 0001:00001b30       ??_C@_1DM@KGHDGBCM@?$AAa?$AAp?$AAi?$AA?9?$AAm?$AAs?$AA?9?$AAw?$AAi?$AAn?$AA?9?$AAc?$AAo?$AAr?$AAe?$AA?9?$AAx?$AAs?$AAt?$AAa?$AAt?$AAe?$AA?9?$AAl?$AA2?$AA?9?$AA1?$AA?9?$AA0?$AA?$AA@ 0000000180002b30     libucrt:winapi_thunks.obj
 0001:00001b70       ??_C@_1EO@IJIOEFOH@?$AAa?$AAp?$AAi?$AA?9?$AAm?$AAs?$AA?9?$AAw?$AAi?$AAn?$AA?9?$AAr?$AAt?$AAc?$AAo?$AAr?$AAe?$AA?9?$AAn?$AAt?$AAu?$AAs?$AAe?$AAr?$AA?9?$AAw?$AAi?$AAn?$AAd?$AAo?$AAw?$AA?9@ 0000000180002b70     libucrt:winapi_thunks.obj
 0001:00001bc0       ??_C@_1FG@HHGEKANL@?$AAa?$AAp?$AAi?$AA?9?$AAm?$AAs?$AA?9?$AAw?$AAi?$AAn?$AA?9?$AAs?$AAe?$AAc?$AAu?$AAr?$AAi?$AAt?$AAy?$AA?9?$AAs?$AAy?$AAs?$AAt?$AAe?$AAm?$AAf?$AAu?$AAn?$AAc?$AAt?$AAi@ 0000000180002bc0     libucrt:winapi_thunks.obj
 0001:00001c20       ??_C@_1EG@DBIOJECG@?$AAe?$AAx?$AAt?$AA?9?$AAm?$AAs?$AA?9?$AAw?$AAi?$AAn?$AA?9?$AAn?$AAt?$AAu?$AAs?$AAe?$AAr?$AA?9?$AAd?$AAi?$AAa?$AAl?$AAo?$AAg?$AAb?$AAo?$AAx?$AA?9?$AAl?$AA1?$AA?9?$AA1@ 0000000180002c20     libucrt:winapi_thunks.obj
 0001:00001c70       ??_C@_1EO@FIHMJCLF@?$AAe?$AAx?$AAt?$AA?9?$AAm?$AAs?$AA?9?$AAw?$AAi?$AAn?$AA?9?$AAn?$AAt?$AAu?$AAs?$AAe?$AAr?$AA?9?$AAw?$AAi?$AAn?$AAd?$AAo?$AAw?$AAs?$AAt?$AAa?$AAt?$AAi?$AAo?$AAn?$AA?9@ 0000000180002c70     libucrt:winapi_thunks.obj
 0001:00001cc0       ??_C@_1BC@DNHGCMLG@?$AAa?$AAd?$AAv?$AAa?$AAp?$AAi?$AA3?$AA2?$AA?$AA@ 0000000180002cc0     libucrt:winapi_thunks.obj
 0001:00001cd8       ??_C@_1BC@GDMECMAK@?$AAk?$AAe?$AAr?$AAn?$AAe?$AAl?$AA3?$AA2?$AA?$AA@ 0000000180002cd8     libucrt:winapi_thunks.obj
 0001:00001cf0       ??_C@_1M@OAIMIKLP@?$AAn?$AAt?$AAd?$AAl?$AAl?$AA?$AA@ 0000000180002cf0     libucrt:winapi_thunks.obj
 0001:00001d00       ??_C@_1EG@DPGNFKGC@?$AAa?$AAp?$AAi?$AA?9?$AAm?$AAs?$AA?9?$AAw?$AAi?$AAn?$AA?9?$AAa?$AAp?$AAp?$AAm?$AAo?$AAd?$AAe?$AAl?$AA?9?$AAr?$AAu?$AAn?$AAt?$AAi?$AAm?$AAe?$AA?9?$AAl?$AA1?$AA?9?$AA1@ 0000000180002d00     libucrt:winapi_thunks.obj
 0001:00001d48       ??_C@_1O@BCCLBEOE@?$AAu?$AAs?$AAe?$AAr?$AA3?$AA2?$AA?$AA@ 0000000180002d48     libucrt:winapi_thunks.obj
 0001:00001d58       ??_C@_1BA@PFFKHIOG@?$AAa?$AAp?$AAi?$AA?9?$AAm?$AAs?$AA?9?$AA?$AA@ 0000000180002d58     libucrt:winapi_thunks.obj
 0001:00001d68       ??_C@_1BA@IAIFMGEF@?$AAe?$AAx?$AAt?$AA?9?$AAm?$AAs?$AA?9?$AA?$AA@ 0000000180002d68     libucrt:winapi_thunks.obj
 0001:00001d80       ??_C@_0BA@FHFNEAED@AreFileApisANSI?$AA@ 0000000180002d80     libucrt:winapi_thunks.obj
 0001:00001d98       ??_C@_08KNHFBNJ@FlsAlloc?$AA@ 0000000180002d98     libucrt:winapi_thunks.obj
 0001:00001db0       ??_C@_07PEJMOBNF@FlsFree?$AA@ 0000000180002db0     libucrt:winapi_thunks.obj
 0001:00001dc0       ??_C@_0M@GDNOONDI@FlsGetValue?$AA@ 0000000180002dc0     libucrt:winapi_thunks.obj
 0001:00001dd8       ??_C@_0M@JCPCPOEF@FlsSetValue?$AA@ 0000000180002dd8     libucrt:winapi_thunks.obj
 0001:00001df0       ??_C@_0BM@HCFOFFN@InitializeCriticalSectionEx?$AA@ 0000000180002df0     libucrt:winapi_thunks.obj
 0001:00001e18       ??_C@_0O@KKBNKAPF@LCMapStringEx?$AA@ 0000000180002e18     libucrt:winapi_thunks.obj
 0001:00001e30       ??_C@_0BB@HBDEELFH@LocaleNameToLCID?$AA@ 0000000180002e30     libucrt:winapi_thunks.obj
 0001:00001e48       ??_C@_0CF@OJOFEIGO@AppPolicyGetProcessTerminationMe@ 0000000180002e48     libucrt:winapi_thunks.obj
 0001:00001e70       __lc_time_c                0000000180002e70     libucrt:nlsdata.obj
 0001:00002130       ??_C@_03KOEHGMDN@Sun?$AA@  0000000180003130     libucrt:nlsdata.obj
 0001:00002134       ??_C@_03PDAGKDH@Mon?$AA@   0000000180003134     libucrt:nlsdata.obj
 0001:00002138       ??_C@_03NAGEINEP@Tue?$AA@  0000000180003138     libucrt:nlsdata.obj
 0001:0000213c       ??_C@_03MHOMLAJA@Wed?$AA@  000000018000313c     libucrt:nlsdata.obj
 0001:00002140       ??_C@_03IOFIKPDN@Thu?$AA@  0000000180003140     libucrt:nlsdata.obj
 0001:00002144       ??_C@_03IDIOELNC@Fri?$AA@  0000000180003144     libucrt:nlsdata.obj
 0001:00002148       ??_C@_03FEFJNEK@Sat?$AA@   0000000180003148     libucrt:nlsdata.obj
 0001:0000214c       ??_C@_06OOPIFAJ@Sunday?$AA@ 000000018000314c     libucrt:nlsdata.obj
 0001:00002154       ??_C@_06JLEDEDGH@Monday?$AA@ 0000000180003154     libucrt:nlsdata.obj
 0001:00002160       ??_C@_07BAAGCFCM@Tuesday?$AA@ 0000000180003160     libucrt:nlsdata.obj
 0001:00002168       ??_C@_09DLIGFAKA@Wednesday?$AA@ 0000000180003168     libucrt:nlsdata.obj
 0001:00002178       ??_C@_08HACCIKIA@Thursday?$AA@ 0000000180003178     libucrt:nlsdata.obj
 0001:00002184       ??_C@_06JECMNKMI@Friday?$AA@ 0000000180003184     libucrt:nlsdata.obj
 0001:00002190       ??_C@_08INBOOONO@Saturday?$AA@ 0000000180003190     libucrt:nlsdata.obj
 0001:0000219c       ??_C@_03JIHJHPIE@Jan?$AA@  000000018000319c     libucrt:nlsdata.obj
 0001:000021a0       ??_C@_03HJBDCHOM@Feb?$AA@  00000001800031a0     libucrt:nlsdata.obj
 0001:000021a4       ??_C@_03ODNJBKGA@Mar?$AA@  00000001800031a4     libucrt:nlsdata.obj
 0001:000021a8       ??_C@_03LEOLGMJP@Apr?$AA@  00000001800031a8     libucrt:nlsdata.obj
 0001:000021ac       ??_C@_03CNMDKL@May?$AA@    00000001800031ac     libucrt:nlsdata.obj
 0001:000021b0       ??_C@_03IDFGHECI@Jun?$AA@  00000001800031b0     libucrt:nlsdata.obj
 0001:000021b4       ??_C@_03LBGABGKK@Jul?$AA@  00000001800031b4     libucrt:nlsdata.obj
 0001:000021b8       ??_C@_03IFJFEIGA@Aug?$AA@  00000001800031b8     libucrt:nlsdata.obj
 0001:000021bc       ??_C@_03GGCAPAJC@Sep?$AA@  00000001800031bc     libucrt:nlsdata.obj
 0001:000021c0       ??_C@_03BMAOKBAD@Oct?$AA@  00000001800031c0     libucrt:nlsdata.obj
 0001:000021c4       ??_C@_03JPJOFNIA@Nov?$AA@  00000001800031c4     libucrt:nlsdata.obj
 0001:000021c8       ??_C@_03MKABNOCG@Dec?$AA@  00000001800031c8     libucrt:nlsdata.obj
 0001:000021d0       ??_C@_07CGJPFGJA@January?$AA@ 00000001800031d0     libucrt:nlsdata.obj
 0001:000021d8       ??_C@_08GNJGEPFN@February?$AA@ 00000001800031d8     libucrt:nlsdata.obj
 0001:000021e4       ??_C@_05HPCKOFNC@March?$AA@ 00000001800031e4     libucrt:nlsdata.obj
 0001:000021ec       ??_C@_05DMJDNLEJ@April?$AA@ 00000001800031ec     libucrt:nlsdata.obj
 0001:000021f4       ??_C@_04CNLMGBGM@June?$AA@ 00000001800031f4     libucrt:nlsdata.obj
 0001:000021fc       ??_C@_04MIEPOIFP@July?$AA@ 00000001800031fc     libucrt:nlsdata.obj
 0001:00002204       ??_C@_06LBBHFDDG@August?$AA@ 0000000180003204     libucrt:nlsdata.obj
 0001:00002210       ??_C@_09BHHEALKD@September?$AA@ 0000000180003210     libucrt:nlsdata.obj
 0001:00002220       ??_C@_07JJNFCEND@October?$AA@ 0000000180003220     libucrt:nlsdata.obj
 0001:00002228       ??_C@_08HCHEGEOA@November?$AA@ 0000000180003228     libucrt:nlsdata.obj
 0001:00002238       ??_C@_08EDHMEBNP@December?$AA@ 0000000180003238     libucrt:nlsdata.obj
 0001:00002244       ??_C@_02DEDBPAFC@AM?$AA@   0000000180003244     libucrt:nlsdata.obj
 0001:00002248       ??_C@_02CJNFDJBF@PM?$AA@   0000000180003248     libucrt:nlsdata.obj
 0001:00002250       ??_C@_08BPBNCDIB@MM?1dd?1yy?$AA@ 0000000180003250     libucrt:nlsdata.obj
 0001:00002260       ??_C@_0BE@CKGJFCPC@dddd?0?5MMMM?5dd?0?5yyyy?$AA@ 0000000180003260     libucrt:nlsdata.obj
 0001:00002278       ??_C@_08JCCMCCIL@HH?3mm?3ss?$AA@ 0000000180003278     libucrt:nlsdata.obj
 0001:00002288       ??_C@_17MBGCMIPB@?$AAS?$AAu?$AAn?$AA?$AA@ 0000000180003288     libucrt:nlsdata.obj
 0001:00002290       ??_C@_17KBOMKBF@?$AAM?$AAo?$AAn?$AA?$AA@ 0000000180003290     libucrt:nlsdata.obj
 0001:00002298       ??_C@_17BMKGEGOJ@?$AAT?$AAu?$AAe?$AA?$AA@ 0000000180003298     libucrt:nlsdata.obj
 0001:000022a0       ??_C@_17CJEDCEPE@?$AAW?$AAe?$AAd?$AA?$AA@ 00000001800032a0     libucrt:nlsdata.obj
 0001:000022a8       ??_C@_17PDPHAADD@?$AAT?$AAh?$AAu?$AA?$AA@ 00000001800032a8     libucrt:nlsdata.obj
 0001:000022b0       ??_C@_17HFOLPPLP@?$AAF?$AAr?$AAi?$AA?$AA@ 00000001800032b0     libucrt:nlsdata.obj
 0001:000022b8       ??_C@_17GGIBDPIH@?$AAS?$AAa?$AAt?$AA?$AA@ 00000001800032b8     libucrt:nlsdata.obj
 0001:000022c0       ??_C@_1O@IHNHDHPB@?$AAS?$AAu?$AAn?$AAd?$AAa?$AAy?$AA?$AA@ 00000001800032c0     libucrt:nlsdata.obj
 0001:000022d0       ??_C@_1O@MMNBFLIA@?$AAM?$AAo?$AAn?$AAd?$AAa?$AAy?$AA?$AA@ 00000001800032d0     libucrt:nlsdata.obj
 0001:000022e0       ??_C@_1BA@ENFBFFEK@?$AAT?$AAu?$AAe?$AAs?$AAd?$AAa?$AAy?$AA?$AA@ 00000001800032e0     libucrt:nlsdata.obj
 0001:000022f0       ??_C@_1BE@EBOGMDOH@?$AAW?$AAe?$AAd?$AAn?$AAe?$AAs?$AAd?$AAa?$AAy?$AA?$AA@ 00000001800032f0     libucrt:nlsdata.obj
 0001:00002308       ??_C@_1BC@HHMNLIHE@?$AAT?$AAh?$AAu?$AAr?$AAs?$AAd?$AAa?$AAy?$AA?$AA@ 0000000180003308     libucrt:nlsdata.obj
 0001:00002320       ??_C@_1O@PDICJHAG@?$AAF?$AAr?$AAi?$AAd?$AAa?$AAy?$AA?$AA@ 0000000180003320     libucrt:nlsdata.obj
 0001:00002330       ??_C@_1BC@ENMNNPAJ@?$AAS?$AAa?$AAt?$AAu?$AAr?$AAd?$AAa?$AAy?$AA?$AA@ 0000000180003330     libucrt:nlsdata.obj
 0001:00002348       ??_C@_17DKNBKCHM@?$AAJ?$AAa?$AAn?$AA?$AA@ 0000000180003348     libucrt:nlsdata.obj
 0001:00002350       ??_C@_17LMDJEKJN@?$AAF?$AAe?$AAb?$AA?$AA@ 0000000180003350     libucrt:nlsdata.obj
 0001:00002358       ??_C@_17CKNLEDEC@?$AAM?$AAa?$AAr?$AA?$AA@ 0000000180003358     libucrt:nlsdata.obj
 0001:00002360       ??_C@_17LFPOIHDD@?$AAA?$AAp?$AAr?$AA?$AA@ 0000000180003360     libucrt:nlsdata.obj
 0001:00002368       ??_C@_17PNNKMEED@?$AAM?$AAa?$AAy?$AA?$AA@ 0000000180003368     libucrt:nlsdata.obj
 0001:00002370       ??_C@_17KCJGOCPB@?$AAJ?$AAu?$AAn?$AA?$AA@ 0000000180003370     libucrt:nlsdata.obj
 0001:00002378       ??_C@_17IJPCKHK@?$AAJ?$AAu?$AAl?$AA?$AA@ 0000000180003378     libucrt:nlsdata.obj
 0001:00002380       ??_C@_17ICPELBCN@?$AAA?$AAu?$AAg?$AA?$AA@ 0000000180003380     libucrt:nlsdata.obj
 0001:00002388       ??_C@_17HCHCOKMG@?$AAS?$AAe?$AAp?$AA?$AA@ 0000000180003388     libucrt:nlsdata.obj
 0001:00002390       ??_C@_17FNLKOI@?$AAO?$AAc?$AAt?$AA?$AA@ 0000000180003390     libucrt:nlsdata.obj
 0001:00002398       ??_C@_17BBDMLCIG@?$AAN?$AAo?$AAv?$AA?$AA@ 0000000180003398     libucrt:nlsdata.obj
 0001:000023a0       ??_C@_17EGKACKIF@?$AAD?$AAe?$AAc?$AA?$AA@ 00000001800033a0     libucrt:nlsdata.obj
 0001:000023a8       ??_C@_1BA@EFMEIEBA@?$AAJ?$AAa?$AAn?$AAu?$AAa?$AAr?$AAy?$AA?$AA@ 00000001800033a8     libucrt:nlsdata.obj
 0001:000023b8       ??_C@_1BC@JGDDFFAM@?$AAF?$AAe?$AAb?$AAr?$AAu?$AAa?$AAr?$AAy?$AA?$AA@ 00000001800033b8     libucrt:nlsdata.obj
 0001:000023d0       ??_C@_1M@IKEENEDF@?$AAM?$AAa?$AAr?$AAc?$AAh?$AA?$AA@ 00000001800033d0     libucrt:nlsdata.obj
 0001:000023e0       ??_C@_1M@GJNLMHFD@?$AAA?$AAp?$AAr?$AAi?$AAl?$AA?$AA@ 00000001800033e0     libucrt:nlsdata.obj
 0001:000023f0       ??_C@_19EPFLPGAP@?$AAJ?$AAu?$AAn?$AAe?$AA?$AA@ 00000001800033f0     libucrt:nlsdata.obj
 0001:00002400       ??_C@_19BIFMLPCD@?$AAJ?$AAu?$AAl?$AAy?$AA?$AA@ 0000000180003400     libucrt:nlsdata.obj
 0001:00002410       ??_C@_1O@PAHLKOAC@?$AAA?$AAu?$AAg?$AAu?$AAs?$AAt?$AA?$AA@ 0000000180003410     libucrt:nlsdata.obj
 0001:00002420       ??_C@_1BE@DKAAMBJL@?$AAS?$AAe?$AAp?$AAt?$AAe?$AAm?$AAb?$AAe?$AAr?$AA?$AA@ 0000000180003420     libucrt:nlsdata.obj
 0001:00002438       ??_C@_1BA@EPANDLNG@?$AAO?$AAc?$AAt?$AAo?$AAb?$AAe?$AAr?$AA?$AA@ 0000000180003438     libucrt:nlsdata.obj
 0001:00002448       ??_C@_1BC@BGLIFPF@?$AAN?$AAo?$AAv?$AAe?$AAm?$AAb?$AAe?$AAr?$AA?$AA@ 0000000180003448     libucrt:nlsdata.obj
 0001:00002460       ??_C@_1BC@FEMKIFH@?$AAD?$AAe?$AAc?$AAe?$AAm?$AAb?$AAe?$AAr?$AA?$AA@ 0000000180003460     libucrt:nlsdata.obj
 0001:00002474       ??_C@_15ODEHAHHF@?$AAA?$AAM?$AA?$AA@ 0000000180003474     libucrt:nlsdata.obj
 0001:0000247c       ??_C@_15CLMNNGEL@?$AAP?$AAM?$AA?$AA@ 000000018000347c     libucrt:nlsdata.obj
 0001:00002488       ??_C@_1BC@IEBCMHCM@?$AAM?$AAM?$AA?1?$AAd?$AAd?$AA?1?$AAy?$AAy?$AA?$AA@ 0000000180003488     libucrt:nlsdata.obj
 0001:000024a0       ??_C@_1CI@KNAKOEBC@?$AAd?$AAd?$AAd?$AAd?$AA?0?$AA?5?$AAM?$AAM?$AAM?$AAM?$AA?5?$AAd?$AAd?$AA?0?$AA?5?$AAy?$AAy?$AAy?$AAy?$AA?$AA@ 00000001800034a0     libucrt:nlsdata.obj
 0001:000024c8       ??_C@_1BC@GDGBMEMK@?$AAH?$AAH?$AA?3?$AAm?$AAm?$AA?3?$AAs?$AAs?$AA?$AA@ 00000001800034c8     libucrt:nlsdata.obj
 0001:000024e0       ??_C@_1M@BMHNFIME@?$AAe?$AAn?$AA?9?$AAU?$AAS?$AA?$AA@ 00000001800034e0     libucrt:nlsdata.obj
 0001:000024f0       __newctype                 00000001800034f0     libucrt:ctype.obj
 0001:000027f0       __newclmap                 00000001800037f0     libucrt:ctype.obj
 0001:00002970       __newcumap                 0000000180003970     libucrt:ctype.obj
 0001:00003930       ??_C@_15EMKDOKLE@?$AAa?$AAr?$AA?$AA@ 0000000180004930     libucrt:lcidtoname_downlevel.obj
 0001:00003938       ??_C@_15KNPADPLH@?$AAb?$AAg?$AA?$AA@ 0000000180004938     libucrt:lcidtoname_downlevel.obj
 0001:00003940       ??_C@_15EDMHLDMO@?$AAc?$AAa?$AA?$AA@ 0000000180004940     libucrt:lcidtoname_downlevel.obj
 0001:00003948       ??_C@_1O@BPEAJADD@?$AAz?$AAh?$AA?9?$AAC?$AAH?$AAS?$AA?$AA@ 0000000180004948     libucrt:lcidtoname_downlevel.obj
 0001:00003958       ??_C@_15LJNHCMNK@?$AAc?$AAs?$AA?$AA@ 0000000180004958     libucrt:lcidtoname_downlevel.obj
 0001:00003960       ??_C@_15FOMCIDHG@?$AAd?$AAa?$AA?$AA@ 0000000180004960     libucrt:lcidtoname_downlevel.obj
 0001:00003968       ??_C@_15NBKABECB@?$AAd?$AAe?$AA?$AA@ 0000000180004968     libucrt:lcidtoname_downlevel.obj
 0001:00003970       ??_C@_15GHPEIIAO@?$AAe?$AAl?$AA?$AA@ 0000000180004970     libucrt:lcidtoname_downlevel.obj
 0001:00003978       ??_C@_15MNPNEAIF@?$AAe?$AAn?$AA?$AA@ 0000000180004978     libucrt:lcidtoname_downlevel.obj
 0001:00003980       ??_C@_15GPIOMPMH@?$AAe?$AAs?$AA?$AA@ 0000000180004980     libucrt:lcidtoname_downlevel.obj
 0001:00003988       ??_C@_15NGLOAKJC@?$AAf?$AAi?$AA?$AA@ 0000000180004988     libucrt:lcidtoname_downlevel.obj
 0001:00003990       ??_C@_15FBKGNKAM@?$AAf?$AAr?$AA?$AA@ 0000000180004990     libucrt:lcidtoname_downlevel.obj
 0001:00003998       ??_C@_15KGGCNEFK@?$AAh?$AAe?$AA?$AA@ 0000000180004998     libucrt:lcidtoname_downlevel.obj
 0001:000039a0       ??_C@_15PGHLIDMF@?$AAh?$AAu?$AA?$AA@ 00000001800049a0     libucrt:lcidtoname_downlevel.obj
 0001:000039a8       ??_C@_15BIEMAPLM@?$AAi?$AAs?$AA?$AA@ 00000001800049a8     libucrt:lcidtoname_downlevel.obj
 0001:000039b0       ??_C@_15IFJLDHAF@?$AAi?$AAt?$AA?$AA@ 00000001800049b0     libucrt:lcidtoname_downlevel.obj
 0001:000039b8       ??_C@_15GEMIOCAG@?$AAj?$AAa?$AA?$AA@ 00000001800049b8     libucrt:lcidtoname_downlevel.obj
 0001:000039c0       ??_C@_15EPELEGJA@?$AAk?$AAo?$AA?$AA@ 00000001800049c0     libucrt:lcidtoname_downlevel.obj
 0001:000039c8       ??_C@_15NDDHIMN@?$AAn?$AAl?$AA?$AA@ 00000001800049c8     libucrt:lcidtoname_downlevel.obj
 0001:000039d0       ??_C@_15BPIGNHCD@?$AAn?$AAo?$AA?$AA@ 00000001800049d0     libucrt:lcidtoname_downlevel.obj
 0001:000039d8       ??_C@_15DEOPBLCG@?$AAp?$AAl?$AA?$AA@ 00000001800049d8     libucrt:lcidtoname_downlevel.obj
 0001:000039e0       ??_C@_15KBECGEFG@?$AAp?$AAt?$AA?$AA@ 00000001800049e0     libucrt:lcidtoname_downlevel.obj
 0001:000039e8       ??_C@_15GLJCBFMD@?$AAr?$AAo?$AA?$AA@ 00000001800049e8     libucrt:lcidtoname_downlevel.obj
 0001:000039f0       ??_C@_15FEDGKCDI@?$AAr?$AAu?$AA?$AA@ 00000001800049f0     libucrt:lcidtoname_downlevel.obj
 0001:000039f8       ??_C@_15GLKMLLHM@?$AAh?$AAr?$AA?$AA@ 00000001800049f8     libucrt:lcidtoname_downlevel.obj
 0001:00003a00       ??_C@_15CPKMFBDB@?$AAs?$AAk?$AA?$AA@ 0000000180004a00     libucrt:lcidtoname_downlevel.obj
 0001:00003a08       ??_C@_15BAAIOGMK@?$AAs?$AAq?$AA?$AA@ 0000000180004a08     libucrt:lcidtoname_downlevel.obj
 0001:00003a10       ??_C@_15INNPNOHD@?$AAs?$AAv?$AA?$AA@ 0000000180004a10     libucrt:lcidtoname_downlevel.obj
 0001:00003a18       ??_C@_15CABMMOGH@?$AAt?$AAh?$AA?$AA@ 0000000180004a18     libucrt:lcidtoname_downlevel.obj
 0001:00003a20       ??_C@_15BPLIHJJM@?$AAt?$AAr?$AA?$AA@ 0000000180004a20     libucrt:lcidtoname_downlevel.obj
 0001:00003a28       ??_C@_15NEOEKKDJ@?$AAu?$AAr?$AA?$AA@ 0000000180004a28     libucrt:lcidtoname_downlevel.obj
 0001:00003a30       ??_C@_15NFICGAJK@?$AAi?$AAd?$AA?$AA@ 0000000180004a30     libucrt:lcidtoname_downlevel.obj
 0001:00003a38       ??_C@_15PJPFLCCM@?$AAu?$AAk?$AA?$AA@ 0000000180004a38     libucrt:lcidtoname_downlevel.obj
 0001:00003a40       ??_C@_15HPJPHDM@?$AAb?$AAe?$AA?$AA@ 0000000180004a40     libucrt:lcidtoname_downlevel.obj
 0001:00003a48       ??_C@_15LCHLGJII@?$AAs?$AAl?$AA?$AA@ 0000000180004a48     libucrt:lcidtoname_downlevel.obj
 0001:00003a50       ??_C@_15PCFJPHHO@?$AAe?$AAt?$AA?$AA@ 0000000180004a50     libucrt:lcidtoname_downlevel.obj
 0001:00003a58       ??_C@_15HPFPGODN@?$AAl?$AAv?$AA?$AA@ 0000000180004a58     libucrt:lcidtoname_downlevel.obj
 0001:00003a60       ??_C@_15NFFGKGLG@?$AAl?$AAt?$AA?$AA@ 0000000180004a60     libucrt:lcidtoname_downlevel.obj
 0001:00003a68       ??_C@_15BDAKCCHN@?$AAf?$AAa?$AA?$AA@ 0000000180004a68     libucrt:lcidtoname_downlevel.obj
 0001:00003a70       ??_C@_15NFGIAIAJ@?$AAv?$AAi?$AA?$AA@ 0000000180004a70     libucrt:lcidtoname_downlevel.obj
 0001:00003a78       ??_C@_15LMKNDMHN@?$AAh?$AAy?$AA?$AA@ 0000000180004a78     libucrt:lcidtoname_downlevel.obj
 0001:00003a80       ??_C@_15IJBHMCFL@?$AAa?$AAz?$AA?$AA@ 0000000180004a80     libucrt:lcidtoname_downlevel.obj
 0001:00003a88       ??_C@_15EKOFJABL@?$AAe?$AAu?$AA?$AA@ 0000000180004a88     libucrt:lcidtoname_downlevel.obj
 0001:00003a90       ??_C@_15BGHADCNK@?$AAm?$AAk?$AA?$AA@ 0000000180004a90     libucrt:lcidtoname_downlevel.obj
 0001:00003a98       ??_C@_15JDNICKHM@?$AAa?$AAf?$AA?$AA@ 0000000180004a98     libucrt:lcidtoname_downlevel.obj
 0001:00003aa0       ??_C@_15KPJEDBKD@?$AAk?$AAa?$AA?$AA@ 0000000180004aa0     libucrt:lcidtoname_downlevel.obj
 0001:00003aa8       ??_C@_15PDNFFFEO@?$AAf?$AAo?$AA?$AA@ 0000000180004aa8     libucrt:lcidtoname_downlevel.obj
 0001:00003ab0       ??_C@_15OMLEGLOC@?$AAh?$AAi?$AA?$AA@ 0000000180004ab0     libucrt:lcidtoname_downlevel.obj
 0001:00003ab8       ??_C@_15IDNNENKK@?$AAm?$AAs?$AA?$AA@ 0000000180004ab8     libucrt:lcidtoname_downlevel.obj
 0001:00003ac0       ??_C@_15MACJNBMH@?$AAk?$AAk?$AA?$AA@ 0000000180004ac0     libucrt:lcidtoname_downlevel.obj
 0001:00003ac8       ??_C@_15DKDJEOND@?$AAk?$AAy?$AA?$AA@ 0000000180004ac8     libucrt:lcidtoname_downlevel.obj
 0001:00003ad0       ??_C@_15DFGDLJBG@?$AAs?$AAw?$AA?$AA@ 0000000180004ad0     libucrt:lcidtoname_downlevel.obj
 0001:00003ad8       ??_C@_15BBFAICNG@?$AAu?$AAz?$AA?$AA@ 0000000180004ad8     libucrt:lcidtoname_downlevel.obj
 0001:00003ae0       ??_C@_15DKNDCGEA@?$AAt?$AAt?$AA?$AA@ 0000000180004ae0     libucrt:lcidtoname_downlevel.obj
 0001:00003ae8       ??_C@_15MGIFMDPL@?$AAp?$AAa?$AA?$AA@ 0000000180004ae8     libucrt:lcidtoname_downlevel.obj
 0001:00003af0       ??_C@_15HCNDBBA@?$AAg?$AAu?$AA?$AA@ 0000000180004af0     libucrt:lcidtoname_downlevel.obj
 0001:00003af8       ??_C@_15FNBEIBON@?$AAt?$AAa?$AA?$AA@ 0000000180004af8     libucrt:lcidtoname_downlevel.obj
 0001:00003b00       ??_C@_15NCHGBGLK@?$AAt?$AAe?$AA?$AA@ 0000000180004b00     libucrt:lcidtoname_downlevel.obj
 0001:00003b08       ??_C@_15PHPHCBPF@?$AAk?$AAn?$AA?$AA@ 0000000180004b08     libucrt:lcidtoname_downlevel.obj
 0001:00003b10       ??_C@_15DLGBCKMP@?$AAm?$AAr?$AA?$AA@ 0000000180004b10     libucrt:lcidtoname_downlevel.obj
 0001:00003b18       ??_C@_15EABBLBFF@?$AAs?$AAa?$AA?$AA@ 0000000180004b18     libucrt:lcidtoname_downlevel.obj
 0001:00003b20       ??_C@_15CBKOMCOI@?$AAm?$AAn?$AA?$AA@ 0000000180004b20     libucrt:lcidtoname_downlevel.obj
 0001:00003b28       ??_C@_15CKDMCJAF@?$AAg?$AAl?$AA?$AA@ 0000000180004b28     libucrt:lcidtoname_downlevel.obj
 0001:00003b30       ??_C@_17CNJFBPG@?$AAk?$AAo?$AAk?$AA?$AA@ 0000000180004b30     libucrt:lcidtoname_downlevel.obj
 0001:00003b38       ??_C@_17FFBJICPL@?$AAs?$AAy?$AAr?$AA?$AA@ 0000000180004b38     libucrt:lcidtoname_downlevel.obj
 0001:00003b40       ??_C@_17KPNDCPAF@?$AAd?$AAi?$AAv?$AA?$AA@ 0000000180004b40     libucrt:lcidtoname_downlevel.obj
 0001:00003b48       ??_C@_11LOCGONAA@?$AA?$AA@ 0000000180004b48     libucrt:lcidtoname_downlevel.obj
 0001:00003b50       ??_C@_1M@OKAHONE@?$AAa?$AAr?$AA?9?$AAS?$AAA?$AA?$AA@ 0000000180004b50     libucrt:lcidtoname_downlevel.obj
 0001:00003b60       ??_C@_1M@FFFIGIGK@?$AAb?$AAg?$AA?9?$AAB?$AAG?$AA?$AA@ 0000000180004b60     libucrt:lcidtoname_downlevel.obj
 0001:00003b70       ??_C@_1M@BJNKEDC@?$AAc?$AAa?$AA?9?$AAE?$AAS?$AA?$AA@ 0000000180004b70     libucrt:lcidtoname_downlevel.obj
 0001:00003b80       ??_C@_1M@IJJHFJHA@?$AAc?$AAs?$AA?9?$AAC?$AAZ?$AA?$AA@ 0000000180004b80     libucrt:lcidtoname_downlevel.obj
 0001:00003b90       ??_C@_1M@CLPEOBGI@?$AAd?$AAa?$AA?9?$AAD?$AAK?$AA?$AA@ 0000000180004b90     libucrt:lcidtoname_downlevel.obj
 0001:00003ba0       ??_C@_1M@MCMADGCB@?$AAd?$AAe?$AA?9?$AAD?$AAE?$AA?$AA@ 0000000180004ba0     libucrt:lcidtoname_downlevel.obj
 0001:00003bb0       ??_C@_1M@OOCKEMAM@?$AAe?$AAl?$AA?9?$AAG?$AAR?$AA?$AA@ 0000000180004bb0     libucrt:lcidtoname_downlevel.obj
 0001:00003bc0       ??_C@_1M@DDNJFGID@?$AAf?$AAi?$AA?9?$AAF?$AAI?$AA?$AA@ 0000000180004bc0     libucrt:lcidtoname_downlevel.obj
 0001:00003bd0       ??_C@_1M@GLIPPMAC@?$AAf?$AAr?$AA?9?$AAF?$AAR?$AA?$AA@ 0000000180004bd0     libucrt:lcidtoname_downlevel.obj
 0001:00003be0       ??_C@_1M@GFMCHPE@?$AAh?$AAe?$AA?9?$AAI?$AAL?$AA?$AA@ 0000000180004be0     libucrt:lcidtoname_downlevel.obj
 0001:00003bf0       ??_C@_1M@MHLPGNKM@?$AAh?$AAu?$AA?9?$AAH?$AAU?$AA?$AA@ 0000000180004bf0     libucrt:lcidtoname_downlevel.obj
 0001:00003c00       ??_C@_1M@LPDDNNPN@?$AAi?$AAs?$AA?9?$AAI?$AAS?$AA?$AA@ 0000000180004c00     libucrt:lcidtoname_downlevel.obj
 0001:00003c10       ??_C@_1M@MADIPODN@?$AAi?$AAt?$AA?9?$AAI?$AAT?$AA?$AA@ 0000000180004c10     libucrt:lcidtoname_downlevel.obj
 0001:00003c20       ??_C@_1M@IHBJJGG@?$AAn?$AAl?$AA?9?$AAN?$AAL?$AA?$AA@ 0000000180004c20     libucrt:lcidtoname_downlevel.obj
 0001:00003c30       ??_C@_1M@EANAGDL@?$AAn?$AAb?$AA?9?$AAN?$AAO?$AA?$AA@ 0000000180004c30     libucrt:lcidtoname_downlevel.obj
 0001:00003c40       ??_C@_1M@NEIEMEGP@?$AAp?$AAl?$AA?9?$AAP?$AAL?$AA?$AA@ 0000000180004c40     libucrt:lcidtoname_downlevel.obj
 0001:00003c50       ??_C@_1M@BOCFIGEP@?$AAp?$AAt?$AA?9?$AAB?$AAR?$AA?$AA@ 0000000180004c50     libucrt:lcidtoname_downlevel.obj
 0001:00003c60       ??_C@_1M@IMPFOPBG@?$AAr?$AAo?$AA?9?$AAR?$AAO?$AA?$AA@ 0000000180004c60     libucrt:lcidtoname_downlevel.obj
 0001:00003c70       ??_C@_1M@IDNNEJMM@?$AAr?$AAu?$AA?9?$AAR?$AAU?$AA?$AA@ 0000000180004c70     libucrt:lcidtoname_downlevel.obj
 0001:00003c80       ??_C@_1M@LILEEOGM@?$AAh?$AAr?$AA?9?$AAH?$AAR?$AA?$AA@ 0000000180004c80     libucrt:lcidtoname_downlevel.obj
 0001:00003c90       ??_C@_1M@FKIFEHPB@?$AAs?$AAk?$AA?9?$AAS?$AAK?$AA?$AA@ 0000000180004c90     libucrt:lcidtoname_downlevel.obj
 0001:00003ca0       ??_C@_1M@LJMAMNPJ@?$AAs?$AAq?$AA?9?$AAA?$AAL?$AA?$AA@ 0000000180004ca0     libucrt:lcidtoname_downlevel.obj
 0001:00003cb0       ??_C@_1M@GIAKDKJK@?$AAs?$AAv?$AA?9?$AAS?$AAE?$AA?$AA@ 0000000180004cb0     libucrt:lcidtoname_downlevel.obj
 0001:00003cc0       ??_C@_1M@MKJKIKCL@?$AAt?$AAh?$AA?9?$AAT?$AAH?$AA?$AA@ 0000000180004cc0     libucrt:lcidtoname_downlevel.obj
 0001:00003cd0       ??_C@_1M@MFLCCMPB@?$AAt?$AAr?$AA?9?$AAT?$AAR?$AA?$AA@ 0000000180004cd0     libucrt:lcidtoname_downlevel.obj
 0001:00003ce0       ??_C@_1M@OIJHDKJN@?$AAu?$AAr?$AA?9?$AAP?$AAK?$AA?$AA@ 0000000180004ce0     libucrt:lcidtoname_downlevel.obj
 0001:00003cf0       ??_C@_1M@LHIPCIEK@?$AAi?$AAd?$AA?9?$AAI?$AAD?$AA?$AA@ 0000000180004cf0     libucrt:lcidtoname_downlevel.obj
 0001:00003d00       ??_C@_1M@MFMOBGI@?$AAu?$AAk?$AA?9?$AAU?$AAA?$AA?$AA@ 0000000180004d00     libucrt:lcidtoname_downlevel.obj
 0001:00003d10       ??_C@_1M@OBGLJIPL@?$AAb?$AAe?$AA?9?$AAB?$AAY?$AA?$AA@ 0000000180004d10     libucrt:lcidtoname_downlevel.obj
 0001:00003d20       ??_C@_1M@BCFAJEAD@?$AAs?$AAl?$AA?9?$AAS?$AAI?$AA?$AA@ 0000000180004d20     libucrt:lcidtoname_downlevel.obj
 0001:00003d30       ??_C@_1M@FKFFEDDN@?$AAe?$AAt?$AA?9?$AAE?$AAE?$AA?$AA@ 0000000180004d30     libucrt:lcidtoname_downlevel.obj
 0001:00003d40       ??_C@_1M@KGKKAACI@?$AAl?$AAv?$AA?9?$AAL?$AAV?$AA?$AA@ 0000000180004d40     libucrt:lcidtoname_downlevel.obj
 0001:00003d50       ??_C@_1M@IFGBIJO@?$AAl?$AAt?$AA?9?$AAL?$AAT?$AA?$AA@ 0000000180004d50     libucrt:lcidtoname_downlevel.obj
 0001:00003d60       ??_C@_1M@FGEAHEDM@?$AAf?$AAa?$AA?9?$AAI?$AAR?$AA?$AA@ 0000000180004d60     libucrt:lcidtoname_downlevel.obj
 0001:00003d70       ??_C@_1M@KBMAIBFN@?$AAv?$AAi?$AA?9?$AAV?$AAN?$AA?$AA@ 0000000180004d70     libucrt:lcidtoname_downlevel.obj
 0001:00003d80       ??_C@_1M@GPCBKDJK@?$AAh?$AAy?$AA?9?$AAA?$AAM?$AA?$AA@ 0000000180004d80     libucrt:lcidtoname_downlevel.obj
 0001:00003d90       ??_C@_1BG@BECMDDJB@?$AAa?$AAz?$AA?9?$AAA?$AAZ?$AA?9?$AAL?$AAa?$AAt?$AAn?$AA?$AA@ 0000000180004d90     libucrt:lcidtoname_downlevel.obj
 0001:00003da8       ??_C@_1M@MAOFCAEA@?$AAe?$AAu?$AA?9?$AAE?$AAS?$AA?$AA@ 0000000180004da8     libucrt:lcidtoname_downlevel.obj
 0001:00003db8       ??_C@_1M@IGHABKPI@?$AAm?$AAk?$AA?9?$AAM?$AAK?$AA?$AA@ 0000000180004db8     libucrt:lcidtoname_downlevel.obj
 0001:00003dc8       ??_C@_1M@IAIGNEJG@?$AAt?$AAn?$AA?9?$AAZ?$AAA?$AA?$AA@ 0000000180004dc8     libucrt:lcidtoname_downlevel.obj
 0001:00003dd8       ??_C@_1M@IIJCOJFA@?$AAx?$AAh?$AA?9?$AAZ?$AAA?$AA?$AA@ 0000000180004dd8     libucrt:lcidtoname_downlevel.obj
 0001:00003de8       ??_C@_1M@LGPJHNJH@?$AAz?$AAu?$AA?9?$AAZ?$AAA?$AA?$AA@ 0000000180004de8     libucrt:lcidtoname_downlevel.obj
 0001:00003df8       ??_C@_1M@HOKAOIO@?$AAa?$AAf?$AA?9?$AAZ?$AAA?$AA?$AA@ 0000000180004df8     libucrt:lcidtoname_downlevel.obj
 0001:00003e08       ??_C@_1M@DPCLHLIE@?$AAk?$AAa?$AA?9?$AAG?$AAE?$AA?$AA@ 0000000180004e08     libucrt:lcidtoname_downlevel.obj
 0001:00003e18       ??_C@_1M@BLKMHJBI@?$AAf?$AAo?$AA?9?$AAF?$AAO?$AA?$AA@ 0000000180004e18     libucrt:lcidtoname_downlevel.obj
 0001:00003e28       ??_C@_1M@LGGJAPPB@?$AAh?$AAi?$AA?9?$AAI?$AAN?$AA?$AA@ 0000000180004e28     libucrt:lcidtoname_downlevel.obj
 0001:00003e38       ??_C@_1M@FIKPIHFE@?$AAm?$AAt?$AA?9?$AAM?$AAT?$AA?$AA@ 0000000180004e38     libucrt:lcidtoname_downlevel.obj
 0001:00003e48       ??_C@_1M@HEGGPBFA@?$AAs?$AAe?$AA?9?$AAN?$AAO?$AA?$AA@ 0000000180004e48     libucrt:lcidtoname_downlevel.obj
 0001:00003e58       ??_C@_1M@EIBJEEPA@?$AAm?$AAs?$AA?9?$AAM?$AAY?$AA?$AA@ 0000000180004e58     libucrt:lcidtoname_downlevel.obj
 0001:00003e68       ??_C@_1M@FHLBGMPP@?$AAk?$AAk?$AA?9?$AAK?$AAZ?$AA?$AA@ 0000000180004e68     libucrt:lcidtoname_downlevel.obj
 0001:00003e78       ??_C@_1M@NGJJLCGI@?$AAk?$AAy?$AA?9?$AAK?$AAG?$AA?$AA@ 0000000180004e78     libucrt:lcidtoname_downlevel.obj
 0001:00003e88       ??_C@_1M@GIENNBFC@?$AAs?$AAw?$AA?9?$AAK?$AAE?$AA?$AA@ 0000000180004e88     libucrt:lcidtoname_downlevel.obj
 0001:00003e98       ??_C@_1BG@NDGMJIMJ@?$AAu?$AAz?$AA?9?$AAU?$AAZ?$AA?9?$AAL?$AAa?$AAt?$AAn?$AA?$AA@ 0000000180004e98     libucrt:lcidtoname_downlevel.obj
 0001:00003eb0       ??_C@_1M@IDCCIHBC@?$AAt?$AAt?$AA?9?$AAR?$AAU?$AA?$AA@ 0000000180004eb0     libucrt:lcidtoname_downlevel.obj
 0001:00003ec0       ??_C@_1M@LOICPMOJ@?$AAb?$AAn?$AA?9?$AAI?$AAN?$AA?$AA@ 0000000180004ec0     libucrt:lcidtoname_downlevel.obj
 0001:00003ed0       ??_C@_1M@KPKKNEAH@?$AAp?$AAa?$AA?9?$AAI?$AAN?$AA?$AA@ 0000000180004ed0     libucrt:lcidtoname_downlevel.obj
 0001:00003ee0       ??_C@_1M@PJGPPBOG@?$AAg?$AAu?$AA?9?$AAI?$AAN?$AA?$AA@ 0000000180004ee0     libucrt:lcidtoname_downlevel.obj
 0001:00003ef0       ??_C@_1M@KMKMOPHI@?$AAt?$AAa?$AA?9?$AAI?$AAN?$AA?$AA@ 0000000180004ef0     libucrt:lcidtoname_downlevel.obj
 0001:00003f00       ??_C@_1M@KFEHEPAC@?$AAt?$AAe?$AA?9?$AAI?$AAN?$AA?$AA@ 0000000180004f00     libucrt:lcidtoname_downlevel.obj
 0001:00003f10       ??_C@_1M@CDCLMGHI@?$AAk?$AAn?$AA?9?$AAI?$AAN?$AA?$AA@ 0000000180004f10     libucrt:lcidtoname_downlevel.obj
 0001:00003f20       ??_C@_1M@MIODLDKF@?$AAm?$AAl?$AA?9?$AAI?$AAN?$AA?$AA@ 0000000180004f20     libucrt:lcidtoname_downlevel.obj
 0001:00003f30       ??_C@_1M@PBIEACPO@?$AAm?$AAr?$AA?9?$AAI?$AAN?$AA?$AA@ 0000000180004f30     libucrt:lcidtoname_downlevel.obj
 0001:00003f40       ??_C@_1M@NIDEAGPH@?$AAs?$AAa?$AA?9?$AAI?$AAN?$AA?$AA@ 0000000180004f40     libucrt:lcidtoname_downlevel.obj
 0001:00003f50       ??_C@_1M@FHIHCBIO@?$AAm?$AAn?$AA?9?$AAM?$AAN?$AA?$AA@ 0000000180004f50     libucrt:lcidtoname_downlevel.obj
 0001:00003f60       ??_C@_1M@JAIJPENP@?$AAc?$AAy?$AA?9?$AAG?$AAB?$AA?$AA@ 0000000180004f60     libucrt:lcidtoname_downlevel.obj
 0001:00003f70       ??_C@_1M@PHGFBEPN@?$AAg?$AAl?$AA?9?$AAE?$AAS?$AA?$AA@ 0000000180004f70     libucrt:lcidtoname_downlevel.obj
 0001:00003f80       ??_C@_1O@KPIPDNCP@?$AAk?$AAo?$AAk?$AA?9?$AAI?$AAN?$AA?$AA@ 0000000180004f80     libucrt:lcidtoname_downlevel.obj
 0001:00003f90       ??_C@_1O@KNHJLDJA@?$AAs?$AAy?$AAr?$AA?9?$AAS?$AAY?$AA?$AA@ 0000000180004f90     libucrt:lcidtoname_downlevel.obj
 0001:00003fa0       ??_C@_1O@MKEKBLAH@?$AAd?$AAi?$AAv?$AA?9?$AAM?$AAV?$AA?$AA@ 0000000180004fa0     libucrt:lcidtoname_downlevel.obj
 0001:00003fb0       ??_C@_1O@OHDCKDDF@?$AAq?$AAu?$AAz?$AA?9?$AAB?$AAO?$AA?$AA@ 0000000180004fb0     libucrt:lcidtoname_downlevel.obj
 0001:00003fc0       ??_C@_1M@LEPJNLFD@?$AAn?$AAs?$AA?9?$AAZ?$AAA?$AA?$AA@ 0000000180004fc0     libucrt:lcidtoname_downlevel.obj
 0001:00003fd0       ??_C@_1M@OMLEIIJB@?$AAm?$AAi?$AA?9?$AAN?$AAZ?$AA?$AA@ 0000000180004fd0     libucrt:lcidtoname_downlevel.obj
 0001:00003fe0       ??_C@_1M@PMPEAILG@?$AAa?$AAr?$AA?9?$AAI?$AAQ?$AA?$AA@ 0000000180004fe0     libucrt:lcidtoname_downlevel.obj
 0001:00003ff0       ??_C@_1M@CNKPNOEE@?$AAd?$AAe?$AA?9?$AAC?$AAH?$AA?$AA@ 0000000180004ff0     libucrt:lcidtoname_downlevel.obj
 0001:00004000       ??_C@_1M@LKMGMLKO@?$AAe?$AAn?$AA?9?$AAG?$AAB?$AA?$AA@ 0000000180005000     libucrt:lcidtoname_downlevel.obj
 0001:00004010       ??_C@_1M@PGKJFFGL@?$AAe?$AAs?$AA?9?$AAM?$AAX?$AA?$AA@ 0000000180005010     libucrt:lcidtoname_downlevel.obj
 0001:00004020       ??_C@_1M@DNNANBDC@?$AAf?$AAr?$AA?9?$AAB?$AAE?$AA?$AA@ 0000000180005020     libucrt:lcidtoname_downlevel.obj
 0001:00004030       ??_C@_1M@HLGMDFHM@?$AAi?$AAt?$AA?9?$AAC?$AAH?$AA?$AA@ 0000000180005030     libucrt:lcidtoname_downlevel.obj
 0001:00004040       ??_C@_1M@CLLBGJH@?$AAn?$AAl?$AA?9?$AAB?$AAE?$AA?$AA@ 0000000180005040     libucrt:lcidtoname_downlevel.obj
 0001:00004050       ??_C@_1M@BODBOGLF@?$AAn?$AAn?$AA?9?$AAN?$AAO?$AA?$AA@ 0000000180005050     libucrt:lcidtoname_downlevel.obj
 0001:00004060       ??_C@_1M@HFFAHKAD@?$AAp?$AAt?$AA?9?$AAP?$AAT?$AA?$AA@ 0000000180005060     libucrt:lcidtoname_downlevel.obj
 0001:00004070       ??_C@_1BG@LNOAKHIE@?$AAs?$AAr?$AA?9?$AAS?$AAP?$AA?9?$AAL?$AAa?$AAt?$AAn?$AA?$AA@ 0000000180005070     libucrt:lcidtoname_downlevel.obj
 0001:00004088       ??_C@_1M@HBMHBGAK@?$AAs?$AAv?$AA?9?$AAF?$AAI?$AA?$AA@ 0000000180005088     libucrt:lcidtoname_downlevel.obj
 0001:00004098       ??_C@_1BG@DGCJGJBE@?$AAa?$AAz?$AA?9?$AAA?$AAZ?$AA?9?$AAC?$AAy?$AAr?$AAl?$AA?$AA@ 0000000180005098     libucrt:lcidtoname_downlevel.obj
 0001:000040b0       ??_C@_1M@KEJDAAHB@?$AAs?$AAe?$AA?9?$AAS?$AAE?$AA?$AA@ 00000001800050b0     libucrt:lcidtoname_downlevel.obj
 0001:000040c0       ??_C@_1M@HEIBJJAD@?$AAm?$AAs?$AA?9?$AAB?$AAN?$AA?$AA@ 00000001800050c0     libucrt:lcidtoname_downlevel.obj
 0001:000040d0       ??_C@_1BG@PBGJMCEM@?$AAu?$AAz?$AA?9?$AAU?$AAZ?$AA?9?$AAC?$AAy?$AAr?$AAl?$AA?$AA@ 00000001800050d0     libucrt:lcidtoname_downlevel.obj
 0001:000040e8       ??_C@_1O@LAOBCMDF@?$AAq?$AAu?$AAz?$AA?9?$AAE?$AAC?$AA?$AA@ 00000001800050e8     libucrt:lcidtoname_downlevel.obj
 0001:000040f8       ??_C@_1M@POEEMAIO@?$AAa?$AAr?$AA?9?$AAE?$AAG?$AA?$AA@ 00000001800050f8     libucrt:lcidtoname_downlevel.obj
 0001:00004108       ??_C@_1M@EFAKDEDL@?$AAz?$AAh?$AA?9?$AAH?$AAK?$AA?$AA@ 0000000180005108     libucrt:lcidtoname_downlevel.obj
 0001:00004118       ??_C@_1M@HKKIJHGI@?$AAd?$AAe?$AA?9?$AAA?$AAT?$AA?$AA@ 0000000180005118     libucrt:lcidtoname_downlevel.obj
 0001:00004128       ??_C@_1M@KBFBEHJF@?$AAe?$AAn?$AA?9?$AAA?$AAU?$AA?$AA@ 0000000180005128     libucrt:lcidtoname_downlevel.obj
 0001:00004138       ??_C@_1M@MNPLFAAH@?$AAe?$AAs?$AA?9?$AAE?$AAS?$AA?$AA@ 0000000180005138     libucrt:lcidtoname_downlevel.obj
 0001:00004148       ??_C@_1M@HJOOJFMA@?$AAf?$AAr?$AA?9?$AAC?$AAA?$AA?$AA@ 0000000180005148     libucrt:lcidtoname_downlevel.obj
 0001:00004158       ??_C@_1BG@JPOFPNAB@?$AAs?$AAr?$AA?9?$AAS?$AAP?$AA?9?$AAC?$AAy?$AAr?$AAl?$AA?$AA@ 0000000180005158     libucrt:lcidtoname_downlevel.obj
 0001:00004170       ??_C@_1M@LNFOCMOB@?$AAs?$AAe?$AA?9?$AAF?$AAI?$AA?$AA@ 0000000180005170     libucrt:lcidtoname_downlevel.obj
 0001:00004180       ??_C@_1O@MGJBOAMB@?$AAq?$AAu?$AAz?$AA?9?$AAP?$AAE?$AA?$AA@ 0000000180005180     libucrt:lcidtoname_downlevel.obj
 0001:00004190       ??_C@_1M@GJINLBOK@?$AAa?$AAr?$AA?9?$AAL?$AAY?$AA?$AA@ 0000000180005190     libucrt:lcidtoname_downlevel.obj
 0001:000041a0       ??_C@_1M@GGMNHJNL@?$AAz?$AAh?$AA?9?$AAS?$AAG?$AA?$AA@ 00000001800051a0     libucrt:lcidtoname_downlevel.obj
 0001:000041b0       ??_C@_1M@HOIKODND@?$AAd?$AAe?$AA?9?$AAL?$AAU?$AA?$AA@ 00000001800051b0     libucrt:lcidtoname_downlevel.obj
 0001:000041c0       ??_C@_1M@DDOCCGFG@?$AAe?$AAn?$AA?9?$AAC?$AAA?$AA?$AA@ 00000001800051c0     libucrt:lcidtoname_downlevel.obj
 0001:000041d0       ??_C@_1M@BNOEMJLF@?$AAe?$AAs?$AA?9?$AAG?$AAT?$AA?$AA@ 00000001800051d0     libucrt:lcidtoname_downlevel.obj
 0001:000041e0       ??_C@_1M@EOGNKEK@?$AAf?$AAr?$AA?9?$AAC?$AAH?$AA?$AA@ 00000001800051e0     libucrt:lcidtoname_downlevel.obj
 0001:000041f0       ??_C@_1M@FLIDJFHL@?$AAh?$AAr?$AA?9?$AAB?$AAA?$AA?$AA@ 00000001800051f0     libucrt:lcidtoname_downlevel.obj
 0001:00004200       ??_C@_1O@FMCELNAJ@?$AAs?$AAm?$AAj?$AA?9?$AAN?$AAO?$AA?$AA@ 0000000180005200     libucrt:lcidtoname_downlevel.obj
 0001:00004210       ??_C@_1M@JHGLJMGJ@?$AAa?$AAr?$AA?9?$AAD?$AAZ?$AA?$AA@ 0000000180005210     libucrt:lcidtoname_downlevel.obj
 0001:00004220       ??_C@_1M@JKKFDCNP@?$AAz?$AAh?$AA?9?$AAM?$AAO?$AA?$AA@ 0000000180005220     libucrt:lcidtoname_downlevel.obj
 0001:00004230       ??_C@_1M@GEEFALPE@?$AAd?$AAe?$AA?9?$AAL?$AAI?$AA?$AA@ 0000000180005230     libucrt:lcidtoname_downlevel.obj
 0001:00004240       ??_C@_1M@IGEOFBG@?$AAe?$AAn?$AA?9?$AAN?$AAZ?$AA?$AA@ 0000000180005240     libucrt:lcidtoname_downlevel.obj
 0001:00004250       ??_C@_1M@KDBONEHP@?$AAe?$AAs?$AA?9?$AAC?$AAR?$AA?$AA@ 0000000180005250     libucrt:lcidtoname_downlevel.obj
 0001:00004260       ??_C@_1M@FHMDOHNN@?$AAf?$AAr?$AA?9?$AAL?$AAU?$AA?$AA@ 0000000180005260     libucrt:lcidtoname_downlevel.obj
 0001:00004270       ??_C@_1BG@NFKKMAFG@?$AAb?$AAs?$AA?9?$AAB?$AAA?$AA?9?$AAL?$AAa?$AAt?$AAn?$AA?$AA@ 0000000180005270     libucrt:lcidtoname_downlevel.obj
 0001:00004288       ??_C@_1O@IMNBEMCI@?$AAs?$AAm?$AAj?$AA?9?$AAS?$AAE?$AA?$AA@ 0000000180005288     libucrt:lcidtoname_downlevel.obj
 0001:00004298       ??_C@_1M@DHHMBNDP@?$AAa?$AAr?$AA?9?$AAM?$AAA?$AA?$AA@ 0000000180005298     libucrt:lcidtoname_downlevel.obj
 0001:000042a8       ??_C@_1M@BNBLJCGH@?$AAe?$AAn?$AA?9?$AAI?$AAE?$AA?$AA@ 00000001800052a8     libucrt:lcidtoname_downlevel.obj
 0001:000042b8       ??_C@_1M@GEPAFMDL@?$AAe?$AAs?$AA?9?$AAP?$AAA?$AA?$AA@ 00000001800052b8     libucrt:lcidtoname_downlevel.obj
 0001:000042c8       ??_C@_1M@OJONDMDL@?$AAf?$AAr?$AA?9?$AAM?$AAC?$AA?$AA@ 00000001800052c8     libucrt:lcidtoname_downlevel.obj
 0001:000042d8       ??_C@_1BG@OBCNFJB@?$AAs?$AAr?$AA?9?$AAB?$AAA?$AA?9?$AAL?$AAa?$AAt?$AAn?$AA?$AA@ 00000001800052d8     libucrt:lcidtoname_downlevel.obj
 0001:000042f0       ??_C@_1O@KEMEEGPO@?$AAs?$AAm?$AAa?$AA?9?$AAN?$AAO?$AA?$AA@ 00000001800052f0     libucrt:lcidtoname_downlevel.obj
 0001:00004300       ??_C@_1M@ELMGFODK@?$AAa?$AAr?$AA?9?$AAT?$AAN?$AA?$AA@ 0000000180005300     libucrt:lcidtoname_downlevel.obj
 0001:00004310       ??_C@_1M@BHDLHFAF@?$AAe?$AAn?$AA?9?$AAZ?$AAA?$AA?$AA@ 0000000180005310     libucrt:lcidtoname_downlevel.obj
 0001:00004320       ??_C@_1M@BMGIGLIF@?$AAe?$AAs?$AA?9?$AAD?$AAO?$AA?$AA@ 0000000180005320     libucrt:lcidtoname_downlevel.obj
 0001:00004330       ??_C@_1BG@CMBHIPBE@?$AAs?$AAr?$AA?9?$AAB?$AAA?$AA?9?$AAC?$AAy?$AAr?$AAl?$AA?$AA@ 0000000180005330     libucrt:lcidtoname_downlevel.obj
 0001:00004348       ??_C@_1O@HEDBLHNP@?$AAs?$AAm?$AAa?$AA?9?$AAS?$AAE?$AA?$AA@ 0000000180005348     libucrt:lcidtoname_downlevel.obj
 0001:00004358       ??_C@_1M@DAGCADIM@?$AAa?$AAr?$AA?9?$AAO?$AAM?$AA?$AA@ 0000000180005358     libucrt:lcidtoname_downlevel.obj
 0001:00004368       ??_C@_1M@FODLMICG@?$AAe?$AAn?$AA?9?$AAJ?$AAM?$AA?$AA@ 0000000180005368     libucrt:lcidtoname_downlevel.obj
 0001:00004378       ??_C@_1M@DNMLCIHB@?$AAe?$AAs?$AA?9?$AAV?$AAE?$AA?$AA@ 0000000180005378     libucrt:lcidtoname_downlevel.obj
 0001:00004388       ??_C@_1O@EOKHMKJK@?$AAs?$AAm?$AAs?$AA?9?$AAF?$AAI?$AA?$AA@ 0000000180005388     libucrt:lcidtoname_downlevel.obj
 0001:00004398       ??_C@_1M@CAFJMKOF@?$AAa?$AAr?$AA?9?$AAY?$AAE?$AA?$AA@ 0000000180005398     libucrt:lcidtoname_downlevel.obj
 0001:000043a8       ??_C@_1M@CBFHIJLI@?$AAe?$AAn?$AA?9?$AAC?$AAB?$AA?$AA@ 00000001800053a8     libucrt:lcidtoname_downlevel.obj
 0001:000043b8       ??_C@_1M@BGNFLDN@?$AAe?$AAs?$AA?9?$AAC?$AAO?$AA?$AA@ 00000001800053b8     libucrt:lcidtoname_downlevel.obj
 0001:000043c8       ??_C@_1O@JMPHMAMC@?$AAs?$AAm?$AAn?$AA?9?$AAF?$AAI?$AA?$AA@ 00000001800053c8     libucrt:lcidtoname_downlevel.obj
 0001:000043d8       ??_C@_1M@JLANABKE@?$AAa?$AAr?$AA?9?$AAS?$AAY?$AA?$AA@ 00000001800053d8     libucrt:lcidtoname_downlevel.obj
 0001:000043e8       ??_C@_1M@HPKGCFGN@?$AAe?$AAn?$AA?9?$AAB?$AAZ?$AA?$AA@ 00000001800053e8     libucrt:lcidtoname_downlevel.obj
 0001:000043f8       ??_C@_1M@OLJCMLGM@?$AAe?$AAs?$AA?9?$AAP?$AAE?$AA?$AA@ 00000001800053f8     libucrt:lcidtoname_downlevel.obj
 0001:00004408       ??_C@_1M@MKKGFKLE@?$AAa?$AAr?$AA?9?$AAJ?$AAO?$AA?$AA@ 0000000180005408     libucrt:lcidtoname_downlevel.obj
 0001:00004418       ??_C@_1M@EKPGLDNI@?$AAe?$AAn?$AA?9?$AAT?$AAT?$AA?$AA@ 0000000180005418     libucrt:lcidtoname_downlevel.obj
 0001:00004428       ??_C@_1M@OONGHFHE@?$AAe?$AAs?$AA?9?$AAA?$AAR?$AA?$AA@ 0000000180005428     libucrt:lcidtoname_downlevel.obj
 0001:00004438       ??_C@_1M@OOJFGBHE@?$AAa?$AAr?$AA?9?$AAL?$AAB?$AA?$AA@ 0000000180005438     libucrt:lcidtoname_downlevel.obj
 0001:00004448       ??_C@_1M@GCEJHNEG@?$AAe?$AAn?$AA?9?$AAZ?$AAW?$AA?$AA@ 0000000180005448     libucrt:lcidtoname_downlevel.obj
 0001:00004458       ??_C@_1M@JNOCAHJI@?$AAe?$AAs?$AA?9?$AAE?$AAC?$AA?$AA@ 0000000180005458     libucrt:lcidtoname_downlevel.obj
 0001:00004468       ??_C@_1M@JEFHPGGB@?$AAa?$AAr?$AA?9?$AAK?$AAW?$AA?$AA@ 0000000180005468     libucrt:lcidtoname_downlevel.obj
 0001:00004478       ??_C@_1M@MLKIBJOJ@?$AAe?$AAn?$AA?9?$AAP?$AAH?$AA?$AA@ 0000000180005478     libucrt:lcidtoname_downlevel.obj
 0001:00004488       ??_C@_1M@BDNIPEND@?$AAe?$AAs?$AA?9?$AAC?$AAL?$AA?$AA@ 0000000180005488     libucrt:lcidtoname_downlevel.obj
 0001:00004498       ??_C@_1M@MPNMEKBD@?$AAa?$AAr?$AA?9?$AAA?$AAE?$AA?$AA@ 0000000180005498     libucrt:lcidtoname_downlevel.obj
 0001:000044a8       ??_C@_1M@KBJALCPI@?$AAe?$AAs?$AA?9?$AAU?$AAY?$AA?$AA@ 00000001800054a8     libucrt:lcidtoname_downlevel.obj
 0001:000044b8       ??_C@_1M@LLCCOAGA@?$AAa?$AAr?$AA?9?$AAB?$AAH?$AA?$AA@ 00000001800054b8     libucrt:lcidtoname_downlevel.obj
 0001:000044c8       ??_C@_1M@PBFNCDEL@?$AAe?$AAs?$AA?9?$AAP?$AAY?$AA?$AA@ 00000001800054c8     libucrt:lcidtoname_downlevel.obj
 0001:000044d8       ??_C@_1M@EDGINPNP@?$AAa?$AAr?$AA?9?$AAQ?$AAA?$AA?$AA@ 00000001800054d8     libucrt:lcidtoname_downlevel.obj
 0001:000044e8       ??_C@_1M@MKDBIIJI@?$AAe?$AAs?$AA?9?$AAB?$AAO?$AA?$AA@ 00000001800054e8     libucrt:lcidtoname_downlevel.obj
 0001:000044f8       ??_C@_1M@CPKKEBLD@?$AAe?$AAs?$AA?9?$AAS?$AAV?$AA?$AA@ 00000001800054f8     libucrt:lcidtoname_downlevel.obj
 0001:00004508       ??_C@_1M@NDBGMMJL@?$AAe?$AAs?$AA?9?$AAH?$AAN?$AA?$AA@ 0000000180005508     libucrt:lcidtoname_downlevel.obj
 0001:00004518       ??_C@_1M@JIJIBHDP@?$AAe?$AAs?$AA?9?$AAN?$AAI?$AA?$AA@ 0000000180005518     libucrt:lcidtoname_downlevel.obj
 0001:00004528       ??_C@_1M@CGFMKEEK@?$AAe?$AAs?$AA?9?$AAP?$AAR?$AA?$AA@ 0000000180005528     libucrt:lcidtoname_downlevel.obj
 0001:00004538       ??_C@_1O@ICJHKIIK@?$AAz?$AAh?$AA?9?$AAC?$AAH?$AAT?$AA?$AA@ 0000000180005538     libucrt:lcidtoname_downlevel.obj
 0001:00004548       ??_C@_15CLNEJCE@?$AAs?$AAr?$AA?$AA@ 0000000180005548     libucrt:lcidtoname_downlevel.obj
 0001:00005390       ??_C@_1M@KAHEKEIG@?$AAa?$AAf?$AA?9?$AAz?$AAa?$AA?$AA@ 0000000180006390     libucrt:lcidtoname_downlevel.obj
 0001:000053a0       ??_C@_1M@GIECOABL@?$AAa?$AAr?$AA?9?$AAa?$AAe?$AA?$AA@ 00000001800063a0     libucrt:lcidtoname_downlevel.obj
 0001:000053b0       ??_C@_1M@BMLMEKGI@?$AAa?$AAr?$AA?9?$AAb?$AAh?$AA?$AA@ 00000001800063b0     libucrt:lcidtoname_downlevel.obj
 0001:000053c0       ??_C@_1M@DAPFDGGB@?$AAa?$AAr?$AA?9?$AAd?$AAz?$AA?$AA@ 00000001800063c0     libucrt:lcidtoname_downlevel.obj
 0001:000053d0       ??_C@_1M@FJNKGKIG@?$AAa?$AAr?$AA?9?$AAe?$AAg?$AA?$AA@ 00000001800063d0     libucrt:lcidtoname_downlevel.obj
 0001:000053e0       ??_C@_1M@FLGKKCLO@?$AAa?$AAr?$AA?9?$AAi?$AAq?$AA?$AA@ 00000001800063e0     libucrt:lcidtoname_downlevel.obj
 0001:000053f0       ??_C@_1M@GNDIPALM@?$AAa?$AAr?$AA?9?$AAj?$AAo?$AA?$AA@ 00000001800063f0     libucrt:lcidtoname_downlevel.obj
 0001:00005400       ??_C@_1M@DDMJFMGJ@?$AAa?$AAr?$AA?9?$AAk?$AAw?$AA?$AA@ 0000000180006400     libucrt:lcidtoname_downlevel.obj
 0001:00005410       ??_C@_1M@EJALMLHM@?$AAa?$AAr?$AA?9?$AAl?$AAb?$AA?$AA@ 0000000180006410     libucrt:lcidtoname_downlevel.obj
 0001:00005420       ??_C@_1M@MOBDBLOC@?$AAa?$AAr?$AA?9?$AAl?$AAy?$AA?$AA@ 0000000180006420     libucrt:lcidtoname_downlevel.obj
 0001:00005430       ??_C@_1M@JAOCLHDH@?$AAa?$AAr?$AA?9?$AAm?$AAa?$AA?$AA@ 0000000180006430     libucrt:lcidtoname_downlevel.obj
 0001:00005440       ??_C@_1M@JHPMKJIE@?$AAa?$AAr?$AA?9?$AAo?$AAm?$AA?$AA@ 0000000180006440     libucrt:lcidtoname_downlevel.obj
 0001:00005450       ??_C@_1M@OEPGHFNH@?$AAa?$AAr?$AA?9?$AAq?$AAa?$AA?$AA@ 0000000180006450     libucrt:lcidtoname_downlevel.obj
 0001:00005460       ??_C@_1M@KJDONENM@?$AAa?$AAr?$AA?9?$AAs?$AAa?$AA?$AA@ 0000000180006460     libucrt:lcidtoname_downlevel.obj
 0001:00005470       ??_C@_1M@DMJDKLKM@?$AAa?$AAr?$AA?9?$AAs?$AAy?$AA?$AA@ 0000000180006470     libucrt:lcidtoname_downlevel.obj
 0001:00005480       ??_C@_1M@OMFIPEDC@?$AAa?$AAr?$AA?9?$AAt?$AAn?$AA?$AA@ 0000000180006480     libucrt:lcidtoname_downlevel.obj
 0001:00005490       ??_C@_1M@IHMHGAON@?$AAa?$AAr?$AA?9?$AAy?$AAe?$AA?$AA@ 0000000180006490     libucrt:lcidtoname_downlevel.obj
 0001:000054a0       ??_C@_1BG@KDCPGJGB@?$AAa?$AAz?$AA?9?$AAa?$AAz?$AA?9?$AAc?$AAy?$AAr?$AAl?$AA?$AA@ 00000001800064a0     libucrt:lcidtoname_downlevel.obj
 0001:000054b8       ??_C@_1BG@IBCKDDOE@?$AAa?$AAz?$AA?9?$AAa?$AAz?$AA?9?$AAl?$AAa?$AAt?$AAn?$AA?$AA@ 00000001800064b8     libucrt:lcidtoname_downlevel.obj
 0001:000054d0       ??_C@_1M@EGPFDCPD@?$AAb?$AAe?$AA?9?$AAb?$AAy?$AA?$AA@ 00000001800064d0     libucrt:lcidtoname_downlevel.obj
 0001:000054e0       ??_C@_1M@PCMGMCGC@?$AAb?$AAg?$AA?9?$AAb?$AAg?$AA?$AA@ 00000001800064e0     libucrt:lcidtoname_downlevel.obj
 0001:000054f0       ??_C@_1M@BJBMFGOB@?$AAb?$AAn?$AA?9?$AAi?$AAn?$AA?$AA@ 00000001800064f0     libucrt:lcidtoname_downlevel.obj
 0001:00005500       ??_C@_1BG@EAKMMACD@?$AAb?$AAs?$AA?9?$AAb?$AAa?$AA?9?$AAl?$AAa?$AAt?$AAn?$AA?$AA@ 0000000180006500     libucrt:lcidtoname_downlevel.obj
 0001:00005518       ??_C@_1M@KGADAODK@?$AAc?$AAa?$AA?9?$AAe?$AAs?$AA?$AA@ 0000000180006518     libucrt:lcidtoname_downlevel.obj
 0001:00005528       ??_C@_1M@COAJPDHI@?$AAc?$AAs?$AA?9?$AAc?$AAz?$AA?$AA@ 0000000180006528     libucrt:lcidtoname_downlevel.obj
 0001:00005538       ??_C@_1M@DHBHFONH@?$AAc?$AAy?$AA?9?$AAg?$AAb?$AA?$AA@ 0000000180006538     libucrt:lcidtoname_downlevel.obj
 0001:00005548       ??_C@_1M@IMGKELGA@?$AAd?$AAa?$AA?9?$AAd?$AAk?$AA?$AA@ 0000000180006548     libucrt:lcidtoname_downlevel.obj
 0001:00005558       ??_C@_1M@NNDGDNGA@?$AAd?$AAe?$AA?9?$AAa?$AAt?$AA?$AA@ 0000000180006558     libucrt:lcidtoname_downlevel.obj
 0001:00005568       ??_C@_1M@IKDBHEEM@?$AAd?$AAe?$AA?9?$AAc?$AAh?$AA?$AA@ 0000000180006568     libucrt:lcidtoname_downlevel.obj
 0001:00005578       ??_C@_1M@GFFOJMCJ@?$AAd?$AAe?$AA?9?$AAd?$AAe?$AA?$AA@ 0000000180006578     libucrt:lcidtoname_downlevel.obj
 0001:00005588       ??_C@_1M@MDNLKBPM@?$AAd?$AAe?$AA?9?$AAl?$AAi?$AA?$AA@ 0000000180006588     libucrt:lcidtoname_downlevel.obj
 0001:00005598       ??_C@_1M@NJBEEJNL@?$AAd?$AAe?$AA?9?$AAl?$AAu?$AA?$AA@ 0000000180006598     libucrt:lcidtoname_downlevel.obj
 0001:000055a8       ??_C@_1O@GNNELBAP@?$AAd?$AAi?$AAv?$AA?9?$AAm?$AAv?$AA?$AA@ 00000001800065a8     libucrt:lcidtoname_downlevel.obj
 0001:000055b8       ??_C@_1M@EJLEOGAE@?$AAe?$AAl?$AA?9?$AAg?$AAr?$AA?$AA@ 00000001800065b8     libucrt:lcidtoname_downlevel.obj
 0001:000055c8       ??_C@_1M@GMPONJN@?$AAe?$AAn?$AA?9?$AAa?$AAu?$AA?$AA@ 00000001800065c8     libucrt:lcidtoname_downlevel.obj
 0001:000055d8       ??_C@_1M@NIDIIPGF@?$AAe?$AAn?$AA?9?$AAb?$AAz?$AA?$AA@ 00000001800065d8     libucrt:lcidtoname_downlevel.obj
 0001:000055e8       ??_C@_1M@JEHMIMFO@?$AAe?$AAn?$AA?9?$AAc?$AAa?$AA?$AA@ 00000001800065e8     libucrt:lcidtoname_downlevel.obj
 0001:000055f8       ??_C@_1M@IGMJCDLA@?$AAe?$AAn?$AA?9?$AAc?$AAb?$AA?$AA@ 00000001800065f8     libucrt:lcidtoname_downlevel.obj
 0001:00005608       ??_C@_1M@BNFIGBKG@?$AAe?$AAn?$AA?9?$AAg?$AAb?$AA?$AA@ 0000000180006608     libucrt:lcidtoname_downlevel.obj
 0001:00005618       ??_C@_1M@LKIFDIGP@?$AAe?$AAn?$AA?9?$AAi?$AAe?$AA?$AA@ 0000000180006618     libucrt:lcidtoname_downlevel.obj
 0001:00005628       ??_C@_1M@PJKFGCCO@?$AAe?$AAn?$AA?9?$AAj?$AAm?$AA?$AA@ 0000000180006628     libucrt:lcidtoname_downlevel.obj
 0001:00005638       ??_C@_1M@KPPKEPBO@?$AAe?$AAn?$AA?9?$AAn?$AAz?$AA?$AA@ 0000000180006638     libucrt:lcidtoname_downlevel.obj
 0001:00005648       ??_C@_1M@GMDGLDOB@?$AAe?$AAn?$AA?9?$AAp?$AAh?$AA?$AA@ 0000000180006648     libucrt:lcidtoname_downlevel.obj
 0001:00005658       ??_C@_1M@ONGIBJNA@?$AAe?$AAn?$AA?9?$AAt?$AAt?$AA?$AA@ 0000000180006658     libucrt:lcidtoname_downlevel.obj
 0001:00005668       ??_C@_1M@LLODPCMM@?$AAe?$AAn?$AA?9?$AAu?$AAs?$AA?$AA@ 0000000180006668     libucrt:lcidtoname_downlevel.obj
 0001:00005678       ??_C@_1M@LAKFNPAN@?$AAe?$AAn?$AA?9?$AAz?$AAa?$AA?$AA@ 0000000180006678     libucrt:lcidtoname_downlevel.obj
 0001:00005688       ??_C@_1M@MFNHNHEO@?$AAe?$AAn?$AA?9?$AAz?$AAw?$AA?$AA@ 0000000180006688     libucrt:lcidtoname_downlevel.obj
 0001:00005698       ??_C@_1M@EJEINPHM@?$AAe?$AAs?$AA?9?$AAa?$AAr?$AA?$AA@ 0000000180006698     libucrt:lcidtoname_downlevel.obj
 0001:000056a8       ??_C@_1M@GNKPCCJA@?$AAe?$AAs?$AA?9?$AAb?$AAo?$AA?$AA@ 00000001800066a8     libucrt:lcidtoname_downlevel.obj
 0001:000056b8       ??_C@_1M@LEEGFONL@?$AAe?$AAs?$AA?9?$AAc?$AAl?$AA?$AA@ 00000001800066b8     libucrt:lcidtoname_downlevel.obj
 0001:000056c8       ??_C@_1M@KGPDPBDF@?$AAe?$AAs?$AA?9?$AAc?$AAo?$AA?$AA@ 00000001800066c8     libucrt:lcidtoname_downlevel.obj
 0001:000056d8       ??_C@_1M@EIAHOHH@?$AAe?$AAs?$AA?9?$AAc?$AAr?$AA?$AA@ 00000001800066d8     libucrt:lcidtoname_downlevel.obj
 0001:000056e8       ??_C@_1M@LLPGMBIN@?$AAe?$AAs?$AA?9?$AAd?$AAo?$AA?$AA@ 00000001800066e8     libucrt:lcidtoname_downlevel.obj
 0001:000056f8       ??_C@_1M@DKHMKNJA@?$AAe?$AAs?$AA?9?$AAe?$AAc?$AA?$AA@ 00000001800066f8     libucrt:lcidtoname_downlevel.obj
 0001:00005708       ??_C@_1M@GKGFPKAP@?$AAe?$AAs?$AA?9?$AAe?$AAs?$AA?$AA@ 0000000180006708     libucrt:lcidtoname_downlevel.obj
 0001:00005718       ??_C@_1M@LKHKGDLN@?$AAe?$AAs?$AA?9?$AAg?$AAt?$AA?$AA@ 0000000180006718     libucrt:lcidtoname_downlevel.obj
 0001:00005728       ??_C@_1M@HEIIGGJD@?$AAe?$AAs?$AA?9?$AAh?$AAn?$AA?$AA@ 0000000180006728     libucrt:lcidtoname_downlevel.obj
 0001:00005738       ??_C@_1M@FBDHPPGD@?$AAe?$AAs?$AA?9?$AAm?$AAx?$AA?$AA@ 0000000180006738     libucrt:lcidtoname_downlevel.obj
 0001:00005748       ??_C@_1M@DPAGLNDH@?$AAe?$AAs?$AA?9?$AAn?$AAi?$AA?$AA@ 0000000180006748     libucrt:lcidtoname_downlevel.obj
 0001:00005758       ??_C@_1M@MDGOPGDD@?$AAe?$AAs?$AA?9?$AAp?$AAa?$AA?$AA@ 0000000180006758     libucrt:lcidtoname_downlevel.obj
 0001:00005768       ??_C@_1M@EMAMGBGE@?$AAe?$AAs?$AA?9?$AAp?$AAe?$AA?$AA@ 0000000180006768     libucrt:lcidtoname_downlevel.obj
 0001:00005778       ??_C@_1M@IBMCAOEC@?$AAe?$AAs?$AA?9?$AAp?$AAr?$AA?$AA@ 0000000180006778     libucrt:lcidtoname_downlevel.obj
 0001:00005788       ??_C@_1M@FGMDIJED@?$AAe?$AAs?$AA?9?$AAp?$AAy?$AA?$AA@ 0000000180006788     libucrt:lcidtoname_downlevel.obj
 0001:00005798       ??_C@_1M@IIDEOLLL@?$AAe?$AAs?$AA?9?$AAs?$AAv?$AA?$AA@ 0000000180006798     libucrt:lcidtoname_downlevel.obj
 0001:000057a8       ??_C@_1M@GAOBIPA@?$AAe?$AAs?$AA?9?$AAu?$AAy?$AA?$AA@ 00000001800067a8     libucrt:lcidtoname_downlevel.obj
 0001:000057b8       ??_C@_1M@JKFFICHJ@?$AAe?$AAs?$AA?9?$AAv?$AAe?$AA?$AA@ 00000001800067b8     libucrt:lcidtoname_downlevel.obj
 0001:000057c8       ??_C@_1M@PNMLOJDF@?$AAe?$AAt?$AA?9?$AAe?$AAe?$AA?$AA@ 00000001800067c8     libucrt:lcidtoname_downlevel.obj
 0001:000057d8       ??_C@_1M@GHHLIKEI@?$AAe?$AAu?$AA?9?$AAe?$AAs?$AA?$AA@ 00000001800067d8     libucrt:lcidtoname_downlevel.obj
 0001:000057e8       ??_C@_1M@PBNONODE@?$AAf?$AAa?$AA?9?$AAi?$AAr?$AA?$AA@ 00000001800067e8     libucrt:lcidtoname_downlevel.obj
 0001:000057f8       ??_C@_1M@JEEHPMIL@?$AAf?$AAi?$AA?9?$AAf?$AAi?$AA?$AA@ 00000001800067f8     libucrt:lcidtoname_downlevel.obj
 0001:00005808       ??_C@_1M@LMDCNDBA@?$AAf?$AAo?$AA?9?$AAf?$AAo?$AA?$AA@ 0000000180006808     libucrt:lcidtoname_downlevel.obj
 0001:00005818       ??_C@_1M@JKEOHLDK@?$AAf?$AAr?$AA?9?$AAb?$AAe?$AA?$AA@ 0000000180006818     libucrt:lcidtoname_downlevel.obj
 0001:00005828       ??_C@_1M@NOHADPMI@?$AAf?$AAr?$AA?9?$AAc?$AAa?$AA?$AA@ 0000000180006828     libucrt:lcidtoname_downlevel.obj
 0001:00005838       ??_C@_1M@KDHIHAEC@?$AAf?$AAr?$AA?9?$AAc?$AAh?$AA?$AA@ 0000000180006838     libucrt:lcidtoname_downlevel.obj
 0001:00005848       ??_C@_1M@MMBBFGAK@?$AAf?$AAr?$AA?9?$AAf?$AAr?$AA?$AA@ 0000000180006848     libucrt:lcidtoname_downlevel.obj
 0001:00005858       ??_C@_1M@PAFNENNF@?$AAf?$AAr?$AA?9?$AAl?$AAu?$AA?$AA@ 0000000180006858     libucrt:lcidtoname_downlevel.obj
 0001:00005868       ??_C@_1M@EOHDJGDD@?$AAf?$AAr?$AA?9?$AAm?$AAc?$AA?$AA@ 0000000180006868     libucrt:lcidtoname_downlevel.obj
 0001:00005878       ??_C@_1M@FAPLLOPF@?$AAg?$AAl?$AA?9?$AAe?$AAs?$AA?$AA@ 0000000180006878     libucrt:lcidtoname_downlevel.obj
 0001:00005888       ??_C@_1M@FOPBFLOO@?$AAg?$AAu?$AA?9?$AAi?$AAn?$AA?$AA@ 0000000180006888     libucrt:lcidtoname_downlevel.obj
 0001:00005898       ??_C@_1M@KBMCINPM@?$AAh?$AAe?$AA?9?$AAi?$AAl?$AA?$AA@ 0000000180006898     libucrt:lcidtoname_downlevel.obj
 0001:000058a8       ??_C@_1M@BBPHKFPJ@?$AAh?$AAi?$AA?9?$AAi?$AAn?$AA?$AA@ 00000001800068a8     libucrt:lcidtoname_downlevel.obj
 0001:000058b8       ??_C@_1M@PMBNDPHD@?$AAh?$AAr?$AA?9?$AAb?$AAa?$AA?$AA@ 00000001800068b8     libucrt:lcidtoname_downlevel.obj
 0001:000058c8       ??_C@_1M@BPCKOEGE@?$AAh?$AAr?$AA?9?$AAh?$AAr?$AA?$AA@ 00000001800068c8     libucrt:lcidtoname_downlevel.obj
 0001:000058d8       ??_C@_1M@GACBMHKE@?$AAh?$AAu?$AA?9?$AAh?$AAu?$AA?$AA@ 00000001800068d8     libucrt:lcidtoname_downlevel.obj
 0001:000058e8       ??_C@_1M@MILPAJJC@?$AAh?$AAy?$AA?9?$AAa?$AAm?$AA?$AA@ 00000001800068e8     libucrt:lcidtoname_downlevel.obj
 0001:000058f8       ??_C@_1M@BABBICEC@?$AAi?$AAd?$AA?9?$AAi?$AAd?$AA?$AA@ 00000001800068f8     libucrt:lcidtoname_downlevel.obj
 0001:00005908       ??_C@_1M@BIKNHHPF@?$AAi?$AAs?$AA?9?$AAi?$AAs?$AA?$AA@ 0000000180006908     libucrt:lcidtoname_downlevel.obj
 0001:00005918       ??_C@_1M@NMPCJPHE@?$AAi?$AAt?$AA?9?$AAc?$AAh?$AA?$AA@ 0000000180006918     libucrt:lcidtoname_downlevel.obj
 0001:00005928       ??_C@_1M@GHKGFEDF@?$AAi?$AAt?$AA?9?$AAi?$AAt?$AA?$AA@ 0000000180006928     libucrt:lcidtoname_downlevel.obj
 0001:00005938       ??_C@_1M@NIEJCJJA@?$AAj?$AAa?$AA?9?$AAj?$AAp?$AA?$AA@ 0000000180006938     libucrt:lcidtoname_downlevel.obj
 0001:00005948       ??_C@_1M@JILFNBIM@?$AAk?$AAa?$AA?9?$AAg?$AAe?$AA?$AA@ 0000000180006948     libucrt:lcidtoname_downlevel.obj
 0001:00005958       ??_C@_1M@PACPMGPH@?$AAk?$AAk?$AA?9?$AAk?$AAz?$AA?$AA@ 0000000180006958     libucrt:lcidtoname_downlevel.obj
 0001:00005968       ??_C@_1M@IELFGMHA@?$AAk?$AAn?$AA?9?$AAi?$AAn?$AA?$AA@ 0000000180006968     libucrt:lcidtoname_downlevel.obj
 0001:00005978       ??_C@_1O@IBBJHCH@?$AAk?$AAo?$AAk?$AA?9?$AAi?$AAn?$AA?$AA@ 0000000180006978     libucrt:lcidtoname_downlevel.obj
 0001:00005988       ??_C@_1M@DMHAEOGC@?$AAk?$AAo?$AA?9?$AAk?$AAr?$AA?$AA@ 0000000180006988     libucrt:lcidtoname_downlevel.obj
 0001:00005998       ??_C@_1M@HBAHBIGA@?$AAk?$AAy?$AA?9?$AAk?$AAg?$AA?$AA@ 0000000180006998     libucrt:lcidtoname_downlevel.obj
 0001:000059a8       ??_C@_1M@KPMILCJG@?$AAl?$AAt?$AA?9?$AAl?$AAt?$AA?$AA@ 00000001800069a8     libucrt:lcidtoname_downlevel.obj
 0001:000059b8       ??_C@_1M@BDEKKCA@?$AAl?$AAv?$AA?9?$AAl?$AAv?$AA?$AA@ 00000001800069b8     libucrt:lcidtoname_downlevel.obj
 0001:000059c8       ??_C@_1M@ELCKCCJJ@?$AAm?$AAi?$AA?9?$AAn?$AAz?$AA?$AA@ 00000001800069c8     libucrt:lcidtoname_downlevel.obj
 0001:000059d8       ??_C@_1M@CBOOLAPA@?$AAm?$AAk?$AA?9?$AAm?$AAk?$AA?$AA@ 00000001800069d8     libucrt:lcidtoname_downlevel.obj
 0001:000059e8       ??_C@_1M@GPHNBJKN@?$AAm?$AAl?$AA?9?$AAi?$AAn?$AA?$AA@ 00000001800069e8     libucrt:lcidtoname_downlevel.obj
 0001:000059f8       ??_C@_1M@PABJILIG@?$AAm?$AAn?$AA?9?$AAm?$AAn?$AA?$AA@ 00000001800069f8     libucrt:lcidtoname_downlevel.obj
 0001:00005a08       ??_C@_1M@FGBKKIPG@?$AAm?$AAr?$AA?9?$AAi?$AAn?$AA?$AA@ 0000000180006a08     libucrt:lcidtoname_downlevel.obj
 0001:00005a18       ??_C@_1M@NDBPDDAL@?$AAm?$AAs?$AA?9?$AAb?$AAn?$AA?$AA@ 0000000180006a18     libucrt:lcidtoname_downlevel.obj
 0001:00005a28       ??_C@_1M@OPIHOOPI@?$AAm?$AAs?$AA?9?$AAm?$AAy?$AA?$AA@ 0000000180006a28     libucrt:lcidtoname_downlevel.obj
 0001:00005a38       ??_C@_1M@PPDBCNFM@?$AAm?$AAt?$AA?9?$AAm?$AAt?$AA?$AA@ 0000000180006a38     libucrt:lcidtoname_downlevel.obj
 0001:00005a48       ??_C@_1M@KDJDKMDD@?$AAn?$AAb?$AA?9?$AAn?$AAo?$AA?$AA@ 0000000180006a48     libucrt:lcidtoname_downlevel.obj
 0001:00005a58       ??_C@_1M@KFCFLMJP@?$AAn?$AAl?$AA?9?$AAb?$AAe?$AA?$AA@ 0000000180006a58     libucrt:lcidtoname_downlevel.obj
 0001:00005a68       ??_C@_1M@KPOPDDGO@?$AAn?$AAl?$AA?9?$AAn?$AAl?$AA?$AA@ 0000000180006a68     libucrt:lcidtoname_downlevel.obj
 0001:00005a78       ??_C@_1M@LJKPEMLN@?$AAn?$AAn?$AA?9?$AAn?$AAo?$AA?$AA@ 0000000180006a78     libucrt:lcidtoname_downlevel.obj
 0001:00005a88       ??_C@_1M@BDGHHBFL@?$AAn?$AAs?$AA?9?$AAz?$AAa?$AA?$AA@ 0000000180006a88     libucrt:lcidtoname_downlevel.obj
 0001:00005a98       ??_C@_1M@IDEHOAP@?$AAp?$AAa?$AA?9?$AAi?$AAn?$AA?$AA@ 0000000180006a98     libucrt:lcidtoname_downlevel.obj
 0001:00005aa8       ??_C@_1M@HDBKGOGH@?$AAp?$AAl?$AA?9?$AAp?$AAl?$AA?$AA@ 0000000180006aa8     libucrt:lcidtoname_downlevel.obj
 0001:00005ab8       ??_C@_1M@LJLLCMEH@?$AAp?$AAt?$AA?9?$AAb?$AAr?$AA?$AA@ 0000000180006ab8     libucrt:lcidtoname_downlevel.obj
 0001:00005ac8       ??_C@_1M@NCMONAAL@?$AAp?$AAt?$AA?9?$AAp?$AAt?$AA?$AA@ 0000000180006ac8     libucrt:lcidtoname_downlevel.obj
 0001:00005ad8       ??_C@_1O@EAKMAJDN@?$AAq?$AAu?$AAz?$AA?9?$AAb?$AAo?$AA?$AA@ 0000000180006ad8     libucrt:lcidtoname_downlevel.obj
 0001:00005ae8       ??_C@_1O@BHHPIGDN@?$AAq?$AAu?$AAz?$AA?9?$AAe?$AAc?$AA?$AA@ 0000000180006ae8     libucrt:lcidtoname_downlevel.obj
 0001:00005af8       ??_C@_1O@GBAPEKMJ@?$AAq?$AAu?$AAz?$AA?9?$AAp?$AAe?$AA?$AA@ 0000000180006af8     libucrt:lcidtoname_downlevel.obj
 0001:00005b08       ??_C@_1M@CLGLEFBO@?$AAr?$AAo?$AA?9?$AAr?$AAo?$AA?$AA@ 0000000180006b08     libucrt:lcidtoname_downlevel.obj
 0001:00005b18       ??_C@_1M@CEEDODME@?$AAr?$AAu?$AA?9?$AAr?$AAu?$AA?$AA@ 0000000180006b18     libucrt:lcidtoname_downlevel.obj
 0001:00005b28       ??_C@_1M@HPKKKMPP@?$AAs?$AAa?$AA?9?$AAi?$AAn?$AA?$AA@ 0000000180006b28     libucrt:lcidtoname_downlevel.obj
 0001:00005b38       ??_C@_1M@BKMAIGOJ@?$AAs?$AAe?$AA?9?$AAf?$AAi?$AA?$AA@ 0000000180006b38     libucrt:lcidtoname_downlevel.obj
 0001:00005b48       ??_C@_1M@NDPIFLFI@?$AAs?$AAe?$AA?9?$AAn?$AAo?$AA?$AA@ 0000000180006b48     libucrt:lcidtoname_downlevel.obj
 0001:00005b58       ??_C@_1M@DANKKHJ@?$AAs?$AAe?$AA?9?$AAs?$AAe?$AA?$AA@ 0000000180006b58     libucrt:lcidtoname_downlevel.obj
 0001:00005b68       ??_C@_1M@PNBLONPJ@?$AAs?$AAk?$AA?9?$AAs?$AAk?$AA?$AA@ 0000000180006b68     libucrt:lcidtoname_downlevel.obj
 0001:00005b78       ??_C@_1M@LFMODOAL@?$AAs?$AAl?$AA?9?$AAs?$AAi?$AA?$AA@ 0000000180006b78     libucrt:lcidtoname_downlevel.obj
 0001:00005b88       ??_C@_1O@DFKOMPG@?$AAs?$AAm?$AAa?$AA?9?$AAn?$AAo?$AA?$AA@ 0000000180006b88     libucrt:lcidtoname_downlevel.obj
 0001:00005b98       ??_C@_1O@NDKPBNNH@?$AAs?$AAm?$AAa?$AA?9?$AAs?$AAe?$AA?$AA@ 0000000180006b98     libucrt:lcidtoname_downlevel.obj
 0001:00005ba8       ??_C@_1O@PLLKBHAB@?$AAs?$AAm?$AAj?$AA?9?$AAn?$AAo?$AA?$AA@ 0000000180006ba8     libucrt:lcidtoname_downlevel.obj
 0001:00005bb8       ??_C@_1O@CLEPOGCA@?$AAs?$AAm?$AAj?$AA?9?$AAs?$AAe?$AA?$AA@ 0000000180006bb8     libucrt:lcidtoname_downlevel.obj
 0001:00005bc8       ??_C@_1O@DLGJGKMK@?$AAs?$AAm?$AAn?$AA?9?$AAf?$AAi?$AA?$AA@ 0000000180006bc8     libucrt:lcidtoname_downlevel.obj
 0001:00005bd8       ??_C@_1O@OJDJGAJC@?$AAs?$AAm?$AAs?$AA?9?$AAf?$AAi?$AA?$AA@ 0000000180006bd8     libucrt:lcidtoname_downlevel.obj
 0001:00005be8       ??_C@_1M@BOFOGHPB@?$AAs?$AAq?$AA?9?$AAa?$AAl?$AA?$AA@ 0000000180006be8     libucrt:lcidtoname_downlevel.obj
 0001:00005bf8       ??_C@_1BG@LJBBIPGB@?$AAs?$AAr?$AA?9?$AAb?$AAa?$AA?9?$AAc?$AAy?$AAr?$AAl?$AA?$AA@ 0000000180006bf8     libucrt:lcidtoname_downlevel.obj
 0001:00005c10       ??_C@_1BG@JLBENFOE@?$AAs?$AAr?$AA?9?$AAb?$AAa?$AA?9?$AAl?$AAa?$AAt?$AAn?$AA?$AA@ 0000000180006c10     libucrt:lcidtoname_downlevel.obj
 0001:00005c28       ??_C@_1BG@KODPNHE@?$AAs?$AAr?$AA?9?$AAs?$AAp?$AA?9?$AAc?$AAy?$AAr?$AAl?$AA?$AA@ 0000000180006c28     libucrt:lcidtoname_downlevel.obj
 0001:00005c40       ??_C@_1BG@CIOGKHPB@?$AAs?$AAr?$AA?9?$AAs?$AAp?$AA?9?$AAl?$AAa?$AAt?$AAn?$AA?$AA@ 0000000180006c40     libucrt:lcidtoname_downlevel.obj
 0001:00005c58       ??_C@_1M@NGFJLMAC@?$AAs?$AAv?$AA?9?$AAf?$AAi?$AA?$AA@ 0000000180006c58     libucrt:lcidtoname_downlevel.obj
 0001:00005c68       ??_C@_1M@MPJEJAJC@?$AAs?$AAv?$AA?9?$AAs?$AAe?$AA?$AA@ 0000000180006c68     libucrt:lcidtoname_downlevel.obj
 0001:00005c78       ??_C@_1M@MPNDHLFK@?$AAs?$AAw?$AA?9?$AAk?$AAe?$AA?$AA@ 0000000180006c78     libucrt:lcidtoname_downlevel.obj
 0001:00005c88       ??_C@_1O@KOHBJJI@?$AAs?$AAy?$AAr?$AA?9?$AAs?$AAy?$AA?$AA@ 0000000180006c88     libucrt:lcidtoname_downlevel.obj
 0001:00005c98       ??_C@_1M@LDCEFHA@?$AAt?$AAa?$AA?9?$AAi?$AAn?$AA?$AA@ 0000000180006c98     libucrt:lcidtoname_downlevel.obj
 0001:00005ca8       ??_C@_1M@CNJOFAK@?$AAt?$AAe?$AA?9?$AAi?$AAn?$AA?$AA@ 0000000180006ca8     libucrt:lcidtoname_downlevel.obj
 0001:00005cb8       ??_C@_1M@GNAECACD@?$AAt?$AAh?$AA?9?$AAt?$AAh?$AA?$AA@ 0000000180006cb8     libucrt:lcidtoname_downlevel.obj
 0001:00005cc8       ??_C@_1M@CHBIHOJO@?$AAt?$AAn?$AA?9?$AAz?$AAa?$AA?$AA@ 0000000180006cc8     libucrt:lcidtoname_downlevel.obj
 0001:00005cd8       ??_C@_1M@GCCMIGPJ@?$AAt?$AAr?$AA?9?$AAt?$AAr?$AA?$AA@ 0000000180006cd8     libucrt:lcidtoname_downlevel.obj
 0001:00005ce8       ??_C@_1M@CELMCNBK@?$AAt?$AAt?$AA?9?$AAr?$AAu?$AA?$AA@ 0000000180006ce8     libucrt:lcidtoname_downlevel.obj
 0001:00005cf8       ??_C@_1M@KLMCELGA@?$AAu?$AAk?$AA?9?$AAu?$AAa?$AA?$AA@ 0000000180006cf8     libucrt:lcidtoname_downlevel.obj
 0001:00005d08       ??_C@_1M@EPAJJAJF@?$AAu?$AAr?$AA?9?$AAp?$AAk?$AA?$AA@ 0000000180006d08     libucrt:lcidtoname_downlevel.obj
 0001:00005d18       ??_C@_1BG@GEGPMCDJ@?$AAu?$AAz?$AA?9?$AAu?$AAz?$AA?9?$AAc?$AAy?$AAr?$AAl?$AA?$AA@ 0000000180006d18     libucrt:lcidtoname_downlevel.obj
 0001:00005d30       ??_C@_1BG@EGGKJILM@?$AAu?$AAz?$AA?9?$AAu?$AAz?$AA?9?$AAl?$AAa?$AAt?$AAn?$AA?$AA@ 0000000180006d30     libucrt:lcidtoname_downlevel.obj
 0001:00005d48       ??_C@_1M@GFOCLFF@?$AAv?$AAi?$AA?9?$AAv?$AAn?$AA?$AA@ 0000000180006d48     libucrt:lcidtoname_downlevel.obj
 0001:00005d58       ??_C@_1M@CPAMEDFI@?$AAx?$AAh?$AA?9?$AAz?$AAa?$AA?$AA@ 0000000180006d58     libucrt:lcidtoname_downlevel.obj
 0001:00005d68       ??_C@_1O@EBKIFIGN@?$AAz?$AAh?$AA?9?$AAc?$AAh?$AAs?$AA?$AA@ 0000000180006d68     libucrt:lcidtoname_downlevel.obj
 0001:00005d78       ??_C@_1O@NMHPGANE@?$AAz?$AAh?$AA?9?$AAc?$AAh?$AAt?$AA?$AA@ 0000000180006d78     libucrt:lcidtoname_downlevel.obj
 0001:00005d88       ??_C@_1M@LPINJOMC@?$AAz?$AAh?$AA?9?$AAc?$AAn?$AA?$AA@ 0000000180006d88     libucrt:lcidtoname_downlevel.obj
 0001:00005d98       ??_C@_1M@OCJEJODD@?$AAz?$AAh?$AA?9?$AAh?$AAk?$AA?$AA@ 0000000180006d98     libucrt:lcidtoname_downlevel.obj
 0001:00005da8       ??_C@_1M@DNDLJINH@?$AAz?$AAh?$AA?9?$AAm?$AAo?$AA?$AA@ 0000000180006da8     libucrt:lcidtoname_downlevel.obj
 0001:00005db8       ??_C@_1M@MBFDNDND@?$AAz?$AAh?$AA?9?$AAs?$AAg?$AA?$AA@ 0000000180006db8     libucrt:lcidtoname_downlevel.obj
 0001:00005dc8       ??_C@_1M@IMEPLEPE@?$AAz?$AAh?$AA?9?$AAt?$AAw?$AA?$AA@ 0000000180006dc8     libucrt:lcidtoname_downlevel.obj
 0001:00005dd8       ??_C@_1M@BBGHNHJP@?$AAz?$AAu?$AA?9?$AAz?$AAa?$AA?$AA@ 0000000180006dd8     libucrt:lcidtoname_downlevel.obj
 0001:00005de4       ??_C@_00CNPNBAHC@?$AA@     0000000180006de4     libucrt:mbrtowc.obj
 0001:00006040       ??_C@_1BA@BALFACEM@?$AAC?$AAO?$AAN?$AAO?$AAU?$AAT?$AA$?$AA?$AA@ 0000000180007040     libucrt:initcon.obj
 0001:00006050       __log10_256_lead           0000000180007050     libucrt:log10_256_lead_tail_table.obj
 0001:00006860       __log10_256_tail           0000000180007860     libucrt:log10_256_lead_tail_table.obj
 0001:00007070       __log_F_inv_qword          0000000180008070     libucrt:log_f_inv_qword_table.obj
 0001:00007880       ??_C@_05HGHHAHAP@log10?$AA@ 0000000180008880     libucrt:log_special.obj
 0001:000078d0       _load_config_used          00000001800088d0     LIBCMT:loadcfg.obj
 0001:000079d0       ??_R4exception@std@@6B@    00000001800089d0     LIBCMT:throw_bad_alloc.obj
 0001:000079f8       ??_R3exception@std@@8      00000001800089f8     LIBCMT:throw_bad_alloc.obj
 0001:00007a10       ??_R2exception@std@@8      0000000180008a10     LIBCMT:throw_bad_alloc.obj
 0001:00007a20       ??_R1A@?0A@EA@exception@std@@8 0000000180008a20     LIBCMT:throw_bad_alloc.obj
 0001:00007a48       ??_R4bad_alloc@std@@6B@    0000000180008a48     LIBCMT:throw_bad_alloc.obj
 0001:00007a70       ??_R3bad_alloc@std@@8      0000000180008a70     LIBCMT:throw_bad_alloc.obj
 0001:00007a88       ??_R2bad_alloc@std@@8      0000000180008a88     LIBCMT:throw_bad_alloc.obj
 0001:00007aa0       ??_R1A@?0A@EA@bad_alloc@std@@8 0000000180008aa0     LIBCMT:throw_bad_alloc.obj
 0001:00007ac8       ??_R4bad_array_new_length@std@@6B@ 0000000180008ac8     LIBCMT:throw_bad_alloc.obj
 0001:00007af0       ??_R3bad_array_new_length@std@@8 0000000180008af0     LIBCMT:throw_bad_alloc.obj
 0001:00007b08       ??_R2bad_array_new_length@std@@8 0000000180008b08     LIBCMT:throw_bad_alloc.obj
 0001:00007b28       ??_R1A@?0A@EA@bad_array_new_length@std@@8 0000000180008b28     LIBCMT:throw_bad_alloc.obj
 0001:00007b50       ??_R4type_info@@6B@        0000000180008b50     LIBCMT:std_type_info_static.obj
 0001:00007b78       ??_R3type_info@@8          0000000180008b78     LIBCMT:std_type_info_static.obj
 0001:00007b90       ??_R2type_info@@8          0000000180008b90     LIBCMT:std_type_info_static.obj
 0001:00007ba0       ??_R1A@?0A@EA@type_info@@8 0000000180008ba0     LIBCMT:std_type_info_static.obj
 0001:00007e78       __rtc_iaa                  0000000180008e78     LIBCMT:initsect.obj
 0001:00007e80       __rtc_izz                  0000000180008e80     LIBCMT:initsect.obj
 0001:00007e88       __rtc_taa                  0000000180008e88     LIBCMT:initsect.obj
 0001:00007e90       __rtc_tzz                  0000000180008e90     LIBCMT:initsect.obj
 0001:00007eb0       __chkstk                   0000000180008eb0 f   chkstk.obj
 0001:00007eb0       _alloca_probe              0000000180008eb0 f   chkstk.obj
 0001:00008330       ?ReadFileLines@@YAXPEAXKPEAPEA_WPEA_WPEAI3@Z 0000000180009330 f   TmpPanel.obj
 0001:00008aa0       AnalyseW                   0000000180009aa0 f   TmpPanel.obj
 0001:00008b00       ClosePanelW                0000000180009b00 f   TmpPanel.obj
 0001:00008b30       ConfigureW                 0000000180009b30 f   TmpPanel.obj
 0001:00008b40       ExitFARW                   0000000180009b40 f   TmpPanel.obj
 0001:00008b80       GetFindDataW               0000000180009b80 f   TmpPanel.obj
 0001:00008ba0       GetGlobalInfoW             0000000180009ba0 f   TmpPanel.obj
 0001:00008c20       GetOpenPanelInfoW          0000000180009c20 f   TmpPanel.obj
 0001:00008c30       GetPluginInfoW             0000000180009c30 f   TmpPanel.obj
 0001:00008d00       OpenW                      0000000180009d00 f   TmpPanel.obj
 0001:00009110       ProcessPanelEventW         000000018000a110 f   TmpPanel.obj
 0001:00009130       ProcessPanelInputW         000000018000a130 f   TmpPanel.obj
 0001:00009150       PutFilesW                  000000018000a150 f   TmpPanel.obj
 0001:00009190       SetDirectoryW              000000018000a190 f   TmpPanel.obj
 0001:000091b0       SetFindListW               000000018000a1b0 f   TmpPanel.obj
 0001:000091d0       SetStartupInfoW            000000018000a1d0 f   TmpPanel.obj
 0001:00009320       ??1?$DialogBuilderBase@UFarDialogItem@@@@MEAA@XZ 000000018000a320 f i TmpCfg.obj
 0001:000093a0       ??_G?$DialogBuilderBase@UFarDialogItem@@@@MEAAPEAXI@Z 000000018000a3a0 f i TmpCfg.obj
 0001:000093a0       ??_E?$DialogBuilderBase@UFarDialogItem@@@@MEAAPEAXI@Z 000000018000a3a0 f i TmpCfg.obj
 0001:000093e0       ??_E?$DialogItemBinding@UFarDialogItem@@@@UEAAPEAXI@Z 000000018000a3e0 f i TmpCfg.obj
 0001:000093e0       ??_G?$DialogItemBinding@UFarDialogItem@@@@UEAAPEAXI@Z 000000018000a3e0 f i TmpCfg.obj
 0001:00009410       ??_EPluginEditFieldBinding@@UEAAPEAXI@Z 000000018000a410 f i TmpCfg.obj
 0001:00009410       ??_GPluginCheckBoxBinding@@UEAAPEAXI@Z 000000018000a410 f i TmpCfg.obj
 0001:00009410       ??_EPluginCheckBoxBinding@@UEAAPEAXI@Z 000000018000a410 f i TmpCfg.obj
 0001:00009410       ??_GPluginEditFieldBinding@@UEAAPEAXI@Z 000000018000a410 f i TmpCfg.obj
 0001:00009440       ??_EPluginDialogBuilder@@UEAAPEAXI@Z 000000018000a440 f i TmpCfg.obj
 0001:00009440       ??_GPluginDialogBuilder@@UEAAPEAXI@Z 000000018000a440 f i TmpCfg.obj
 0001:00009490       ??_GPluginIntEditFieldBinding@@UEAAPEAXI@Z 000000018000a490 f i TmpCfg.obj
 0001:00009490       ??_EPluginUIntEditFieldBinding@@UEAAPEAXI@Z 000000018000a490 f i TmpCfg.obj
 0001:00009490       ??_EPluginIntEditFieldBinding@@UEAAPEAXI@Z 000000018000a490 f i TmpCfg.obj
 0001:00009490       ??_GPluginUIntEditFieldBinding@@UEAAPEAXI@Z 000000018000a490 f i TmpCfg.obj
 0001:000094c0       ??_GPluginRadioButtonBinding@@UEAAPEAXI@Z 000000018000a4c0 f i TmpCfg.obj
 0001:000094c0       ??_EPluginRadioButtonBinding@@UEAAPEAXI@Z 000000018000a4c0 f i TmpCfg.obj
 0001:000094f0       ?AddButtons@?$DialogBuilderBase@UFarDialogItem@@@@QEAAXHPEBHHH@Z 000000018000a4f0 f i TmpCfg.obj
 0001:00009800       ?AddDialogItem@?$DialogBuilderBase@UFarDialogItem@@@@IEAAPEAUFarDialogItem@@W4FARDIALOGITEMTYPES@@PEB_W@Z 000000018000a800 f i TmpCfg.obj
 0001:000099b0       ?AddUIntEditField@?$DialogBuilderBase@UFarDialogItem@@@@UEAAPEAUFarDialogItem@@PEAIH@Z 000000018000a9b0 f i TmpCfg.obj
 0001:000099b0       ?AddIntEditField@?$DialogBuilderBase@UFarDialogItem@@@@UEAAPEAUFarDialogItem@@PEAHH@Z 000000018000a9b0 f i TmpCfg.obj
 0001:000099b0       ?GetLangString@?$DialogBuilderBase@UFarDialogItem@@@@MEAAPEB_WH@Z 000000018000a9b0 f i TmpCfg.obj
 0001:000099b0       ?CreateRadioButtonBinding@?$DialogBuilderBase@UFarDialogItem@@@@MEAAPEAU?$DialogItemBinding@UFarDialogItem@@@@PEAH@Z 000000018000a9b0 f i TmpCfg.obj
 0001:000099b0       ?CreateCheckBoxBinding@?$DialogBuilderBase@UFarDialogItem@@@@MEAAPEAU?$DialogItemBinding@UFarDialogItem@@@@PEAHH@Z 000000018000a9b0 f i TmpCfg.obj
 0001:000099c0       ?AddIntEditField@PluginDialogBuilder@@UEAAPEAUFarDialogItem@@PEAHH@Z 000000018000a9c0 f i TmpCfg.obj
 0001:00009b20       ?AddUIntEditField@PluginDialogBuilder@@UEAAPEAUFarDialogItem@@PEAIH@Z 000000018000ab20 f i TmpCfg.obj
 0001:00009c80       ?Config@@YAHXZ             000000018000ac80 f   TmpCfg.obj
 0001:0000b5f0       ?CreateCheckBoxBinding@PluginDialogBuilder@@MEAAPEAU?$DialogItemBinding@UFarDialogItem@@@@PEAHH@Z 000000018000c5f0 f i TmpCfg.obj
 0001:0000b670       ?CreateRadioButtonBinding@PluginDialogBuilder@@MEAAPEAU?$DialogItemBinding@UFarDialogItem@@@@PEAH@Z 000000018000c670 f i TmpCfg.obj
 0001:0000b6e0       ?DoShowDialog@?$DialogBuilderBase@UFarDialogItem@@@@MEAA_JXZ 000000018000c6e0 f i TmpCfg.obj
 0001:0000b6f0       ?DoShowDialog@PluginDialogBuilder@@MEAA_JXZ 000000018000c6f0 f i TmpCfg.obj
 0001:0000b7a0       ?EndColumns@?$DialogBuilderBase@UFarDialogItem@@@@QEAAXXZ 000000018000c7a0 f i TmpCfg.obj
 0001:0000b8c0       ?GetLangString@PluginDialogBuilder@@MEAAPEB_WH@Z 000000018000c8c0 f i TmpCfg.obj
 0001:0000b8d0       ?GetOptions@@YAXXZ         000000018000c8d0 f   TmpCfg.obj
 0001:0000be70       ?SaveValue@?$DialogItemBinding@UFarDialogItem@@@@UEAAXPEAUFarDialogItem@@H@Z 000000018000ce70 f i TmpCfg.obj
 0001:0000be70       _guard_check_icall_nop     000000018000ce70 f i LIBCMT:guard_support.obj
 0001:0000be70       ?InitDialogItem@?$DialogBuilderBase@UFarDialogItem@@@@MEAAXPEAUFarDialogItem@@PEB_W@Z 000000018000ce70 f i TmpCfg.obj
 0001:0000be80       ?InitDialogItem@PluginDialogBuilder@@MEAAXPEAUFarDialogItem@@PEB_W@Z 000000018000ce80 f i TmpCfg.obj
 0001:0000beb0       ?SaveValue@PluginCheckBoxBinding@@UEAAXPEAUFarDialogItem@@H@Z 000000018000ceb0 f i TmpCfg.obj
 0001:0000bf10       ?SaveValue@PluginEditFieldBinding@@UEAAXPEAUFarDialogItem@@H@Z 000000018000cf10 f i TmpCfg.obj
 0001:0000bf50       ?SaveValue@PluginIntEditFieldBinding@@UEAAXPEAUFarDialogItem@@H@Z 000000018000cf50 f i TmpCfg.obj
 0001:0000bfa0       ?SaveValue@PluginRadioButtonBinding@@UEAAXPEAUFarDialogItem@@H@Z 000000018000cfa0 f i TmpCfg.obj
 0001:0000bff0       ?SaveValue@PluginUIntEditFieldBinding@@UEAAXPEAUFarDialogItem@@H@Z 000000018000cff0 f i TmpCfg.obj
 0001:0000c040       ?TextWidth@?$DialogBuilderBase@UFarDialogItem@@@@MEAAHAEBUFarDialogItem@@@Z 000000018000d040 f i TmpCfg.obj
 0001:0000c050       ?TextWidth@PluginDialogBuilder@@MEAAHAEBUFarDialogItem@@@Z 000000018000d050 f i TmpCfg.obj
 0001:0000c060       ?UpdateBorderSize@?$DialogBuilderBase@UFarDialogItem@@@@IEAAXXZ 000000018000d060 f i TmpCfg.obj
 0001:0000c240       ??0TmpPanel@@QEAA@PEB_W@Z  000000018000d240 f   TmpClass.obj
 0001:0000c2e0       ??1TmpPanel@@QEAA@XZ       000000018000d2e0 f   TmpClass.obj
 0001:0000c320       ?BeginPutFiles@TmpPanel@@QEAAPEAXXZ 000000018000d320 f   TmpClass.obj
 0001:0000c3d0       ?CommitPutFiles@TmpPanel@@QEAAXPEAXH@Z 000000018000d3d0 f   TmpClass.obj
 0001:0000c500       ?GetFileInfoAndValidate@TmpPanel@@SA_NPEB_WPEAUPluginPanelItem@@H@Z 000000018000d500 f   TmpClass.obj
 0001:0000c820       ?GetFindData@TmpPanel@@QEAAHPEAPEAUPluginPanelItem@@PEA_K_K@Z 000000018000d820 f   TmpClass.obj
 0001:0000c9b0       ?GetOpenPanelInfo@TmpPanel@@QEAAXPEAUOpenPanelInfo@@@Z 000000018000d9b0 f   TmpClass.obj
 0001:0000cbb0       ?Inflate@SimpleString@@QEAAX_K@Z 000000018000dbb0 f i TmpClass.obj
 0001:0000cc40       ?IsCurrentFileCorrect@TmpPanel@@AEAA_NPEAPEA_W@Z 000000018000dc40 f   TmpClass.obj
 0001:0000cd80       ?ProcessEvent@TmpPanel@@QEAAH_JPEAX@Z 000000018000dd80 f   TmpClass.obj
 0001:0000cf20       ?ProcessKey@TmpPanel@@QEAAHPEBU_INPUT_RECORD@@@Z 000000018000df20 f   TmpClass.obj
 0001:0000d510       ?ProcessSaveListKey@TmpPanel@@AEAAXXZ 000000018000e510 f   TmpClass.obj
 0001:0000d860       ?PutDirectoryContents@TmpPanel@@QEAAHPEB_W@Z 000000018000e860 f   TmpClass.obj
 0001:0000da80       ?PutFiles@TmpPanel@@QEAAHPEAUPluginPanelItem@@_KHPEB_W_K@Z 000000018000ea80 f   TmpClass.obj
 0001:0000dc30       ?PutOneFile@TmpPanel@@QEAAHPEB_W@Z 000000018000ec30 f   TmpClass.obj
 0001:0000dd00       ?RemoveEmptyItems@TmpPanel@@AEAAXXZ 000000018000ed00 f   TmpClass.obj
 0001:0000de80       ?Replace@SimpleString@@QEAAAEAV1@_K0PEB_W0@Z 000000018000ee80 f i TmpClass.obj
 0001:0000e040       ?SaveListFile@TmpPanel@@AEAAXPEB_W@Z 000000018000f040 f   TmpClass.obj
 0001:0000e320       ?SetDirectory@TmpPanel@@QEAAHPEB_W_K@Z 000000018000f320 f   TmpClass.obj
 0001:0000e380       ?SetFindList@TmpPanel@@QEAAHPEBUPluginPanelItem@@_K@Z 000000018000f380 f   TmpClass.obj
 0001:0000e590       ?SortListCmp@@YAHPEBX0PEAX@Z 000000018000f590 f   TmpClass.obj
 0001:0000e5f0       ?SwitchToPanel@TmpPanel@@AEAAXH@Z 000000018000f5f0 f   TmpClass.obj
 0001:0000e6b0       ?UpdateItems@TmpPanel@@AEAAXHH@Z 000000018000f6b0 f   TmpClass.obj
 0001:0000ec20       ?ExpandEnvStrs@@YAPEA_WPEB_WAEAVStrBuf@@@Z 000000018000fc20 f   TmpMix.obj
 0001:0000ed20       ?FindListFile@@YA_NPEB_WAEAVStrBuf@@@Z 000000018000fd20 f   TmpMix.obj
 0001:0000f150       ?FormNtPath@@YAPEA_WPEB_WAEAVStrBuf@@@Z 0000000180010150 f   TmpMix.obj
 0001:0000f260       ?FreePanelItems@@YAXPEAUPluginPanelItem@@_K@Z 0000000180010260 f   TmpMix.obj
 0001:0000f2d0       ?GetFullPath@@YAPEA_WPEB_WAEAVStrBuf@@@Z 00000001800102d0 f   TmpMix.obj
 0001:0000f390       ?GetMsg@@YAPEB_WH@Z        0000000180010390 f   TmpMix.obj
 0001:0000f3b0       ?GoToFile@@YAXPEB_WH@Z     00000001800103b0 f   TmpMix.obj
 0001:0000f5f0       ?Grow@StrBuf@@QEAAX_K@Z    00000001800105f0 f i TmpMix.obj
 0001:0000f640       ?IsTextUTF8@@YA_NPEBD_K@Z  0000000180010640 f   TmpMix.obj
 0001:0000f6e0       ?ParseParam@@YAPEA_WAEAPEA_W@Z 00000001800106e0 f   TmpMix.obj
 0001:0000f740       ?WFD2FFD@@YAXAEAU_WIN32_FIND_DATAW@@AEAUPluginPanelItem@@@Z 0000000180010740 f   TmpMix.obj
 0001:0000f7a0       ??2@YAPEAX_K@Z             00000001800107a0 f   LIBCMT:new_scalar.obj
 0001:0000f7dc       ??_V@YAXPEAX@Z             00000001800107dc f   LIBCMT:delete_array.obj
 0001:0000f7dc       ??3@YAXPEAX_K@Z            00000001800107dc f   LIBCMT:delete_scalar_size.obj
 0001:0000f7e4       ??_U@YAPEAX_K@Z            00000001800107e4 f   LIBCMT:new_array.obj
 0001:0000fb1c       _DllMainCRTStartup         0000000180010b1c f   LIBCMT:dll_dllmain.obj
 0001:0000fb5c       ??0bad_alloc@std@@QEAA@AEBV01@@Z 0000000180010b5c f i LIBCMT:throw_bad_alloc.obj
 0001:0000fb9c       ??0bad_alloc@std@@QEAA@XZ  0000000180010b9c f i LIBCMT:throw_bad_alloc.obj
 0001:0000fbbc       ??0bad_array_new_length@std@@QEAA@AEBV01@@Z 0000000180010bbc f i LIBCMT:throw_bad_alloc.obj
 0001:0000fbfc       ??0bad_array_new_length@std@@QEAA@XZ 0000000180010bfc f i LIBCMT:throw_bad_alloc.obj
 0001:0000fc1c       ??0exception@std@@QEAA@AEBV01@@Z 0000000180010c1c f i LIBCMT:throw_bad_alloc.obj
 0001:0000fc54       ??1bad_alloc@std@@UEAA@XZ  0000000180010c54 f i LIBCMT:throw_bad_alloc.obj
 0001:0000fc54       ??1bad_array_new_length@std@@UEAA@XZ 0000000180010c54 f i LIBCMT:throw_bad_alloc.obj
 0001:0000fc68       ??_Gbad_array_new_length@std@@UEAAPEAXI@Z 0000000180010c68 f i LIBCMT:throw_bad_alloc.obj
 0001:0000fc68       ??_Gbad_alloc@std@@UEAAPEAXI@Z 0000000180010c68 f i LIBCMT:throw_bad_alloc.obj
 0001:0000fc68       ??_Gexception@std@@UEAAPEAXI@Z 0000000180010c68 f i LIBCMT:throw_bad_alloc.obj
 0001:0000fc68       ??_Eexception@std@@UEAAPEAXI@Z 0000000180010c68 f i LIBCMT:throw_bad_alloc.obj
 0001:0000fc68       ??_Ebad_array_new_length@std@@UEAAPEAXI@Z 0000000180010c68 f i LIBCMT:throw_bad_alloc.obj
 0001:0000fc68       ??_Ebad_alloc@std@@UEAAPEAXI@Z 0000000180010c68 f i LIBCMT:throw_bad_alloc.obj
 0001:0000fcac       ?__scrt_throw_std_bad_alloc@@YAXXZ 0000000180010cac f   LIBCMT:throw_bad_alloc.obj
 0001:0000fccc       ?__scrt_throw_std_bad_array_new_length@@YAXXZ 0000000180010ccc f   LIBCMT:throw_bad_alloc.obj
 0001:0000fcec       ?what@exception@std@@UEBAPEBDXZ 0000000180010cec f i LIBCMT:throw_bad_alloc.obj
 0001:0000fd00       ??3@YAXPEAX@Z              0000000180010d00 f   LIBCMT:delete_scalar.obj
 0001:0000fd08       __security_init_cookie     0000000180010d08 f   LIBCMT:gs_support.obj
 0001:0000fdb4       DllMain                    0000000180010db4 f   LIBCMT:dll_dllmain_stub.obj
 0001:0000fdb4       _get_startup_argv_mode     0000000180010db4 f   LIBCMT:argv_mode.obj
 0001:0000fdbc       ?__scrt_initialize_type_info@@YAXXZ 0000000180010dbc f   LIBCMT:tncleanup.obj
 0001:0000fdcc       ?__scrt_uninitialize_type_info@@YAXXZ 0000000180010dcc f   LIBCMT:tncleanup.obj
 0001:0000fdd8       __local_stdio_printf_options 0000000180010dd8 f i LIBCMT:default_local_stdio_options.obj
 0001:0000fde0       __local_stdio_scanf_options 0000000180010de0 f i LIBCMT:default_local_stdio_options.obj
 0001:0000fde8       __scrt_initialize_default_local_stdio_options 0000000180010de8 f   LIBCMT:default_local_stdio_options.obj
 0001:0000fe04       __scrt_acquire_startup_lock 0000000180010e04 f   LIBCMT:utility.obj
 0001:0000fe40       __scrt_dllmain_after_initialize_c 0000000180010e40 f   LIBCMT:utility.obj
 0001:0000fe74       __scrt_dllmain_before_initialize_c 0000000180010e74 f   LIBCMT:utility.obj
 0001:0000fe8c       __scrt_dllmain_crt_thread_attach 0000000180010e8c f   LIBCMT:utility.obj
 0001:0000feb4       __scrt_dllmain_crt_thread_detach 0000000180010eb4 f   LIBCMT:utility.obj
 0001:0000fecc       __scrt_dllmain_exception_filter 0000000180010ecc f   LIBCMT:utility.obj
 0001:0000ff2c       __scrt_dllmain_uninitialize_c 0000000180010f2c f   LIBCMT:utility.obj
 0001:0000ff5c       __scrt_dllmain_uninitialize_critical 0000000180010f5c f   LIBCMT:utility.obj
 0001:0000ff70       __scrt_initialize_crt      0000000180010f70 f   LIBCMT:utility.obj
 0001:0000ffbc       __scrt_initialize_onexit_tables 0000000180010fbc f   LIBCMT:utility.obj
 0001:00010094       __scrt_is_nonwritable_in_current_image 0000000180011094 f   LIBCMT:utility.obj
 0001:00010130       __scrt_release_startup_lock 0000000180011130 f   LIBCMT:utility.obj
 0001:00010154       __scrt_uninitialize_crt    0000000180011154 f   LIBCMT:utility.obj
 0001:00010180       __scrt_get_dyn_tls_init_callback 0000000180011180 f   LIBCMT:dyn_tls_init.obj
 0001:00010188       __crt_debugger_hook        0000000180011188 f   LIBCMT:utility_desktop.obj
 0001:00010190       __scrt_fastfail            0000000180011190 f   LIBCMT:utility_desktop.obj
 0001:000102dc       _RTC_Initialize            00000001800112dc f   LIBCMT:initsect.obj
 0001:00010318       _RTC_Terminate             0000000180011318 f   LIBCMT:initsect.obj
 0001:00010354       ??_Etype_info@@UEAAPEAXI@Z 0000000180011354 f i LIBCMT:std_type_info_static.obj
 0001:00010354       ??_Gtype_info@@UEAAPEAXI@Z 0000000180011354 f i LIBCMT:std_type_info_static.obj
 0001:00010380       __isa_available_init       0000000180011380 f   LIBCMT:cpu_disp.obj
 0001:0001053c       __scrt_is_ucrt_dll_in_use  000000018001153c f   LIBCMT:ucrt_detection.obj
 0001:00010560       memcpy_repmovs             0000000180011560 f   libvcruntime:memcpy.obj
 0001:00010580       memmove                    0000000180011580 f   libvcruntime:memcpy.obj
 0001:00010580       memcpy                     0000000180011580 f   libvcruntime:memcpy.obj
 0001:000109d0       memset_repmovs             00000001800119d0 f   libvcruntime:memset.obj
 0001:000109f0       memset                     00000001800119f0 f   libvcruntime:memset.obj
 0001:00010b80       wcschr                     0000000180011b80 f   libvcruntime:wcschr.obj
 0001:00010c14       wcsrchr                    0000000180011c14 f   libvcruntime:wcsrchr.obj
 0001:00010ce0       memcmp                     0000000180011ce0 f   libvcruntime:memcmp.obj
 0001:00010da8       __C_specific_handler       0000000180011da8 f   libvcruntime:riscchandler.obj
 0001:00010fb4       __std_exception_copy       0000000180011fb4 f   libvcruntime:std_exception.obj
 0001:00011044       __std_exception_destroy    0000000180012044 f   libvcruntime:std_exception.obj
 0001:0001106c       _CxxThrowException         000000018001206c f   libvcruntime:throw.obj
 0001:0001112c       __std_type_info_destroy_list 000000018001212c f   libvcruntime:std_type_info.obj
 0001:00011158       __vcrt_initialize          0000000180012158 f   libvcruntime:initialization.obj
 0001:0001118c       __vcrt_thread_attach       000000018001218c f   libvcruntime:initialization.obj
 0001:000111a0       __vcrt_thread_detach       00000001800121a0 f   libvcruntime:initialization.obj
 0001:000111b4       __vcrt_uninitialize        00000001800121b4 f   libvcruntime:initialization.obj
 0001:000111d4       __vcrt_uninitialize_critical 00000001800121d4 f   libvcruntime:initialization.obj
 0001:00011200       _NLG_Notify                0000000180012200 f   libvcruntime:notify.obj
 0001:00011220       __NLG_Dispatch2            0000000180012220 f   libvcruntime:notify.obj
 0001:00011230       __NLG_Return2              0000000180012230 f   libvcruntime:notify.obj
 0001:00011234       __except_validate_context_record 0000000180012234 f   libvcruntime:jbcxrval.obj
 0001:0001126c       __DestructExceptionObject  000000018001226c f   libvcruntime:ehhelpers.obj
 0001:000112e0       ?_CallMemberFunction0@@YAXQEAX0@Z 00000001800122e0 f i libvcruntime:ehhelpers.obj
 0001:000112e4       __vcrt_freefls             00000001800122e4 f   libvcruntime:per_thread_data.obj
 0001:00011304       __vcrt_freeptd             0000000180012304 f   libvcruntime:per_thread_data.obj
 0001:00011354       __vcrt_getptd_noexit       0000000180012354 f   libvcruntime:per_thread_data.obj
 0001:00011420       __vcrt_initialize_ptd      0000000180012420 f   libvcruntime:per_thread_data.obj
 0001:00011474       __vcrt_uninitialize_ptd    0000000180012474 f   libvcruntime:per_thread_data.obj
 0001:00011498       __vcrt_initialize_locks    0000000180012498 f   libvcruntime:locks.obj
 0001:000114e0       __vcrt_uninitialize_locks  00000001800124e0 f   libvcruntime:locks.obj
 0001:000116f0       __vcrt_FlsAlloc            00000001800126f0 f   libvcruntime:winapi_downlevel.obj
 0001:00011738       __vcrt_FlsFree             0000000180012738 f   libvcruntime:winapi_downlevel.obj
 0001:00011780       __vcrt_FlsGetValue         0000000180012780 f   libvcruntime:winapi_downlevel.obj
 0001:000117c8       __vcrt_FlsSetValue         00000001800127c8 f   libvcruntime:winapi_downlevel.obj
 0001:0001181c       __vcrt_InitializeCriticalSectionEx 000000018001281c f   libvcruntime:winapi_downlevel.obj
 0001:00011880       __vcrt_initialize_winapi_thunks 0000000180012880 f   libvcruntime:winapi_downlevel.obj
 0001:000118b0       __vcrt_uninitialize_winapi_thunks 00000001800128b0 f   libvcruntime:winapi_downlevel.obj
 0001:000118f0       __vcrt_initialize_pure_virtual_call_handler 00000001800128f0 f   libvcruntime:purevirt_data.obj
 0001:00011910       _CallSettingFrame          0000000180012910 f   libvcruntime:handlers.obj
 0001:00011960       _CallSettingFrameEncoded   0000000180012960 f   libvcruntime:handlers.obj
 0001:000119a8       calloc                     00000001800129a8 f   libucrt:calloc.obj
 0001:000119b0       free                       00000001800129b0 f   libucrt:free.obj
 0001:000119c4       malloc                     00000001800129c4 f   libucrt:malloc.obj
 0001:000119cc       realloc                    00000001800129cc f   libucrt:realloc.obj
 0001:000119d4       __acrt_initialize_new_handler 00000001800129d4 f   libucrt:new_handler.obj
 0001:000119dc       _callnewh                  00000001800129dc f   libucrt:new_handler.obj
 0001:00011a0c       _query_new_handler         0000000180012a0c f   libucrt:new_handler.obj
 0001:00011a40       _initterm                  0000000180012a40 f   libucrt:initterm.obj
 0001:00011aa4       _initterm_e                0000000180012aa4 f   libucrt:initterm.obj
 0001:00011ae4       _seh_filter_dll            0000000180012ae4 f   libucrt:exception_filter.obj
 0001:00011af8       _seh_filter_exe            0000000180012af8 f   libucrt:exception_filter.obj
 0001:00011ee8       __acrt_initialize_thread_local_exit_callback 0000000180012ee8 f   libucrt:exit.obj
 0001:00011ef0       _cexit                     0000000180012ef0 f   libucrt:exit.obj
 0001:00011f00       _exit                      0000000180012f00 f   libucrt:exit.obj
 0001:00011f0c       _is_c_termination_complete 0000000180012f0c f   libucrt:exit.obj
 0001:000120d8       __acrt_allocate_buffer_for_argv 00000001800130d8 f   libucrt:argv_parsing.obj
 0001:00012138       _configure_narrow_argv     0000000180013138 f   libucrt:argv_parsing.obj
 0001:000124b0       __dcrt_uninitialize_environments_nolock 00000001800134b0 f   libucrt:environment_initialization.obj
 0001:000124e8       _initialize_narrow_environment 00000001800134e8 f   libucrt:environment_initialization.obj
 0001:00012644       _execute_onexit_table      0000000180013644 f   libucrt:onexit.obj
 0001:00012680       _initialize_onexit_table   0000000180013680 f   libucrt:onexit.obj
 0001:000126e0       __acrt_uninitialize_command_line 00000001800136e0 f   libucrt:argv_data.obj
 0001:000127d8       __acrt_initialize          00000001800137d8 f   libucrt:initialization.obj
 0001:000127ec       __acrt_thread_attach       00000001800137ec f   libucrt:initialization.obj
 0001:00012800       __acrt_thread_detach       0000000180013800 f   libucrt:initialization.obj
 0001:00012810       __acrt_uninitialize        0000000180013810 f   libucrt:initialization.obj
 0001:00012848       __acrt_uninitialize_critical 0000000180013848 f   libucrt:initialization.obj
 0001:00012858       terminate                  0000000180013858 f   libucrt:terminate.obj
 0001:00012878       _wcsdup                    0000000180013878 f   libucrt:wcsdup.obj
 0001:00012878       wcsdup                     0000000180013878 f   libucrt:wcsdup.obj
 0001:000128fc       strcpy_s                   00000001800138fc f   libucrt:strcpy_s.obj
 0001:0001295c       ??0_LocaleUpdate@@QEAA@QEAU__crt_locale_pointers@@@Z 000000018001395c f i libucrt:output.obj
 0001:00012a10       strncmp                    0000000180013a10 f   libucrt:strncmp.obj
 0001:00012a90       abort                      0000000180013a90 f   libucrt:abort.obj
 0001:00012ae8       wcsncmp                    0000000180013ae8 f   libucrt:wcsncmp.obj
 0001:00012b14       _calloc_base               0000000180013b14 f   libucrt:calloc_base.obj
 0001:00012b8c       _free_base                 0000000180013b8c f   libucrt:free_base.obj
 0001:00012bcc       _malloc_base               0000000180013bcc f   libucrt:malloc_base.obj
 0001:00012c2c       _realloc_base              0000000180013c2c f   libucrt:realloc_base.obj
 0001:00012ca8       __acrt_initialize_locks    0000000180013ca8 f   libucrt:locks.obj
 0001:00012cf0       __acrt_lock                0000000180013cf0 f   libucrt:locks.obj
 0001:00012d0c       __acrt_uninitialize_locks  0000000180013d0c f   libucrt:locks.obj
 0001:00012d44       __acrt_unlock              0000000180013d44 f   libucrt:locks.obj
 0001:000130d8       __acrt_freeptd             00000001800140d8 f   libucrt:per_thread_data.obj
 0001:0001311c       __acrt_getptd              000000018001411c f   libucrt:per_thread_data.obj
 0001:000131f0       __acrt_getptd_head         00000001800141f0 f   libucrt:per_thread_data.obj
 0001:00013298       __acrt_getptd_noexit       0000000180014298 f   libucrt:per_thread_data.obj
 0001:00013364       __acrt_initialize_ptd      0000000180014364 f   libucrt:per_thread_data.obj
 0001:000133a0       __acrt_uninitialize_ptd    00000001800143a0 f   libucrt:per_thread_data.obj
 0001:000133c4       __acrt_get_process_end_policy 00000001800143c4 f   libucrt:win_policies.obj
 0001:00013400       __acrt_call_reportfault    0000000180014400 f   libucrt:invalid_parameter.obj
 0001:0001355c       __acrt_initialize_invalid_parameter_handler 000000018001455c f   libucrt:invalid_parameter.obj
 0001:00013564       _invalid_parameter         0000000180014564 f   libucrt:invalid_parameter.obj
 0001:00013614       _invalid_parameter_noinfo  0000000180014614 f   libucrt:invalid_parameter.obj
 0001:00013634       _invoke_watson             0000000180014634 f   libucrt:invalid_parameter.obj
 0001:0001367c       __acrt_errno_from_os_error 000000018001467c f   libucrt:errno.obj
 0001:000136c4       __acrt_errno_map_os_error  00000001800146c4 f   libucrt:errno.obj
 0001:00013714       __doserrno                 0000000180014714 f   libucrt:errno.obj
 0001:00013734       _errno                     0000000180014734 f   libucrt:errno.obj
 0001:00013768       ??$__acrt_mbs_to_wcs_cp@U__crt_win32_buffer_internal_dynamic_resizing@@@@YAHQEBDAEAV?$__crt_win32_buffer@_WU__crt_win32_buffer_internal_dynamic_resizing@@@@I@Z 0000000180014768 f i libucrt:argv_wildcards.obj
 0001:000138e0       ??$__acrt_wcs_to_mbs_cp@U__crt_win32_buffer_internal_dynamic_resizing@@@@YAHQEB_WAEAV?$__crt_win32_buffer@DU__crt_win32_buffer_internal_dynamic_resizing@@@@I@Z 00000001800148e0 f i libucrt:argv_wildcards.obj
 0001:00014110       __acrt_expand_narrow_argv_wildcards 0000000180015110 f   libucrt:argv_wildcards.obj
 0001:00014118       ??$__acrt_wcs_to_mbs_cp@U__crt_win32_buffer_no_resizing@@@@YAHQEB_WAEAV?$__crt_win32_buffer@DU__crt_win32_buffer_no_resizing@@@@I@Z 0000000180015118 f i libucrt:getmodulefilenamea.obj
 0001:0001422c       __acrt_GetModuleFileNameA  000000018001522c f   libucrt:getmodulefilenamea.obj
 0001:00014a78       __acrt_initialize_multibyte 0000000180015a78 f   libucrt:mbctype.obj
 0001:00014ad8       __acrt_update_thread_multibyte_data 0000000180015ad8 f   libucrt:mbctype.obj
 0001:00014af4       _setmbcp_nolock            0000000180015af4 f   libucrt:mbctype.obj
 0001:00014e28       _ismbblead                 0000000180015e28 f   libucrt:ismbbyte.obj
 0001:00014e3c       __acrt_initialize_command_line 0000000180015e3c f   libucrt:argv_data.obj
 0001:00014e64       wcscpy_s                   0000000180015e64 f   libucrt:wcscpy_s.obj
 0001:00014ecc       __acrt_MultiByteToWideChar 0000000180015ecc f   libucrt:multibytetowidechar.obj
 0001:00014f28       __acrt_WideCharToMultiByte 0000000180015f28 f   libucrt:widechartomultibyte.obj
 0001:00014fc0       __dcrt_get_narrow_environment_from_os 0000000180015fc0 f   libucrt:get_environment_from_os.obj
 0001:000150c4       _recalloc_base             00000001800160c4 f   libucrt:recalloc.obj
 0001:00015334       __acrt_AppPolicyGetProcessTerminationMethodInternal 0000000180016334 f   libucrt:winapi_thunks.obj
 0001:00015384       __acrt_AreFileApisANSI     0000000180016384 f   libucrt:winapi_thunks.obj
 0001:000153c0       __acrt_FlsAlloc            00000001800163c0 f   libucrt:winapi_thunks.obj
 0001:00015408       __acrt_FlsFree             0000000180016408 f   libucrt:winapi_thunks.obj
 0001:00015450       __acrt_FlsGetValue         0000000180016450 f   libucrt:winapi_thunks.obj
 0001:00015498       __acrt_FlsSetValue         0000000180016498 f   libucrt:winapi_thunks.obj
 0001:000154ec       __acrt_InitializeCriticalSectionEx 00000001800164ec f   libucrt:winapi_thunks.obj
 0001:00015550       __acrt_LCMapStringEx       0000000180016550 f   libucrt:winapi_thunks.obj
 0001:0001562c       __acrt_LocaleNameToLCID    000000018001662c f   libucrt:winapi_thunks.obj
 0001:0001567c       __acrt_initialize_winapi_thunks 000000018001667c f   libucrt:winapi_thunks.obj
 0001:000156b0       __acrt_uninitialize_winapi_thunks 00000001800166b0 f   libucrt:winapi_thunks.obj
 0001:000156f4       __acrt_initialize_heap     00000001800166f4 f   libucrt:heap_handle.obj
 0001:00015710       __acrt_uninitialize_heap   0000000180016710 f   libucrt:heap_handle.obj
 0001:00015918       __acrt_initialize_lowio    0000000180016918 f   libucrt:ioinit.obj
 0001:00015954       __acrt_uninitialize_lowio  0000000180016954 f   libucrt:ioinit.obj
 0001:00015994       __acrt_execute_initializers 0000000180016994 f   libucrt:shared_initialization.obj
 0001:00015a14       __acrt_execute_uninitializers 0000000180016a14 f   libucrt:shared_initialization.obj
 0001:00015a98       __acrt_get_sigabrt_handler 0000000180016a98 f   libucrt:signal.obj
 0001:00015ac8       __acrt_initialize_signal_handlers 0000000180016ac8 f   libucrt:signal.obj
 0001:00015ae8       raise                      0000000180016ae8 f   libucrt:signal.obj
 0001:00015d54       __acrt_has_user_matherr    0000000180016d54 f   libucrt:matherr.obj
 0001:00015d74       __acrt_initialize_user_matherr 0000000180016d74 f   libucrt:matherr.obj
 0001:00015d7c       __acrt_invoke_user_matherr 0000000180016d7c f   libucrt:matherr.obj
 0001:00015f88       __acrt_stdio_flush_nolock  0000000180016f88 f   libucrt:fflush.obj
 0001:00016004       _fflush_nolock             0000000180017004 f   libucrt:fflush.obj
 0001:00016050       _flushall                  0000000180017050 f   libucrt:fflush.obj
 0001:00016058       __acrt_initialize_stdio    0000000180017058 f   libucrt:_file.obj
 0001:00016178       __acrt_uninitialize_stdio  0000000180017178 f   libucrt:_file.obj
 0001:000161d4       _lock_file                 00000001800171d4 f   libucrt:_file.obj
 0001:000161e0       _unlock_file               00000001800171e0 f   libucrt:_file.obj
 0001:000161ec       _mbtowc_l                  00000001800171ec f   libucrt:mbtowc.obj
 0001:00016368       mbtowc                     0000000180017368 f   libucrt:mbtowc.obj
 0001:00016370       __acrt_update_locale_info  0000000180017370 f   libucrt:locale_update.obj
 0001:000163a4       __acrt_update_multibyte_info 00000001800173a4 f   libucrt:locale_update.obj
 0001:000163d8       _fileno                    00000001800173d8 f   libucrt:fileno.obj
 0001:00016470       __acrt_set_locale_changed  0000000180017470 f   libucrt:wsetlocale.obj
 0001:0001647c       __acrt_uninitialize_locale 000000018001747c f   libucrt:wsetlocale.obj
 0001:000164ac       __pctype_func              00000001800174ac f   libucrt:ctype.obj
 0001:000164dc       _query_new_mode            00000001800174dc f   libucrt:new_mode.obj
 0001:000164e4       __acrt_add_locale_ref      00000001800174e4 f   libucrt:locale_refcounting.obj
 0001:00016570       __acrt_free_locale         0000000180017570 f   libucrt:locale_refcounting.obj
 0001:000166e8       __acrt_locale_add_lc_time_reference 00000001800176e8 f   libucrt:locale_refcounting.obj
 0001:00016710       __acrt_locale_free_lc_time_if_unreferenced 0000000180017710 f   libucrt:locale_refcounting.obj
 0001:00016748       __acrt_locale_release_lc_time_reference 0000000180017748 f   libucrt:locale_refcounting.obj
 0001:00016770       __acrt_release_locale_ref  0000000180017770 f   libucrt:locale_refcounting.obj
 0001:00016818       __acrt_update_thread_locale_data 0000000180017818 f   libucrt:locale_refcounting.obj
 0001:00016888       _updatetlocinfoEx_nolock   0000000180017888 f   libucrt:locale_refcounting.obj
 0001:000168f0       qsort                      00000001800178f0 f   libucrt:qsort.obj
 0001:00016cb0       strncpy_s                  0000000180017cb0 f   libucrt:strncpy_s.obj
 0001:00016e30       strpbrk                    0000000180017e30 f   libucrt:strpbrk.obj
 0001:00017210       _mbsdec                    0000000180018210 f   libucrt:mbsdec.obj
 0001:00017218       _mbsdec_l                  0000000180018218 f   libucrt:mbsdec.obj
 0001:000172ac       __acrt_GetStringTypeA      00000001800182ac f   libucrt:getstringtypea.obj
 0001:00017754       __acrt_LCMapStringA        0000000180018754 f   libucrt:lcmapstringa.obj
 0001:00017804       _msize_base                0000000180018804 f   libucrt:msize.obj
 0001:00017928       __acrt_DownlevelLocaleNameToLCID 0000000180018928 f   libucrt:lcidtoname_downlevel.obj
 0001:0001795c       __acrt_lowio_create_handle_array 000000018001895c f   libucrt:osfinfo.obj
 0001:00017a04       __acrt_lowio_destroy_handle_array 0000000180018a04 f   libucrt:osfinfo.obj
 0001:00017a54       __acrt_lowio_ensure_fh_exists 0000000180018a54 f   libucrt:osfinfo.obj
 0001:00017afc       __acrt_lowio_lock_fh       0000000180018afc f   libucrt:osfinfo.obj
 0001:00017b24       __acrt_lowio_unlock_fh     0000000180018b24 f   libucrt:osfinfo.obj
 0001:00017b4c       _free_osfhnd               0000000180018b4c f   libucrt:osfinfo.obj
 0001:00017c08       _get_osfhandle             0000000180018c08 f   libucrt:osfinfo.obj
 0001:00017d0c       _commit                    0000000180018d0c f   libucrt:commit.obj
 0001:0001860c       _write                     000000018001960c f   libucrt:write.obj
 0001:000186f8       _write_nolock              00000001800196f8 f   libucrt:write.obj
 0001:000189d4       _fcloseall                 00000001800199d4 f   libucrt:closeall.obj
 0001:00018a88       __acrt_stdio_free_buffer_nolock 0000000180019a88 f   libucrt:_freebuf.obj
 0001:00018ac8       _isatty                    0000000180019ac8 f   libucrt:isatty.obj
 0001:00018b28       _isleadbyte_l              0000000180019b28 f i libucrt:_wctype.obj
 0001:00018b74       ?__mbrtowc_utf8@__crt_mbstring@@YA_KPEA_WPEBD_KPEAU_Mbstatet@@@Z 0000000180019b74 f   libucrt:mbrtowc.obj
 0001:00018bb0       ?__mbsrtowcs_utf8@__crt_mbstring@@YA_KPEA_WPEAPEBD_KPEAU_Mbstatet@@@Z 0000000180019bb0 f   libucrt:mbrtowc.obj
 0001:00018d28       __acrt_locale_free_monetary 0000000180019d28 f   libucrt:initmon.obj
 0001:00018e34       __acrt_locale_free_numeric 0000000180019e34 f   libucrt:initnum.obj
 0001:00018ef8       __acrt_locale_free_time    0000000180019ef8 f   libucrt:inittime.obj
 0001:00019000       __strncnt                  000000018001a000 f   libucrt:strncnt.obj
 0001:00019018       _query_app_type            000000018001a018 f   libucrt:report_runtime_error.obj
 0001:000190bc       _lseeki64_nolock           000000018001a0bc f   libucrt:lseek.obj
 0001:000190c4       _putwch_nolock             000000018001a0c4 f   libucrt:putwch.obj
 0001:00019100       _fclose_nolock             000000018001a100 f   libucrt:fclose.obj
 0001:00019184       fclose                     000000018001a184 f   libucrt:fclose.obj
 0001:000191e8       ?__mbrtoc32_utf8@__crt_mbstring@@YA_KPEA_UPEBD_KPEAU_Mbstatet@@@Z 000000018001a1e8 f   libucrt:mbrtoc32.obj
 0001:000193d0       log10                      000000018001a3d0 f   libucrt:log10.obj
 0001:0001997c       __dcrt_lowio_ensure_console_output_initialized 000000018001a97c f   libucrt:initcon.obj
 0001:000199d0       __dcrt_terminate_console_output 000000018001a9d0 f   libucrt:initcon.obj
 0001:000199ec       __dcrt_write_console       000000018001a9ec f   libucrt:initcon.obj
 0001:00019b20       _close                     000000018001ab20 f   libucrt:close.obj
 0001:00019bc4       _close_nolock              000000018001abc4 f   libucrt:close.obj
 0001:00019c84       ?__acrt_stdio_free_stream@@YAXV__crt_stdio_stream@@@Z 000000018001ac84 f   libucrt:stream.obj
 0001:00019dc4       _handle_error              000000018001adc4 f   libucrt:libm_error.obj
 0001:00019ef0       __acrt_initialize_fma3     000000018001aef0 f   libucrt:fma3_available.obj
 0001:00019f60       _log10_special             000000018001af60 f   libucrt:log_special.obj
 0001:0001a030       _get_fpsr                  000000018001b030 f   libucrt:fpsr.obj
 0001:0001a040       _set_fpsr                  000000018001b040 f   libucrt:fpsr.obj
 0001:0001a04a       _fclrf                     000000018001b04a f   libucrt:fpsr.obj
 0001:0001a05e       _frnd                      000000018001b05e f   libucrt:fpsr.obj
 0001:0001a080       _raise_exc                 000000018001b080 f   libucrt:fpexcept.obj
 0001:0001a0a8       _raise_exc_ex              000000018001b0a8 f   libucrt:fpexcept.obj
 0001:0001a3b8       _set_errno_from_matherr    000000018001b3b8 f   libucrt:fpexcept.obj
 0001:0001a3e8       _clrfp                     000000018001b3e8 f   libucrt:fpctrl.obj
 0001:0001a408       _ctrlfp                    000000018001b408 f   libucrt:fpctrl.obj
 0001:0001a484       _set_statfp                000000018001b484 f   libucrt:fpctrl.obj
 0001:0001a4a4       _statfp                    000000018001b4a4 f   libucrt:fpctrl.obj
 0001:0001a4b5       IsProcessorFeaturePresent  000000018001b4b5 f   kernel32:KERNEL32.dll
 0001:0001a4c0       _FindPESection             000000018001b4c0 f   LIBCMT:pesect.obj
 0001:0001a510       _IsNonwritableInCurrentImage 000000018001b510 f   LIBCMT:pesect.obj
 0001:0001a560       _ValidateImageBase         000000018001b560 f   LIBCMT:pesect.obj
 0001:0001a590       __GSHandlerCheck           000000018001b590 f   LIBCMT:gshandler.obj
 0001:0001a5b0       __GSHandlerCheckCommon     000000018001b5b0 f   LIBCMT:gshandler.obj
 0001:0001a620       __security_check_cookie    000000018001b620 f   LIBCMT:amdsecgs.obj
 0001:0001a644       __raise_securityfailure    000000018001b644 f   LIBCMT:gs_report.obj
 0001:0001a678       __report_gsfailure         000000018001b678 f   LIBCMT:gs_report.obj
 0001:0001a74c       __report_rangecheckfailure 000000018001b74c f   LIBCMT:gs_report.obj
 0001:0001a760       __report_securityfailure   000000018001b760 f   LIBCMT:gs_report.obj
 0001:0001a8f0       _guard_dispatch_icall_nop  000000018001b8f0 f   LIBCMT:guard_dispatch.obj
 0001:0001bde0       _TI2?AVbad_alloc@std@@     000000018001cde0     LIBCMT:throw_bad_alloc.obj
 0001:0001be00       _CTA2?AVbad_alloc@std@@    000000018001ce00     LIBCMT:throw_bad_alloc.obj
 0001:0001be18       _CT??_R0?AVbad_alloc@std@@@8??0bad_alloc@std@@QEAA@AEBV01@@Z24 000000018001ce18     LIBCMT:throw_bad_alloc.obj
 0001:0001be40       _CT??_R0?AVexception@std@@@8??0exception@std@@QEAA@AEBV01@@Z24 000000018001ce40     LIBCMT:throw_bad_alloc.obj
 0001:0001be68       _TI3?AVbad_array_new_length@std@@ 000000018001ce68     LIBCMT:throw_bad_alloc.obj
 0001:0001be88       _CTA3?AVbad_array_new_length@std@@ 000000018001ce88     LIBCMT:throw_bad_alloc.obj
 0001:0001bea8       _CT??_R0?AVbad_array_new_length@std@@@8??0bad_array_new_length@std@@QEAA@AEBV01@@Z24 000000018001cea8     LIBCMT:throw_bad_alloc.obj
 0002:00000038       __scrt_native_dllmain_reason 000000018001e038     LIBCMT:utility.obj
 0002:00000040       __security_cookie_complement 000000018001e040     LIBCMT:gs_cookie.obj
 0002:00000048       __security_cookie          000000018001e048     LIBCMT:gs_cookie.obj
 0002:00000050       __isa_available            000000018001e050     LIBCMT:cpu_disp.obj
 0002:00000054       __isa_enabled              000000018001e054     LIBCMT:cpu_disp.obj
 0002:00000058       __memcpy_nt_iters          000000018001e058     LIBCMT:cpu_disp.obj
 0002:00000070       __abort_behavior           000000018001e070     libucrt:abort.obj
 0002:00000390       __acrt_initial_multibyte_data 000000018001e390     libucrt:mbctype.obj
 0002:000005c0       __acrt_initial_locale_data 000000018001e5c0     libucrt:nlsdata.obj
 0002:00000718       __acrt_initial_locale_pointers 000000018001e718     libucrt:nlsdata.obj
 0002:00000728       __acrt_wide_c_locale_string 000000018001e728     libucrt:nlsdata.obj
 0002:00000730       _iob                       000000018001e730     libucrt:_file.obj
 0002:00000838       __globallocalestatus       000000018001e838     libucrt:glstatus.obj
 0002:00000840       __acrt_lconv_c             000000018001e840     libucrt:localeconv.obj
 0002:000008d8       __acrt_lconv_static_decimal 000000018001e8d8     libucrt:localeconv.obj
 0002:000008dc       __acrt_lconv_static_W_decimal 000000018001e8dc     libucrt:localeconv.obj
 0002:000008e0       _lookuptrailbytes          000000018001e8e0     libucrt:read.obj
 0002:00000a00       _fltused                   000000018001ea00     LIBCMT:fltused.obj
 0002:00000a08       ??_R0?AVbad_alloc@std@@@8  000000018001ea08     LIBCMT:throw_bad_alloc.obj
 0002:00000a30       ??_R0?AVexception@std@@@8  000000018001ea30     LIBCMT:throw_bad_alloc.obj
 0002:00000a58       ??_R0?AVbad_array_new_length@std@@@8 000000018001ea58     LIBCMT:throw_bad_alloc.obj
 0002:00000a88       ??_R0?AVtype_info@@@8      000000018001ea88     LIBCMT:std_type_info_static.obj
 0002:00000ab0       ?CommonPanels@@3PAU_PluginPanels@@A 000000018001eab0     TmpPanel.obj
 0002:00000b50       ?CurrentCommonPanel@@3IA   000000018001eb50     TmpPanel.obj
 0002:00000b60       ?Info@@3UPluginStartupInfo@@A 000000018001eb60     TmpPanel.obj
 0002:00000c70       ?FSF@@3UFarStandardFunctions@@A 000000018001ec70     TmpPanel.obj
 0002:00000e10       ?Opt@@3Uoptions_s@@A       000000018001ee10     TmpCfg.obj
 0002:00001464       ?StartupOptFullScreenPanel@@3HA 000000018001f464     TmpCfg.obj
 0002:00001468       ?StartupOptCommonPanel@@3HA 000000018001f468     TmpCfg.obj
 0002:0000146c       ?StartupOpenFrom@@3HA      000000018001f46c     TmpCfg.obj
 0002:00001790       ?__type_info_root_node@@3U__type_info_node@@A 000000018001f790     LIBCMT:tncleanup.obj
 0002:000017a0       ?_OptionsStorage@?1??__local_stdio_printf_options@@9@4_KA 000000018001f7a0     LIBCMT:default_local_stdio_options.obj
 0002:000017a8       ?_OptionsStorage@?1??__local_stdio_scanf_options@@9@4_KA 000000018001f7a8     LIBCMT:default_local_stdio_options.obj
 0002:000017b0       __scrt_current_native_startup_state 000000018001f7b0     LIBCMT:utility.obj
 0002:000017b8       __scrt_native_startup_lock 000000018001f7b8     LIBCMT:utility.obj
 0002:000017f8       __scrt_debugger_hook_flag  000000018001f7f8     LIBCMT:utility_desktop.obj
 0002:000017fc       __favor                    000000018001f7fc     LIBCMT:cpu_disp.obj
 0002:00001800       ?__WinRTOutOfMemoryExceptionCallback@@3P6APEAXXZEA 000000018001f800     libvcruntime:ehhelpers.obj
 0002:00001808       ?pArgList@UnDecorator@@0PEAVReplicator@@EA 000000018001f808     libvcruntime:undname.obj
 0002:00001810       ?pZNameList@UnDecorator@@0PEAVReplicator@@EA 000000018001f810     libvcruntime:undname.obj
 0002:00001818       ?pTemplateArgList@UnDecorator@@0PEAVReplicator@@EA 000000018001f818     libvcruntime:undname.obj
 0002:00001820       ?gName@UnDecorator@@0PEBDEB 000000018001f820     libvcruntime:undname.obj
 0002:00001828       ?name@UnDecorator@@0PEBDEB 000000018001f828     libvcruntime:undname.obj
 0002:00001830       ?disableFlags@UnDecorator@@0KA 000000018001f830     libvcruntime:undname.obj
 0002:00001834       ?fExplicitTemplateParams@UnDecorator@@0_NA 000000018001f834     libvcruntime:undname.obj
 0002:00001835       ?fGetTemplateArgumentList@UnDecorator@@0_NA 000000018001f835     libvcruntime:undname.obj
 0002:00001838       ?m_pGetParameter@UnDecorator@@0P6APEADJ@ZEA 000000018001f838     libvcruntime:undname.obj
 0002:00001840       ?m_CHPENameOffset@UnDecorator@@0KA 000000018001f840     libvcruntime:undname.obj
 0002:00001844       ?m_recursionLevel@UnDecorator@@0KA 000000018001f844     libvcruntime:undname.obj
 0002:00001970       __pPurecall                000000018001f970     libvcruntime:purevirt_data.obj
 0002:00001990       ?c_exit_complete@?1???R<lambda_6e4b09c48022b2350581041d5f6b0c4c>@@QEBA@XZ@4_NA 000000018001f990     libucrt:exit.obj
 0002:00001aa8       _environ_table             000000018001faa8     libucrt:environment_initialization.obj
 0002:00001ab0       _wenviron_table            000000018001fab0     libucrt:environment_initialization.obj
 0002:00001ab8       __dcrt_initial_wide_environment 000000018001fab8     libucrt:environment_initialization.obj
 0002:00001ac0       __dcrt_initial_narrow_environment 000000018001fac0     libucrt:environment_initialization.obj
 0002:00001ac8       __acrt_atexit_table        000000018001fac8     libucrt:onexit.obj
 0002:00001ae0       __acrt_at_quick_exit_table 000000018001fae0     libucrt:onexit.obj
 0002:00001d40       _mbctype                   000000018001fd40     libucrt:mbctype.obj
 0002:00001d48       _mbcasemap                 000000018001fd48     libucrt:mbctype.obj
 0002:00001d50       __acrt_current_multibyte_data 000000018001fd50     libucrt:mbctype.obj
 0002:00001d60       _pgmptr                    000000018001fd60     libucrt:argv_data.obj
 0002:00001d68       __argc                     000000018001fd68     libucrt:argv_data.obj
 0002:00001d70       __argv                     000000018001fd70     libucrt:argv_data.obj
 0002:00001d78       __wargv                    000000018001fd78     libucrt:argv_data.obj
 0002:00001d80       _acmdln                    000000018001fd80     libucrt:argv_data.obj
 0002:00001d88       _wcmdln                    000000018001fd88     libucrt:argv_data.obj
 0002:00001f40       __acrt_heap                000000018001ff40     libucrt:heap_handle.obj
 0002:00001f50       __pioinfo                  000000018001ff50     libucrt:ioinit.obj
 0002:00002350       _nhandle                   0000000180020350     libucrt:ioinit.obj
 0002:00002380       __acrt_current_locale_data 0000000180020380     libucrt:nlsdata.obj
 0002:00002388       _nstream                   0000000180020388     libucrt:_file.obj
 0002:00002390       __piob                     0000000180020390     libucrt:_file.obj
 0002:00002398       __acrt_stdout_buffer       0000000180020398     libucrt:_sftbuf.obj
 0002:000023a0       __acrt_stderr_buffer       00000001800203a0     libucrt:_sftbuf.obj
 0002:000023b0       __acrt_locale_changed_data 00000001800203b0     libucrt:wsetlocale.obj
 0002:000023b8       __acrt_lconv_static_null   00000001800203b8     libucrt:localeconv.obj
 0002:000023bc       __acrt_lconv_static_W_null 00000001800203bc     libucrt:localeconv.obj
 0002:000023d0       __fma3_is_available        00000001800203d0     libucrt:fma3_available.obj
 0002:000023d4       __use_fma3_lib             00000001800203d4     libucrt:fma3_available.obj
 0002:00002950       __scrt_ucrt_dll_is_in_use  0000000180020950     <common>
 0002:00002958       __dyn_tls_init_callback    0000000180020958     <common>
 0004:00000000       __imp_IsTextUnicode        0000000180023000     advapi32:ADVAPI32.dll
 0004:00000008       \177ADVAPI32_NULL_THUNK_DATA 0000000180023008     advapi32:ADVAPI32.dll
 0004:00000010       __imp_DeleteFileW          0000000180023010     kernel32:KERNEL32.dll
 0004:00000018       __imp_GetFileSize          0000000180023018     kernel32:KERNEL32.dll
 0004:00000020       __imp_CloseHandle          0000000180023020     kernel32:KERNEL32.dll
 0004:00000028       __imp_WaitForSingleObject  0000000180023028     kernel32:KERNEL32.dll
 0004:00000030       __imp_CreateProcessW       0000000180023030     kernel32:KERNEL32.dll
 0004:00000038       __imp_CreateFileMappingW   0000000180023038     kernel32:KERNEL32.dll
 0004:00000040       __imp_MapViewOfFile        0000000180023040     kernel32:KERNEL32.dll
 0004:00000048       __imp_UnmapViewOfFile      0000000180023048     kernel32:KERNEL32.dll
 0004:00000050       __imp_lstrcmpW             0000000180023050     kernel32:KERNEL32.dll
 0004:00000058       __imp_lstrcmpiW            0000000180023058     kernel32:KERNEL32.dll
 0004:00000060       __imp_lstrcpynW            0000000180023060     kernel32:KERNEL32.dll
 0004:00000068       __imp_lstrcpyW             0000000180023068     kernel32:KERNEL32.dll
 0004:00000070       __imp_lstrcatW             0000000180023070     kernel32:KERNEL32.dll
 0004:00000078       __imp_CreateFileW          0000000180023078     kernel32:KERNEL32.dll
 0004:00000080       __imp_MultiByteToWideChar  0000000180023080     kernel32:KERNEL32.dll
 0004:00000088       __imp_GetConsoleTitleW     0000000180023088     kernel32:KERNEL32.dll
 0004:00000090       __imp_SetConsoleTitleW     0000000180023090     kernel32:KERNEL32.dll
 0004:00000098       __imp_FindClose            0000000180023098     kernel32:KERNEL32.dll
 0004:000000a0       __imp_FindFirstFileW       00000001800230a0     kernel32:KERNEL32.dll
 0004:000000a8       __imp_FindNextFileW        00000001800230a8     kernel32:KERNEL32.dll
 0004:000000b0       __imp_GetFileAttributesW   00000001800230b0     kernel32:KERNEL32.dll
 0004:000000b8       __imp_GetFileTime          00000001800230b8     kernel32:KERNEL32.dll
 0004:000000c0       __imp_WriteFile            00000001800230c0     kernel32:KERNEL32.dll
 0004:000000c8       __imp_WideCharToMultiByte  00000001800230c8     kernel32:KERNEL32.dll
 0004:000000d0       __imp_ExpandEnvironmentStringsW 00000001800230d0     kernel32:KERNEL32.dll
 0004:000000d8       __imp_SearchPathW          00000001800230d8     kernel32:KERNEL32.dll
 0004:000000e0       __imp_WriteConsoleW        00000001800230e0     kernel32:KERNEL32.dll
 0004:000000e8       __imp_lstrlenW             00000001800230e8     kernel32:KERNEL32.dll
 0004:000000f0       __imp_GetStdHandle         00000001800230f0     kernel32:KERNEL32.dll
 0004:000000f8       __imp_QueryPerformanceCounter 00000001800230f8     kernel32:KERNEL32.dll
 0004:00000100       __imp_GetCurrentProcessId  0000000180023100     kernel32:KERNEL32.dll
 0004:00000108       __imp_GetCurrentThreadId   0000000180023108     kernel32:KERNEL32.dll
 0004:00000110       __imp_GetSystemTimeAsFileTime 0000000180023110     kernel32:KERNEL32.dll
 0004:00000118       __imp_InitializeSListHead  0000000180023118     kernel32:KERNEL32.dll
 0004:00000120       __imp_RtlCaptureContext    0000000180023120     kernel32:KERNEL32.dll
 0004:00000128       __imp_RtlLookupFunctionEntry 0000000180023128     kernel32:KERNEL32.dll
 0004:00000130       __imp_RtlVirtualUnwind     0000000180023130     kernel32:KERNEL32.dll
 0004:00000138       __imp_IsDebuggerPresent    0000000180023138     kernel32:KERNEL32.dll
 0004:00000140       __imp_UnhandledExceptionFilter 0000000180023140     kernel32:KERNEL32.dll
 0004:00000148       __imp_SetUnhandledExceptionFilter 0000000180023148     kernel32:KERNEL32.dll
 0004:00000150       __imp_GetStartupInfoW      0000000180023150     kernel32:KERNEL32.dll
 0004:00000158       __imp_IsProcessorFeaturePresent 0000000180023158     kernel32:KERNEL32.dll
 0004:00000160       __imp_GetModuleHandleW     0000000180023160     kernel32:KERNEL32.dll
 0004:00000168       __imp_RtlUnwindEx          0000000180023168     kernel32:KERNEL32.dll
 0004:00000170       __imp_RtlPcToFileHeader    0000000180023170     kernel32:KERNEL32.dll
 0004:00000178       __imp_RaiseException       0000000180023178     kernel32:KERNEL32.dll
 0004:00000180       __imp_InterlockedFlushSList 0000000180023180     kernel32:KERNEL32.dll
 0004:00000188       __imp_GetLastError         0000000180023188     kernel32:KERNEL32.dll
 0004:00000190       __imp_SetLastError         0000000180023190     kernel32:KERNEL32.dll
 0004:00000198       __imp_EnterCriticalSection 0000000180023198     kernel32:KERNEL32.dll
 0004:000001a0       __imp_LeaveCriticalSection 00000001800231a0     kernel32:KERNEL32.dll
 0004:000001a8       __imp_DeleteCriticalSection 00000001800231a8     kernel32:KERNEL32.dll
 0004:000001b0       __imp_InitializeCriticalSectionAndSpinCount 00000001800231b0     kernel32:KERNEL32.dll
 0004:000001b8       __imp_TlsAlloc             00000001800231b8     kernel32:KERNEL32.dll
 0004:000001c0       __imp_TlsGetValue          00000001800231c0     kernel32:KERNEL32.dll
 0004:000001c8       __imp_TlsSetValue          00000001800231c8     kernel32:KERNEL32.dll
 0004:000001d0       __imp_TlsFree              00000001800231d0     kernel32:KERNEL32.dll
 0004:000001d8       __imp_FreeLibrary          00000001800231d8     kernel32:KERNEL32.dll
 0004:000001e0       __imp_GetProcAddress       00000001800231e0     kernel32:KERNEL32.dll
 0004:000001e8       __imp_LoadLibraryExW       00000001800231e8     kernel32:KERNEL32.dll
 0004:000001f0       __imp_GetCurrentProcess    00000001800231f0     kernel32:KERNEL32.dll
 0004:000001f8       __imp_ExitProcess          00000001800231f8     kernel32:KERNEL32.dll
 0004:00000200       __imp_TerminateProcess     0000000180023200     kernel32:KERNEL32.dll
 0004:00000208       __imp_GetModuleHandleExW   0000000180023208     kernel32:KERNEL32.dll
 0004:00000210       __imp_GetModuleFileNameW   0000000180023210     kernel32:KERNEL32.dll
 0004:00000218       __imp_HeapAlloc            0000000180023218     kernel32:KERNEL32.dll
 0004:00000220       __imp_HeapFree             0000000180023220     kernel32:KERNEL32.dll
 0004:00000228       __imp_HeapReAlloc          0000000180023228     kernel32:KERNEL32.dll
 0004:00000230       __imp_FindFirstFileExW     0000000180023230     kernel32:KERNEL32.dll
 0004:00000238       __imp_IsValidCodePage      0000000180023238     kernel32:KERNEL32.dll
 0004:00000240       __imp_GetACP               0000000180023240     kernel32:KERNEL32.dll
 0004:00000248       __imp_GetOEMCP             0000000180023248     kernel32:KERNEL32.dll
 0004:00000250       __imp_GetCPInfo            0000000180023250     kernel32:KERNEL32.dll
 0004:00000258       __imp_GetCommandLineA      0000000180023258     kernel32:KERNEL32.dll
 0004:00000260       __imp_GetCommandLineW      0000000180023260     kernel32:KERNEL32.dll
 0004:00000268       __imp_GetEnvironmentStringsW 0000000180023268     kernel32:KERNEL32.dll
 0004:00000270       __imp_FreeEnvironmentStringsW 0000000180023270     kernel32:KERNEL32.dll
 0004:00000278       __imp_LCMapStringW         0000000180023278     kernel32:KERNEL32.dll
 0004:00000280       __imp_GetProcessHeap       0000000180023280     kernel32:KERNEL32.dll
 0004:00000288       __imp_GetFileType          0000000180023288     kernel32:KERNEL32.dll
 0004:00000290       __imp_GetStringTypeW       0000000180023290     kernel32:KERNEL32.dll
 0004:00000298       __imp_HeapSize             0000000180023298     kernel32:KERNEL32.dll
 0004:000002a0       __imp_SetStdHandle         00000001800232a0     kernel32:KERNEL32.dll
 0004:000002a8       __imp_FlushFileBuffers     00000001800232a8     kernel32:KERNEL32.dll
 0004:000002b0       __imp_GetConsoleCP         00000001800232b0     kernel32:KERNEL32.dll
 0004:000002b8       __imp_GetConsoleMode       00000001800232b8     kernel32:KERNEL32.dll
 0004:000002c0       __imp_SetFilePointerEx     00000001800232c0     kernel32:KERNEL32.dll
 0004:000002c8       \177KERNEL32_NULL_THUNK_DATA 00000001800232c8     kernel32:KERNEL32.dll
 0004:000002d0       __imp_ShellExecuteW        00000001800232d0     shell32:SHELL32.dll
 0004:000002d8       \177SHELL32_NULL_THUNK_DATA 00000001800232d8     shell32:SHELL32.dll
 0004:000002e0       __guard_check_icall_fptr   00000001800232e0     LIBCMT:guard_support.obj
 0004:000002e8       __guard_dispatch_icall_fptr 00000001800232e8     LIBCMT:guard_support.obj
 0004:000002f0       __IMPORT_DESCRIPTOR_KERNEL32 00000001800232f0     kernel32:KERNEL32.dll
 0004:00000304       __IMPORT_DESCRIPTOR_ADVAPI32 0000000180023304     advapi32:ADVAPI32.dll
 0004:00000318       __IMPORT_DESCRIPTOR_SHELL32 0000000180023318     shell32:SHELL32.dll
 0004:0000032c       __NULL_IMPORT_DESCRIPTOR   000000018002332c     kernel32:KERNEL32.dll

 entry point at        0001:0000fb1c

 Static symbols

 0001:000001a0       ?ParamsStr@?4??OpenW@@9@4QAY07$$CB_WA 00000001800011a0     TmpPanel.obj
 0001:000006fc       ?bom@?9??SaveListFile@TmpPanel@@AEAAXPEB_W@Z@4GB 00000001800016fc     TmpClass.obj
 0001:000006fe       ?bomhi@?M@??SaveListFile@TmpPanel@@AEAAXPEB_W@Z@4EB 00000001800016fe     TmpClass.obj
 0001:00000700       ?bomlo@?M@??SaveListFile@TmpPanel@@AEAAXPEB_W@Z@4GB 0000000180001700     TmpClass.obj
 0001:00000710       ?fmt1@?1??ProcessPanelSwitchMenu@TmpPanel@@AEAAXXZ@4QB_WB 0000000180001710     TmpClass.obj
 0001:00000890       ?ExceptionTemplate@?1??_CxxThrowException@@9@4UEHExceptionRecord@@B 0000000180001890     libvcruntime:throw.obj
 0001:000008e0       ?tokenTable@@3QBQEBDB      00000001800018e0     libvcruntime:undname.obj
 0001:00000960       ?nameTable@@3QBQEBDB       0000000180001960     libvcruntime:undname.obj
 0001:00000bf0       ?rttiTable@@3QBQEBDB       0000000180001bf0     libvcruntime:undname.obj
 0001:000012a8       ?module_names@?A0xbfd18cd1@@3QBQEB_WB 00000001800022a8     libvcruntime:winapi_downlevel.obj
 0001:00001378       ?candidate_modules@?1??try_get_FlsAlloc@@YAP6AKP6AXPEAX@Z@ZXZ@4QBW4module_id@?A0xbfd18cd1@@B 0000000180002378     libvcruntime:winapi_downlevel.obj
 0001:00001390       ?candidate_modules@?1??try_get_FlsFree@@YAP6AHK@ZXZ@4QBW4module_id@?A0xbfd18cd1@@B 0000000180002390     libvcruntime:winapi_downlevel.obj
 0001:000013a0       ?candidate_modules@?1??try_get_FlsGetValue@@YAP6APEAXK@ZXZ@4QBW4module_id@?A0xbfd18cd1@@B 00000001800023a0     libvcruntime:winapi_downlevel.obj
 0001:000013b8       ?candidate_modules@?1??try_get_FlsSetValue@@YAP6AHKPEAX@ZXZ@4QBW4module_id@?A0xbfd18cd1@@B 00000001800023b8     libvcruntime:winapi_downlevel.obj
 0001:000013d0       ?candidate_modules@?1??try_get_InitializeCriticalSectionEx@@YAP6AHPEAU_RTL_CRITICAL_SECTION@@KK@ZXZ@4QBW4module_id@?A0xbfd18cd1@@B 00000001800023d0     libvcruntime:winapi_downlevel.obj
 0001:00001500       __acrt_initializers        0000000180002500     libucrt:initialization.obj
 0001:00001600       ?errtable@@3QBUerrentry@?A0x31fdb9ec@@B 0000000180002600     libucrt:errno.obj
 0001:00001768       ?_mb_locale_names@@3QBQEB_WB 0000000180002768     libucrt:mbctype.obj
 0001:000017d0       ?module_names@?A0x391cf84c@@3QBQEB_WB 00000001800027d0     libucrt:winapi_thunks.obj
 0001:00001d78       ?candidate_modules@?1??try_get_AreFileApisANSI@@YAP6AHXZXZ@4QBW4module_id@?A0x391cf84c@@B 0000000180002d78     libucrt:winapi_thunks.obj
 0001:00001d90       ?candidate_modules@?1??try_get_FlsAlloc@@YAP6AKP6AXPEAX@Z@ZXZ@4QBW4module_id@?A0x391cf84c@@B 0000000180002d90     libucrt:winapi_thunks.obj
 0001:00001da8       ?candidate_modules@?1??try_get_FlsFree@@YAP6AHK@ZXZ@4QBW4module_id@?A0x391cf84c@@B 0000000180002da8     libucrt:winapi_thunks.obj
 0001:00001db8       ?candidate_modules@?1??try_get_FlsGetValue@@YAP6APEAXK@ZXZ@4QBW4module_id@?A0x391cf84c@@B 0000000180002db8     libucrt:winapi_thunks.obj
 0001:00001dd0       ?candidate_modules@?1??try_get_FlsSetValue@@YAP6AHKPEAX@ZXZ@4QBW4module_id@?A0x391cf84c@@B 0000000180002dd0     libucrt:winapi_thunks.obj
 0001:00001de8       ?candidate_modules@?1??try_get_InitializeCriticalSectionEx@@YAP6AHPEAU_RTL_CRITICAL_SECTION@@KK@ZXZ@4QBW4module_id@?A0x391cf84c@@B 0000000180002de8     libucrt:winapi_thunks.obj
 0001:00001e10       ?candidate_modules@?1??try_get_LCMapStringEx@@YAP6AHPEB_WK0HPEA_WHPEAU_nlsversioninfo@@PEAX_J@ZXZ@4QBW4module_id@?A0x391cf84c@@B 0000000180002e10     libucrt:winapi_thunks.obj
 0001:00001e28       ?candidate_modules@?1??try_get_LocaleNameToLCID@@YAP6AKPEB_WK@ZXZ@4QBW4module_id@?A0x391cf84c@@B 0000000180002e28     libucrt:winapi_thunks.obj
 0001:00001e44       ?candidate_modules@?1??try_get_AppPolicyGetProcessTerminationMethod@@YAP6AJPEAXPEAW4AppPolicyProcessTerminationMethod@@@ZXZ@4QBW4module_id@?A0x391cf84c@@B 0000000180002e44     libucrt:winapi_thunks.obj
 0001:00002af0       ?LcidToLocaleNameTable@?A0x881e4c05@@3QBULcidToLocaleName@1@B 0000000180003af0     libucrt:lcidtoname_downlevel.obj
 0001:00004550       ?LocaleNameToIndexTable@?A0x881e4c05@@3QBULocaleNameIndex@1@B 0000000180005550     libucrt:lcidtoname_downlevel.obj
 0001:00005df0       __real_ninf                0000000180006df0     libucrt:log10.obj
 0001:00005e00       __real_inf                 0000000180006e00     libucrt:log10.obj
 0001:00005e10       __real_neg_qnan            0000000180006e10     libucrt:log10.obj
 0001:00005e20       __real_qnanbit             0000000180006e20     libucrt:log10.obj
 0001:00005e30       __int_1023                 0000000180006e30     libucrt:log10.obj
 0001:00005e40       __mask_001                 0000000180006e40     libucrt:log10.obj
 0001:00005e50       __mask_mant                0000000180006e50     libucrt:log10.obj
 0001:00005e60       __mask_mant_top8           0000000180006e60     libucrt:log10.obj
 0001:00005e70       __mask_mant9               0000000180006e70     libucrt:log10.obj
 0001:00005e80       __real_log10_e             0000000180006e80     libucrt:log10.obj
 0001:00005e90       __real_log10_e_lead        0000000180006e90     libucrt:log10.obj
 0001:00005ea0       __real_log10_e_tail        0000000180006ea0     libucrt:log10.obj
 0001:00005eb0       __real_log10_2_lead        0000000180006eb0     libucrt:log10.obj
 0001:00005ec0       __real_log10_2_tail        0000000180006ec0     libucrt:log10.obj
 0001:00005ed0       __real_two                 0000000180006ed0     libucrt:log10.obj
 0001:00005ee0       __real_one                 0000000180006ee0     libucrt:log10.obj
 0001:00005ef0       __real_half                0000000180006ef0     libucrt:log10.obj
 0001:00005f00       __mask_100                 0000000180006f00     libucrt:log10.obj
 0001:00005f10       __real_1_over_512          0000000180006f10     libucrt:log10.obj
 0001:00005f20       __real_1_over_2            0000000180006f20     libucrt:log10.obj
 0001:00005f30       __real_1_over_3            0000000180006f30     libucrt:log10.obj
 0001:00005f40       __real_1_over_4            0000000180006f40     libucrt:log10.obj
 0001:00005f50       __real_1_over_5            0000000180006f50     libucrt:log10.obj
 0001:00005f60       __real_1_over_6            0000000180006f60     libucrt:log10.obj
 0001:00005f70       __real_neg_1023            0000000180006f70     libucrt:log10.obj
 0001:00005f80       __mask_2045                0000000180006f80     libucrt:log10.obj
 0001:00005f90       __real_threshold           0000000180006f90     libucrt:log10.obj
 0001:00005fa0       __real_near_one_lt         0000000180006fa0     libucrt:log10.obj
 0001:00005fb0       __real_near_one_gt         0000000180006fb0     libucrt:log10.obj
 0001:00005fc0       __real_min_norm            0000000180006fc0     libucrt:log10.obj
 0001:00005fd0       __real_notsign             0000000180006fd0     libucrt:log10.obj
 0001:00005fe0       __real_ca1                 0000000180006fe0     libucrt:log10.obj
 0001:00005ff0       __real_ca2                 0000000180006ff0     libucrt:log10.obj
 0001:00006000       __real_ca3                 0000000180007000     libucrt:log10.obj
 0001:00006010       __real_ca4                 0000000180007010     libucrt:log10.obj
 0001:00006020       __mask_lower               0000000180007020     libucrt:log10.obj
 0001:00006030       __flag_x_zero              0000000180007030     libucrt:log10.obj
 0001:00006034       __flag_x_neg               0000000180007034     libucrt:log10.obj
 0001:00006038       __flag_x_nan               0000000180007038     libucrt:log10.obj
 0001:00007890       __real@433fffffffffffff    0000000180008890     libucrt:fpsr.obj
 0001:00007898       __real@c33fffffffffffff    0000000180008898     libucrt:fpsr.obj
 0001:000078a0       GS_ExceptionPointers       00000001800088a0     LIBCMT:gs_report.obj
 0001:00007ea0       $$000000                   0000000180008ea0     chkstk.obj
 0001:00007f10       ?OpenPanelFromOutput@@YAPEAXPEA_W@Z 0000000180008f10 f   TmpPanel.obj
 0001:00008250       ?ProcessList@@YAXPEAXPEA_WH@Z 0000000180009250 f   TmpPanel.obj
 0001:000085d0       ?ReadFileList@@YAXPEA_WPEAHPEAPEAPEA_W@Z 00000001800095d0 f   TmpPanel.obj
 0001:00008730       ?ShowMenuFromList@@YAXPEA_W@Z 0000000180009730 f   TmpPanel.obj
 0001:000097cc       $LN39                      000000018000a7cc     TmpCfg.obj
 0001:0000b40c       $LN540                     000000018000c40c     TmpCfg.obj
 0001:0000b43c       $LN539                     000000018000c43c     TmpCfg.obj
 0001:0000b46c       $LN538                     000000018000c46c     TmpCfg.obj
 0001:0000b49c       $LN537                     000000018000c49c     TmpCfg.obj
 0001:0000b4cc       $LN536                     000000018000c4cc     TmpCfg.obj
 0001:0000b4fc       $LN535                     000000018000c4fc     TmpCfg.obj
 0001:0000b52c       $LN534                     000000018000c52c     TmpCfg.obj
 0001:0000b55c       $LN533                     000000018000c55c     TmpCfg.obj
 0001:0000b58c       $LN532                     000000018000c58c     TmpCfg.obj
 0001:0000b5bc       $LN531                     000000018000c5bc     TmpCfg.obj
 0001:0000b88c       $LN24                      000000018000c88c     TmpCfg.obj
 0001:0000c204       $LN36                      000000018000d204     TmpCfg.obj
 0001:0000f7ec       ?dllmain_crt_dispatch@@YAHQEAUHINSTANCE__@@KQEAX@Z 00000001800107ec f   LIBCMT:dll_dllmain.obj
 0001:0000f83c       ?dllmain_crt_process_attach@@YAHQEAUHINSTANCE__@@QEAX@Z 000000018001083c f   LIBCMT:dll_dllmain.obj
 0001:0000f958       ?dllmain_crt_process_detach@@YAH_N@Z 0000000180010958 f   LIBCMT:dll_dllmain.obj
 0001:0000f9e8       ?dllmain_dispatch@@YAHQEAUHINSTANCE__@@KQEAX@Z 00000001800109e8 f   LIBCMT:dll_dllmain.obj
 0001:00010550       $$000000                   0000000180011550     libvcruntime:memcpy.obj
 0001:00010607       MoveSmall                  0000000180011607     libvcruntime:memcpy.obj
 0001:000109c0       $$000000                   00000001800119c0     libvcruntime:memset.obj
 0001:00010abc       MsetTab                    0000000180011abc     libvcruntime:memset.obj
 0001:00010cd0       $$000000                   0000000180011cd0     libvcruntime:memcmp.obj
 0001:000111f0       $$000000                   00000001800121f0     libvcruntime:notify.obj
 0001:00011518       ?try_get_function@@YAPEAXW4function_id@?A0xbfd18cd1@@QEBDQEBW4module_id@2@2@Z 0000000180012518 f   libvcruntime:winapi_downlevel.obj
 0001:00011900       $$000000                   0000000180012900     libvcruntime:handlers.obj
 0001:00011c7c       ??$?RV<lambda_d80eeec6fff315bfe5c115232f3240e3>@@AEAV<lambda_6e4b09c48022b2350581041d5f6b0c4c>@@V<lambda_2358e3775559c9db80273638284d5e45>@@@?$__crt_seh_guarded_call@X@@QEAAX$$QEAV<lambda_d80eeec6fff315bfe5c115232f3240e3>@@AEAV<lambda_6e4b09c48022b2350581041d5f6b0c4c>@@$$QEAV<lambda_2358e3775559c9db80273638284d5e45>@@@Z 0000000180012c7c f   libucrt:exit.obj
 0001:00011cb4       ??R<lambda_6e4b09c48022b2350581041d5f6b0c4c>@@QEBA@XZ 0000000180012cb4 f   libucrt:exit.obj
 0001:00011d78       ?atexit_exception_filter@@YAHK@Z 0000000180012d78 f   libucrt:exit.obj
 0001:00011d84       ?common_exit@@YAXHW4_crt_exit_cleanup_mode@@W4_crt_exit_return_mode@@@Z 0000000180012d84 f   libucrt:exit.obj
 0001:00011e40       ?exit_or_terminate_process@@YAXI@Z 0000000180012e40 f   libucrt:exit.obj
 0001:00011e8c       ?try_cor_exit_process@@YAXI@Z 0000000180012e8c f   libucrt:exit.obj
 0001:00011f14       ??$parse_command_line@D@@YAXPEADPEAPEAD0PEA_K2@Z 0000000180012f14 f   libucrt:argv_parsing.obj
 0001:000122c0       ??$common_initialize_environment_nolock@D@@YAHXZ 00000001800132c0 f   libucrt:environment_initialization.obj
 0001:0001232c       ??$create_environment@D@@YAQEAPEADQEAD@Z 000000018001332c f   libucrt:environment_initialization.obj
 0001:00012434       ??$free_environment@_W@@YAXQEAPEA_W@Z 0000000180013434 f   libucrt:environment_initialization.obj
 0001:00012434       ??$free_environment@D@@YAXQEAPEAD@Z 0000000180013434 f   libucrt:environment_initialization.obj
 0001:00012478       ??$uninitialize_environment_internal@D@@YAXAEAPEAPEAD@Z 0000000180013478 f   libucrt:environment_initialization.obj
 0001:00012494       ??$uninitialize_environment_internal@_W@@YAXAEAPEAPEA_W@Z 0000000180013494 f   libucrt:environment_initialization.obj
 0001:000124f0       ??$?RV<lambda_7777bce6b2f8c936911f934f8298dc43>@@AEAV<lambda_f03950bc5685219e0bcd2087efbe011e>@@V<lambda_3883c3dff614d5e0c5f61bb1ac94921c>@@@?$__crt_seh_guarded_call@H@@QEAAH$$QEAV<lambda_7777bce6b2f8c936911f934f8298dc43>@@AEAV<lambda_f03950bc5685219e0bcd2087efbe011e>@@$$QEAV<lambda_3883c3dff614d5e0c5f61bb1ac94921c>@@@Z 00000001800134f0 f   libucrt:onexit.obj
 0001:0001252c       ??R<lambda_f03950bc5685219e0bcd2087efbe011e>@@QEBAHXZ 000000018001352c f   libucrt:onexit.obj
 0001:000126a8       initialize_global_variables 00000001800136a8 f   libucrt:initialization.obj
 0001:000126bc       initialize_c               00000001800136bc f   libucrt:initialization.obj
 0001:000126e0       initialize_global_state_isolation 00000001800136e0 f   libucrt:initialization.obj
 0001:000126e0       uninitialize_c             00000001800136e0 f   libucrt:initialization.obj
 0001:000126e0       uninitialize_global_state_isolation 00000001800136e0 f   libucrt:initialization.obj
 0001:000126e0       initialize_environment     00000001800136e0 f   libucrt:initialization.obj
 0001:000126e0       report_memory_leaks        00000001800136e0 f   libucrt:initialization.obj
 0001:000126e4       uninitialize_environment   00000001800136e4 f   libucrt:initialization.obj
 0001:000126f4       initialize_pointers        00000001800136f4 f   libucrt:initialization.obj
 0001:00012734       uninitialize_vcruntime     0000000180013734 f   libucrt:initialization.obj
 0001:0001273c       uninitialize_allocated_memory 000000018001373c f   libucrt:initialization.obj
 0001:0001277c       uninitialize_allocated_io_buffers 000000018001377c f   libucrt:initialization.obj
 0001:00012a00       $$000000                   0000000180013a00     libucrt:strncmp.obj
 0001:00012d60       ??$?RV<lambda_0ae27a3a962d80f24befdcbee591983d>@@AEAV<lambda_8d0ee55de4b1038c4002e0adecdf1839>@@V<lambda_dc504788e8f1664fe9b84e20bfb512f2>@@@?$__crt_seh_guarded_call@X@@QEAAX$$QEAV<lambda_0ae27a3a962d80f24befdcbee591983d>@@AEAV<lambda_8d0ee55de4b1038c4002e0adecdf1839>@@$$QEAV<lambda_dc504788e8f1664fe9b84e20bfb512f2>@@@Z 0000000180013d60 f   libucrt:per_thread_data.obj
 0001:00012da0       ??$?RV<lambda_2d41944a1d46af3157314b8a01080d33>@@AEAV<lambda_8f455de75cd7d7f24b4096f044d8b9e6>@@V<lambda_aa500f224e6afead328df44964fe2772>@@@?$__crt_seh_guarded_call@X@@QEAAX$$QEAV<lambda_2d41944a1d46af3157314b8a01080d33>@@AEAV<lambda_8f455de75cd7d7f24b4096f044d8b9e6>@@$$QEAV<lambda_aa500f224e6afead328df44964fe2772>@@@Z 0000000180013da0 f   libucrt:per_thread_data.obj
 0001:00012de0       ??$?RV<lambda_aa87e3671a710a21b5dc78c0bdf72e11>@@AEAV<lambda_92619d2358a28f41a33ba319515a20b9>@@V<lambda_6992ecaafeb10aed2b74cb1fae11a551>@@@?$__crt_seh_guarded_call@X@@QEAAX$$QEAV<lambda_aa87e3671a710a21b5dc78c0bdf72e11>@@AEAV<lambda_92619d2358a28f41a33ba319515a20b9>@@$$QEAV<lambda_6992ecaafeb10aed2b74cb1fae11a551>@@@Z 0000000180013de0 f   libucrt:per_thread_data.obj
 0001:00012e28       ??$?RV<lambda_f2e299630e499de9f9a165e60fcd3db5>@@AEAV<lambda_2ae9d31cdba2644fcbeaf08da7c24588>@@V<lambda_40d01ff24d0e7b3814fdbdcee8eab3c7>@@@?$__crt_seh_guarded_call@X@@QEAAX$$QEAV<lambda_f2e299630e499de9f9a165e60fcd3db5>@@AEAV<lambda_2ae9d31cdba2644fcbeaf08da7c24588>@@$$QEAV<lambda_40d01ff24d0e7b3814fdbdcee8eab3c7>@@@Z 0000000180013e28 f   libucrt:per_thread_data.obj
 0001:00012e88       ?construct_ptd_array@@YAXQEAU__acrt_ptd@@@Z 0000000180013e88 f   libucrt:per_thread_data.obj
 0001:00012f58       ?destroy_fls@@YAXPEAX@Z    0000000180013f58 f   libucrt:per_thread_data.obj
 0001:00012f78       ?destroy_ptd_array@@YAXQEAU__acrt_ptd@@@Z 0000000180013f78 f   libucrt:per_thread_data.obj
 0001:00013070       ?replace_current_thread_locale_nolock@@YAXQEAU__acrt_ptd@@QEAU__crt_locale_data@@@Z 0000000180014070 f   libucrt:per_thread_data.obj
 0001:00013754       ?<lambda_invoker_cdecl>@<lambda_c2303d2482d7c3675ea2e24c4cfb6115>@@CAHPEBX0@Z 0000000180014754 f   libucrt:argv_wildcards.obj
 0001:00013a6c       ??$common_expand_argv_wildcards@D@@YAHQEAPEADQEAPEAPEAD@Z 0000000180014a6c f   libucrt:argv_wildcards.obj
 0001:00013c78       ??$copy_and_add_argument_to_buffer@D@@YAHQEBD0_KAEAV?$argument_list@D@?A0x5f5c8891@@@Z 0000000180014c78 f   libucrt:argv_wildcards.obj
 0001:00013e00       ??$expand_argument_wildcards@D@@YAHQEAD0AEAV?$argument_list@D@?A0x5f5c8891@@@Z 0000000180014e00 f   libucrt:argv_wildcards.obj
 0001:0001434c       ??$?RV<lambda_efdfa57d1f175319df784efa44bb7b81>@@AEAV<lambda_5f0a4c1567f8adc6734073e5d1e1b35c>@@V<lambda_2e8a7d3640ea6ccb4c2413664c2db6fd>@@@?$__crt_seh_guarded_call@X@@QEAAX$$QEAV<lambda_efdfa57d1f175319df784efa44bb7b81>@@AEAV<lambda_5f0a4c1567f8adc6734073e5d1e1b35c>@@$$QEAV<lambda_2e8a7d3640ea6ccb4c2413664c2db6fd>@@@Z 000000018001534c f   libucrt:mbctype.obj
 0001:00014508       ?getSystemCP@@YAHH@Z       0000000180015508 f   libucrt:mbctype.obj
 0001:00014588       ?setSBCS@@YAXPEAU__crt_multibyte_data@@@Z 0000000180015588 f   libucrt:mbctype.obj
 0001:00014618       ?setSBUpLow@@YAXPEAU__crt_multibyte_data@@@Z 0000000180015618 f   libucrt:mbctype.obj
 0001:000147fc       ?setmbcp_internal@@YAHH_NQEAU__acrt_ptd@@QEAPEAU__crt_multibyte_data@@@Z 00000001800157fc f   libucrt:mbctype.obj
 0001:000149c0       ?update_thread_multibyte_data_internal@@YAPEAU__crt_multibyte_data@@QEAU__acrt_ptd@@QEAPEAU1@@Z 00000001800159c0 f   libucrt:mbctype.obj
 0001:00014db0       ?x_ismbbtype_l@@YAHPEAU__crt_locale_pointers@@IHH@Z 0000000180015db0 f   libucrt:ismbbyte.obj
 0001:0001515c       ?try_get_function@@YAPEAXW4function_id@?A0x391cf84c@@QEBDQEBW4module_id@2@2@Z 000000018001615c f   libucrt:winapi_thunks.obj
 0001:0001571c       ?initialize_inherited_file_handles_nolock@@YAXXZ 000000018001671c f   libucrt:ioinit.obj
 0001:0001580c       ?initialize_stdio_handles_nolock@@YAXXZ 000000018001680c f   libucrt:ioinit.obj
 0001:00015a50       ??$?RV<lambda_450d765d439847d4c735a33c368b5fc0>@@AEAV<lambda_44731a7d0e6d81c3e6aa82d741081786>@@V<lambda_601a2a7da3b7a96e9554ac7215c4b07c>@@@?$__crt_seh_guarded_call@P6AXH@Z@@QEAAP6AXH@Z$$QEAV<lambda_450d765d439847d4c735a33c368b5fc0>@@AEAV<lambda_44731a7d0e6d81c3e6aa82d741081786>@@$$QEAV<lambda_601a2a7da3b7a96e9554ac7215c4b07c>@@@Z 0000000180016a50 f   libucrt:signal.obj
 0001:00015dac       ??$?RV<lambda_842d9ff0dc9ef11c61343bbaebe7f885>@@AEAV<lambda_c5860995281e5c4ce005b3de8f5874ee>@@V<lambda_d90129c13df834fdcbf8d2b88dafcf2d>@@@?$__crt_seh_guarded_call@X@@QEAAX$$QEAV<lambda_842d9ff0dc9ef11c61343bbaebe7f885>@@AEAV<lambda_c5860995281e5c4ce005b3de8f5874ee>@@$$QEAV<lambda_d90129c13df834fdcbf8d2b88dafcf2d>@@@Z 0000000180016dac f   libucrt:fflush.obj
 0001:00015e48       ??$?RV<lambda_886d6c58226a84441f68b9f2b8217b83>@@AEAV<lambda_ab61a845afdef5b7c387490eaf3616ee>@@V<lambda_f7f22ab5edc0698d5f6905b0d3f44752>@@@?$__crt_seh_guarded_call@X@@QEAAX$$QEAV<lambda_886d6c58226a84441f68b9f2b8217b83>@@AEAV<lambda_ab61a845afdef5b7c387490eaf3616ee>@@$$QEAV<lambda_f7f22ab5edc0698d5f6905b0d3f44752>@@@Z 0000000180016e48 f   libucrt:fflush.obj
 0001:00015f28       ?common_flush_all@@YAH_N@Z 0000000180016f28 f   libucrt:fflush.obj
 0001:00016400       ??$?RV<lambda_410d79af7f07d98d83a3f525b3859a53>@@AEAV<lambda_3e16ef9562a7dcce91392c22ab16ea36>@@V<lambda_38119f0e861e05405d8a144b9b982f0a>@@@?$__crt_seh_guarded_call@X@@QEAAX$$QEAV<lambda_410d79af7f07d98d83a3f525b3859a53>@@AEAV<lambda_3e16ef9562a7dcce91392c22ab16ea36>@@$$QEAV<lambda_38119f0e861e05405d8a144b9b982f0a>@@@Z 0000000180017400 f   libucrt:wsetlocale.obj
 0001:00016d84       fallbackMethod             0000000180017d84 f   libucrt:strpbrk.obj
 0001:00017154       $LN78                      0000000180018154     libucrt:strpbrk.obj
 0001:00017190       $LN77                      0000000180018190     libucrt:strpbrk.obj
 0001:000171d0       $LN76                      00000001800181d0     libucrt:strpbrk.obj
 0001:0001743c       ?__acrt_LCMapStringA_stat@@YAHPEAU__crt_locale_pointers@@PEB_WKPEBDHPEADHHH@Z 000000018001843c f   libucrt:lcmapstringa.obj
 0001:000177ec       ?initialize_multibyte@@YAHXZ 00000001800187ec f   libucrt:multibyte_initializer.obj
 0001:00017840       ?GetTableIndexFromLocaleName@@YAHPEB_W@Z 0000000180018840 f   libucrt:lcidtoname_downlevel.obj
 0001:00017c80       ??$?RV<lambda_a37b2b86f63e897a80ea819b0eb08c01>@@AEAV<lambda_38ce7e780aa69e748d6df282ebc68efe>@@V<lambda_99fb1378e971ab6e7edea83e3a7a83a2>@@@?$__crt_seh_guarded_call@H@@QEAAH$$QEAV<lambda_a37b2b86f63e897a80ea819b0eb08c01>@@AEAV<lambda_38ce7e780aa69e748d6df282ebc68efe>@@$$QEAV<lambda_99fb1378e971ab6e7edea83e3a7a83a2>@@@Z 0000000180018c80 f   libucrt:commit.obj
 0001:00017da0       ?write_double_translated_ansi_nolock@@YA?AUwrite_result@?A0x17268360@@HQEBDI@Z 0000000180018da0 f   libucrt:write.obj
 0001:0001827c       ?write_text_ansi_nolock@@YA?AUwrite_result@?A0x17268360@@HQEBDI@Z 000000018001927c f   libucrt:write.obj
 0001:00018380       ?write_text_utf16le_nolock@@YA?AUwrite_result@?A0x17268360@@HQEBDI@Z 0000000180019380 f   libucrt:write.obj
 0001:0001849c       ?write_text_utf8_nolock@@YA?AUwrite_result@?A0x17268360@@HQEBDI@Z 000000018001949c f   libucrt:write.obj
 0001:00018ea0       ?free_crt_array_internal@@YAXQEAPEBX_K@Z 0000000180019ea0 f   libucrt:inittime.obj
 0001:00019020       ??$common_lseek_nolock@_J@@YA_JH_JH@Z 000000018001a020 f   libucrt:lseek.obj
 0001:000193d0       $$000000                   000000018001a3d0     libucrt:log10.obj
 0001:00019aac       ??$?RV<lambda_751a882b2c74d4b022dec766aa51a29a>@@AEAV<lambda_628dfdc04ba53c8bfc02c9951375f3f5>@@V<lambda_f6c7be5f7998530c34de24c7437d6b54>@@@?$__crt_seh_guarded_call@H@@QEAAH$$QEAV<lambda_751a882b2c74d4b022dec766aa51a29a>@@AEAV<lambda_628dfdc04ba53c8bfc02c9951375f3f5>@@$$QEAV<lambda_f6c7be5f7998530c34de24c7437d6b54>@@@Z 000000018001aaac f   libucrt:close.obj
 0001:00019ca0       _call_matherr              000000018001aca0 f   libucrt:libm_error.obj
 0001:00019d08       _exception_enabled         000000018001ad08 f   libucrt:libm_error.obj
 0001:00019f80       _log_special_common        000000018001af80 f   libucrt:log_special.obj
 0001:0001a020       $$000000                   000000018001b020     libucrt:fpsr.obj
 0001:0001a610       $$000000                   000000018001b610     LIBCMT:amdsecgs.obj
 0001:0001a7fc       capture_current_context    000000018001b7fc f   LIBCMT:gs_report.obj
 0001:0001a86c       capture_previous_context   000000018001b86c f   LIBCMT:gs_report.obj
 0001:0001a8e0       $$000000                   000000018001b8e0     LIBCMT:guard_dispatch.obj
 0001:0001a900       ?fin$0@?0??dllmain_crt_process_attach@@YAHQEAUHINSTANCE__@@QEAX@Z@4HA 000000018001b900 f   LIBCMT:dll_dllmain.obj
 0001:0001a917       ?fin$0@?0??dllmain_crt_process_detach@@YAH_N@Z@4HA 000000018001b917 f   LIBCMT:dll_dllmain.obj
 0001:0001a933       ?filt$0@?0??dllmain_dispatch@@YAHQEAUHINSTANCE__@@KQEAX@Z@4HA 000000018001b933 f   LIBCMT:dll_dllmain.obj
 0001:0001a969       __scrt_is_nonwritable_in_current_image$filt$0 000000018001b969 f   LIBCMT:utility.obj
 0001:0001a981       __DestructExceptionObject$filt$0 000000018001b981 f   libvcruntime:ehhelpers.obj
 0001:0001a999       _query_new_handler$fin$0   000000018001b999 f   libucrt:new_handler.obj
 0001:0001a9af       ?fin$0@?0???$?RV<lambda_0ae27a3a962d80f24befdcbee591983d>@@AEAV<lambda_8d0ee55de4b1038c4002e0adecdf1839>@@V<lambda_dc504788e8f1664fe9b84e20bfb512f2>@@@?$__crt_seh_guarded_call@X@@QEAAX$$QEAV<lambda_0ae27a3a962d80f24befdcbee591983d>@@AEAV<lambda_8d0ee55de4b1038c4002e0adecdf1839>@@$$QEAV<lambda_dc504788e8f1664fe9b84e20bfb512f2>@@@Z@4HA 000000018001b9af f   libucrt:per_thread_data.obj
 0001:0001a9af       ?fin$0@?0???$?RV<lambda_2d41944a1d46af3157314b8a01080d33>@@AEAV<lambda_8f455de75cd7d7f24b4096f044d8b9e6>@@V<lambda_aa500f224e6afead328df44964fe2772>@@@?$__crt_seh_guarded_call@X@@QEAAX$$QEAV<lambda_2d41944a1d46af3157314b8a01080d33>@@AEAV<lambda_8f455de75cd7d7f24b4096f044d8b9e6>@@$$QEAV<lambda_aa500f224e6afead328df44964fe2772>@@@Z@4HA 000000018001b9af f   libucrt:per_thread_data.obj
 0001:0001a9af       ?fin$0@?0???$?RV<lambda_aa87e3671a710a21b5dc78c0bdf72e11>@@AEAV<lambda_92619d2358a28f41a33ba319515a20b9>@@V<lambda_6992ecaafeb10aed2b74cb1fae11a551>@@@?$__crt_seh_guarded_call@X@@QEAAX$$QEAV<lambda_aa87e3671a710a21b5dc78c0bdf72e11>@@AEAV<lambda_92619d2358a28f41a33ba319515a20b9>@@$$QEAV<lambda_6992ecaafeb10aed2b74cb1fae11a551>@@@Z@4HA 000000018001b9af f   libucrt:per_thread_data.obj
 0001:0001a9af       ?fin$0@?0???$?RV<lambda_f2e299630e499de9f9a165e60fcd3db5>@@AEAV<lambda_2ae9d31cdba2644fcbeaf08da7c24588>@@V<lambda_40d01ff24d0e7b3814fdbdcee8eab3c7>@@@?$__crt_seh_guarded_call@X@@QEAAX$$QEAV<lambda_f2e299630e499de9f9a165e60fcd3db5>@@AEAV<lambda_2ae9d31cdba2644fcbeaf08da7c24588>@@$$QEAV<lambda_40d01ff24d0e7b3814fdbdcee8eab3c7>@@@Z@4HA 000000018001b9af f   libucrt:per_thread_data.obj
 0001:0001a9af       ?fin$0@?0???$?RV<lambda_450d765d439847d4c735a33c368b5fc0>@@AEAV<lambda_44731a7d0e6d81c3e6aa82d741081786>@@V<lambda_601a2a7da3b7a96e9554ac7215c4b07c>@@@?$__crt_seh_guarded_call@P6AXH@Z@@QEAAP6AXH@Z$$QEAV<lambda_450d765d439847d4c735a33c368b5fc0>@@AEAV<lambda_44731a7d0e6d81c3e6aa82d741081786>@@$$QEAV<lambda_601a2a7da3b7a96e9554ac7215c4b07c>@@@Z@4HA 000000018001b9af f   libucrt:signal.obj
 0001:0001a9af       ?fin$0@?0???$?RV<lambda_d80eeec6fff315bfe5c115232f3240e3>@@AEAV<lambda_6e4b09c48022b2350581041d5f6b0c4c>@@V<lambda_2358e3775559c9db80273638284d5e45>@@@?$__crt_seh_guarded_call@X@@QEAAX$$QEAV<lambda_d80eeec6fff315bfe5c115232f3240e3>@@AEAV<lambda_6e4b09c48022b2350581041d5f6b0c4c>@@$$QEAV<lambda_2358e3775559c9db80273638284d5e45>@@@Z@4HA 000000018001b9af f   libucrt:exit.obj
 0001:0001a9af       ?fin$0@?0???$?RV<lambda_7777bce6b2f8c936911f934f8298dc43>@@AEAV<lambda_f03950bc5685219e0bcd2087efbe011e>@@V<lambda_3883c3dff614d5e0c5f61bb1ac94921c>@@@?$__crt_seh_guarded_call@H@@QEAAH$$QEAV<lambda_7777bce6b2f8c936911f934f8298dc43>@@AEAV<lambda_f03950bc5685219e0bcd2087efbe011e>@@$$QEAV<lambda_3883c3dff614d5e0c5f61bb1ac94921c>@@@Z@4HA 000000018001b9af f   libucrt:onexit.obj
 0001:0001a9af       ?fin$0@?0???$?RV<lambda_efdfa57d1f175319df784efa44bb7b81>@@AEAV<lambda_5f0a4c1567f8adc6734073e5d1e1b35c>@@V<lambda_2e8a7d3640ea6ccb4c2413664c2db6fd>@@@?$__crt_seh_guarded_call@X@@QEAAX$$QEAV<lambda_efdfa57d1f175319df784efa44bb7b81>@@AEAV<lambda_5f0a4c1567f8adc6734073e5d1e1b35c>@@$$QEAV<lambda_2e8a7d3640ea6ccb4c2413664c2db6fd>@@@Z@4HA 000000018001b9af f   libucrt:mbctype.obj
 0001:0001a9c9       ?filt$0@?0???R<lambda_6e4b09c48022b2350581041d5f6b0c4c>@@QEBA@XZ@4HA 000000018001b9c9 f   libucrt:exit.obj
 0001:0001a9e4       ?fin$0@?0??update_thread_multibyte_data_internal@@YAPEAU__crt_multibyte_data@@QEAU__acrt_ptd@@QEAPEAU1@@Z@4HA 000000018001b9e4 f   libucrt:mbctype.obj
 0001:0001a9fd       __acrt_lowio_ensure_fh_exists$fin$0 000000018001b9fd f   libucrt:osfinfo.obj
 0001:0001a9fd       __acrt_initialize_lowio$fin$0 000000018001b9fd f   libucrt:ioinit.obj
 0001:0001aa16       raise$fin$0                000000018001ba16 f   libucrt:signal.obj
 0001:0001aa37       ?fin$0@?0???$?RV<lambda_842d9ff0dc9ef11c61343bbaebe7f885>@@AEAV<lambda_c5860995281e5c4ce005b3de8f5874ee>@@V<lambda_d90129c13df834fdcbf8d2b88dafcf2d>@@@?$__crt_seh_guarded_call@X@@QEAAX$$QEAV<lambda_842d9ff0dc9ef11c61343bbaebe7f885>@@AEAV<lambda_c5860995281e5c4ce005b3de8f5874ee>@@$$QEAV<lambda_d90129c13df834fdcbf8d2b88dafcf2d>@@@Z@4HA 000000018001ba37 f   libucrt:fflush.obj
 0001:0001aa52       ?fin$0@?0???$?RV<lambda_886d6c58226a84441f68b9f2b8217b83>@@AEAV<lambda_ab61a845afdef5b7c387490eaf3616ee>@@V<lambda_f7f22ab5edc0698d5f6905b0d3f44752>@@@?$__crt_seh_guarded_call@X@@QEAAX$$QEAV<lambda_886d6c58226a84441f68b9f2b8217b83>@@AEAV<lambda_ab61a845afdef5b7c387490eaf3616ee>@@$$QEAV<lambda_f7f22ab5edc0698d5f6905b0d3f44752>@@@Z@4HA 000000018001ba52 f   libucrt:fflush.obj
 0001:0001aa6f       ?fin$0@?0???$?RV<lambda_410d79af7f07d98d83a3f525b3859a53>@@AEAV<lambda_3e16ef9562a7dcce91392c22ab16ea36>@@V<lambda_38119f0e861e05405d8a144b9b982f0a>@@@?$__crt_seh_guarded_call@X@@QEAAX$$QEAV<lambda_410d79af7f07d98d83a3f525b3859a53>@@AEAV<lambda_3e16ef9562a7dcce91392c22ab16ea36>@@$$QEAV<lambda_38119f0e861e05405d8a144b9b982f0a>@@@Z@4HA 000000018001ba6f f   libucrt:wsetlocale.obj
 0001:0001aa89       __acrt_update_thread_locale_data$fin$0 000000018001ba89 f   libucrt:locale_refcounting.obj
 0001:0001aaa2       ?fin$0@?0???$?RV<lambda_a37b2b86f63e897a80ea819b0eb08c01>@@AEAV<lambda_38ce7e780aa69e748d6df282ebc68efe>@@V<lambda_99fb1378e971ab6e7edea83e3a7a83a2>@@@?$__crt_seh_guarded_call@H@@QEAAH$$QEAV<lambda_a37b2b86f63e897a80ea819b0eb08c01>@@AEAV<lambda_38ce7e780aa69e748d6df282ebc68efe>@@$$QEAV<lambda_99fb1378e971ab6e7edea83e3a7a83a2>@@@Z@4HA 000000018001baa2 f   libucrt:commit.obj
 0001:0001aaa2       ?fin$0@?0???$?RV<lambda_751a882b2c74d4b022dec766aa51a29a>@@AEAV<lambda_628dfdc04ba53c8bfc02c9951375f3f5>@@V<lambda_f6c7be5f7998530c34de24c7437d6b54>@@@?$__crt_seh_guarded_call@H@@QEAAH$$QEAV<lambda_751a882b2c74d4b022dec766aa51a29a>@@AEAV<lambda_628dfdc04ba53c8bfc02c9951375f3f5>@@$$QEAV<lambda_f6c7be5f7998530c34de24c7437d6b54>@@@Z@4HA 000000018001baa2 f   libucrt:close.obj
 0001:0001aabc       _write$fin$0               000000018001babc f   libucrt:write.obj
 0001:0001aad3       _fcloseall$fin$0           000000018001bad3 f   libucrt:closeall.obj
 0001:0001aaec       fclose$fin$0               000000018001baec f   libucrt:fclose.obj
 0001:0001ab04       _ctrlfp$filt$0             000000018001bb04 f   libucrt:fpctrl.obj
 0001:0001ab30       _IsNonwritableInCurrentImage$filt$0 000000018001bb30 f   LIBCMT:pesect.obj
 0001:0001ab50       $xdatasym                  000000018001bb50     chkstk.obj
 0001:0001ab58       $unwind$_set_statfp        000000018001bb58     libucrt:fpctrl.obj
 0001:0001ab58       $unwind$??_GPluginUIntEditFieldBinding@@UEAAPEAXI@Z 000000018001bb58     TmpCfg.obj
 0001:0001ab58       $unwind$__acrt_get_process_end_policy 000000018001bb58     libucrt:win_policies.obj
 0001:0001ab58       $unwind$?SaveValue@PluginUIntEditFieldBinding@@UEAAXPEAUFarDialogItem@@H@Z 000000018001bb58     TmpCfg.obj
 0001:0001ab58       $unwind$initialize_pointers 000000018001bb58     libucrt:initialization.obj
 0001:0001ab58       $unwind$uninitialize_allocated_memory 000000018001bb58     libucrt:initialization.obj
 0001:0001ab58       $unwind$__acrt_uninitialize_locks 000000018001bb58     libucrt:locks.obj
 0001:0001ab58       $unwind$_callnewh          000000018001bb58     libucrt:new_handler.obj
 0001:0001ab58       $unwind$??_GPluginIntEditFieldBinding@@UEAAPEAXI@Z 000000018001bb58     TmpCfg.obj
 0001:0001ab58       $unwind$__acrt_FlsGetValue 000000018001bb58     libucrt:winapi_thunks.obj
 0001:0001ab58       $unwind$?SaveValue@PluginIntEditFieldBinding@@UEAAXPEAUFarDialogItem@@H@Z 000000018001bb58     TmpCfg.obj
 0001:0001ab58       $unwind$__acrt_initialize_locks 000000018001bb58     libucrt:locks.obj
 0001:0001ab58       $unwind$?WFD2FFD@@YAXAEAU_WIN32_FIND_DATAW@@AEAUPluginPanelItem@@@Z 000000018001bb58     TmpMix.obj
 0001:0001ab58       $unwind$?FormNtPath@@YAPEA_WPEB_WAEAVStrBuf@@@Z 000000018001bb58     TmpMix.obj
 0001:0001ab58       $unwind$??_GPluginEditFieldBinding@@UEAAPEAXI@Z 000000018001bb58     TmpCfg.obj
 0001:0001ab58       $unwind$strcpy_s           000000018001bb58     libucrt:strcpy_s.obj
 0001:0001ab58       $unwind$__scrt_uninitialize_crt 000000018001bb58     LIBCMT:utility.obj
 0001:0001ab58       $unwind$?SaveValue@PluginEditFieldBinding@@UEAAXPEAUFarDialogItem@@H@Z 000000018001bb58     TmpCfg.obj
 0001:0001ab58       $unwind$__scrt_initialize_crt 000000018001bb58     LIBCMT:utility.obj
 0001:0001ab58       $unwind$__acrt_FlsFree     000000018001bb58     libucrt:winapi_thunks.obj
 0001:0001ab58       $unwind$__acrt_FlsAlloc    000000018001bb58     libucrt:winapi_thunks.obj
 0001:0001ab58       $unwind$ClosePanelW        000000018001bb58     TmpPanel.obj
 0001:0001ab58       $unwind$__vcrt_FlsGetValue 000000018001bb58     libvcruntime:winapi_downlevel.obj
 0001:0001ab58       $unwind$__scrt_release_startup_lock 000000018001bb58     LIBCMT:utility.obj
 0001:0001ab58       $unwind$??_Gtype_info@@UEAAPEAXI@Z 000000018001bb58     LIBCMT:std_type_info_static.obj
 0001:0001ab58       $unwind$__vcrt_FlsFree     000000018001bb58     libvcruntime:winapi_downlevel.obj
 0001:0001ab58       $unwind$_fflush_nolock     000000018001bb58     libucrt:fflush.obj
 0001:0001ab58       $unwind$??_GPluginRadioButtonBinding@@UEAAPEAXI@Z 000000018001bb58     TmpCfg.obj
 0001:0001ab58       $unwind$__acrt_uninitialize_winapi_thunks 000000018001bb58     libucrt:winapi_thunks.obj
 0001:0001ab58       $unwind$??1TmpPanel@@QEAA@XZ 000000018001bb58     TmpClass.obj
 0001:0001ab58       $unwind$__vcrt_FlsAlloc    000000018001bb58     libvcruntime:winapi_downlevel.obj
 0001:0001ab58       $unwind$_calloc_base       000000018001bb58     libucrt:calloc_base.obj
 0001:0001ab58       $unwind$__vcrt_uninitialize_locks 000000018001bb58     libvcruntime:locks.obj
 0001:0001ab58       $unwind$?try_cor_exit_process@@YAXI@Z 000000018001bb58     libucrt:exit.obj
 0001:0001ab58       $unwind$__std_exception_destroy 000000018001bb58     libvcruntime:std_exception.obj
 0001:0001ab58       $unwind$??_GPluginCheckBoxBinding@@UEAAPEAXI@Z 000000018001bb58     TmpCfg.obj
 0001:0001ab58       $unwind$__vcrt_initialize_locks 000000018001bb58     libvcruntime:locks.obj
 0001:0001ab58       $unwind$AnalyseW           000000018001bb58     TmpPanel.obj
 0001:0001ab58       $unwind$??0bad_array_new_length@std@@QEAA@AEBV01@@Z 000000018001bb58     LIBCMT:throw_bad_alloc.obj
 0001:0001ab58       $unwind$__acrt_freeptd     000000018001bb58     libucrt:per_thread_data.obj
 0001:0001ab58       $unwind$??0bad_alloc@std@@QEAA@AEBV01@@Z 000000018001bb58     LIBCMT:throw_bad_alloc.obj
 0001:0001ab58       $unwind$__std_type_info_destroy_list 000000018001bb58     libvcruntime:std_type_info.obj
 0001:0001ab58       $unwind$?SaveValue@PluginCheckBoxBinding@@UEAAXPEAUFarDialogItem@@H@Z 000000018001bb58     TmpCfg.obj
 0001:0001ab58       $unwind$__vcrt_freeptd     000000018001bb58     libvcruntime:per_thread_data.obj
 0001:0001ab58       $unwind$?exit_or_terminate_process@@YAXI@Z 000000018001bb58     libucrt:exit.obj
 0001:0001ab58       $unwind$__acrt_uninitialize_stdio 000000018001bb58     libucrt:_file.obj
 0001:0001ab58       $unwind$??_G?$DialogItemBinding@UFarDialogItem@@@@UEAAPEAXI@Z 000000018001bb58     TmpCfg.obj
 0001:0001ab58       $unwind$_malloc_base       000000018001bb58     libucrt:malloc_base.obj
 0001:0001ab58       $unwind$__acrt_update_locale_info 000000018001bb58     libucrt:locale_update.obj
 0001:0001ab58       $unwind$??2@YAPEAX_K@Z     000000018001bb58     LIBCMT:new_scalar.obj
 0001:0001ab58       $unwind$__acrt_update_multibyte_info 000000018001bb58     libucrt:locale_update.obj
 0001:0001ab58       $unwind$??0exception@std@@QEAA@AEBV01@@Z 000000018001bb58     LIBCMT:throw_bad_alloc.obj
 0001:0001ab58       $unwind$__raise_securityfailure 000000018001bb58     LIBCMT:gs_report.obj
 0001:0001ab58       $unwind$?EndColumns@?$DialogBuilderBase@UFarDialogItem@@@@QEAAXXZ 000000018001bb58     TmpCfg.obj
 0001:0001ab58       $unwind$_clrfp             000000018001bb58     libucrt:fpctrl.obj
 0001:0001ab58       $unwind$?Inflate@SimpleString@@QEAAX_K@Z 000000018001bb58     TmpClass.obj
 0001:0001ab58       $unwind$wcscpy_s           000000018001bb58     libucrt:wcscpy_s.obj
 0001:0001ab58       $unwind$__acrt_getptd_head 000000018001bb58     libucrt:per_thread_data.obj
 0001:0001ab58       $unwind$__acrt_allocate_buffer_for_argv 000000018001bb58     libucrt:argv_parsing.obj
 0001:0001ab58       $unwind$__acrt_stdio_free_buffer_nolock 000000018001bb58     libucrt:_freebuf.obj
 0001:0001ab58       $unwind$__acrt_AppPolicyGetProcessTerminationMethodInternal 000000018001bb58     libucrt:winapi_thunks.obj
 0001:0001ab60       $unwind$GetGlobalInfoW     000000018001bb60     TmpPanel.obj
 0001:0001ab60       $unwind$_isatty            000000018001bb60     libucrt:isatty.obj
 0001:0001ab60       $unwind$__acrt_thread_attach 000000018001bb60     libucrt:initialization.obj
 0001:0001ab60       $unwind$__pctype_func      000000018001bb60     libucrt:ctype.obj
 0001:0001ab60       $unwind$__acrt_thread_detach 000000018001bb60     libucrt:initialization.obj
 0001:0001ab60       $unwind$?dllmain_crt_dispatch@@YAHQEAUHINSTANCE__@@KQEAX@Z 000000018001bb60     LIBCMT:dll_dllmain.obj
 0001:0001ab60       $unwind$__acrt_initialize_command_line 000000018001bb60     libucrt:argv_data.obj
 0001:0001ab60       $unwind$__acrt_uninitialize_ptd 000000018001bb60     libucrt:per_thread_data.obj
 0001:0001ab60       $unwind$__acrt_initialize_ptd 000000018001bb60     libucrt:per_thread_data.obj
 0001:0001ab60       $unwind$__acrt_uninitialize_critical 000000018001bb60     libucrt:initialization.obj
 0001:0001ab60       $unwind$_errno             000000018001bb60     libucrt:errno.obj
 0001:0001ab60       $unwind$initialize_c       000000018001bb60     libucrt:initialization.obj
 0001:0001ab60       $unwind$__acrt_uninitialize 000000018001bb60     libucrt:initialization.obj
 0001:0001ab60       $unwind$_fileno            000000018001bb60     libucrt:fileno.obj
 0001:0001ab60       $unwind$__doserrno         000000018001bb60     libucrt:errno.obj
 0001:0001ab60       $unwind$ProcessPanelEventW 000000018001bb60     TmpPanel.obj
 0001:0001ab60       $unwind$uninitialize_environment 000000018001bb60     libucrt:initialization.obj
 0001:0001ab60       $unwind$__vcrt_thread_detach 000000018001bb60     libvcruntime:initialization.obj
 0001:0001ab60       $unwind$__vcrt_initialize_ptd 000000018001bb60     libvcruntime:per_thread_data.obj
 0001:0001ab60       $unwind$__vcrt_thread_attach 000000018001bb60     libvcruntime:initialization.obj
 0001:0001ab60       $unwind$__vcrt_uninitialize_ptd 000000018001bb60     libvcruntime:per_thread_data.obj
 0001:0001ab60       $unwind$__vcrt_uninitialize_critical 000000018001bb60     libvcruntime:initialization.obj
 0001:0001ab60       $unwind$__vcrt_uninitialize 000000018001bb60     libvcruntime:initialization.obj
 0001:0001ab60       $unwind$__vcrt_initialize  000000018001bb60     libvcruntime:initialization.obj
 0001:0001ab60       $unwind$__report_rangecheckfailure 000000018001bb60     LIBCMT:gs_report.obj
 0001:0001ab60       $unwind$_invoke_watson     000000018001bb60     libucrt:invalid_parameter.obj
 0001:0001ab60       $unwind$__acrt_initialize_heap 000000018001bb60     libucrt:heap_handle.obj
 0001:0001ab60       $unwind$__vcrt_freefls     000000018001bb60     libvcruntime:per_thread_data.obj
 0001:0001ab60       $unwind$ProcessPanelInputW 000000018001bb60     TmpPanel.obj
 0001:0001ab60       $unwind$GetFindDataW       000000018001bb60     TmpPanel.obj
 0001:0001ab60       $unwind$__scrt_initialize_default_local_stdio_options 000000018001bb60     LIBCMT:default_local_stdio_options.obj
 0001:0001ab60       $unwind$__dcrt_uninitialize_environments_nolock 000000018001bb60     libucrt:environment_initialization.obj
 0001:0001ab60       $unwind$SetStartupInfoW    000000018001bb60     TmpPanel.obj
 0001:0001ab60       $unwind$__acrt_update_thread_multibyte_data 000000018001bb60     libucrt:mbctype.obj
 0001:0001ab60       $unwind$__scrt_dllmain_before_initialize_c 000000018001bb60     LIBCMT:utility.obj
 0001:0001ab60       $unwind$??$uninitialize_environment_internal@D@@YAXAEAPEAPEAD@Z 000000018001bb60     libucrt:environment_initialization.obj
 0001:0001ab60       $unwind$__scrt_acquire_startup_lock 000000018001bb60     LIBCMT:utility.obj
 0001:0001ab60       $unwind$??$uninitialize_environment_internal@_W@@YAXAEAPEAPEA_W@Z 000000018001bb60     libucrt:environment_initialization.obj
 0001:0001ab60       $unwind$__GSHandlerCheck   000000018001bb60     LIBCMT:gshandler.obj
 0001:0001ab60       $unwind$__scrt_dllmain_after_initialize_c 000000018001bb60     LIBCMT:utility.obj
 0001:0001ab60       $unwind$__acrt_AreFileApisANSI 000000018001bb60     libucrt:winapi_thunks.obj
 0001:0001ab60       $unwind$SetFindListW       000000018001bb60     TmpPanel.obj
 0001:0001ab60       $unwind$__scrt_dllmain_uninitialize_c 000000018001bb60     LIBCMT:utility.obj
 0001:0001ab60       $unwind$abort              000000018001bb60     libucrt:abort.obj
 0001:0001ab60       $unwind$__acrt_initialize_multibyte 000000018001bb60     libucrt:mbctype.obj
 0001:0001ab60       $unwind$?initialize_multibyte@@YAHXZ 000000018001bb60     libucrt:multibyte_initializer.obj
 0001:0001ab60       $unwind$__scrt_dllmain_uninitialize_critical 000000018001bb60     LIBCMT:utility.obj
 0001:0001ab60       $unwind$__acrt_release_locale_ref 000000018001bb60     libucrt:locale_refcounting.obj
 0001:0001ab60       $unwind$__scrt_dllmain_crt_thread_attach 000000018001bb60     LIBCMT:utility.obj
 0001:0001ab60       $unwind$_msize_base        000000018001bb60     libucrt:msize.obj
 0001:0001ab60       $unwind$ConfigureW         000000018001bb60     TmpPanel.obj
 0001:0001ab60       $unwind$_statfp            000000018001bb60     libucrt:fpctrl.obj
 0001:0001ab60       $unwind$SetDirectoryW      000000018001bb60     TmpPanel.obj
 0001:0001ab60       $unwind$__acrt_DownlevelLocaleNameToLCID 000000018001bb60     libucrt:lcidtoname_downlevel.obj
 0001:0001ab60       $unwind$__dcrt_terminate_console_output 000000018001bb60     libucrt:initcon.obj
 0001:0001ab60       $unwind$_get_osfhandle     000000018001bb60     libucrt:osfinfo.obj
 0001:0001ab60       $unwind$uninitialize_allocated_io_buffers 000000018001bb60     libucrt:initialization.obj
 0001:0001ab60       $unwind$__scrt_dllmain_crt_thread_detach 000000018001bb60     LIBCMT:utility.obj
 0001:0001ab60       $unwind$_set_errno_from_matherr 000000018001bb60     libucrt:fpexcept.obj
 0001:0001ab68       $unwind$?Grow@StrBuf@@QEAAX_K@Z 000000018001bb68     TmpMix.obj
 0001:0001ab68       $unwind$_RTC_Initialize    000000018001bb68     LIBCMT:initsect.obj
 0001:0001ab68       $unwind$??_G?$DialogBuilderBase@UFarDialogItem@@@@MEAAPEAXI@Z 000000018001bb68     TmpCfg.obj
 0001:0001ab68       $unwind$ExitFARW           000000018001bb68     TmpPanel.obj
 0001:0001ab68       $unwind$__acrt_execute_uninitializers 000000018001bb68     libucrt:shared_initialization.obj
 0001:0001ab68       $unwind$??_GPluginDialogBuilder@@UEAAPEAXI@Z 000000018001bb68     TmpCfg.obj
 0001:0001ab68       $unwind$_RTC_Terminate     000000018001bb68     LIBCMT:initsect.obj
 0001:0001ab68       $unwind$GetPluginInfoW     000000018001bb68     TmpPanel.obj
 0001:0001ab68       $unwind$__vcrt_FlsSetValue 000000018001bb68     libvcruntime:winapi_downlevel.obj
 0001:0001ab68       $unwind$??0TmpPanel@@QEAA@PEB_W@Z 000000018001bb68     TmpClass.obj
 0001:0001ab68       $unwind$_fclose_nolock     000000018001bb68     libucrt:fclose.obj
 0001:0001ab68       $unwind$?replace_current_thread_locale_nolock@@YAXQEAU__acrt_ptd@@QEAU__crt_locale_data@@@Z 000000018001bb68     libucrt:per_thread_data.obj
 0001:0001ab68       $unwind$__acrt_uninitialize_lowio 000000018001bb68     libucrt:ioinit.obj
 0001:0001ab68       $unwind$__acrt_FlsSetValue 000000018001bb68     libucrt:winapi_thunks.obj
 0001:0001ab68       $unwind$??$common_initialize_environment_nolock@D@@YAHXZ 000000018001bb68     libucrt:environment_initialization.obj
 0001:0001ab68       $unwind$?SaveValue@PluginRadioButtonBinding@@UEAAXPEAUFarDialogItem@@H@Z 000000018001bb68     TmpCfg.obj
 0001:0001ab68       $unwind$_initterm_e        000000018001bb68     libucrt:initterm.obj
 0001:0001ab68       $unwind$?ParseParam@@YAPEA_WAEAPEA_W@Z 000000018001bb68     TmpMix.obj
 0001:0001ab68       $unwind$_realloc_base      000000018001bb68     libucrt:realloc_base.obj
 0001:0001ab68       $unwind$??_Gbad_array_new_length@std@@UEAAPEAXI@Z 000000018001bb68     LIBCMT:throw_bad_alloc.obj
 0001:0001ab68       $unwind$?CreateRadioButtonBinding@PluginDialogBuilder@@MEAAPEAU?$DialogItemBinding@UFarDialogItem@@@@PEAH@Z 000000018001bb68     TmpCfg.obj
 0001:0001ab68       $unwind$??_Gbad_alloc@std@@UEAAPEAXI@Z 000000018001bb68     LIBCMT:throw_bad_alloc.obj
 0001:0001ab68       $unwind$_close_nolock      000000018001bb68     libucrt:close.obj
 0001:0001ab68       $unwind$strncpy_s          000000018001bb68     libucrt:strncpy_s.obj
 0001:0001ab68       $unwind$??_Gexception@std@@UEAAPEAXI@Z 000000018001bb68     LIBCMT:throw_bad_alloc.obj
 0001:0001ab68       $unwind$_updatetlocinfoEx_nolock 000000018001bb68     libucrt:locale_refcounting.obj
 0001:0001ab68       $unwind$__acrt_errno_map_os_error 000000018001bb68     libucrt:errno.obj
 0001:0001ab68       $unwind$?InitDialogItem@PluginDialogBuilder@@MEAAXPEAUFarDialogItem@@PEB_W@Z 000000018001bb68     TmpCfg.obj
 0001:0001ab68       $unwind$__acrt_LocaleNameToLCID 000000018001bb68     libucrt:winapi_thunks.obj
 0001:0001ab68       $unwind$?SetDirectory@TmpPanel@@QEAAHPEB_W_K@Z 000000018001bb68     TmpClass.obj
 0001:0001ab68       $unwind$?SortListCmp@@YAHPEBX0PEAX@Z 000000018001bb68     TmpClass.obj
 0001:0001ab74       $unwind$OpenW              000000018001bb74     TmpPanel.obj
 0001:0001ab80       $chain$4$OpenW             000000018001bb80     TmpPanel.obj
 0001:0001aba4       $chain$5$OpenW             000000018001bba4     TmpPanel.obj
 0001:0001abb4       $unwind$_invalid_parameter_noinfo 000000018001bbb4     libucrt:invalid_parameter.obj
 0001:0001abb4       $unwind$PutFilesW          000000018001bbb4     TmpPanel.obj
 0001:0001abb4       $unwind$_log10_special     000000018001bbb4     libucrt:log_special.obj
 0001:0001abbc       $unwind$?ProcessList@@YAXPEAXPEA_WH@Z 000000018001bbbc     TmpPanel.obj
 0001:0001abd0       $unwind$?ShowMenuFromList@@YAXPEA_W@Z 000000018001bbd0     TmpPanel.obj
 0001:0001abdc       $chain$1$?ShowMenuFromList@@YAXPEA_W@Z 000000018001bbdc     TmpPanel.obj
 0001:0001abf4       $chain$4$?ShowMenuFromList@@YAXPEA_W@Z 000000018001bbf4     TmpPanel.obj
 0001:0001ac10       $chain$5$?ShowMenuFromList@@YAXPEA_W@Z 000000018001bc10     TmpPanel.obj
 0001:0001ac24       $chain$6$?ShowMenuFromList@@YAXPEA_W@Z 000000018001bc24     TmpPanel.obj
 0001:0001ac34       $chain$7$?ShowMenuFromList@@YAXPEA_W@Z 000000018001bc34     TmpPanel.obj
 0001:0001ac44       $chain$8$?ShowMenuFromList@@YAXPEA_W@Z 000000018001bc44     TmpPanel.obj
 0001:0001ac54       $unwind$?OpenPanelFromOutput@@YAPEAXPEA_W@Z 000000018001bc54     TmpPanel.obj
 0001:0001ac68       $chain$1$?OpenPanelFromOutput@@YAPEAXPEA_W@Z 000000018001bc68     TmpPanel.obj
 0001:0001ac80       $chain$2$?OpenPanelFromOutput@@YAPEAXPEA_W@Z 000000018001bc80     TmpPanel.obj
 0001:0001ac94       $chain$3$?OpenPanelFromOutput@@YAPEAXPEA_W@Z 000000018001bc94     TmpPanel.obj
 0001:0001aca4       $chain$4$?OpenPanelFromOutput@@YAPEAXPEA_W@Z 000000018001bca4     TmpPanel.obj
 0001:0001acb4       $unwind$?ReadFileLines@@YAXPEAXKPEAPEA_WPEA_WPEAI3@Z 000000018001bcb4     TmpPanel.obj
 0001:0001acc8       $chain$1$?ReadFileLines@@YAXPEAXKPEAPEA_WPEA_WPEAI3@Z 000000018001bcc8     TmpPanel.obj
 0001:0001ace0       $chain$2$?ReadFileLines@@YAXPEAXKPEAPEA_WPEA_WPEAI3@Z 000000018001bce0     TmpPanel.obj
 0001:0001acf0       $unwind$?ReadFileList@@YAXPEA_WPEAHPEAPEAPEA_W@Z 000000018001bcf0     TmpPanel.obj
 0001:0001ad00       $chain$0$?ReadFileList@@YAXPEA_WPEAHPEAPEAPEA_W@Z 000000018001bd00     TmpPanel.obj
 0001:0001ad14       $chain$1$?ReadFileList@@YAXPEA_WPEAHPEAPEAPEA_W@Z 000000018001bd14     TmpPanel.obj
 0001:0001ad24       $unwind$?AddIntEditField@PluginDialogBuilder@@UEAAPEAUFarDialogItem@@PEAHH@Z 000000018001bd24     TmpCfg.obj
 0001:0001ad24       $unwind$?GetOpenPanelInfo@TmpPanel@@QEAAXPEAUOpenPanelInfo@@@Z 000000018001bd24     TmpClass.obj
 0001:0001ad24       $unwind$?AddUIntEditField@PluginDialogBuilder@@UEAAPEAUFarDialogItem@@PEAIH@Z 000000018001bd24     TmpCfg.obj
 0001:0001ad24       $unwind$?AddDialogItem@?$DialogBuilderBase@UFarDialogItem@@@@IEAAPEAUFarDialogItem@@W4FARDIALOGITEMTYPES@@PEB_W@Z 000000018001bd24     TmpCfg.obj
 0001:0001ad3c       $unwind$?UpdateBorderSize@?$DialogBuilderBase@UFarDialogItem@@@@IEAAXXZ 000000018001bd3c     TmpCfg.obj
 0001:0001ad4c       $chain$1$?UpdateBorderSize@?$DialogBuilderBase@UFarDialogItem@@@@IEAAXXZ 000000018001bd4c     TmpCfg.obj
 0001:0001ad64       $chain$2$?UpdateBorderSize@?$DialogBuilderBase@UFarDialogItem@@@@IEAAXXZ 000000018001bd64     TmpCfg.obj
 0001:0001ad78       $chain$3$?UpdateBorderSize@?$DialogBuilderBase@UFarDialogItem@@@@IEAAXXZ 000000018001bd78     TmpCfg.obj
 0001:0001ad88       $chain$4$?UpdateBorderSize@?$DialogBuilderBase@UFarDialogItem@@@@IEAAXXZ 000000018001bd88     TmpCfg.obj
 0001:0001ad98       $unwind$?SwitchToPanel@TmpPanel@@AEAAXH@Z 000000018001bd98     TmpClass.obj
 0001:0001ad98       $unwind$??1?$DialogBuilderBase@UFarDialogItem@@@@MEAA@XZ 000000018001bd98     TmpCfg.obj
 0001:0001ada4       $chain$0$??1?$DialogBuilderBase@UFarDialogItem@@@@MEAA@XZ 000000018001bda4     TmpCfg.obj
 0001:0001adb8       $chain$1$??1?$DialogBuilderBase@UFarDialogItem@@@@MEAA@XZ 000000018001bdb8     TmpCfg.obj
 0001:0001adc8       $chain$0$?EndColumns@?$DialogBuilderBase@UFarDialogItem@@@@QEAAXXZ 000000018001bdc8     TmpCfg.obj
 0001:0001addc       $chain$2$?EndColumns@?$DialogBuilderBase@UFarDialogItem@@@@QEAAXXZ 000000018001bddc     TmpCfg.obj
 0001:0001adf4       $chain$3$?EndColumns@?$DialogBuilderBase@UFarDialogItem@@@@QEAAXXZ 000000018001bdf4     TmpCfg.obj
 0001:0001ae04       $chain$4$?EndColumns@?$DialogBuilderBase@UFarDialogItem@@@@QEAAXXZ 000000018001be04     TmpCfg.obj
 0001:0001ae14       $unwind$?AddButtons@?$DialogBuilderBase@UFarDialogItem@@@@QEAAXHPEBHHH@Z 000000018001be14     TmpCfg.obj
 0001:0001ae20       $chain$4$?AddButtons@?$DialogBuilderBase@UFarDialogItem@@@@QEAAXHPEBHHH@Z 000000018001be20     TmpCfg.obj
 0001:0001ae44       $chain$5$?AddButtons@?$DialogBuilderBase@UFarDialogItem@@@@QEAAXHPEBHHH@Z 000000018001be44     TmpCfg.obj
 0001:0001ae54       $unwind$?DoShowDialog@PluginDialogBuilder@@MEAA_JXZ 000000018001be54     TmpCfg.obj
 0001:0001ae60       $unwind$_exception_enabled 000000018001be60     libucrt:libm_error.obj
 0001:0001ae60       $unwind$_DllMainCRTStartup 000000018001be60     LIBCMT:dll_dllmain.obj
 0001:0001ae60       $unwind$__vcrt_getptd_noexit 000000018001be60     libvcruntime:per_thread_data.obj
 0001:0001ae60       $unwind$__acrt_InitializeCriticalSectionEx 000000018001be60     libucrt:winapi_thunks.obj
 0001:0001ae60       $unwind$??$common_lseek_nolock@_J@@YA_JH_JH@Z 000000018001be60     libucrt:lseek.obj
 0001:0001ae60       $unwind$?free_crt_array_internal@@YAXQEAPEBX_K@Z 000000018001be60     libucrt:inittime.obj
 0001:0001ae60       $unwind$__acrt_stdio_flush_nolock 000000018001be60     libucrt:fflush.obj
 0001:0001ae60       $unwind$?CreateCheckBoxBinding@PluginDialogBuilder@@MEAAPEAU?$DialogItemBinding@UFarDialogItem@@@@PEAHH@Z 000000018001be60     TmpCfg.obj
 0001:0001ae60       $unwind$__acrt_getptd_noexit 000000018001be60     libucrt:per_thread_data.obj
 0001:0001ae60       $unwind$__acrt_getptd      000000018001be60     libucrt:per_thread_data.obj
 0001:0001ae60       $unwind$??0_LocaleUpdate@@QEAA@QEAU__crt_locale_pointers@@@Z 000000018001be60     libucrt:output.obj
 0001:0001ae60       $unwind$__acrt_execute_initializers 000000018001be60     libucrt:shared_initialization.obj
 0001:0001ae60       $unwind$__vcrt_InitializeCriticalSectionEx 000000018001be60     libvcruntime:winapi_downlevel.obj
 0001:0001ae70       $unwind$?Config@@YAHXZ     000000018001be70     TmpCfg.obj
 0001:0001ae90       $unwind$?GetOptions@@YAXXZ 000000018001be90     TmpCfg.obj
 0001:0001aea4       $unwind$?RemoveEmptyItems@TmpPanel@@AEAAXXZ 000000018001bea4     TmpClass.obj
 0001:0001aeac       $chain$3$?RemoveEmptyItems@TmpPanel@@AEAAXXZ 000000018001beac     TmpClass.obj
 0001:0001aecc       $chain$4$?RemoveEmptyItems@TmpPanel@@AEAAXXZ 000000018001becc     TmpClass.obj
 0001:0001aee0       $chain$5$?RemoveEmptyItems@TmpPanel@@AEAAXXZ 000000018001bee0     TmpClass.obj
 0001:0001aef0       $chain$6$?RemoveEmptyItems@TmpPanel@@AEAAXXZ 000000018001bef0     TmpClass.obj
 0001:0001af00       $unwind$?UpdateItems@TmpPanel@@AEAAXHH@Z 000000018001bf00     TmpClass.obj
 0001:0001af10       $chain$2$?UpdateItems@TmpPanel@@AEAAXHH@Z 000000018001bf10     TmpClass.obj
 0001:0001af2c       $chain$3$?UpdateItems@TmpPanel@@AEAAXHH@Z 000000018001bf2c     TmpClass.obj
 0001:0001af40       $chain$4$?UpdateItems@TmpPanel@@AEAAXHH@Z 000000018001bf40     TmpClass.obj
 0001:0001af50       $chain$5$?UpdateItems@TmpPanel@@AEAAXHH@Z 000000018001bf50     TmpClass.obj
 0001:0001af60       $unwind$?ProcessSaveListKey@TmpPanel@@AEAAXXZ 000000018001bf60     TmpClass.obj
 0001:0001af6c       $chain$3$?ProcessSaveListKey@TmpPanel@@AEAAXXZ 000000018001bf6c     TmpClass.obj
 0001:0001af8c       $chain$4$?ProcessSaveListKey@TmpPanel@@AEAAXXZ 000000018001bf8c     TmpClass.obj
 0001:0001afa8       $chain$5$?ProcessSaveListKey@TmpPanel@@AEAAXXZ 000000018001bfa8     TmpClass.obj
 0001:0001afb8       $chain$0$?SwitchToPanel@TmpPanel@@AEAAXH@Z 000000018001bfb8     TmpClass.obj
 0001:0001afcc       $chain$1$?SwitchToPanel@TmpPanel@@AEAAXH@Z 000000018001bfcc     TmpClass.obj
 0001:0001afdc       $unwind$?SaveListFile@TmpPanel@@AEAAXPEB_W@Z 000000018001bfdc     TmpClass.obj
 0001:0001afe4       $chain$1$?SaveListFile@TmpPanel@@AEAAXPEB_W@Z 000000018001bfe4     TmpClass.obj
 0001:0001affc       $chain$5$?SaveListFile@TmpPanel@@AEAAXPEB_W@Z 000000018001bffc     TmpClass.obj
 0001:0001b01c       $chain$6$?SaveListFile@TmpPanel@@AEAAXPEB_W@Z 000000018001c01c     TmpClass.obj
 0001:0001b02c       $chain$7$?SaveListFile@TmpPanel@@AEAAXPEB_W@Z 000000018001c02c     TmpClass.obj
 0001:0001b03c       $unwind$?IsCurrentFileCorrect@TmpPanel@@AEAA_NPEAPEA_W@Z 000000018001c03c     TmpClass.obj
 0001:0001b054       $unwind$?GetFindData@TmpPanel@@QEAAHPEAPEAUPluginPanelItem@@PEA_K_K@Z 000000018001c054     TmpClass.obj
 0001:0001b06c       $unwind$?try_get_function@@YAPEAXW4function_id@?A0xbfd18cd1@@QEBDQEBW4module_id@2@2@Z 000000018001c06c     libvcruntime:winapi_downlevel.obj
 0001:0001b06c       $unwind$?try_get_function@@YAPEAXW4function_id@?A0x391cf84c@@QEBDQEBW4module_id@2@2@Z 000000018001c06c     libucrt:winapi_thunks.obj
 0001:0001b06c       $unwind$?PutFiles@TmpPanel@@QEAAHPEAUPluginPanelItem@@_KHPEB_W_K@Z 000000018001c06c     TmpClass.obj
 0001:0001b088       $unwind$?BeginPutFiles@TmpPanel@@QEAAPEAXXZ 000000018001c088     TmpClass.obj
 0001:0001b090       $unwind$?CommitPutFiles@TmpPanel@@QEAAXPEAXH@Z 000000018001c090     TmpClass.obj
 0001:0001b09c       $chain$0$?CommitPutFiles@TmpPanel@@QEAAXPEAXH@Z 000000018001c09c     TmpClass.obj
 0001:0001b0b0       $chain$2$?CommitPutFiles@TmpPanel@@QEAAXPEAXH@Z 000000018001c0b0     TmpClass.obj
 0001:0001b0c8       $chain$3$?CommitPutFiles@TmpPanel@@QEAAXPEAXH@Z 000000018001c0c8     TmpClass.obj
 0001:0001b0d8       $chain$4$?CommitPutFiles@TmpPanel@@QEAAXPEAXH@Z 000000018001c0d8     TmpClass.obj
 0001:0001b0e8       $unwind$?PutDirectoryContents@TmpPanel@@QEAAHPEB_W@Z 000000018001c0e8     TmpClass.obj
 0001:0001b0f4       $chain$0$?PutDirectoryContents@TmpPanel@@QEAAHPEB_W@Z 000000018001c0f4     TmpClass.obj
 0001:0001b108       $chain$1$?PutDirectoryContents@TmpPanel@@QEAAHPEB_W@Z 000000018001c108     TmpClass.obj
 0001:0001b11c       $chain$2$?PutDirectoryContents@TmpPanel@@QEAAHPEB_W@Z 000000018001c11c     TmpClass.obj
 0001:0001b12c       $chain$3$?PutDirectoryContents@TmpPanel@@QEAAHPEB_W@Z 000000018001c12c     TmpClass.obj
 0001:0001b13c       $unwind$?PutOneFile@TmpPanel@@QEAAHPEB_W@Z 000000018001c13c     TmpClass.obj
 0001:0001b148       $chain$0$?PutOneFile@TmpPanel@@QEAAHPEB_W@Z 000000018001c148     TmpClass.obj
 0001:0001b15c       $chain$2$?PutOneFile@TmpPanel@@QEAAHPEB_W@Z 000000018001c15c     TmpClass.obj
 0001:0001b170       $unwind$?SetFindList@TmpPanel@@QEAAHPEBUPluginPanelItem@@_K@Z 000000018001c170     TmpClass.obj
 0001:0001b188       $chain$0$?SetFindList@TmpPanel@@QEAAHPEBUPluginPanelItem@@_K@Z 000000018001c188     TmpClass.obj
 0001:0001b19c       $chain$1$?SetFindList@TmpPanel@@QEAAHPEBUPluginPanelItem@@_K@Z 000000018001c19c     TmpClass.obj
 0001:0001b1ac       $unwind$?ProcessEvent@TmpPanel@@QEAAH_JPEAX@Z 000000018001c1ac     TmpClass.obj
 0001:0001b1b4       $chain$1$?ProcessEvent@TmpPanel@@QEAAH_JPEAX@Z 000000018001c1b4     TmpClass.obj
 0001:0001b1cc       $chain$2$?ProcessEvent@TmpPanel@@QEAAH_JPEAX@Z 000000018001c1cc     TmpClass.obj
 0001:0001b1e0       $chain$3$?ProcessEvent@TmpPanel@@QEAAH_JPEAX@Z 000000018001c1e0     TmpClass.obj
 0001:0001b1f0       $chain$4$?ProcessEvent@TmpPanel@@QEAAH_JPEAX@Z 000000018001c1f0     TmpClass.obj
 0001:0001b200       $unwind$?ProcessKey@TmpPanel@@QEAAHPEBU_INPUT_RECORD@@@Z 000000018001c200     TmpClass.obj
 0001:0001b21c       $chain$0$?ProcessKey@TmpPanel@@QEAAHPEBU_INPUT_RECORD@@@Z 000000018001c21c     TmpClass.obj
 0001:0001b230       $chain$1$?ProcessKey@TmpPanel@@QEAAHPEBU_INPUT_RECORD@@@Z 000000018001c230     TmpClass.obj
 0001:0001b230       $chain$3$?ProcessKey@TmpPanel@@QEAAHPEBU_INPUT_RECORD@@@Z 000000018001c230     TmpClass.obj
 0001:0001b240       $chain$2$?ProcessKey@TmpPanel@@QEAAHPEBU_INPUT_RECORD@@@Z 000000018001c240     TmpClass.obj
 0001:0001b254       $unwind$?GetFileInfoAndValidate@TmpPanel@@SA_NPEB_WPEAUPluginPanelItem@@H@Z 000000018001c254     TmpClass.obj
 0001:0001b270       $unwind$?Replace@SimpleString@@QEAAAEAV1@_K0PEB_W0@Z 000000018001c270     TmpClass.obj
 0001:0001b280       $chain$1$?Replace@SimpleString@@QEAAAEAV1@_K0PEB_W0@Z 000000018001c280     TmpClass.obj
 0001:0001b298       $chain$2$?Replace@SimpleString@@QEAAAEAV1@_K0PEB_W0@Z 000000018001c298     TmpClass.obj
 0001:0001b2ac       $chain$3$?Replace@SimpleString@@QEAAAEAV1@_K0PEB_W0@Z 000000018001c2ac     TmpClass.obj
 0001:0001b2bc       $chain$4$?Replace@SimpleString@@QEAAAEAV1@_K0PEB_W0@Z 000000018001c2bc     TmpClass.obj
 0001:0001b2cc       $unwind$?GoToFile@@YAXPEB_WH@Z 000000018001c2cc     TmpMix.obj
 0001:0001b2ec       $unwind$?FreePanelItems@@YAXPEAUPluginPanelItem@@_K@Z 000000018001c2ec     TmpMix.obj
 0001:0001b2f8       $chain$0$?FreePanelItems@@YAXPEAUPluginPanelItem@@_K@Z 000000018001c2f8     TmpMix.obj
 0001:0001b30c       $chain$1$?FreePanelItems@@YAXPEAUPluginPanelItem@@_K@Z 000000018001c30c     TmpMix.obj
 0001:0001b31c       $unwind$?IsTextUTF8@@YA_NPEBD_K@Z 000000018001c31c     TmpMix.obj
 0001:0001b328       $chain$1$?FormNtPath@@YAPEA_WPEB_WAEAVStrBuf@@@Z 000000018001c328     TmpMix.obj
 0001:0001b340       $chain$2$?FormNtPath@@YAPEA_WPEB_WAEAVStrBuf@@@Z 000000018001c340     TmpMix.obj
 0001:0001b350       $unwind$_initterm          000000018001c350     libucrt:initterm.obj
 0001:0001b350       $unwind$_recalloc_base     000000018001c350     libucrt:recalloc.obj
 0001:0001b350       $unwind$?setSBCS@@YAXPEAU__crt_multibyte_data@@@Z 000000018001c350     libucrt:mbctype.obj
 0001:0001b350       $unwind$_seh_filter_exe    000000018001c350     libucrt:exception_filter.obj
 0001:0001b350       $unwind$?GetFullPath@@YAPEA_WPEB_WAEAVStrBuf@@@Z 000000018001c350     TmpMix.obj
 0001:0001b350       $unwind$__scrt_dllmain_exception_filter 000000018001c350     LIBCMT:utility.obj
 0001:0001b350       $unwind$__acrt_lowio_create_handle_array 000000018001c350     libucrt:osfinfo.obj
 0001:0001b350       $unwind$?ExpandEnvStrs@@YAPEA_WPEB_WAEAVStrBuf@@@Z 000000018001c350     TmpMix.obj
 0001:0001b350       $unwind$__acrt_free_locale 000000018001c350     libucrt:locale_refcounting.obj
 0001:0001b364       $unwind$?FindListFile@@YA_NPEB_WAEAVStrBuf@@@Z 000000018001c364     TmpMix.obj
 0001:0001b364       $unwind$??$copy_and_add_argument_to_buffer@D@@YAHQEBD0_KAEAV?$argument_list@D@?A0x5f5c8891@@@Z 000000018001c364     libucrt:argv_wildcards.obj
 0001:0001b380       $unwind$?dllmain_crt_process_attach@@YAHQEAUHINSTANCE__@@QEAX@Z 000000018001c380     LIBCMT:dll_dllmain.obj
 0001:0001b3bc       $unwind$?fin$0@?0???$?RV<lambda_842d9ff0dc9ef11c61343bbaebe7f885>@@AEAV<lambda_c5860995281e5c4ce005b3de8f5874ee>@@V<lambda_d90129c13df834fdcbf8d2b88dafcf2d>@@@?$__crt_seh_guarded_call@X@@QEAAX$$QEAV<lambda_842d9ff0dc9ef11c61343bbaebe7f885>@@AEAV<lambda_c5860995281e5c4ce005b3de8f5874ee>@@$$QEAV<lambda_d90129c13df834fdcbf8d2b88dafcf2d>@@@Z@4HA 000000018001c3bc     libucrt:fflush.obj
 0001:0001b3bc       $unwind$?fin$0@?0???$?RV<lambda_886d6c58226a84441f68b9f2b8217b83>@@AEAV<lambda_ab61a845afdef5b7c387490eaf3616ee>@@V<lambda_f7f22ab5edc0698d5f6905b0d3f44752>@@@?$__crt_seh_guarded_call@X@@QEAAX$$QEAV<lambda_886d6c58226a84441f68b9f2b8217b83>@@AEAV<lambda_ab61a845afdef5b7c387490eaf3616ee>@@$$QEAV<lambda_f7f22ab5edc0698d5f6905b0d3f44752>@@@Z@4HA 000000018001c3bc     libucrt:fflush.obj
 0001:0001b3bc       $unwind$?fin$0@?0???$?RV<lambda_aa87e3671a710a21b5dc78c0bdf72e11>@@AEAV<lambda_92619d2358a28f41a33ba319515a20b9>@@V<lambda_6992ecaafeb10aed2b74cb1fae11a551>@@@?$__crt_seh_guarded_call@X@@QEAAX$$QEAV<lambda_aa87e3671a710a21b5dc78c0bdf72e11>@@AEAV<lambda_92619d2358a28f41a33ba319515a20b9>@@$$QEAV<lambda_6992ecaafeb10aed2b74cb1fae11a551>@@@Z@4HA 000000018001c3bc     libucrt:per_thread_data.obj
 0001:0001b3bc       $unwind$?fin$0@?0???$?RV<lambda_450d765d439847d4c735a33c368b5fc0>@@AEAV<lambda_44731a7d0e6d81c3e6aa82d741081786>@@V<lambda_601a2a7da3b7a96e9554ac7215c4b07c>@@@?$__crt_seh_guarded_call@P6AXH@Z@@QEAAP6AXH@Z$$QEAV<lambda_450d765d439847d4c735a33c368b5fc0>@@AEAV<lambda_44731a7d0e6d81c3e6aa82d741081786>@@$$QEAV<lambda_601a2a7da3b7a96e9554ac7215c4b07c>@@@Z@4HA 000000018001c3bc     libucrt:signal.obj
 0001:0001b3bc       $unwind$?fin$0@?0???$?RV<lambda_0ae27a3a962d80f24befdcbee591983d>@@AEAV<lambda_8d0ee55de4b1038c4002e0adecdf1839>@@V<lambda_dc504788e8f1664fe9b84e20bfb512f2>@@@?$__crt_seh_guarded_call@X@@QEAAX$$QEAV<lambda_0ae27a3a962d80f24befdcbee591983d>@@AEAV<lambda_8d0ee55de4b1038c4002e0adecdf1839>@@$$QEAV<lambda_dc504788e8f1664fe9b84e20bfb512f2>@@@Z@4HA 000000018001c3bc     libucrt:per_thread_data.obj
 0001:0001b3bc       $unwind$?fin$0@?0??dllmain_crt_process_attach@@YAHQEAUHINSTANCE__@@QEAX@Z@4HA 000000018001c3bc     LIBCMT:dll_dllmain.obj
 0001:0001b3bc       $unwind$?fin$0@?0???$?RV<lambda_410d79af7f07d98d83a3f525b3859a53>@@AEAV<lambda_3e16ef9562a7dcce91392c22ab16ea36>@@V<lambda_38119f0e861e05405d8a144b9b982f0a>@@@?$__crt_seh_guarded_call@X@@QEAAX$$QEAV<lambda_410d79af7f07d98d83a3f525b3859a53>@@AEAV<lambda_3e16ef9562a7dcce91392c22ab16ea36>@@$$QEAV<lambda_38119f0e861e05405d8a144b9b982f0a>@@@Z@4HA 000000018001c3bc     libucrt:wsetlocale.obj
 0001:0001b3bc       $unwind$?fin$0@?0??dllmain_crt_process_detach@@YAH_N@Z@4HA 000000018001c3bc     LIBCMT:dll_dllmain.obj
 0001:0001b3bc       $unwind$raise$fin$0        000000018001c3bc     libucrt:signal.obj
 0001:0001b3bc       $unwind$?fin$0@?0???$?RV<lambda_f2e299630e499de9f9a165e60fcd3db5>@@AEAV<lambda_2ae9d31cdba2644fcbeaf08da7c24588>@@V<lambda_40d01ff24d0e7b3814fdbdcee8eab3c7>@@@?$__crt_seh_guarded_call@X@@QEAAX$$QEAV<lambda_f2e299630e499de9f9a165e60fcd3db5>@@AEAV<lambda_2ae9d31cdba2644fcbeaf08da7c24588>@@$$QEAV<lambda_40d01ff24d0e7b3814fdbdcee8eab3c7>@@@Z@4HA 000000018001c3bc     libucrt:per_thread_data.obj
 0001:0001b3bc       $unwind$__DestructExceptionObject$filt$0 000000018001c3bc     libvcruntime:ehhelpers.obj
 0001:0001b3bc       $unwind$_query_new_handler$fin$0 000000018001c3bc     libucrt:new_handler.obj
 0001:0001b3bc       $unwind$_fcloseall$fin$0   000000018001c3bc     libucrt:closeall.obj
 0001:0001b3bc       $unwind$?fin$0@?0???$?RV<lambda_2d41944a1d46af3157314b8a01080d33>@@AEAV<lambda_8f455de75cd7d7f24b4096f044d8b9e6>@@V<lambda_aa500f224e6afead328df44964fe2772>@@@?$__crt_seh_guarded_call@X@@QEAAX$$QEAV<lambda_2d41944a1d46af3157314b8a01080d33>@@AEAV<lambda_8f455de75cd7d7f24b4096f044d8b9e6>@@$$QEAV<lambda_aa500f224e6afead328df44964fe2772>@@@Z@4HA 000000018001c3bc     libucrt:per_thread_data.obj
 0001:0001b3bc       $unwind$__acrt_initialize_lowio$fin$0 000000018001c3bc     libucrt:ioinit.obj
 0001:0001b3bc       $unwind$?fin$0@?0???$?RV<lambda_751a882b2c74d4b022dec766aa51a29a>@@AEAV<lambda_628dfdc04ba53c8bfc02c9951375f3f5>@@V<lambda_f6c7be5f7998530c34de24c7437d6b54>@@@?$__crt_seh_guarded_call@H@@QEAAH$$QEAV<lambda_751a882b2c74d4b022dec766aa51a29a>@@AEAV<lambda_628dfdc04ba53c8bfc02c9951375f3f5>@@$$QEAV<lambda_f6c7be5f7998530c34de24c7437d6b54>@@@Z@4HA 000000018001c3bc     libucrt:close.obj
 0001:0001b3bc       $unwind$?filt$0@?0???R<lambda_6e4b09c48022b2350581041d5f6b0c4c>@@QEBA@XZ@4HA 000000018001c3bc     libucrt:exit.obj
 0001:0001b3bc       $unwind$?fin$0@?0???$?RV<lambda_d80eeec6fff315bfe5c115232f3240e3>@@AEAV<lambda_6e4b09c48022b2350581041d5f6b0c4c>@@V<lambda_2358e3775559c9db80273638284d5e45>@@@?$__crt_seh_guarded_call@X@@QEAAX$$QEAV<lambda_d80eeec6fff315bfe5c115232f3240e3>@@AEAV<lambda_6e4b09c48022b2350581041d5f6b0c4c>@@$$QEAV<lambda_2358e3775559c9db80273638284d5e45>@@@Z@4HA 000000018001c3bc     libucrt:exit.obj
 0001:0001b3bc       $unwind$__acrt_update_thread_locale_data$fin$0 000000018001c3bc     libucrt:locale_refcounting.obj
 0001:0001b3bc       $unwind$_write$fin$0       000000018001c3bc     libucrt:write.obj
 0001:0001b3bc       $unwind$fclose$fin$0       000000018001c3bc     libucrt:fclose.obj
 0001:0001b3bc       $unwind$?fin$0@?0???$?RV<lambda_efdfa57d1f175319df784efa44bb7b81>@@AEAV<lambda_5f0a4c1567f8adc6734073e5d1e1b35c>@@V<lambda_2e8a7d3640ea6ccb4c2413664c2db6fd>@@@?$__crt_seh_guarded_call@X@@QEAAX$$QEAV<lambda_efdfa57d1f175319df784efa44bb7b81>@@AEAV<lambda_5f0a4c1567f8adc6734073e5d1e1b35c>@@$$QEAV<lambda_2e8a7d3640ea6ccb4c2413664c2db6fd>@@@Z@4HA 000000018001c3bc     libucrt:mbctype.obj
 0001:0001b3bc       $unwind$?fin$0@?0???$?RV<lambda_a37b2b86f63e897a80ea819b0eb08c01>@@AEAV<lambda_38ce7e780aa69e748d6df282ebc68efe>@@V<lambda_99fb1378e971ab6e7edea83e3a7a83a2>@@@?$__crt_seh_guarded_call@H@@QEAAH$$QEAV<lambda_a37b2b86f63e897a80ea819b0eb08c01>@@AEAV<lambda_38ce7e780aa69e748d6df282ebc68efe>@@$$QEAV<lambda_99fb1378e971ab6e7edea83e3a7a83a2>@@@Z@4HA 000000018001c3bc     libucrt:commit.obj
 0001:0001b3bc       $unwind$_ctrlfp$filt$0     000000018001c3bc     libucrt:fpctrl.obj
 0001:0001b3bc       $unwind$?fin$0@?0??update_thread_multibyte_data_internal@@YAPEAU__crt_multibyte_data@@QEAU__acrt_ptd@@QEAPEAU1@@Z@4HA 000000018001c3bc     libucrt:mbctype.obj
 0001:0001b3bc       $unwind$_IsNonwritableInCurrentImage$filt$0 000000018001c3bc     LIBCMT:pesect.obj
 0001:0001b3bc       $unwind$?fin$0@?0???$?RV<lambda_7777bce6b2f8c936911f934f8298dc43>@@AEAV<lambda_f03950bc5685219e0bcd2087efbe011e>@@V<lambda_3883c3dff614d5e0c5f61bb1ac94921c>@@@?$__crt_seh_guarded_call@H@@QEAAH$$QEAV<lambda_7777bce6b2f8c936911f934f8298dc43>@@AEAV<lambda_f03950bc5685219e0bcd2087efbe011e>@@$$QEAV<lambda_3883c3dff614d5e0c5f61bb1ac94921c>@@@Z@4HA 000000018001c3bc     libucrt:onexit.obj
 0001:0001b3bc       $unwind$__acrt_lowio_ensure_fh_exists$fin$0 000000018001c3bc     libucrt:osfinfo.obj
 0001:0001b3c4       $unwind$?dllmain_crt_process_detach@@YAH_N@Z 000000018001c3c4     LIBCMT:dll_dllmain.obj
 0001:0001b3fc       $unwind$?dllmain_dispatch@@YAHQEAUHINSTANCE__@@KQEAX@Z 000000018001c3fc     LIBCMT:dll_dllmain.obj
 0001:0001b424       $unwind$?filt$0@?0??dllmain_dispatch@@YAHQEAUHINSTANCE__@@KQEAX@Z@4HA 000000018001c424     LIBCMT:dll_dllmain.obj
 0001:0001b42c       $unwind$?__scrt_throw_std_bad_alloc@@YAXXZ 000000018001c42c     LIBCMT:throw_bad_alloc.obj
 0001:0001b42c       $unwind$?__scrt_throw_std_bad_array_new_length@@YAXXZ 000000018001c42c     LIBCMT:throw_bad_alloc.obj
 0001:0001b42c       $unwind$_raise_exc         000000018001c42c     libucrt:fpexcept.obj
 0001:0001b434       $unwind$__security_init_cookie 000000018001c434     LIBCMT:gs_support.obj
 0001:0001b440       $unwind$__scrt_is_nonwritable_in_current_image 000000018001c440     LIBCMT:utility.obj
 0001:0001b460       $unwind$__scrt_is_nonwritable_in_current_image$filt$0 000000018001c460     LIBCMT:utility.obj
 0001:0001b468       $unwind$__dcrt_lowio_ensure_console_output_initialized 000000018001c468     libucrt:initcon.obj
 0001:0001b468       $unwind$?getSystemCP@@YAHH@Z 000000018001c468     libucrt:mbctype.obj
 0001:0001b468       $unwind$__scrt_initialize_onexit_tables 000000018001c468     LIBCMT:utility.obj
 0001:0001b468       $unwind$_isleadbyte_l      000000018001c468     libucrt:_wctype.obj
 0001:0001b470       $unwind$__scrt_fastfail    000000018001c470     LIBCMT:utility_desktop.obj
 0001:0001b480       $unwind$__isa_available_init 000000018001c480     LIBCMT:cpu_disp.obj
 0001:0001b498       $xdatasym                  000000018001c498     LIBCMT:guard_dispatch.obj
 0001:0001b4a0       $xdatasym                  000000018001c4a0     libvcruntime:memcpy.obj
 0001:0001b4b0       $xdatasym                  000000018001c4b0     libvcruntime:memset.obj
 0001:0001b4c0       $unwind$wcschr             000000018001c4c0     libvcruntime:wcschr.obj
 0001:0001b4c8       $xdatasym                  000000018001c4c8     libvcruntime:memcmp.obj
 0001:0001b4cc       $unwind$__C_specific_handler 000000018001c4cc     libvcruntime:riscchandler.obj
 0001:0001b4e8       $unwind$__std_exception_copy 000000018001c4e8     libvcruntime:std_exception.obj
 0001:0001b4e8       $unwind$_free_osfhnd       000000018001c4e8     libucrt:osfinfo.obj
 0001:0001b4fc       $unwind$_CxxThrowException 000000018001c4fc     libvcruntime:throw.obj
 0001:0001b510       $xdatasym                  000000018001c510     libvcruntime:notify.obj
 0001:0001b51c       $unwind$__DestructExceptionObject 000000018001c51c     libvcruntime:ehhelpers.obj
 0001:0001b53c       $unwind$__vcrt_initialize_winapi_thunks 000000018001c53c     libvcruntime:winapi_downlevel.obj
 0001:0001b53c       $unwind$__acrt_initialize_winapi_thunks 000000018001c53c     libucrt:winapi_thunks.obj
 0001:0001b544       $unwind$__vcrt_uninitialize_winapi_thunks 000000018001c544     libvcruntime:winapi_downlevel.obj
 0001:0001b550       $xdatasym                  000000018001c550     libvcruntime:handlers.obj
 0001:0001b560       $unwind$_query_new_handler 000000018001c560     libucrt:new_handler.obj
 0001:0001b580       $unwind$?common_exit@@YAXHW4_crt_exit_cleanup_mode@@W4_crt_exit_return_mode@@@Z 000000018001c580     libucrt:exit.obj
 0001:0001b58c       $unwind$??R<lambda_6e4b09c48022b2350581041d5f6b0c4c>@@QEBA@XZ 000000018001c58c     libucrt:exit.obj
 0001:0001b5ac       $unwind$??$?RV<lambda_d80eeec6fff315bfe5c115232f3240e3>@@AEAV<lambda_6e4b09c48022b2350581041d5f6b0c4c>@@V<lambda_2358e3775559c9db80273638284d5e45>@@@?$__crt_seh_guarded_call@X@@QEAAX$$QEAV<lambda_d80eeec6fff315bfe5c115232f3240e3>@@AEAV<lambda_6e4b09c48022b2350581041d5f6b0c4c>@@$$QEAV<lambda_2358e3775559c9db80273638284d5e45>@@@Z 000000018001c5ac     libucrt:exit.obj
 0001:0001b5d0       $unwind$_configure_narrow_argv 000000018001c5d0     libucrt:argv_parsing.obj
 0001:0001b5e4       $unwind$??$parse_command_line@D@@YAXPEADPEAPEAD0PEA_K2@Z 000000018001c5e4     libucrt:argv_parsing.obj
 0001:0001b600       $unwind$??$free_environment@D@@YAXQEAPEAD@Z 000000018001c600     libucrt:environment_initialization.obj
 0001:0001b600       $unwind$??$free_environment@_W@@YAXQEAPEA_W@Z 000000018001c600     libucrt:environment_initialization.obj
 0001:0001b60c       $unwind$??$create_environment@D@@YAQEAPEADQEAD@Z 000000018001c60c     libucrt:environment_initialization.obj
 0001:0001b624       $unwind$_execute_onexit_table 000000018001c624     libucrt:onexit.obj
 0001:0001b62c       $unwind$??R<lambda_f03950bc5685219e0bcd2087efbe011e>@@QEBAHXZ 000000018001c62c     libucrt:onexit.obj
 0001:0001b644       $unwind$??$?RV<lambda_7777bce6b2f8c936911f934f8298dc43>@@AEAV<lambda_f03950bc5685219e0bcd2087efbe011e>@@V<lambda_3883c3dff614d5e0c5f61bb1ac94921c>@@@?$__crt_seh_guarded_call@H@@QEAAH$$QEAV<lambda_7777bce6b2f8c936911f934f8298dc43>@@AEAV<lambda_f03950bc5685219e0bcd2087efbe011e>@@$$QEAV<lambda_3883c3dff614d5e0c5f61bb1ac94921c>@@@Z 000000018001c644     libucrt:onexit.obj
 0001:0001b668       $unwind$terminate          000000018001c668     libucrt:terminate.obj
 0001:0001b688       $unwind$_wcsdup            000000018001c688     libucrt:wcsdup.obj
 0001:0001b688       $unwind$_invalid_parameter 000000018001c688     libucrt:invalid_parameter.obj
 0001:0001b6a0       $xdatasym                  000000018001c6a0     libucrt:strncmp.obj
 0001:0001b6a4       $unwind$?destroy_fls@@YAXPEAX@Z 000000018001c6a4     libucrt:per_thread_data.obj
 0001:0001b6a4       $unwind$__acrt_locale_free_lc_time_if_unreferenced 000000018001c6a4     libucrt:locale_refcounting.obj
 0001:0001b6a4       $unwind$_free_base         000000018001c6a4     libucrt:free_base.obj
 0001:0001b6a4       $unwind$__acrt_locale_free_numeric 000000018001c6a4     libucrt:initnum.obj
 0001:0001b6ac       $unwind$?construct_ptd_array@@YAXQEAU__acrt_ptd@@@Z 000000018001c6ac     libucrt:per_thread_data.obj
 0001:0001b6b4       $unwind$?destroy_ptd_array@@YAXQEAU__acrt_ptd@@@Z 000000018001c6b4     libucrt:per_thread_data.obj
 0001:0001b6bc       $unwind$??$?RV<lambda_0ae27a3a962d80f24befdcbee591983d>@@AEAV<lambda_8d0ee55de4b1038c4002e0adecdf1839>@@V<lambda_dc504788e8f1664fe9b84e20bfb512f2>@@@?$__crt_seh_guarded_call@X@@QEAAX$$QEAV<lambda_0ae27a3a962d80f24befdcbee591983d>@@AEAV<lambda_8d0ee55de4b1038c4002e0adecdf1839>@@$$QEAV<lambda_dc504788e8f1664fe9b84e20bfb512f2>@@@Z 000000018001c6bc     libucrt:per_thread_data.obj
 0001:0001b6e0       $unwind$??$?RV<lambda_aa87e3671a710a21b5dc78c0bdf72e11>@@AEAV<lambda_92619d2358a28f41a33ba319515a20b9>@@V<lambda_6992ecaafeb10aed2b74cb1fae11a551>@@@?$__crt_seh_guarded_call@X@@QEAAX$$QEAV<lambda_aa87e3671a710a21b5dc78c0bdf72e11>@@AEAV<lambda_92619d2358a28f41a33ba319515a20b9>@@$$QEAV<lambda_6992ecaafeb10aed2b74cb1fae11a551>@@@Z 000000018001c6e0     libucrt:per_thread_data.obj
 0001:0001b704       $unwind$??$?RV<lambda_f2e299630e499de9f9a165e60fcd3db5>@@AEAV<lambda_2ae9d31cdba2644fcbeaf08da7c24588>@@V<lambda_40d01ff24d0e7b3814fdbdcee8eab3c7>@@@?$__crt_seh_guarded_call@X@@QEAAX$$QEAV<lambda_f2e299630e499de9f9a165e60fcd3db5>@@AEAV<lambda_2ae9d31cdba2644fcbeaf08da7c24588>@@$$QEAV<lambda_40d01ff24d0e7b3814fdbdcee8eab3c7>@@@Z 000000018001c704     libucrt:per_thread_data.obj
 0001:0001b728       $unwind$??$?RV<lambda_2d41944a1d46af3157314b8a01080d33>@@AEAV<lambda_8f455de75cd7d7f24b4096f044d8b9e6>@@V<lambda_aa500f224e6afead328df44964fe2772>@@@?$__crt_seh_guarded_call@X@@QEAAX$$QEAV<lambda_2d41944a1d46af3157314b8a01080d33>@@AEAV<lambda_8f455de75cd7d7f24b4096f044d8b9e6>@@$$QEAV<lambda_aa500f224e6afead328df44964fe2772>@@@Z 000000018001c728     libucrt:per_thread_data.obj
 0001:0001b74c       $unwind$__acrt_call_reportfault 000000018001c74c     libucrt:invalid_parameter.obj
 0001:0001b76c       $unwind$??$__acrt_mbs_to_wcs_cp@U__crt_win32_buffer_internal_dynamic_resizing@@@@YAHQEBDAEAV?$__crt_win32_buffer@_WU__crt_win32_buffer_internal_dynamic_resizing@@@@I@Z 000000018001c76c     libucrt:argv_wildcards.obj
 0001:0001b784       $unwind$??$__acrt_wcs_to_mbs_cp@U__crt_win32_buffer_internal_dynamic_resizing@@@@YAHQEB_WAEAV?$__crt_win32_buffer@DU__crt_win32_buffer_internal_dynamic_resizing@@@@I@Z 000000018001c784     libucrt:argv_wildcards.obj
 0001:0001b784       $unwind$__dcrt_get_narrow_environment_from_os 000000018001c784     libucrt:get_environment_from_os.obj
 0001:0001b79c       $unwind$??$common_expand_argv_wildcards@D@@YAHQEAPEADQEAPEAPEAD@Z 000000018001c79c     libucrt:argv_wildcards.obj
 0001:0001b7b4       $unwind$??$expand_argument_wildcards@D@@YAHQEAD0AEAV?$argument_list@D@?A0x5f5c8891@@@Z 000000018001c7b4     libucrt:argv_wildcards.obj
 0001:0001b7d8       $unwind$__acrt_GetModuleFileNameA 000000018001c7d8     libucrt:getmodulefilenamea.obj
 0001:0001b7f4       $unwind$__dcrt_write_console 000000018001c7f4     libucrt:initcon.obj
 0001:0001b7f4       $unwind$??$__acrt_wcs_to_mbs_cp@U__crt_win32_buffer_no_resizing@@@@YAHQEB_WAEAV?$__crt_win32_buffer@DU__crt_win32_buffer_no_resizing@@@@I@Z 000000018001c7f4     libucrt:getmodulefilenamea.obj
 0001:0001b808       $unwind$_setmbcp_nolock    000000018001c808     libucrt:mbctype.obj
 0001:0001b828       $unwind$?update_thread_multibyte_data_internal@@YAPEAU__crt_multibyte_data@@QEAU__acrt_ptd@@QEAPEAU1@@Z 000000018001c828     libucrt:mbctype.obj
 0001:0001b850       $unwind$?setmbcp_internal@@YAHH_NQEAU__acrt_ptd@@QEAPEAU__crt_multibyte_data@@@Z 000000018001c850     libucrt:mbctype.obj
 0001:0001b860       $unwind$?setSBUpLow@@YAXPEAU__crt_multibyte_data@@@Z 000000018001c860     libucrt:mbctype.obj
 0001:0001b87c       $unwind$??$?RV<lambda_efdfa57d1f175319df784efa44bb7b81>@@AEAV<lambda_5f0a4c1567f8adc6734073e5d1e1b35c>@@V<lambda_2e8a7d3640ea6ccb4c2413664c2db6fd>@@@?$__crt_seh_guarded_call@X@@QEAAX$$QEAV<lambda_efdfa57d1f175319df784efa44bb7b81>@@AEAV<lambda_5f0a4c1567f8adc6734073e5d1e1b35c>@@$$QEAV<lambda_2e8a7d3640ea6ccb4c2413664c2db6fd>@@@Z 000000018001c87c     libucrt:mbctype.obj
 0001:0001b8a0       $unwind$?x_ismbbtype_l@@YAHPEAU__crt_locale_pointers@@IHH@Z 000000018001c8a0     libucrt:ismbbyte.obj
 0001:0001b8b0       $unwind$__GSHandlerCheckCommon 000000018001c8b0     LIBCMT:gshandler.obj
 0001:0001b8b0       $unwind$__acrt_WideCharToMultiByte 000000018001c8b0     libucrt:widechartomultibyte.obj
 0001:0001b8b8       $unwind$_mbtowc_l          000000018001c8b8     libucrt:mbtowc.obj
 0001:0001b8b8       $unwind$__acrt_LCMapStringEx 000000018001c8b8     libucrt:winapi_thunks.obj
 0001:0001b8cc       $unwind$__acrt_initialize_lowio 000000018001c8cc     libucrt:ioinit.obj
 0001:0001b8ec       $unwind$?initialize_inherited_file_handles_nolock@@YAXXZ 000000018001c8ec     libucrt:ioinit.obj
 0001:0001b908       $unwind$__acrt_initialize_stdio 000000018001c908     libucrt:_file.obj
 0001:0001b908       $unwind$?initialize_stdio_handles_nolock@@YAXXZ 000000018001c908     libucrt:ioinit.obj
 0001:0001b920       $unwind$__acrt_uninitialize_locale 000000018001c920     libucrt:wsetlocale.obj
 0001:0001b920       $unwind$__acrt_get_sigabrt_handler 000000018001c920     libucrt:signal.obj
 0001:0001b928       $unwind$raise              000000018001c928     libucrt:signal.obj
 0001:0001b964       $unwind$??$?RV<lambda_450d765d439847d4c735a33c368b5fc0>@@AEAV<lambda_44731a7d0e6d81c3e6aa82d741081786>@@V<lambda_601a2a7da3b7a96e9554ac7215c4b07c>@@@?$__crt_seh_guarded_call@P6AXH@Z@@QEAAP6AXH@Z$$QEAV<lambda_450d765d439847d4c735a33c368b5fc0>@@AEAV<lambda_44731a7d0e6d81c3e6aa82d741081786>@@$$QEAV<lambda_601a2a7da3b7a96e9554ac7215c4b07c>@@@Z 000000018001c964     libucrt:signal.obj
 0001:0001b988       $unwind$?common_flush_all@@YAH_N@Z 000000018001c988     libucrt:fflush.obj
 0001:0001b990       $unwind$??$?RV<lambda_842d9ff0dc9ef11c61343bbaebe7f885>@@AEAV<lambda_c5860995281e5c4ce005b3de8f5874ee>@@V<lambda_d90129c13df834fdcbf8d2b88dafcf2d>@@@?$__crt_seh_guarded_call@X@@QEAAX$$QEAV<lambda_842d9ff0dc9ef11c61343bbaebe7f885>@@AEAV<lambda_c5860995281e5c4ce005b3de8f5874ee>@@$$QEAV<lambda_d90129c13df834fdcbf8d2b88dafcf2d>@@@Z 000000018001c990     libucrt:fflush.obj
 0001:0001b9b4       $unwind$??$?RV<lambda_886d6c58226a84441f68b9f2b8217b83>@@AEAV<lambda_ab61a845afdef5b7c387490eaf3616ee>@@V<lambda_f7f22ab5edc0698d5f6905b0d3f44752>@@@?$__crt_seh_guarded_call@X@@QEAAX$$QEAV<lambda_886d6c58226a84441f68b9f2b8217b83>@@AEAV<lambda_ab61a845afdef5b7c387490eaf3616ee>@@$$QEAV<lambda_f7f22ab5edc0698d5f6905b0d3f44752>@@@Z 000000018001c9b4     libucrt:fflush.obj
 0001:0001b9dc       $unwind$??$?RV<lambda_410d79af7f07d98d83a3f525b3859a53>@@AEAV<lambda_3e16ef9562a7dcce91392c22ab16ea36>@@V<lambda_38119f0e861e05405d8a144b9b982f0a>@@@?$__crt_seh_guarded_call@X@@QEAAX$$QEAV<lambda_410d79af7f07d98d83a3f525b3859a53>@@AEAV<lambda_3e16ef9562a7dcce91392c22ab16ea36>@@$$QEAV<lambda_38119f0e861e05405d8a144b9b982f0a>@@@Z 000000018001c9dc     libucrt:wsetlocale.obj
 0001:0001ba04       $unwind$__acrt_update_thread_locale_data 000000018001ca04     libucrt:locale_refcounting.obj
 0001:0001ba28       $unwind$qsort              000000018001ca28     libucrt:qsort.obj
 0001:0001ba40       $chain$4$qsort             000000018001ca40     libucrt:qsort.obj
 0001:0001ba64       $chain$5$qsort             000000018001ca64     libucrt:qsort.obj
 0001:0001ba74       $unwind$strpbrk            000000018001ca74     libucrt:strpbrk.obj
 0001:0001ba84       $unwind$fallbackMethod     000000018001ca84     libucrt:strpbrk.obj
 0001:0001ba94       $unwind$_mbsdec_l          000000018001ca94     libucrt:mbsdec.obj
 0001:0001baa0       $unwind$__acrt_GetStringTypeA 000000018001caa0     libucrt:getstringtypea.obj
 0001:0001bac8       $unwind$__acrt_LCMapStringA 000000018001cac8     libucrt:lcmapstringa.obj
 0001:0001bad8       $unwind$?__acrt_LCMapStringA_stat@@YAHPEAU__crt_locale_pointers@@PEB_WKPEBDHPEADHHH@Z 000000018001cad8     libucrt:lcmapstringa.obj
 0001:0001bb00       $unwind$?GetTableIndexFromLocaleName@@YAHPEB_W@Z 000000018001cb00     libucrt:lcidtoname_downlevel.obj
 0001:0001bb18       $unwind$__acrt_lowio_destroy_handle_array 000000018001cb18     libucrt:osfinfo.obj
 0001:0001bb28       $unwind$__acrt_lowio_ensure_fh_exists 000000018001cb28     libucrt:osfinfo.obj
 0001:0001bb54       $unwind$_commit            000000018001cb54     libucrt:commit.obj
 0001:0001bb54       $unwind$_close             000000018001cb54     libucrt:close.obj
 0001:0001bb5c       $unwind$??$?RV<lambda_a37b2b86f63e897a80ea819b0eb08c01>@@AEAV<lambda_38ce7e780aa69e748d6df282ebc68efe>@@V<lambda_99fb1378e971ab6e7edea83e3a7a83a2>@@@?$__crt_seh_guarded_call@H@@QEAAH$$QEAV<lambda_a37b2b86f63e897a80ea819b0eb08c01>@@AEAV<lambda_38ce7e780aa69e748d6df282ebc68efe>@@$$QEAV<lambda_99fb1378e971ab6e7edea83e3a7a83a2>@@@Z 000000018001cb5c     libucrt:commit.obj
 0001:0001bb80       $unwind$_write             000000018001cb80     libucrt:write.obj
 0001:0001bbb0       $unwind$_write_nolock      000000018001cbb0     libucrt:write.obj
 0001:0001bbc8       $unwind$?write_double_translated_ansi_nolock@@YA?AUwrite_result@?A0x17268360@@HQEBDI@Z 000000018001cbc8     libucrt:write.obj
 0001:0001bbec       $unwind$?write_text_utf16le_nolock@@YA?AUwrite_result@?A0x17268360@@HQEBDI@Z 000000018001cbec     libucrt:write.obj
 0001:0001bbec       $unwind$?write_text_ansi_nolock@@YA?AUwrite_result@?A0x17268360@@HQEBDI@Z 000000018001cbec     libucrt:write.obj
 0001:0001bc0c       $unwind$?write_text_utf8_nolock@@YA?AUwrite_result@?A0x17268360@@HQEBDI@Z 000000018001cc0c     libucrt:write.obj
 0001:0001bc30       $unwind$_fcloseall         000000018001cc30     libucrt:closeall.obj
 0001:0001bc54       $unwind$?__mbrtowc_utf8@__crt_mbstring@@YA_KPEA_WPEBD_KPEAU_Mbstatet@@@Z 000000018001cc54     libucrt:mbrtowc.obj
 0001:0001bc5c       $unwind$?__mbsrtowcs_utf8@__crt_mbstring@@YA_KPEA_WPEAPEBD_KPEAU_Mbstatet@@@Z 000000018001cc5c     libucrt:mbrtowc.obj
 0001:0001bc74       $unwind$__acrt_locale_free_monetary 000000018001cc74     libucrt:initmon.obj
 0001:0001bc7c       $unwind$__acrt_locale_free_time 000000018001cc7c     libucrt:inittime.obj
 0001:0001bc8c       $unwind$_putwch_nolock     000000018001cc8c     libucrt:putwch.obj
 0001:0001bc94       $unwind$fclose             000000018001cc94     libucrt:fclose.obj
 0001:0001bcb8       $unwind$?__mbrtoc32_utf8@__crt_mbstring@@YA_KPEA_UPEBD_KPEAU_Mbstatet@@@Z 000000018001ccb8     libucrt:mbrtoc32.obj
 0001:0001bcd8       $xdatasym                  000000018001ccd8     libucrt:log10.obj
 0001:0001bce4       $unwind$??$?RV<lambda_751a882b2c74d4b022dec766aa51a29a>@@AEAV<lambda_628dfdc04ba53c8bfc02c9951375f3f5>@@V<lambda_f6c7be5f7998530c34de24c7437d6b54>@@@?$__crt_seh_guarded_call@H@@QEAAH$$QEAV<lambda_751a882b2c74d4b022dec766aa51a29a>@@AEAV<lambda_628dfdc04ba53c8bfc02c9951375f3f5>@@$$QEAV<lambda_f6c7be5f7998530c34de24c7437d6b54>@@@Z 000000018001cce4     libucrt:close.obj
 0001:0001bd08       $unwind$_call_matherr      000000018001cd08     libucrt:libm_error.obj
 0001:0001bd10       $unwind$_handle_error      000000018001cd10     libucrt:libm_error.obj
 0001:0001bd30       $unwind$__acrt_initialize_fma3 000000018001cd30     libucrt:fma3_available.obj
 0001:0001bd38       $unwind$_log_special_common 000000018001cd38     libucrt:log_special.obj
 0001:0001bd48       $xdatasym                  000000018001cd48     libucrt:fpsr.obj
 0001:0001bd50       $unwind$_raise_exc_ex      000000018001cd50     libucrt:fpexcept.obj
 0001:0001bd64       $unwind$_ctrlfp            000000018001cd64     libucrt:fpctrl.obj
 0001:0001bd8c       $unwind$_IsNonwritableInCurrentImage 000000018001cd8c     LIBCMT:pesect.obj
 0001:0001bdb0       $xdatasym                  000000018001cdb0     LIBCMT:amdsecgs.obj
 0001:0001bdb4       $unwind$__report_securityfailure 000000018001cdb4     LIBCMT:gs_report.obj
 0001:0001bdbc       $unwind$__report_gsfailure 000000018001cdbc     LIBCMT:gs_report.obj
 0001:0001bdc4       $unwind$capture_current_context 000000018001cdc4     LIBCMT:gs_report.obj
 0001:0001bdd0       $unwind$capture_previous_context 000000018001cdd0     LIBCMT:gs_report.obj
 0001:0001bed0       .edata                     000000018001ced0     TmpPanel.exp
 0001:0001bef8       rgpv                       000000018001cef8     TmpPanel.exp
 0001:0001bf34       rgszName                   000000018001cf34     TmpPanel.exp
 0001:0001bf70       rgwOrd                     000000018001cf70     TmpPanel.exp
 0001:0001bf8e       szName                     000000018001cf8e     TmpPanel.exp
 0001:0001bf9b       $N00001                    000000018001cf9b     TmpPanel.exp
 0001:0001bfa4       $N00002                    000000018001cfa4     TmpPanel.exp
 0001:0001bfb0       $N00003                    000000018001cfb0     TmpPanel.exp
 0001:0001bfbb       $N00004                    000000018001cfbb     TmpPanel.exp
 0001:0001bfc4       $N00005                    000000018001cfc4     TmpPanel.exp
 0001:0001bfd1       $N00006                    000000018001cfd1     TmpPanel.exp
 0001:0001bfe0       $N00007                    000000018001cfe0     TmpPanel.exp
 0001:0001bff2       $N00008                    000000018001cff2     TmpPanel.exp
 0001:0001c001       $N00009                    000000018001d001     TmpPanel.exp
 0001:0001c007       $N00010                    000000018001d007     TmpPanel.exp
 0001:0001c01a       $N00011                    000000018001d01a     TmpPanel.exp
 0001:0001c02d       $N00012                    000000018001d02d     TmpPanel.exp
 0001:0001c037       $N00013                    000000018001d037     TmpPanel.exp
 0001:0001c045       $N00014                    000000018001d045     TmpPanel.exp
 0001:0001c052       $N00015                    000000018001d052     TmpPanel.exp
 0002:00000000       ?FKeys@?1??GetOpenPanelInfo@TmpPanel@@QEAAXPEAUOpenPanelInfo@@@Z@4PAGA 000000018001e000     TmpClass.obj
 0002:00000018       ?kbt@?1??GetOpenPanelInfo@TmpPanel@@QEAAXPEAUOpenPanelInfo@@@Z@4UKeyBarTitles@@A 000000018001e018     TmpClass.obj
 0002:00000028       ?CRLF@?BB@??SaveListFile@TmpPanel@@AEAAXPEB_W@Z@4PEB_WEB 000000018001e028     TmpClass.obj
 0002:00000030       ?CRLF@?BD@??SaveListFile@TmpPanel@@AEAAXPEB_W@Z@4PEBDEB 000000018001e030     TmpClass.obj
 0002:00000060       ?__vcrt_flsindex@@3KA      000000018001e060     libvcruntime:per_thread_data.obj
 0002:00000074       ?__acrt_flsindex@@3KA      000000018001e074     libucrt:per_thread_data.obj
 0002:00000078       ?errno_no_memory@@3HA      000000018001e078     libucrt:errno.obj
 0002:0000007c       ?doserrno_no_memory@@3KA   000000018001e07c     libucrt:errno.obj
 0002:00000080       _mbctypes                  000000018001e080     libucrt:mbctype.obj
 0002:00000190       _mbcasemaps                000000018001e190     libucrt:mbctype.obj
 0002:00000290       ?__rgctypeflag@@3PADA      000000018001e290     libucrt:mbctype.obj
 0002:000002a0       ?__rgcode_page_info@@3PAUcode_page_info@@A 000000018001e2a0     libucrt:mbctype.obj
 0002:000009e0       ?__dcrt_lowio_console_output_handle@@3PEAXEA 000000018001e9e0     libucrt:initcon.obj
 0002:000009f0       ?dazSupported@?1??_ctrlfp@@9@9 000000018001e9f0     libucrt:fpctrl.obj
 0002:00000df8       ?DiskMenuStrings@?4??GetPluginInfoW@@9@4PAPEB_WA 000000018001edf8     TmpPanel.obj
 0002:00000e00       ?PluginMenuStrings@?7??GetPluginInfoW@@9@4PAPEB_WA 000000018001ee00     TmpPanel.obj
 0002:00000e08       ?PluginCfgStrings@?1??GetPluginInfoW@@9@4PAPEB_WA 000000018001ee08     TmpPanel.obj
 0002:00001470       ?Title@?1??GetOpenPanelInfo@TmpPanel@@QEAAXPEAUOpenPanelInfo@@@Z@4PA_WA 000000018001f470     TmpClass.obj
 0002:00001540       ?PanelModesArray@?1??GetOpenPanelInfo@TmpPanel@@QEAAXPEAUOpenPanelInfo@@@Z@4PAUPanelMode@@A 000000018001f540     TmpClass.obj
 0002:00001720       ?kbl@?1??GetOpenPanelInfo@TmpPanel@@QEAAXPEAUOpenPanelInfo@@@Z@4PAUKeyBarLabel@@A 000000018001f720     TmpClass.obj
 0002:00001780       ?__proc_attached@@3HA      000000018001f780     LIBCMT:dll_dllmain.obj
 0002:000017c0       ?is_initialized_as_dll@@3_NA 000000018001f7c0     LIBCMT:utility.obj
 0002:000017c1       ?module_local_atexit_table_initialized@@3_NA 000000018001f7c1     LIBCMT:utility.obj
 0002:000017c8       ?module_local_atexit_table@@3U_onexit_table_t@@A 000000018001f7c8     LIBCMT:utility.obj
 0002:000017e0       ?module_local_at_quick_exit_table@@3U_onexit_table_t@@A 000000018001f7e0     LIBCMT:utility.obj
 0002:00001848       ?heap@@3V_HeapManager@@A   000000018001f848     libvcruntime:undname.obj
 0002:00001870       ?__vcrt_startup_thread_ptd@@3U__vcrt_ptd@@A 000000018001f870     libvcruntime:per_thread_data.obj
 0002:00001900       __vcrt_lock_table          000000018001f900     libvcruntime:locks.obj
 0002:00001928       __vcrt_locks_initialized   000000018001f928     libvcruntime:locks.obj
 0002:00001930       ?module_handles@@3PAPEAUHINSTANCE__@@A 000000018001f930     libvcruntime:winapi_downlevel.obj
 0002:00001948       ?encoded_function_pointers@@3PAPEAXA 000000018001f948     libvcruntime:winapi_downlevel.obj
 0002:00001978       ?__acrt_new_handler@@3V?$dual_state_global@P6AH_K@Z@__crt_state_management@@A 000000018001f978     libucrt:new_handler.obj
 0002:00001980       ?c_termination_complete@@3JA 000000018001f980     libucrt:exit.obj
 0002:00001988       ?thread_local_exit_callback_func@@3P6AXPEAXK0@ZEA 000000018001f988     libucrt:exit.obj
 0002:000019a0       ?program_name@?1???$common_configure_argv@D@@YAHW4_crt_argv_mode@@@Z@4PADA 000000018001f9a0     libucrt:argv_parsing.obj
 0002:00001b00       ?__acrt_lock_table@@3PAU_RTL_CRITICAL_SECTION@@A 000000018001fb00     libucrt:locks.obj
 0002:00001d30       ?__acrt_locks_initialized@@3IA 000000018001fd30     libucrt:locks.obj
 0002:00001d38       ?__acrt_invalid_parameter_handler@@3V?$dual_state_global@P6AXPEB_W00I_K@Z@__crt_state_management@@A 000000018001fd38     libucrt:invalid_parameter.obj
 0002:00001d58       ?fSystemSet@@3HA           000000018001fd58     libucrt:mbctype.obj
 0002:00001d5c       ?initialized@?1??__acrt_initialize_multibyte@@9@4_NA 000000018001fd5c     libucrt:mbctype.obj
 0002:00001d90       ?module_handles@@3PAPEAUHINSTANCE__@@A 000000018001fd90     libucrt:winapi_thunks.obj
 0002:00001e30       ?encoded_function_pointers@@3PAPEAXA 000000018001fe30     libucrt:winapi_thunks.obj
 0002:00002358       ?ctrlc_action@@3V?$dual_state_global@P6AXH@Z@__crt_state_management@@A 0000000180020358     libucrt:signal.obj
 0002:00002360       ?ctrlbreak_action@@3V?$dual_state_global@P6AXH@Z@__crt_state_management@@A 0000000180020360     libucrt:signal.obj
 0002:00002368       ?abort_action@@3V?$dual_state_global@P6AXH@Z@__crt_state_management@@A 0000000180020368     libucrt:signal.obj
 0002:00002370       ?term_action@@3V?$dual_state_global@P6AXH@Z@__crt_state_management@@A 0000000180020370     libucrt:signal.obj
 0002:00002378       ?user_matherr@@3V?$dual_state_global@P6AHPEAU_exception@@@Z@__crt_state_management@@A 0000000180020378     libucrt:matherr.obj
 0002:000023a8       ?internal_state@?1??_mbtowc_l@@9@4U_Mbstatet@@A 00000001800203a8     libucrt:mbtowc.obj
 0002:000023b4       ?__acrt_global_new_mode@@3V?$dual_state_global@J@__crt_state_management@@A 00000001800203b4     libucrt:new_mode.obj
 0002:000023c0       ?__acrt_app_type@@3W4_crt_app_type@@A 00000001800203c0     libucrt:report_runtime_error.obj
 0002:000023c8       ?internal_pst@?1??__mbrtoc32_utf8@__crt_mbstring@@YA_KPEA_UPEBD_KPEAU_Mbstatet@@@Z@4U3@A 00000001800203c8     libucrt:mbrtoc32.obj
 0002:000023e0       GS_ExceptionRecord         00000001800203e0     LIBCMT:gs_report.obj
 0002:00002480       GS_ContextRecord           0000000180020480     LIBCMT:gs_report.obj
 0003:0000000c       $pdata$?OpenPanelFromOutput@@YAPEAXPEA_W@Z 000000018002100c     TmpPanel.obj
 0003:00000018       $pdata$1$?OpenPanelFromOutput@@YAPEAXPEA_W@Z 0000000180021018     TmpPanel.obj
 0003:00000024       $pdata$2$?OpenPanelFromOutput@@YAPEAXPEA_W@Z 0000000180021024     TmpPanel.obj
 0003:00000030       $pdata$3$?OpenPanelFromOutput@@YAPEAXPEA_W@Z 0000000180021030     TmpPanel.obj
 0003:0000003c       $pdata$4$?OpenPanelFromOutput@@YAPEAXPEA_W@Z 000000018002103c     TmpPanel.obj
 0003:00000048       $pdata$?ProcessList@@YAXPEAXPEA_WH@Z 0000000180021048     TmpPanel.obj
 0003:00000054       $pdata$?ReadFileLines@@YAXPEAXKPEAPEA_WPEA_WPEAI3@Z 0000000180021054     TmpPanel.obj
 0003:00000060       $pdata$1$?ReadFileLines@@YAXPEAXKPEAPEA_WPEA_WPEAI3@Z 0000000180021060     TmpPanel.obj
 0003:0000006c       $pdata$2$?ReadFileLines@@YAXPEAXKPEAPEA_WPEA_WPEAI3@Z 000000018002106c     TmpPanel.obj
 0003:00000078       $pdata$?ReadFileList@@YAXPEA_WPEAHPEAPEAPEA_W@Z 0000000180021078     TmpPanel.obj
 0003:00000084       $pdata$0$?ReadFileList@@YAXPEA_WPEAHPEAPEAPEA_W@Z 0000000180021084     TmpPanel.obj
 0003:00000090       $pdata$1$?ReadFileList@@YAXPEA_WPEAHPEAPEAPEA_W@Z 0000000180021090     TmpPanel.obj
 0003:0000009c       $pdata$?ShowMenuFromList@@YAXPEA_W@Z 000000018002109c     TmpPanel.obj
 0003:000000a8       $pdata$1$?ShowMenuFromList@@YAXPEA_W@Z 00000001800210a8     TmpPanel.obj
 0003:000000b4       $pdata$4$?ShowMenuFromList@@YAXPEA_W@Z 00000001800210b4     TmpPanel.obj
 0003:000000c0       $pdata$5$?ShowMenuFromList@@YAXPEA_W@Z 00000001800210c0     TmpPanel.obj
 0003:000000cc       $pdata$6$?ShowMenuFromList@@YAXPEA_W@Z 00000001800210cc     TmpPanel.obj
 0003:000000d8       $pdata$7$?ShowMenuFromList@@YAXPEA_W@Z 00000001800210d8     TmpPanel.obj
 0003:000000e4       $pdata$8$?ShowMenuFromList@@YAXPEA_W@Z 00000001800210e4     TmpPanel.obj
 0003:000000f0       $pdata$AnalyseW            00000001800210f0     TmpPanel.obj
 0003:000000fc       $pdata$ClosePanelW         00000001800210fc     TmpPanel.obj
 0003:00000108       $pdata$ConfigureW          0000000180021108     TmpPanel.obj
 0003:00000114       $pdata$ExitFARW            0000000180021114     TmpPanel.obj
 0003:00000120       $pdata$GetFindDataW        0000000180021120     TmpPanel.obj
 0003:0000012c       $pdata$GetGlobalInfoW      000000018002112c     TmpPanel.obj
 0003:00000138       $pdata$GetPluginInfoW      0000000180021138     TmpPanel.obj
 0003:00000144       $pdata$OpenW               0000000180021144     TmpPanel.obj
 0003:00000150       $pdata$4$OpenW             0000000180021150     TmpPanel.obj
 0003:0000015c       $pdata$5$OpenW             000000018002115c     TmpPanel.obj
 0003:00000168       $pdata$ProcessPanelEventW  0000000180021168     TmpPanel.obj
 0003:00000174       $pdata$ProcessPanelInputW  0000000180021174     TmpPanel.obj
 0003:00000180       $pdata$PutFilesW           0000000180021180     TmpPanel.obj
 0003:0000018c       $pdata$SetDirectoryW       000000018002118c     TmpPanel.obj
 0003:00000198       $pdata$SetFindListW        0000000180021198     TmpPanel.obj
 0003:000001a4       $pdata$SetStartupInfoW     00000001800211a4     TmpPanel.obj
 0003:000001b0       $pdata$??1?$DialogBuilderBase@UFarDialogItem@@@@MEAA@XZ 00000001800211b0     TmpCfg.obj
 0003:000001bc       $pdata$0$??1?$DialogBuilderBase@UFarDialogItem@@@@MEAA@XZ 00000001800211bc     TmpCfg.obj
 0003:000001c8       $pdata$1$??1?$DialogBuilderBase@UFarDialogItem@@@@MEAA@XZ 00000001800211c8     TmpCfg.obj
 0003:000001d4       $pdata$??_G?$DialogBuilderBase@UFarDialogItem@@@@MEAAPEAXI@Z 00000001800211d4     TmpCfg.obj
 0003:000001e0       $pdata$??_G?$DialogItemBinding@UFarDialogItem@@@@UEAAPEAXI@Z 00000001800211e0     TmpCfg.obj
 0003:000001ec       $pdata$??_GPluginEditFieldBinding@@UEAAPEAXI@Z 00000001800211ec     TmpCfg.obj
 0003:000001ec       $pdata$??_GPluginCheckBoxBinding@@UEAAPEAXI@Z 00000001800211ec     TmpCfg.obj
 0003:000001f8       $pdata$??_GPluginDialogBuilder@@UEAAPEAXI@Z 00000001800211f8     TmpCfg.obj
 0003:00000204       $pdata$??_GPluginUIntEditFieldBinding@@UEAAPEAXI@Z 0000000180021204     TmpCfg.obj
 0003:00000204       $pdata$??_GPluginIntEditFieldBinding@@UEAAPEAXI@Z 0000000180021204     TmpCfg.obj
 0003:00000210       $pdata$??_GPluginRadioButtonBinding@@UEAAPEAXI@Z 0000000180021210     TmpCfg.obj
 0003:0000021c       $pdata$?AddButtons@?$DialogBuilderBase@UFarDialogItem@@@@QEAAXHPEBHHH@Z 000000018002121c     TmpCfg.obj
 0003:00000228       $pdata$4$?AddButtons@?$DialogBuilderBase@UFarDialogItem@@@@QEAAXHPEBHHH@Z 0000000180021228     TmpCfg.obj
 0003:00000234       $pdata$5$?AddButtons@?$DialogBuilderBase@UFarDialogItem@@@@QEAAXHPEBHHH@Z 0000000180021234     TmpCfg.obj
 0003:00000240       $pdata$?AddDialogItem@?$DialogBuilderBase@UFarDialogItem@@@@IEAAPEAUFarDialogItem@@W4FARDIALOGITEMTYPES@@PEB_W@Z 0000000180021240     TmpCfg.obj
 0003:0000024c       $pdata$?AddIntEditField@PluginDialogBuilder@@UEAAPEAUFarDialogItem@@PEAHH@Z 000000018002124c     TmpCfg.obj
 0003:00000258       $pdata$?AddUIntEditField@PluginDialogBuilder@@UEAAPEAUFarDialogItem@@PEAIH@Z 0000000180021258     TmpCfg.obj
 0003:00000264       $pdata$?Config@@YAHXZ      0000000180021264     TmpCfg.obj
 0003:00000270       $pdata$?CreateCheckBoxBinding@PluginDialogBuilder@@MEAAPEAU?$DialogItemBinding@UFarDialogItem@@@@PEAHH@Z 0000000180021270     TmpCfg.obj
 0003:0000027c       $pdata$?CreateRadioButtonBinding@PluginDialogBuilder@@MEAAPEAU?$DialogItemBinding@UFarDialogItem@@@@PEAH@Z 000000018002127c     TmpCfg.obj
 0003:00000288       $pdata$?DoShowDialog@PluginDialogBuilder@@MEAA_JXZ 0000000180021288     TmpCfg.obj
 0003:00000294       $pdata$?EndColumns@?$DialogBuilderBase@UFarDialogItem@@@@QEAAXXZ 0000000180021294     TmpCfg.obj
 0003:000002a0       $pdata$0$?EndColumns@?$DialogBuilderBase@UFarDialogItem@@@@QEAAXXZ 00000001800212a0     TmpCfg.obj
 0003:000002ac       $pdata$2$?EndColumns@?$DialogBuilderBase@UFarDialogItem@@@@QEAAXXZ 00000001800212ac     TmpCfg.obj
 0003:000002b8       $pdata$3$?EndColumns@?$DialogBuilderBase@UFarDialogItem@@@@QEAAXXZ 00000001800212b8     TmpCfg.obj
 0003:000002c4       $pdata$4$?EndColumns@?$DialogBuilderBase@UFarDialogItem@@@@QEAAXXZ 00000001800212c4     TmpCfg.obj
 0003:000002d0       $pdata$?GetOptions@@YAXXZ  00000001800212d0     TmpCfg.obj
 0003:000002dc       $pdata$?InitDialogItem@PluginDialogBuilder@@MEAAXPEAUFarDialogItem@@PEB_W@Z 00000001800212dc     TmpCfg.obj
 0003:000002e8       $pdata$?SaveValue@PluginCheckBoxBinding@@UEAAXPEAUFarDialogItem@@H@Z 00000001800212e8     TmpCfg.obj
 0003:000002f4       $pdata$?SaveValue@PluginEditFieldBinding@@UEAAXPEAUFarDialogItem@@H@Z 00000001800212f4     TmpCfg.obj
 0003:00000300       $pdata$?SaveValue@PluginIntEditFieldBinding@@UEAAXPEAUFarDialogItem@@H@Z 0000000180021300     TmpCfg.obj
 0003:0000030c       $pdata$?SaveValue@PluginRadioButtonBinding@@UEAAXPEAUFarDialogItem@@H@Z 000000018002130c     TmpCfg.obj
 0003:00000318       $pdata$?SaveValue@PluginUIntEditFieldBinding@@UEAAXPEAUFarDialogItem@@H@Z 0000000180021318     TmpCfg.obj
 0003:00000324       $pdata$?UpdateBorderSize@?$DialogBuilderBase@UFarDialogItem@@@@IEAAXXZ 0000000180021324     TmpCfg.obj
 0003:00000330       $pdata$1$?UpdateBorderSize@?$DialogBuilderBase@UFarDialogItem@@@@IEAAXXZ 0000000180021330     TmpCfg.obj
 0003:0000033c       $pdata$2$?UpdateBorderSize@?$DialogBuilderBase@UFarDialogItem@@@@IEAAXXZ 000000018002133c     TmpCfg.obj
 0003:00000348       $pdata$3$?UpdateBorderSize@?$DialogBuilderBase@UFarDialogItem@@@@IEAAXXZ 0000000180021348     TmpCfg.obj
 0003:00000354       $pdata$4$?UpdateBorderSize@?$DialogBuilderBase@UFarDialogItem@@@@IEAAXXZ 0000000180021354     TmpCfg.obj
 0003:00000360       $pdata$??0TmpPanel@@QEAA@PEB_W@Z 0000000180021360     TmpClass.obj
 0003:0000036c       $pdata$??1TmpPanel@@QEAA@XZ 000000018002136c     TmpClass.obj
 0003:00000378       $pdata$?BeginPutFiles@TmpPanel@@QEAAPEAXXZ 0000000180021378     TmpClass.obj
 0003:00000384       $pdata$?CommitPutFiles@TmpPanel@@QEAAXPEAXH@Z 0000000180021384     TmpClass.obj
 0003:00000390       $pdata$0$?CommitPutFiles@TmpPanel@@QEAAXPEAXH@Z 0000000180021390     TmpClass.obj
 0003:0000039c       $pdata$2$?CommitPutFiles@TmpPanel@@QEAAXPEAXH@Z 000000018002139c     TmpClass.obj
 0003:000003a8       $pdata$3$?CommitPutFiles@TmpPanel@@QEAAXPEAXH@Z 00000001800213a8     TmpClass.obj
 0003:000003b4       $pdata$4$?CommitPutFiles@TmpPanel@@QEAAXPEAXH@Z 00000001800213b4     TmpClass.obj
 0003:000003c0       $pdata$?GetFileInfoAndValidate@TmpPanel@@SA_NPEB_WPEAUPluginPanelItem@@H@Z 00000001800213c0     TmpClass.obj
 0003:000003cc       $pdata$?GetFindData@TmpPanel@@QEAAHPEAPEAUPluginPanelItem@@PEA_K_K@Z 00000001800213cc     TmpClass.obj
 0003:000003d8       $pdata$?GetOpenPanelInfo@TmpPanel@@QEAAXPEAUOpenPanelInfo@@@Z 00000001800213d8     TmpClass.obj
 0003:000003e4       $pdata$?Inflate@SimpleString@@QEAAX_K@Z 00000001800213e4     TmpClass.obj
 0003:000003f0       $pdata$?IsCurrentFileCorrect@TmpPanel@@AEAA_NPEAPEA_W@Z 00000001800213f0     TmpClass.obj
 0003:000003fc       $pdata$?ProcessEvent@TmpPanel@@QEAAH_JPEAX@Z 00000001800213fc     TmpClass.obj
 0003:00000408       $pdata$1$?ProcessEvent@TmpPanel@@QEAAH_JPEAX@Z 0000000180021408     TmpClass.obj
 0003:00000414       $pdata$2$?ProcessEvent@TmpPanel@@QEAAH_JPEAX@Z 0000000180021414     TmpClass.obj
 0003:00000420       $pdata$3$?ProcessEvent@TmpPanel@@QEAAH_JPEAX@Z 0000000180021420     TmpClass.obj
 0003:0000042c       $pdata$4$?ProcessEvent@TmpPanel@@QEAAH_JPEAX@Z 000000018002142c     TmpClass.obj
 0003:00000438       $pdata$?ProcessKey@TmpPanel@@QEAAHPEBU_INPUT_RECORD@@@Z 0000000180021438     TmpClass.obj
 0003:00000444       $pdata$0$?ProcessKey@TmpPanel@@QEAAHPEBU_INPUT_RECORD@@@Z 0000000180021444     TmpClass.obj
 0003:00000450       $pdata$1$?ProcessKey@TmpPanel@@QEAAHPEBU_INPUT_RECORD@@@Z 0000000180021450     TmpClass.obj
 0003:0000045c       $pdata$2$?ProcessKey@TmpPanel@@QEAAHPEBU_INPUT_RECORD@@@Z 000000018002145c     TmpClass.obj
 0003:00000468       $pdata$3$?ProcessKey@TmpPanel@@QEAAHPEBU_INPUT_RECORD@@@Z 0000000180021468     TmpClass.obj
 0003:00000474       $pdata$?ProcessSaveListKey@TmpPanel@@AEAAXXZ 0000000180021474     TmpClass.obj
 0003:00000480       $pdata$3$?ProcessSaveListKey@TmpPanel@@AEAAXXZ 0000000180021480     TmpClass.obj
 0003:0000048c       $pdata$4$?ProcessSaveListKey@TmpPanel@@AEAAXXZ 000000018002148c     TmpClass.obj
 0003:00000498       $pdata$5$?ProcessSaveListKey@TmpPanel@@AEAAXXZ 0000000180021498     TmpClass.obj
 0003:000004a4       $pdata$?PutDirectoryContents@TmpPanel@@QEAAHPEB_W@Z 00000001800214a4     TmpClass.obj
 0003:000004b0       $pdata$0$?PutDirectoryContents@TmpPanel@@QEAAHPEB_W@Z 00000001800214b0     TmpClass.obj
 0003:000004bc       $pdata$1$?PutDirectoryContents@TmpPanel@@QEAAHPEB_W@Z 00000001800214bc     TmpClass.obj
 0003:000004c8       $pdata$2$?PutDirectoryContents@TmpPanel@@QEAAHPEB_W@Z 00000001800214c8     TmpClass.obj
 0003:000004d4       $pdata$3$?PutDirectoryContents@TmpPanel@@QEAAHPEB_W@Z 00000001800214d4     TmpClass.obj
 0003:000004e0       $pdata$?PutFiles@TmpPanel@@QEAAHPEAUPluginPanelItem@@_KHPEB_W_K@Z 00000001800214e0     TmpClass.obj
 0003:000004ec       $pdata$?PutOneFile@TmpPanel@@QEAAHPEB_W@Z 00000001800214ec     TmpClass.obj
 0003:000004f8       $pdata$0$?PutOneFile@TmpPanel@@QEAAHPEB_W@Z 00000001800214f8     TmpClass.obj
 0003:00000504       $pdata$2$?PutOneFile@TmpPanel@@QEAAHPEB_W@Z 0000000180021504     TmpClass.obj
 0003:00000510       $pdata$?RemoveEmptyItems@TmpPanel@@AEAAXXZ 0000000180021510     TmpClass.obj
 0003:0000051c       $pdata$3$?RemoveEmptyItems@TmpPanel@@AEAAXXZ 000000018002151c     TmpClass.obj
 0003:00000528       $pdata$4$?RemoveEmptyItems@TmpPanel@@AEAAXXZ 0000000180021528     TmpClass.obj
 0003:00000534       $pdata$5$?RemoveEmptyItems@TmpPanel@@AEAAXXZ 0000000180021534     TmpClass.obj
 0003:00000540       $pdata$6$?RemoveEmptyItems@TmpPanel@@AEAAXXZ 0000000180021540     TmpClass.obj
 0003:0000054c       $pdata$?Replace@SimpleString@@QEAAAEAV1@_K0PEB_W0@Z 000000018002154c     TmpClass.obj
 0003:00000558       $pdata$1$?Replace@SimpleString@@QEAAAEAV1@_K0PEB_W0@Z 0000000180021558     TmpClass.obj
 0003:00000564       $pdata$2$?Replace@SimpleString@@QEAAAEAV1@_K0PEB_W0@Z 0000000180021564     TmpClass.obj
 0003:00000570       $pdata$3$?Replace@SimpleString@@QEAAAEAV1@_K0PEB_W0@Z 0000000180021570     TmpClass.obj
 0003:0000057c       $pdata$4$?Replace@SimpleString@@QEAAAEAV1@_K0PEB_W0@Z 000000018002157c     TmpClass.obj
 0003:00000588       $pdata$?SaveListFile@TmpPanel@@AEAAXPEB_W@Z 0000000180021588     TmpClass.obj
 0003:00000594       $pdata$1$?SaveListFile@TmpPanel@@AEAAXPEB_W@Z 0000000180021594     TmpClass.obj
 0003:000005a0       $pdata$5$?SaveListFile@TmpPanel@@AEAAXPEB_W@Z 00000001800215a0     TmpClass.obj
 0003:000005ac       $pdata$6$?SaveListFile@TmpPanel@@AEAAXPEB_W@Z 00000001800215ac     TmpClass.obj
 0003:000005b8       $pdata$7$?SaveListFile@TmpPanel@@AEAAXPEB_W@Z 00000001800215b8     TmpClass.obj
 0003:000005c4       $pdata$?SetDirectory@TmpPanel@@QEAAHPEB_W_K@Z 00000001800215c4     TmpClass.obj
 0003:000005d0       $pdata$?SetFindList@TmpPanel@@QEAAHPEBUPluginPanelItem@@_K@Z 00000001800215d0     TmpClass.obj
 0003:000005dc       $pdata$0$?SetFindList@TmpPanel@@QEAAHPEBUPluginPanelItem@@_K@Z 00000001800215dc     TmpClass.obj
 0003:000005e8       $pdata$1$?SetFindList@TmpPanel@@QEAAHPEBUPluginPanelItem@@_K@Z 00000001800215e8     TmpClass.obj
 0003:000005f4       $pdata$?SortListCmp@@YAHPEBX0PEAX@Z 00000001800215f4     TmpClass.obj
 0003:00000600       $pdata$?SwitchToPanel@TmpPanel@@AEAAXH@Z 0000000180021600     TmpClass.obj
 0003:0000060c       $pdata$0$?SwitchToPanel@TmpPanel@@AEAAXH@Z 000000018002160c     TmpClass.obj
 0003:00000618       $pdata$1$?SwitchToPanel@TmpPanel@@AEAAXH@Z 0000000180021618     TmpClass.obj
 0003:00000624       $pdata$?UpdateItems@TmpPanel@@AEAAXHH@Z 0000000180021624     TmpClass.obj
 0003:00000630       $pdata$2$?UpdateItems@TmpPanel@@AEAAXHH@Z 0000000180021630     TmpClass.obj
 0003:0000063c       $pdata$3$?UpdateItems@TmpPanel@@AEAAXHH@Z 000000018002163c     TmpClass.obj
 0003:00000648       $pdata$4$?UpdateItems@TmpPanel@@AEAAXHH@Z 0000000180021648     TmpClass.obj
 0003:00000654       $pdata$5$?UpdateItems@TmpPanel@@AEAAXHH@Z 0000000180021654     TmpClass.obj
 0003:00000660       $pdata$?ExpandEnvStrs@@YAPEA_WPEB_WAEAVStrBuf@@@Z 0000000180021660     TmpMix.obj
 0003:0000066c       $pdata$?FindListFile@@YA_NPEB_WAEAVStrBuf@@@Z 000000018002166c     TmpMix.obj
 0003:00000678       $pdata$?FormNtPath@@YAPEA_WPEB_WAEAVStrBuf@@@Z 0000000180021678     TmpMix.obj
 0003:00000684       $pdata$1$?FormNtPath@@YAPEA_WPEB_WAEAVStrBuf@@@Z 0000000180021684     TmpMix.obj
 0003:00000690       $pdata$2$?FormNtPath@@YAPEA_WPEB_WAEAVStrBuf@@@Z 0000000180021690     TmpMix.obj
 0003:0000069c       $pdata$?FreePanelItems@@YAXPEAUPluginPanelItem@@_K@Z 000000018002169c     TmpMix.obj
 0003:000006a8       $pdata$0$?FreePanelItems@@YAXPEAUPluginPanelItem@@_K@Z 00000001800216a8     TmpMix.obj
 0003:000006b4       $pdata$1$?FreePanelItems@@YAXPEAUPluginPanelItem@@_K@Z 00000001800216b4     TmpMix.obj
 0003:000006c0       $pdata$?GetFullPath@@YAPEA_WPEB_WAEAVStrBuf@@@Z 00000001800216c0     TmpMix.obj
 0003:000006cc       $pdata$?GoToFile@@YAXPEB_WH@Z 00000001800216cc     TmpMix.obj
 0003:000006d8       $pdata$?Grow@StrBuf@@QEAAX_K@Z 00000001800216d8     TmpMix.obj
 0003:000006e4       $pdata$?IsTextUTF8@@YA_NPEBD_K@Z 00000001800216e4     TmpMix.obj
 0003:000006f0       $pdata$?ParseParam@@YAPEA_WAEAPEA_W@Z 00000001800216f0     TmpMix.obj
 0003:000006fc       $pdata$?WFD2FFD@@YAXAEAU_WIN32_FIND_DATAW@@AEAUPluginPanelItem@@@Z 00000001800216fc     TmpMix.obj
 0003:00000708       $pdata$??2@YAPEAX_K@Z      0000000180021708     LIBCMT:new_scalar.obj
 0003:00000714       $pdata$?dllmain_crt_dispatch@@YAHQEAUHINSTANCE__@@KQEAX@Z 0000000180021714     LIBCMT:dll_dllmain.obj
 0003:00000720       $pdata$?dllmain_crt_process_attach@@YAHQEAUHINSTANCE__@@QEAX@Z 0000000180021720     LIBCMT:dll_dllmain.obj
 0003:0000072c       $pdata$?dllmain_crt_process_detach@@YAH_N@Z 000000018002172c     LIBCMT:dll_dllmain.obj
 0003:00000738       $pdata$?dllmain_dispatch@@YAHQEAUHINSTANCE__@@KQEAX@Z 0000000180021738     LIBCMT:dll_dllmain.obj
 0003:00000744       $pdata$_DllMainCRTStartup  0000000180021744     LIBCMT:dll_dllmain.obj
 0003:00000750       $pdata$??0bad_alloc@std@@QEAA@AEBV01@@Z 0000000180021750     LIBCMT:throw_bad_alloc.obj
 0003:0000075c       $pdata$??0bad_array_new_length@std@@QEAA@AEBV01@@Z 000000018002175c     LIBCMT:throw_bad_alloc.obj
 0003:00000768       $pdata$??0exception@std@@QEAA@AEBV01@@Z 0000000180021768     LIBCMT:throw_bad_alloc.obj
 0003:00000774       $pdata$??_Gexception@std@@UEAAPEAXI@Z 0000000180021774     LIBCMT:throw_bad_alloc.obj
 0003:00000774       $pdata$??_Gbad_array_new_length@std@@UEAAPEAXI@Z 0000000180021774     LIBCMT:throw_bad_alloc.obj
 0003:00000774       $pdata$??_Gbad_alloc@std@@UEAAPEAXI@Z 0000000180021774     LIBCMT:throw_bad_alloc.obj
 0003:00000780       $pdata$?__scrt_throw_std_bad_alloc@@YAXXZ 0000000180021780     LIBCMT:throw_bad_alloc.obj
 0003:0000078c       $pdata$?__scrt_throw_std_bad_array_new_length@@YAXXZ 000000018002178c     LIBCMT:throw_bad_alloc.obj
 0003:00000798       $pdata$__security_init_cookie 0000000180021798     LIBCMT:gs_support.obj
 0003:000007a4       $pdata$__scrt_initialize_default_local_stdio_options 00000001800217a4     LIBCMT:default_local_stdio_options.obj
 0003:000007b0       $pdata$__scrt_acquire_startup_lock 00000001800217b0     LIBCMT:utility.obj
 0003:000007bc       $pdata$__scrt_dllmain_after_initialize_c 00000001800217bc     LIBCMT:utility.obj
 0003:000007c8       $pdata$__scrt_dllmain_before_initialize_c 00000001800217c8     LIBCMT:utility.obj
 0003:000007d4       $pdata$__scrt_dllmain_crt_thread_attach 00000001800217d4     LIBCMT:utility.obj
 0003:000007e0       $pdata$__scrt_dllmain_crt_thread_detach 00000001800217e0     LIBCMT:utility.obj
 0003:000007ec       $pdata$__scrt_dllmain_exception_filter 00000001800217ec     LIBCMT:utility.obj
 0003:000007f8       $pdata$__scrt_dllmain_uninitialize_c 00000001800217f8     LIBCMT:utility.obj
 0003:00000804       $pdata$__scrt_dllmain_uninitialize_critical 0000000180021804     LIBCMT:utility.obj
 0003:00000810       $pdata$__scrt_initialize_crt 0000000180021810     LIBCMT:utility.obj
 0003:0000081c       $pdata$__scrt_initialize_onexit_tables 000000018002181c     LIBCMT:utility.obj
 0003:00000828       $pdata$__scrt_is_nonwritable_in_current_image 0000000180021828     LIBCMT:utility.obj
 0003:00000834       $pdata$__scrt_release_startup_lock 0000000180021834     LIBCMT:utility.obj
 0003:00000840       $pdata$__scrt_uninitialize_crt 0000000180021840     LIBCMT:utility.obj
 0003:0000084c       $pdata$__scrt_fastfail     000000018002184c     LIBCMT:utility_desktop.obj
 0003:00000858       $pdata$_RTC_Initialize     0000000180021858     LIBCMT:initsect.obj
 0003:00000864       $pdata$_RTC_Terminate      0000000180021864     LIBCMT:initsect.obj
 0003:00000870       $pdata$??_Gtype_info@@UEAAPEAXI@Z 0000000180021870     LIBCMT:std_type_info_static.obj
 0003:0000087c       $pdata$__isa_available_init 000000018002187c     LIBCMT:cpu_disp.obj
 0003:000008b8       $pdata$wcschr              00000001800218b8     libvcruntime:wcschr.obj
 0003:000008d0       $pdata$__C_specific_handler 00000001800218d0     libvcruntime:riscchandler.obj
 0003:000008dc       $pdata$__std_exception_copy 00000001800218dc     libvcruntime:std_exception.obj
 0003:000008e8       $pdata$__std_exception_destroy 00000001800218e8     libvcruntime:std_exception.obj
 0003:000008f4       $pdata$_CxxThrowException  00000001800218f4     libvcruntime:throw.obj
 0003:00000900       $pdata$__std_type_info_destroy_list 0000000180021900     libvcruntime:std_type_info.obj
 0003:0000090c       $pdata$__vcrt_initialize   000000018002190c     libvcruntime:initialization.obj
 0003:00000918       $pdata$__vcrt_thread_attach 0000000180021918     libvcruntime:initialization.obj
 0003:00000924       $pdata$__vcrt_thread_detach 0000000180021924     libvcruntime:initialization.obj
 0003:00000930       $pdata$__vcrt_uninitialize 0000000180021930     libvcruntime:initialization.obj
 0003:0000093c       $pdata$__vcrt_uninitialize_critical 000000018002193c     libvcruntime:initialization.obj
 0003:0000096c       $pdata$__DestructExceptionObject 000000018002196c     libvcruntime:ehhelpers.obj
 0003:00000978       $pdata$__vcrt_freefls      0000000180021978     libvcruntime:per_thread_data.obj
 0003:00000984       $pdata$__vcrt_freeptd      0000000180021984     libvcruntime:per_thread_data.obj
 0003:00000990       $pdata$__vcrt_getptd_noexit 0000000180021990     libvcruntime:per_thread_data.obj
 0003:0000099c       $pdata$__vcrt_initialize_ptd 000000018002199c     libvcruntime:per_thread_data.obj
 0003:000009a8       $pdata$__vcrt_uninitialize_ptd 00000001800219a8     libvcruntime:per_thread_data.obj
 0003:000009b4       $pdata$__vcrt_initialize_locks 00000001800219b4     libvcruntime:locks.obj
 0003:000009c0       $pdata$__vcrt_uninitialize_locks 00000001800219c0     libvcruntime:locks.obj
 0003:000009cc       $pdata$?try_get_function@@YAPEAXW4function_id@?A0xbfd18cd1@@QEBDQEBW4module_id@2@2@Z 00000001800219cc     libvcruntime:winapi_downlevel.obj
 0003:000009d8       $pdata$__vcrt_FlsAlloc     00000001800219d8     libvcruntime:winapi_downlevel.obj
 0003:000009e4       $pdata$__vcrt_FlsFree      00000001800219e4     libvcruntime:winapi_downlevel.obj
 0003:000009f0       $pdata$__vcrt_FlsGetValue  00000001800219f0     libvcruntime:winapi_downlevel.obj
 0003:000009fc       $pdata$__vcrt_FlsSetValue  00000001800219fc     libvcruntime:winapi_downlevel.obj
 0003:00000a08       $pdata$__vcrt_InitializeCriticalSectionEx 0000000180021a08     libvcruntime:winapi_downlevel.obj
 0003:00000a14       $pdata$__vcrt_initialize_winapi_thunks 0000000180021a14     libvcruntime:winapi_downlevel.obj
 0003:00000a20       $pdata$__vcrt_uninitialize_winapi_thunks 0000000180021a20     libvcruntime:winapi_downlevel.obj
 0003:00000a44       $pdata$_callnewh           0000000180021a44     libucrt:new_handler.obj
 0003:00000a50       $pdata$_query_new_handler  0000000180021a50     libucrt:new_handler.obj
 0003:00000a5c       $pdata$_initterm           0000000180021a5c     libucrt:initterm.obj
 0003:00000a68       $pdata$_initterm_e         0000000180021a68     libucrt:initterm.obj
 0003:00000a74       $pdata$_seh_filter_exe     0000000180021a74     libucrt:exception_filter.obj
 0003:00000a80       $pdata$??$?RV<lambda_d80eeec6fff315bfe5c115232f3240e3>@@AEAV<lambda_6e4b09c48022b2350581041d5f6b0c4c>@@V<lambda_2358e3775559c9db80273638284d5e45>@@@?$__crt_seh_guarded_call@X@@QEAAX$$QEAV<lambda_d80eeec6fff315bfe5c115232f3240e3>@@AEAV<lambda_6e4b09c48022b2350581041d5f6b0c4c>@@$$QEAV<lambda_2358e3775559c9db80273638284d5e45>@@@Z 0000000180021a80     libucrt:exit.obj
 0003:00000a8c       $pdata$??R<lambda_6e4b09c48022b2350581041d5f6b0c4c>@@QEBA@XZ 0000000180021a8c     libucrt:exit.obj
 0003:00000a98       $pdata$?common_exit@@YAXHW4_crt_exit_cleanup_mode@@W4_crt_exit_return_mode@@@Z 0000000180021a98     libucrt:exit.obj
 0003:00000aa4       $pdata$?exit_or_terminate_process@@YAXI@Z 0000000180021aa4     libucrt:exit.obj
 0003:00000ab0       $pdata$?try_cor_exit_process@@YAXI@Z 0000000180021ab0     libucrt:exit.obj
 0003:00000abc       $pdata$??$parse_command_line@D@@YAXPEADPEAPEAD0PEA_K2@Z 0000000180021abc     libucrt:argv_parsing.obj
 0003:00000ac8       $pdata$__acrt_allocate_buffer_for_argv 0000000180021ac8     libucrt:argv_parsing.obj
 0003:00000ad4       $pdata$_configure_narrow_argv 0000000180021ad4     libucrt:argv_parsing.obj
 0003:00000ae0       $pdata$??$common_initialize_environment_nolock@D@@YAHXZ 0000000180021ae0     libucrt:environment_initialization.obj
 0003:00000aec       $pdata$??$create_environment@D@@YAQEAPEADQEAD@Z 0000000180021aec     libucrt:environment_initialization.obj
 0003:00000af8       $pdata$??$free_environment@_W@@YAXQEAPEA_W@Z 0000000180021af8     libucrt:environment_initialization.obj
 0003:00000af8       $pdata$??$free_environment@D@@YAXQEAPEAD@Z 0000000180021af8     libucrt:environment_initialization.obj
 0003:00000b04       $pdata$??$uninitialize_environment_internal@D@@YAXAEAPEAPEAD@Z 0000000180021b04     libucrt:environment_initialization.obj
 0003:00000b10       $pdata$??$uninitialize_environment_internal@_W@@YAXAEAPEAPEA_W@Z 0000000180021b10     libucrt:environment_initialization.obj
 0003:00000b1c       $pdata$__dcrt_uninitialize_environments_nolock 0000000180021b1c     libucrt:environment_initialization.obj
 0003:00000b28       $pdata$??$?RV<lambda_7777bce6b2f8c936911f934f8298dc43>@@AEAV<lambda_f03950bc5685219e0bcd2087efbe011e>@@V<lambda_3883c3dff614d5e0c5f61bb1ac94921c>@@@?$__crt_seh_guarded_call@H@@QEAAH$$QEAV<lambda_7777bce6b2f8c936911f934f8298dc43>@@AEAV<lambda_f03950bc5685219e0bcd2087efbe011e>@@$$QEAV<lambda_3883c3dff614d5e0c5f61bb1ac94921c>@@@Z 0000000180021b28     libucrt:onexit.obj
 0003:00000b34       $pdata$??R<lambda_f03950bc5685219e0bcd2087efbe011e>@@QEBAHXZ 0000000180021b34     libucrt:onexit.obj
 0003:00000b40       $pdata$_execute_onexit_table 0000000180021b40     libucrt:onexit.obj
 0003:00000b4c       $pdata$initialize_c        0000000180021b4c     libucrt:initialization.obj
 0003:00000b58       $pdata$uninitialize_environment 0000000180021b58     libucrt:initialization.obj
 0003:00000b64       $pdata$initialize_pointers 0000000180021b64     libucrt:initialization.obj
 0003:00000b70       $pdata$uninitialize_allocated_memory 0000000180021b70     libucrt:initialization.obj
 0003:00000b7c       $pdata$uninitialize_allocated_io_buffers 0000000180021b7c     libucrt:initialization.obj
 0003:00000b88       $pdata$__acrt_thread_attach 0000000180021b88     libucrt:initialization.obj
 0003:00000b94       $pdata$__acrt_thread_detach 0000000180021b94     libucrt:initialization.obj
 0003:00000ba0       $pdata$__acrt_uninitialize 0000000180021ba0     libucrt:initialization.obj
 0003:00000bac       $pdata$__acrt_uninitialize_critical 0000000180021bac     libucrt:initialization.obj
 0003:00000bb8       $pdata$terminate           0000000180021bb8     libucrt:terminate.obj
 0003:00000bc4       $pdata$_wcsdup             0000000180021bc4     libucrt:wcsdup.obj
 0003:00000bd0       $pdata$strcpy_s            0000000180021bd0     libucrt:strcpy_s.obj
 0003:00000bdc       $pdata$??0_LocaleUpdate@@QEAA@QEAU__crt_locale_pointers@@@Z 0000000180021bdc     libucrt:output.obj
 0003:00000bf4       $pdata$abort               0000000180021bf4     libucrt:abort.obj
 0003:00000c00       $pdata$_calloc_base        0000000180021c00     libucrt:calloc_base.obj
 0003:00000c0c       $pdata$_free_base          0000000180021c0c     libucrt:free_base.obj
 0003:00000c18       $pdata$_malloc_base        0000000180021c18     libucrt:malloc_base.obj
 0003:00000c24       $pdata$_realloc_base       0000000180021c24     libucrt:realloc_base.obj
 0003:00000c30       $pdata$__acrt_initialize_locks 0000000180021c30     libucrt:locks.obj
 0003:00000c3c       $pdata$__acrt_uninitialize_locks 0000000180021c3c     libucrt:locks.obj
 0003:00000c48       $pdata$??$?RV<lambda_0ae27a3a962d80f24befdcbee591983d>@@AEAV<lambda_8d0ee55de4b1038c4002e0adecdf1839>@@V<lambda_dc504788e8f1664fe9b84e20bfb512f2>@@@?$__crt_seh_guarded_call@X@@QEAAX$$QEAV<lambda_0ae27a3a962d80f24befdcbee591983d>@@AEAV<lambda_8d0ee55de4b1038c4002e0adecdf1839>@@$$QEAV<lambda_dc504788e8f1664fe9b84e20bfb512f2>@@@Z 0000000180021c48     libucrt:per_thread_data.obj
 0003:00000c54       $pdata$??$?RV<lambda_2d41944a1d46af3157314b8a01080d33>@@AEAV<lambda_8f455de75cd7d7f24b4096f044d8b9e6>@@V<lambda_aa500f224e6afead328df44964fe2772>@@@?$__crt_seh_guarded_call@X@@QEAAX$$QEAV<lambda_2d41944a1d46af3157314b8a01080d33>@@AEAV<lambda_8f455de75cd7d7f24b4096f044d8b9e6>@@$$QEAV<lambda_aa500f224e6afead328df44964fe2772>@@@Z 0000000180021c54     libucrt:per_thread_data.obj
 0003:00000c60       $pdata$??$?RV<lambda_aa87e3671a710a21b5dc78c0bdf72e11>@@AEAV<lambda_92619d2358a28f41a33ba319515a20b9>@@V<lambda_6992ecaafeb10aed2b74cb1fae11a551>@@@?$__crt_seh_guarded_call@X@@QEAAX$$QEAV<lambda_aa87e3671a710a21b5dc78c0bdf72e11>@@AEAV<lambda_92619d2358a28f41a33ba319515a20b9>@@$$QEAV<lambda_6992ecaafeb10aed2b74cb1fae11a551>@@@Z 0000000180021c60     libucrt:per_thread_data.obj
 0003:00000c6c       $pdata$??$?RV<lambda_f2e299630e499de9f9a165e60fcd3db5>@@AEAV<lambda_2ae9d31cdba2644fcbeaf08da7c24588>@@V<lambda_40d01ff24d0e7b3814fdbdcee8eab3c7>@@@?$__crt_seh_guarded_call@X@@QEAAX$$QEAV<lambda_f2e299630e499de9f9a165e60fcd3db5>@@AEAV<lambda_2ae9d31cdba2644fcbeaf08da7c24588>@@$$QEAV<lambda_40d01ff24d0e7b3814fdbdcee8eab3c7>@@@Z 0000000180021c6c     libucrt:per_thread_data.obj
 0003:00000c78       $pdata$?construct_ptd_array@@YAXQEAU__acrt_ptd@@@Z 0000000180021c78     libucrt:per_thread_data.obj
 0003:00000c84       $pdata$?destroy_fls@@YAXPEAX@Z 0000000180021c84     libucrt:per_thread_data.obj
 0003:00000c90       $pdata$?destroy_ptd_array@@YAXQEAU__acrt_ptd@@@Z 0000000180021c90     libucrt:per_thread_data.obj
 0003:00000c9c       $pdata$?replace_current_thread_locale_nolock@@YAXQEAU__acrt_ptd@@QEAU__crt_locale_data@@@Z 0000000180021c9c     libucrt:per_thread_data.obj
 0003:00000ca8       $pdata$__acrt_freeptd      0000000180021ca8     libucrt:per_thread_data.obj
 0003:00000cb4       $pdata$__acrt_getptd       0000000180021cb4     libucrt:per_thread_data.obj
 0003:00000cc0       $pdata$__acrt_getptd_head  0000000180021cc0     libucrt:per_thread_data.obj
 0003:00000ccc       $pdata$__acrt_getptd_noexit 0000000180021ccc     libucrt:per_thread_data.obj
 0003:00000cd8       $pdata$__acrt_initialize_ptd 0000000180021cd8     libucrt:per_thread_data.obj
 0003:00000ce4       $pdata$__acrt_uninitialize_ptd 0000000180021ce4     libucrt:per_thread_data.obj
 0003:00000cf0       $pdata$__acrt_get_process_end_policy 0000000180021cf0     libucrt:win_policies.obj
 0003:00000cfc       $pdata$__acrt_call_reportfault 0000000180021cfc     libucrt:invalid_parameter.obj
 0003:00000d08       $pdata$_invalid_parameter  0000000180021d08     libucrt:invalid_parameter.obj
 0003:00000d14       $pdata$_invalid_parameter_noinfo 0000000180021d14     libucrt:invalid_parameter.obj
 0003:00000d20       $pdata$_invoke_watson      0000000180021d20     libucrt:invalid_parameter.obj
 0003:00000d2c       $pdata$__acrt_errno_map_os_error 0000000180021d2c     libucrt:errno.obj
 0003:00000d38       $pdata$__doserrno          0000000180021d38     libucrt:errno.obj
 0003:00000d44       $pdata$_errno              0000000180021d44     libucrt:errno.obj
 0003:00000d50       $pdata$??$__acrt_mbs_to_wcs_cp@U__crt_win32_buffer_internal_dynamic_resizing@@@@YAHQEBDAEAV?$__crt_win32_buffer@_WU__crt_win32_buffer_internal_dynamic_resizing@@@@I@Z 0000000180021d50     libucrt:argv_wildcards.obj
 0003:00000d5c       $pdata$??$__acrt_wcs_to_mbs_cp@U__crt_win32_buffer_internal_dynamic_resizing@@@@YAHQEB_WAEAV?$__crt_win32_buffer@DU__crt_win32_buffer_internal_dynamic_resizing@@@@I@Z 0000000180021d5c     libucrt:argv_wildcards.obj
 0003:00000d68       $pdata$??$common_expand_argv_wildcards@D@@YAHQEAPEADQEAPEAPEAD@Z 0000000180021d68     libucrt:argv_wildcards.obj
 0003:00000d74       $pdata$??$copy_and_add_argument_to_buffer@D@@YAHQEBD0_KAEAV?$argument_list@D@?A0x5f5c8891@@@Z 0000000180021d74     libucrt:argv_wildcards.obj
 0003:00000d80       $pdata$??$expand_argument_wildcards@D@@YAHQEAD0AEAV?$argument_list@D@?A0x5f5c8891@@@Z 0000000180021d80     libucrt:argv_wildcards.obj
 0003:00000d8c       $pdata$??$__acrt_wcs_to_mbs_cp@U__crt_win32_buffer_no_resizing@@@@YAHQEB_WAEAV?$__crt_win32_buffer@DU__crt_win32_buffer_no_resizing@@@@I@Z 0000000180021d8c     libucrt:getmodulefilenamea.obj
 0003:00000d98       $pdata$__acrt_GetModuleFileNameA 0000000180021d98     libucrt:getmodulefilenamea.obj
 0003:00000da4       $pdata$??$?RV<lambda_efdfa57d1f175319df784efa44bb7b81>@@AEAV<lambda_5f0a4c1567f8adc6734073e5d1e1b35c>@@V<lambda_2e8a7d3640ea6ccb4c2413664c2db6fd>@@@?$__crt_seh_guarded_call@X@@QEAAX$$QEAV<lambda_efdfa57d1f175319df784efa44bb7b81>@@AEAV<lambda_5f0a4c1567f8adc6734073e5d1e1b35c>@@$$QEAV<lambda_2e8a7d3640ea6ccb4c2413664c2db6fd>@@@Z 0000000180021da4     libucrt:mbctype.obj
 0003:00000db0       $pdata$?getSystemCP@@YAHH@Z 0000000180021db0     libucrt:mbctype.obj
 0003:00000dbc       $pdata$?setSBCS@@YAXPEAU__crt_multibyte_data@@@Z 0000000180021dbc     libucrt:mbctype.obj
 0003:00000dc8       $pdata$?setSBUpLow@@YAXPEAU__crt_multibyte_data@@@Z 0000000180021dc8     libucrt:mbctype.obj
 0003:00000dd4       $pdata$?setmbcp_internal@@YAHH_NQEAU__acrt_ptd@@QEAPEAU__crt_multibyte_data@@@Z 0000000180021dd4     libucrt:mbctype.obj
 0003:00000de0       $pdata$?update_thread_multibyte_data_internal@@YAPEAU__crt_multibyte_data@@QEAU__acrt_ptd@@QEAPEAU1@@Z 0000000180021de0     libucrt:mbctype.obj
 0003:00000dec       $pdata$__acrt_initialize_multibyte 0000000180021dec     libucrt:mbctype.obj
 0003:00000df8       $pdata$__acrt_update_thread_multibyte_data 0000000180021df8     libucrt:mbctype.obj
 0003:00000e04       $pdata$_setmbcp_nolock     0000000180021e04     libucrt:mbctype.obj
 0003:00000e10       $pdata$?x_ismbbtype_l@@YAHPEAU__crt_locale_pointers@@IHH@Z 0000000180021e10     libucrt:ismbbyte.obj
 0003:00000e1c       $pdata$__acrt_initialize_command_line 0000000180021e1c     libucrt:argv_data.obj
 0003:00000e28       $pdata$wcscpy_s            0000000180021e28     libucrt:wcscpy_s.obj
 0003:00000e34       $pdata$__acrt_WideCharToMultiByte 0000000180021e34     libucrt:widechartomultibyte.obj
 0003:00000e40       $pdata$__dcrt_get_narrow_environment_from_os 0000000180021e40     libucrt:get_environment_from_os.obj
 0003:00000e4c       $pdata$_recalloc_base      0000000180021e4c     libucrt:recalloc.obj
 0003:00000e58       $pdata$?try_get_function@@YAPEAXW4function_id@?A0x391cf84c@@QEBDQEBW4module_id@2@2@Z 0000000180021e58     libucrt:winapi_thunks.obj
 0003:00000e64       $pdata$__acrt_AppPolicyGetProcessTerminationMethodInternal 0000000180021e64     libucrt:winapi_thunks.obj
 0003:00000e70       $pdata$__acrt_AreFileApisANSI 0000000180021e70     libucrt:winapi_thunks.obj
 0003:00000e7c       $pdata$__acrt_FlsAlloc     0000000180021e7c     libucrt:winapi_thunks.obj
 0003:00000e88       $pdata$__acrt_FlsFree      0000000180021e88     libucrt:winapi_thunks.obj
 0003:00000e94       $pdata$__acrt_FlsGetValue  0000000180021e94     libucrt:winapi_thunks.obj
 0003:00000ea0       $pdata$__acrt_FlsSetValue  0000000180021ea0     libucrt:winapi_thunks.obj
 0003:00000eac       $pdata$__acrt_InitializeCriticalSectionEx 0000000180021eac     libucrt:winapi_thunks.obj
 0003:00000eb8       $pdata$__acrt_LCMapStringEx 0000000180021eb8     libucrt:winapi_thunks.obj
 0003:00000ec4       $pdata$__acrt_LocaleNameToLCID 0000000180021ec4     libucrt:winapi_thunks.obj
 0003:00000ed0       $pdata$__acrt_initialize_winapi_thunks 0000000180021ed0     libucrt:winapi_thunks.obj
 0003:00000edc       $pdata$__acrt_uninitialize_winapi_thunks 0000000180021edc     libucrt:winapi_thunks.obj
 0003:00000ee8       $pdata$__acrt_initialize_heap 0000000180021ee8     libucrt:heap_handle.obj
 0003:00000ef4       $pdata$?initialize_inherited_file_handles_nolock@@YAXXZ 0000000180021ef4     libucrt:ioinit.obj
 0003:00000f00       $pdata$?initialize_stdio_handles_nolock@@YAXXZ 0000000180021f00     libucrt:ioinit.obj
 0003:00000f0c       $pdata$__acrt_initialize_lowio 0000000180021f0c     libucrt:ioinit.obj
 0003:00000f18       $pdata$__acrt_uninitialize_lowio 0000000180021f18     libucrt:ioinit.obj
 0003:00000f24       $pdata$__acrt_execute_initializers 0000000180021f24     libucrt:shared_initialization.obj
 0003:00000f30       $pdata$__acrt_execute_uninitializers 0000000180021f30     libucrt:shared_initialization.obj
 0003:00000f3c       $pdata$??$?RV<lambda_450d765d439847d4c735a33c368b5fc0>@@AEAV<lambda_44731a7d0e6d81c3e6aa82d741081786>@@V<lambda_601a2a7da3b7a96e9554ac7215c4b07c>@@@?$__crt_seh_guarded_call@P6AXH@Z@@QEAAP6AXH@Z$$QEAV<lambda_450d765d439847d4c735a33c368b5fc0>@@AEAV<lambda_44731a7d0e6d81c3e6aa82d741081786>@@$$QEAV<lambda_601a2a7da3b7a96e9554ac7215c4b07c>@@@Z 0000000180021f3c     libucrt:signal.obj
 0003:00000f48       $pdata$__acrt_get_sigabrt_handler 0000000180021f48     libucrt:signal.obj
 0003:00000f54       $pdata$raise               0000000180021f54     libucrt:signal.obj
 0003:00000f60       $pdata$??$?RV<lambda_842d9ff0dc9ef11c61343bbaebe7f885>@@AEAV<lambda_c5860995281e5c4ce005b3de8f5874ee>@@V<lambda_d90129c13df834fdcbf8d2b88dafcf2d>@@@?$__crt_seh_guarded_call@X@@QEAAX$$QEAV<lambda_842d9ff0dc9ef11c61343bbaebe7f885>@@AEAV<lambda_c5860995281e5c4ce005b3de8f5874ee>@@$$QEAV<lambda_d90129c13df834fdcbf8d2b88dafcf2d>@@@Z 0000000180021f60     libucrt:fflush.obj
 0003:00000f6c       $pdata$??$?RV<lambda_886d6c58226a84441f68b9f2b8217b83>@@AEAV<lambda_ab61a845afdef5b7c387490eaf3616ee>@@V<lambda_f7f22ab5edc0698d5f6905b0d3f44752>@@@?$__crt_seh_guarded_call@X@@QEAAX$$QEAV<lambda_886d6c58226a84441f68b9f2b8217b83>@@AEAV<lambda_ab61a845afdef5b7c387490eaf3616ee>@@$$QEAV<lambda_f7f22ab5edc0698d5f6905b0d3f44752>@@@Z 0000000180021f6c     libucrt:fflush.obj
 0003:00000f78       $pdata$?common_flush_all@@YAH_N@Z 0000000180021f78     libucrt:fflush.obj
 0003:00000f84       $pdata$__acrt_stdio_flush_nolock 0000000180021f84     libucrt:fflush.obj
 0003:00000f90       $pdata$_fflush_nolock      0000000180021f90     libucrt:fflush.obj
 0003:00000f9c       $pdata$__acrt_initialize_stdio 0000000180021f9c     libucrt:_file.obj
 0003:00000fa8       $pdata$__acrt_uninitialize_stdio 0000000180021fa8     libucrt:_file.obj
 0003:00000fb4       $pdata$_mbtowc_l           0000000180021fb4     libucrt:mbtowc.obj
 0003:00000fc0       $pdata$__acrt_update_locale_info 0000000180021fc0     libucrt:locale_update.obj
 0003:00000fcc       $pdata$__acrt_update_multibyte_info 0000000180021fcc     libucrt:locale_update.obj
 0003:00000fd8       $pdata$_fileno             0000000180021fd8     libucrt:fileno.obj
 0003:00000fe4       $pdata$??$?RV<lambda_410d79af7f07d98d83a3f525b3859a53>@@AEAV<lambda_3e16ef9562a7dcce91392c22ab16ea36>@@V<lambda_38119f0e861e05405d8a144b9b982f0a>@@@?$__crt_seh_guarded_call@X@@QEAAX$$QEAV<lambda_410d79af7f07d98d83a3f525b3859a53>@@AEAV<lambda_3e16ef9562a7dcce91392c22ab16ea36>@@$$QEAV<lambda_38119f0e861e05405d8a144b9b982f0a>@@@Z 0000000180021fe4     libucrt:wsetlocale.obj
 0003:00000ff0       $pdata$__acrt_uninitialize_locale 0000000180021ff0     libucrt:wsetlocale.obj
 0003:00000ffc       $pdata$__pctype_func       0000000180021ffc     libucrt:ctype.obj
 0003:00001008       $pdata$__acrt_free_locale  0000000180022008     libucrt:locale_refcounting.obj
 0003:00001014       $pdata$__acrt_locale_free_lc_time_if_unreferenced 0000000180022014     libucrt:locale_refcounting.obj
 0003:00001020       $pdata$__acrt_release_locale_ref 0000000180022020     libucrt:locale_refcounting.obj
 0003:0000102c       $pdata$__acrt_update_thread_locale_data 000000018002202c     libucrt:locale_refcounting.obj
 0003:00001038       $pdata$_updatetlocinfoEx_nolock 0000000180022038     libucrt:locale_refcounting.obj
 0003:00001044       $pdata$qsort               0000000180022044     libucrt:qsort.obj
 0003:00001050       $pdata$4$qsort             0000000180022050     libucrt:qsort.obj
 0003:0000105c       $pdata$5$qsort             000000018002205c     libucrt:qsort.obj
 0003:00001068       $pdata$strncpy_s           0000000180022068     libucrt:strncpy_s.obj
 0003:00001074       $pdata$fallbackMethod      0000000180022074     libucrt:strpbrk.obj
 0003:00001080       $pdata$strpbrk             0000000180022080     libucrt:strpbrk.obj
 0003:0000108c       $pdata$_mbsdec_l           000000018002208c     libucrt:mbsdec.obj
 0003:00001098       $pdata$__acrt_GetStringTypeA 0000000180022098     libucrt:getstringtypea.obj
 0003:000010a4       $pdata$?__acrt_LCMapStringA_stat@@YAHPEAU__crt_locale_pointers@@PEB_WKPEBDHPEADHHH@Z 00000001800220a4     libucrt:lcmapstringa.obj
 0003:000010b0       $pdata$__acrt_LCMapStringA 00000001800220b0     libucrt:lcmapstringa.obj
 0003:000010bc       $pdata$?initialize_multibyte@@YAHXZ 00000001800220bc     libucrt:multibyte_initializer.obj
 0003:000010c8       $pdata$_msize_base         00000001800220c8     libucrt:msize.obj
 0003:000010d4       $pdata$?GetTableIndexFromLocaleName@@YAHPEB_W@Z 00000001800220d4     libucrt:lcidtoname_downlevel.obj
 0003:000010e0       $pdata$__acrt_DownlevelLocaleNameToLCID 00000001800220e0     libucrt:lcidtoname_downlevel.obj
 0003:000010ec       $pdata$__acrt_lowio_create_handle_array 00000001800220ec     libucrt:osfinfo.obj
 0003:000010f8       $pdata$__acrt_lowio_destroy_handle_array 00000001800220f8     libucrt:osfinfo.obj
 0003:00001104       $pdata$__acrt_lowio_ensure_fh_exists 0000000180022104     libucrt:osfinfo.obj
 0003:00001110       $pdata$_free_osfhnd        0000000180022110     libucrt:osfinfo.obj
 0003:0000111c       $pdata$_get_osfhandle      000000018002211c     libucrt:osfinfo.obj
 0003:00001128       $pdata$??$?RV<lambda_a37b2b86f63e897a80ea819b0eb08c01>@@AEAV<lambda_38ce7e780aa69e748d6df282ebc68efe>@@V<lambda_99fb1378e971ab6e7edea83e3a7a83a2>@@@?$__crt_seh_guarded_call@H@@QEAAH$$QEAV<lambda_a37b2b86f63e897a80ea819b0eb08c01>@@AEAV<lambda_38ce7e780aa69e748d6df282ebc68efe>@@$$QEAV<lambda_99fb1378e971ab6e7edea83e3a7a83a2>@@@Z 0000000180022128     libucrt:commit.obj
 0003:00001134       $pdata$_commit             0000000180022134     libucrt:commit.obj
 0003:00001140       $pdata$?write_double_translated_ansi_nolock@@YA?AUwrite_result@?A0x17268360@@HQEBDI@Z 0000000180022140     libucrt:write.obj
 0003:0000114c       $pdata$?write_text_ansi_nolock@@YA?AUwrite_result@?A0x17268360@@HQEBDI@Z 000000018002214c     libucrt:write.obj
 0003:00001158       $pdata$?write_text_utf16le_nolock@@YA?AUwrite_result@?A0x17268360@@HQEBDI@Z 0000000180022158     libucrt:write.obj
 0003:00001164       $pdata$?write_text_utf8_nolock@@YA?AUwrite_result@?A0x17268360@@HQEBDI@Z 0000000180022164     libucrt:write.obj
 0003:00001170       $pdata$_write              0000000180022170     libucrt:write.obj
 0003:0000117c       $pdata$_write_nolock       000000018002217c     libucrt:write.obj
 0003:00001188       $pdata$_fcloseall          0000000180022188     libucrt:closeall.obj
 0003:00001194       $pdata$__acrt_stdio_free_buffer_nolock 0000000180022194     libucrt:_freebuf.obj
 0003:000011a0       $pdata$_isatty             00000001800221a0     libucrt:isatty.obj
 0003:000011ac       $pdata$_isleadbyte_l       00000001800221ac     libucrt:_wctype.obj
 0003:000011b8       $pdata$?__mbrtowc_utf8@__crt_mbstring@@YA_KPEA_WPEBD_KPEAU_Mbstatet@@@Z 00000001800221b8     libucrt:mbrtowc.obj
 0003:000011c4       $pdata$?__mbsrtowcs_utf8@__crt_mbstring@@YA_KPEA_WPEAPEBD_KPEAU_Mbstatet@@@Z 00000001800221c4     libucrt:mbrtowc.obj
 0003:000011d0       $pdata$__acrt_locale_free_monetary 00000001800221d0     libucrt:initmon.obj
 0003:000011dc       $pdata$__acrt_locale_free_numeric 00000001800221dc     libucrt:initnum.obj
 0003:000011e8       $pdata$?free_crt_array_internal@@YAXQEAPEBX_K@Z 00000001800221e8     libucrt:inittime.obj
 0003:000011f4       $pdata$__acrt_locale_free_time 00000001800221f4     libucrt:inittime.obj
 0003:00001200       $pdata$??$common_lseek_nolock@_J@@YA_JH_JH@Z 0000000180022200     libucrt:lseek.obj
 0003:0000120c       $pdata$_putwch_nolock      000000018002220c     libucrt:putwch.obj
 0003:00001218       $pdata$_fclose_nolock      0000000180022218     libucrt:fclose.obj
 0003:00001224       $pdata$fclose              0000000180022224     libucrt:fclose.obj
 0003:00001230       $pdata$?__mbrtoc32_utf8@__crt_mbstring@@YA_KPEA_UPEBD_KPEAU_Mbstatet@@@Z 0000000180022230     libucrt:mbrtoc32.obj
 0003:00001248       $pdata$__dcrt_lowio_ensure_console_output_initialized 0000000180022248     libucrt:initcon.obj
 0003:00001254       $pdata$__dcrt_terminate_console_output 0000000180022254     libucrt:initcon.obj
 0003:00001260       $pdata$__dcrt_write_console 0000000180022260     libucrt:initcon.obj
 0003:0000126c       $pdata$??$?RV<lambda_751a882b2c74d4b022dec766aa51a29a>@@AEAV<lambda_628dfdc04ba53c8bfc02c9951375f3f5>@@V<lambda_f6c7be5f7998530c34de24c7437d6b54>@@@?$__crt_seh_guarded_call@H@@QEAAH$$QEAV<lambda_751a882b2c74d4b022dec766aa51a29a>@@AEAV<lambda_628dfdc04ba53c8bfc02c9951375f3f5>@@$$QEAV<lambda_f6c7be5f7998530c34de24c7437d6b54>@@@Z 000000018002226c     libucrt:close.obj
 0003:00001278       $pdata$_close              0000000180022278     libucrt:close.obj
 0003:00001284       $pdata$_close_nolock       0000000180022284     libucrt:close.obj
 0003:00001290       $pdata$_call_matherr       0000000180022290     libucrt:libm_error.obj
 0003:0000129c       $pdata$_exception_enabled  000000018002229c     libucrt:libm_error.obj
 0003:000012a8       $pdata$_handle_error       00000001800222a8     libucrt:libm_error.obj
 0003:000012b4       $pdata$__acrt_initialize_fma3 00000001800222b4     libucrt:fma3_available.obj
 0003:000012c0       $pdata$_log10_special      00000001800222c0     libucrt:log_special.obj
 0003:000012cc       $pdata$_log_special_common 00000001800222cc     libucrt:log_special.obj
 0003:000012e4       $pdata$_raise_exc          00000001800222e4     libucrt:fpexcept.obj
 0003:000012f0       $pdata$_raise_exc_ex       00000001800222f0     libucrt:fpexcept.obj
 0003:000012fc       $pdata$_set_errno_from_matherr 00000001800222fc     libucrt:fpexcept.obj
 0003:00001308       $pdata$_clrfp              0000000180022308     libucrt:fpctrl.obj
 0003:00001314       $pdata$_ctrlfp             0000000180022314     libucrt:fpctrl.obj
 0003:00001320       $pdata$_set_statfp         0000000180022320     libucrt:fpctrl.obj
 0003:0000132c       $pdata$_statfp             000000018002232c     libucrt:fpctrl.obj
 0003:00001338       $pdata$_IsNonwritableInCurrentImage 0000000180022338     LIBCMT:pesect.obj
 0003:00001344       $pdata$__GSHandlerCheck    0000000180022344     LIBCMT:gshandler.obj
 0003:00001350       $pdata$__GSHandlerCheckCommon 0000000180022350     LIBCMT:gshandler.obj
 0003:00001368       $pdata$__raise_securityfailure 0000000180022368     LIBCMT:gs_report.obj
 0003:00001374       $pdata$__report_gsfailure  0000000180022374     LIBCMT:gs_report.obj
 0003:00001380       $pdata$__report_rangecheckfailure 0000000180022380     LIBCMT:gs_report.obj
 0003:0000138c       $pdata$__report_securityfailure 000000018002238c     LIBCMT:gs_report.obj
 0003:00001398       $pdata$capture_current_context 0000000180022398     LIBCMT:gs_report.obj
 0003:000013a4       $pdata$capture_previous_context 00000001800223a4     LIBCMT:gs_report.obj
 0003:000013bc       $pdata$?fin$0@?0??dllmain_crt_process_attach@@YAHQEAUHINSTANCE__@@QEAX@Z@4HA 00000001800223bc     LIBCMT:dll_dllmain.obj
 0003:000013c8       $pdata$?fin$0@?0??dllmain_crt_process_detach@@YAH_N@Z@4HA 00000001800223c8     LIBCMT:dll_dllmain.obj
 0003:000013d4       $pdata$?filt$0@?0??dllmain_dispatch@@YAHQEAUHINSTANCE__@@KQEAX@Z@4HA 00000001800223d4     LIBCMT:dll_dllmain.obj
 0003:000013e0       $pdata$__scrt_is_nonwritable_in_current_image$filt$0 00000001800223e0     LIBCMT:utility.obj
 0003:000013ec       $pdata$__DestructExceptionObject$filt$0 00000001800223ec     libvcruntime:ehhelpers.obj
 0003:000013f8       $pdata$_query_new_handler$fin$0 00000001800223f8     libucrt:new_handler.obj
 0003:00001404       $pdata$?fin$0@?0???$?RV<lambda_0ae27a3a962d80f24befdcbee591983d>@@AEAV<lambda_8d0ee55de4b1038c4002e0adecdf1839>@@V<lambda_dc504788e8f1664fe9b84e20bfb512f2>@@@?$__crt_seh_guarded_call@X@@QEAAX$$QEAV<lambda_0ae27a3a962d80f24befdcbee591983d>@@AEAV<lambda_8d0ee55de4b1038c4002e0adecdf1839>@@$$QEAV<lambda_dc504788e8f1664fe9b84e20bfb512f2>@@@Z@4HA 0000000180022404     libucrt:per_thread_data.obj
 0003:00001404       $pdata$?fin$0@?0???$?RV<lambda_f2e299630e499de9f9a165e60fcd3db5>@@AEAV<lambda_2ae9d31cdba2644fcbeaf08da7c24588>@@V<lambda_40d01ff24d0e7b3814fdbdcee8eab3c7>@@@?$__crt_seh_guarded_call@X@@QEAAX$$QEAV<lambda_f2e299630e499de9f9a165e60fcd3db5>@@AEAV<lambda_2ae9d31cdba2644fcbeaf08da7c24588>@@$$QEAV<lambda_40d01ff24d0e7b3814fdbdcee8eab3c7>@@@Z@4HA 0000000180022404     libucrt:per_thread_data.obj
 0003:00001404       $pdata$?fin$0@?0???$?RV<lambda_aa87e3671a710a21b5dc78c0bdf72e11>@@AEAV<lambda_92619d2358a28f41a33ba319515a20b9>@@V<lambda_6992ecaafeb10aed2b74cb1fae11a551>@@@?$__crt_seh_guarded_call@X@@QEAAX$$QEAV<lambda_aa87e3671a710a21b5dc78c0bdf72e11>@@AEAV<lambda_92619d2358a28f41a33ba319515a20b9>@@$$QEAV<lambda_6992ecaafeb10aed2b74cb1fae11a551>@@@Z@4HA 0000000180022404     libucrt:per_thread_data.obj
 0003:00001404       $pdata$?fin$0@?0???$?RV<lambda_450d765d439847d4c735a33c368b5fc0>@@AEAV<lambda_44731a7d0e6d81c3e6aa82d741081786>@@V<lambda_601a2a7da3b7a96e9554ac7215c4b07c>@@@?$__crt_seh_guarded_call@P6AXH@Z@@QEAAP6AXH@Z$$QEAV<lambda_450d765d439847d4c735a33c368b5fc0>@@AEAV<lambda_44731a7d0e6d81c3e6aa82d741081786>@@$$QEAV<lambda_601a2a7da3b7a96e9554ac7215c4b07c>@@@Z@4HA 0000000180022404     libucrt:signal.obj
 0003:00001404       $pdata$?fin$0@?0???$?RV<lambda_d80eeec6fff315bfe5c115232f3240e3>@@AEAV<lambda_6e4b09c48022b2350581041d5f6b0c4c>@@V<lambda_2358e3775559c9db80273638284d5e45>@@@?$__crt_seh_guarded_call@X@@QEAAX$$QEAV<lambda_d80eeec6fff315bfe5c115232f3240e3>@@AEAV<lambda_6e4b09c48022b2350581041d5f6b0c4c>@@$$QEAV<lambda_2358e3775559c9db80273638284d5e45>@@@Z@4HA 0000000180022404     libucrt:exit.obj
 0003:00001404       $pdata$?fin$0@?0???$?RV<lambda_2d41944a1d46af3157314b8a01080d33>@@AEAV<lambda_8f455de75cd7d7f24b4096f044d8b9e6>@@V<lambda_aa500f224e6afead328df44964fe2772>@@@?$__crt_seh_guarded_call@X@@QEAAX$$QEAV<lambda_2d41944a1d46af3157314b8a01080d33>@@AEAV<lambda_8f455de75cd7d7f24b4096f044d8b9e6>@@$$QEAV<lambda_aa500f224e6afead328df44964fe2772>@@@Z@4HA 0000000180022404     libucrt:per_thread_data.obj
 0003:00001404       $pdata$?fin$0@?0???$?RV<lambda_efdfa57d1f175319df784efa44bb7b81>@@AEAV<lambda_5f0a4c1567f8adc6734073e5d1e1b35c>@@V<lambda_2e8a7d3640ea6ccb4c2413664c2db6fd>@@@?$__crt_seh_guarded_call@X@@QEAAX$$QEAV<lambda_efdfa57d1f175319df784efa44bb7b81>@@AEAV<lambda_5f0a4c1567f8adc6734073e5d1e1b35c>@@$$QEAV<lambda_2e8a7d3640ea6ccb4c2413664c2db6fd>@@@Z@4HA 0000000180022404     libucrt:mbctype.obj
 0003:00001404       $pdata$?fin$0@?0???$?RV<lambda_7777bce6b2f8c936911f934f8298dc43>@@AEAV<lambda_f03950bc5685219e0bcd2087efbe011e>@@V<lambda_3883c3dff614d5e0c5f61bb1ac94921c>@@@?$__crt_seh_guarded_call@H@@QEAAH$$QEAV<lambda_7777bce6b2f8c936911f934f8298dc43>@@AEAV<lambda_f03950bc5685219e0bcd2087efbe011e>@@$$QEAV<lambda_3883c3dff614d5e0c5f61bb1ac94921c>@@@Z@4HA 0000000180022404     libucrt:onexit.obj
 0003:00001410       $pdata$?filt$0@?0???R<lambda_6e4b09c48022b2350581041d5f6b0c4c>@@QEBA@XZ@4HA 0000000180022410     libucrt:exit.obj
 0003:0000141c       $pdata$?fin$0@?0??update_thread_multibyte_data_internal@@YAPEAU__crt_multibyte_data@@QEAU__acrt_ptd@@QEAPEAU1@@Z@4HA 000000018002241c     libucrt:mbctype.obj
 0003:00001428       $pdata$__acrt_lowio_ensure_fh_exists$fin$0 0000000180022428     libucrt:osfinfo.obj
 0003:00001428       $pdata$__acrt_initialize_lowio$fin$0 0000000180022428     libucrt:ioinit.obj
 0003:00001434       $pdata$raise$fin$0         0000000180022434     libucrt:signal.obj
 0003:00001440       $pdata$?fin$0@?0???$?RV<lambda_842d9ff0dc9ef11c61343bbaebe7f885>@@AEAV<lambda_c5860995281e5c4ce005b3de8f5874ee>@@V<lambda_d90129c13df834fdcbf8d2b88dafcf2d>@@@?$__crt_seh_guarded_call@X@@QEAAX$$QEAV<lambda_842d9ff0dc9ef11c61343bbaebe7f885>@@AEAV<lambda_c5860995281e5c4ce005b3de8f5874ee>@@$$QEAV<lambda_d90129c13df834fdcbf8d2b88dafcf2d>@@@Z@4HA 0000000180022440     libucrt:fflush.obj
 0003:0000144c       $pdata$?fin$0@?0???$?RV<lambda_886d6c58226a84441f68b9f2b8217b83>@@AEAV<lambda_ab61a845afdef5b7c387490eaf3616ee>@@V<lambda_f7f22ab5edc0698d5f6905b0d3f44752>@@@?$__crt_seh_guarded_call@X@@QEAAX$$QEAV<lambda_886d6c58226a84441f68b9f2b8217b83>@@AEAV<lambda_ab61a845afdef5b7c387490eaf3616ee>@@$$QEAV<lambda_f7f22ab5edc0698d5f6905b0d3f44752>@@@Z@4HA 000000018002244c     libucrt:fflush.obj
 0003:00001458       $pdata$?fin$0@?0???$?RV<lambda_410d79af7f07d98d83a3f525b3859a53>@@AEAV<lambda_3e16ef9562a7dcce91392c22ab16ea36>@@V<lambda_38119f0e861e05405d8a144b9b982f0a>@@@?$__crt_seh_guarded_call@X@@QEAAX$$QEAV<lambda_410d79af7f07d98d83a3f525b3859a53>@@AEAV<lambda_3e16ef9562a7dcce91392c22ab16ea36>@@$$QEAV<lambda_38119f0e861e05405d8a144b9b982f0a>@@@Z@4HA 0000000180022458     libucrt:wsetlocale.obj
 0003:00001464       $pdata$__acrt_update_thread_locale_data$fin$0 0000000180022464     libucrt:locale_refcounting.obj
 0003:00001470       $pdata$?fin$0@?0???$?RV<lambda_a37b2b86f63e897a80ea819b0eb08c01>@@AEAV<lambda_38ce7e780aa69e748d6df282ebc68efe>@@V<lambda_99fb1378e971ab6e7edea83e3a7a83a2>@@@?$__crt_seh_guarded_call@H@@QEAAH$$QEAV<lambda_a37b2b86f63e897a80ea819b0eb08c01>@@AEAV<lambda_38ce7e780aa69e748d6df282ebc68efe>@@$$QEAV<lambda_99fb1378e971ab6e7edea83e3a7a83a2>@@@Z@4HA 0000000180022470     libucrt:commit.obj
 0003:00001470       $pdata$?fin$0@?0???$?RV<lambda_751a882b2c74d4b022dec766aa51a29a>@@AEAV<lambda_628dfdc04ba53c8bfc02c9951375f3f5>@@V<lambda_f6c7be5f7998530c34de24c7437d6b54>@@@?$__crt_seh_guarded_call@H@@QEAAH$$QEAV<lambda_751a882b2c74d4b022dec766aa51a29a>@@AEAV<lambda_628dfdc04ba53c8bfc02c9951375f3f5>@@$$QEAV<lambda_f6c7be5f7998530c34de24c7437d6b54>@@@Z@4HA 0000000180022470     libucrt:close.obj
 0003:0000147c       $pdata$_write$fin$0        000000018002247c     libucrt:write.obj
 0003:00001488       $pdata$_fcloseall$fin$0    0000000180022488     libucrt:closeall.obj
 0003:00001494       $pdata$fclose$fin$0        0000000180022494     libucrt:fclose.obj
 0003:000014a0       $pdata$_ctrlfp$filt$0      00000001800224a0     libucrt:fpctrl.obj
 0003:000014ac       $pdata$_IsNonwritableInCurrentImage$filt$0 00000001800224ac     LIBCMT:pesect.obj
 0004:000007ec       .idata$6                   00000001800237ec     kernel32:KERNEL32.dll
 0004:0000080a       .idata$6                   000000018002380a     advapi32:ADVAPI32.dll
 0004:00000828       .idata$6                   0000000180023828     shell32:SHELL32.dll
 0005:00000060       $R000000                   0000000180024060     TmpPanel.res
